 ServerApp

 Timestamp is 602f668b (Fri Feb 19 16:19:39 2021)

 Preferred load address is 00400000

 Start         Length     Name                   Class
 0001:00000000 00000af0H .text$di                CODE
 0001:00000af0 00015ba0H .text$mn                CODE
 0001:00016690 00001070H .text$x                 CODE
 0001:00017700 000005d4H .text$yd                CODE
 0002:00000000 0000067cH .idata$5                DATA
 0002:0000067c 00000004H .00cfg                  DATA
 0002:00000680 00000004H .CRT$XCA                DATA
 0002:00000684 00000004H .CRT$XCAA               DATA
 0002:00000688 00000008H .CRT$XCL                DATA
 0002:00000690 00000210H .CRT$XCU                DATA
 0002:000008a0 00000004H .CRT$XCZ                DATA
 0002:000008a4 00000004H .CRT$XIA                DATA
 0002:000008a8 00000004H .CRT$XIAA               DATA
 0002:000008ac 00000004H .CRT$XIAC               DATA
 0002:000008b0 00000004H .CRT$XIZ                DATA
 0002:000008b4 00000004H .CRT$XPA                DATA
 0002:000008b8 00000004H .CRT$XPZ                DATA
 0002:000008bc 00000004H .CRT$XTA                DATA
 0002:000008c0 00000010H .CRT$XTZ                DATA
 0002:000008c4 00000000H .gfids$y                DATA
 0002:000008d0 00007318H .rdata                  DATA
 0002:00007be8 000009d8H .rdata$r                DATA
 0002:000085c0 00000100H .rdata$sxdata           DATA
 0002:000086c0 00000340H .rdata$zzzdbg           DATA
 0002:00008a00 00000004H .rtc$IAA                DATA
 0002:00008a04 00000004H .rtc$IZZ                DATA
 0002:00008a08 00000004H .rtc$TAA                DATA
 0002:00008a0c 00000004H .rtc$TZZ                DATA
 0002:00008a10 00000000H .tls$                   DATA
 0002:00008a10 00000e90H .xdata$x                DATA
 0002:0000989c 00000000H ATL$__a                 DATA
 0002:0000989c 00000000H ATL$__z                 DATA
 0002:000098a0 00000068H .edata                  DATA
 0002:00009908 000001ccH .idata$2                DATA
 0002:00009ad4 00000014H .idata$3                DATA
 0002:00009ae8 0000067cH .idata$4                DATA
 0002:0000a164 000014acH .idata$6                DATA
 0003:00000000 00000250H .data                   DATA
 0003:00000250 00000510H .data$r                 DATA
 0003:00000760 00227488H .bss                    DATA
 0004:00000000 000001b0H .rsrc$01                DATA
 0004:000001b0 00000a38H .rsrc$02                DATA

  Address         Publics by Value              Rva+Base       Lib:Object

 0000:00000000       ___guard_longjmp_count     00000000     <absolute>
 0000:00000000       ___guard_iat_count         00000000     <absolute>
 0000:00000000       ___guard_fids_count        00000000     <absolute>
 0000:00000000       ___guard_longjmp_table     00000000     <absolute>
 0000:00000000       ___hybrid_code_map_count   00000000     <absolute>
 0000:00000000       ___volatile_metadata       00000000     <absolute>
 0000:00000000       ___hybrid_auxiliary_iat    00000000     <absolute>
 0000:00000000       ___dynamic_value_reloc_table 00000000     <absolute>
 0000:00000000       ___guard_fids_table        00000000     <absolute>
 0000:00000000       ___guard_iat_table         00000000     <absolute>
 0000:00000000       ___enclave_config          00000000     <absolute>
 0000:00000000       ___hybrid_code_map         00000000     <absolute>
 0000:00000040       ___safe_se_handler_count   00000040     <absolute>
 0000:00000100       ___guard_flags             00000100     <absolute>
 0000:00000000       ___ImageBase               00400000     <linker-defined>
 0001:00000af0       ___local_stdio_printf_options 00401af0 f i safe_string:safe_string.obj
 0001:00000b00       ?sprintf_s@internal@cf@@YAHPADIPBDAAPAD@Z 00401b00 f   safe_string:safe_string.obj
 0001:00000d40       ??_D?$basic_stringstream@DU?$char_traits@D@std@@V?$allocator@D@2@@std@@QAEXXZ 00401d40 f i safe_string:safe_string.obj
 0001:00000d80       ?strcpy_s@cf@@YAHPADIPBD@Z 00401d80 f   safe_string:safe_string.obj
 0001:00000fb0       ?strncpy_s@cf@@YAHPADIPBDI@Z 00401fb0 f   safe_string:safe_string.obj
 0001:00001200       ?sprintf_s@cf@@YAHPADIPBDZZ 00402200 f   safe_string:safe_string.obj
 0001:00001230       ?_Tidy_deallocate@?$basic_string@DU?$char_traits@D@std@@V?$allocator@D@2@@std@@QAEXXZ 00402230 f i safe_string:safe_string.obj
 0001:00001230       ??1?$basic_string@DU?$char_traits@D@std@@V?$allocator@D@2@@std@@QAE@XZ 00402230 f i safe_string:safe_string.obj
 0001:00001280       ??0?$basic_string@DU?$char_traits@D@std@@V?$allocator@D@2@@std@@QAE@QBD@Z 00402280 f i safe_string:safe_string.obj
 0001:000012c0       ?str@?$basic_stringstream@DU?$char_traits@D@std@@V?$allocator@D@2@@std@@QBE?AV?$basic_string@DU?$char_traits@D@std@@V?$allocator@D@2@@2@XZ 004022c0 f i safe_string:safe_string.obj
 0001:00001380       ??0?$basic_stringstream@DU?$char_traits@D@std@@V?$allocator@D@2@@std@@QAE@H@Z 00402380 f i safe_string:safe_string.obj
 0001:00001440       ?seekpos@?$basic_stringbuf@DU?$char_traits@D@std@@V?$allocator@D@2@@std@@MAE?AV?$fpos@U_Mbstatet@@@2@V32@H@Z 00402440 f i safe_string:safe_string.obj
 0001:00001540       ?seekoff@?$basic_stringbuf@DU?$char_traits@D@std@@V?$allocator@D@2@@std@@MAE?AV?$fpos@U_Mbstatet@@@2@_JHH@Z 00402540 f i safe_string:safe_string.obj
 0001:000016b0       ?underflow@?$basic_stringbuf@DU?$char_traits@D@std@@V?$allocator@D@2@@std@@MAEHXZ 004026b0 f i safe_string:safe_string.obj
 0001:00001710       ?pbackfail@?$basic_stringbuf@DU?$char_traits@D@std@@V?$allocator@D@2@@std@@MAEHH@Z 00402710 f i safe_string:safe_string.obj
 0001:00001770       ?overflow@?$basic_stringbuf@DU?$char_traits@D@std@@V?$allocator@D@2@@std@@MAEHH@Z 00402770 f i safe_string:safe_string.obj
 0001:00001920       ??1?$basic_stringbuf@DU?$char_traits@D@std@@V?$allocator@D@2@@std@@UAE@XZ 00402920 f i safe_string:safe_string.obj
 0001:000019d0       ??_E?$basic_stringstream@DU?$char_traits@D@std@@V?$allocator@D@2@@std@@UAEPAXI@Z 004029d0 f i * CIL library *:* CIL module *
 0001:000019d0       ??_G?$basic_stringstream@DU?$char_traits@D@std@@V?$allocator@D@2@@std@@UAEPAXI@Z 004029d0 f i safe_string:safe_string.obj
 0001:00001a30       ??_G?$basic_stringbuf@DU?$char_traits@D@std@@V?$allocator@D@2@@std@@UAEPAXI@Z 00402a30 f i safe_string:safe_string.obj
 0001:00001a30       ??_E?$basic_stringbuf@DU?$char_traits@D@std@@V?$allocator@D@2@@std@@UAEPAXI@Z 00402a30 f i * CIL library *:* CIL module *
 0001:00001a60       ??1sentry@?$basic_ostream@DU?$char_traits@D@std@@@std@@QAE@XZ 00402a60 f i safe_string:safe_string.obj
 0001:00001ad0       ?assign@?$basic_string@DU?$char_traits@D@std@@V?$allocator@D@2@@std@@QAEAAV12@QBD@Z 00402ad0 f i safe_string:safe_string.obj
 0001:00001b00       ?assign@?$basic_string@DU?$char_traits@D@std@@V?$allocator@D@2@@std@@QAEAAV12@QBDI@Z 00402b00 f i safe_string:safe_string.obj
 0001:00001c30       ?allocate@?$allocator@D@std@@QAEPADI@Z 00402c30 f i safe_string:safe_string.obj
 0001:00001c90       ??1_Sentry_base@?$basic_ostream@DU?$char_traits@D@std@@@std@@QAE@XZ 00402c90 f i safe_string:safe_string.obj
 0001:00001ce0       ??$?6U?$char_traits@D@std@@@std@@YAAAV?$basic_ostream@DU?$char_traits@D@std@@@0@AAV10@PBD@Z 00402ce0 f i safe_string:safe_string.obj
 0001:00001f30       ??$endl@DU?$char_traits@D@std@@@std@@YAAAV?$basic_ostream@DU?$char_traits@D@std@@@0@AAV10@@Z 00402f30 f i safe_string:safe_string.obj
 0001:00001f60       ?_Xlen@?$basic_string@DU?$char_traits@D@std@@V?$allocator@D@2@@std@@SAXXZ 00402f60 f i safe_string:safe_string.obj
 0001:00001f60       ?_Xlen@?$basic_string@_WU?$char_traits@_W@std@@V?$allocator@_W@2@@std@@SAXXZ 00402f60 f i crs_uploader1.obj
 0001:00001f6b       ??_E?$basic_stringstream@DU?$char_traits@D@std@@V?$allocator@D@2@@std@@$4PPPPPPPM@A@AEPAXI@Z 00402f6b f i safe_string:safe_string.obj
 0001:00001f80       ??$_AppendInt@$0BAE@@rwpmlog@@YA_NAAY0BAE@D_J@Z 00402f80 f i RWPMLog.obj
 0001:00001fa0       ??$_AppendStr@$0BAE@@rwpmlog@@YA_NAAY0BAE@DPBD@Z 00402fa0 f i RWPMLog.obj
 0001:00001fc0       ??$sprintf_s@$0EA@@cf@@YAHAAY0EA@DPBDZZ 00402fc0 f i RWPMLog.obj
 0001:00001ff0       ?Log@rwpmlog@@YAXPBDF0_J@Z 00402ff0 f   RWPMLog.obj
 0001:00002060       ?Log@rwpmlog@@YAXPBDFPAY0DC@PAX@Z 00403060 f   RWPMLog.obj
 0001:00002130       ?Log@rwpmlog@@YAXPBDFPBUBATTLE_ROYAL_RESULT@@@Z 00403130 f   RWPMLog.obj
 0001:00002250       ?Log@rwpmlog@@YAXPBDFPBUCLANSTATREPORTDATA@@@Z 00403250 f   RWPMLog.obj
 0001:00002320       ?Log@rwpmlog@@YAXPBDFPBUGAMEPROTO_SC_HOST_USER_STAT@@@Z 00403320 f   RWPMLog.obj
 0001:00002560       ?Log@rwpmlog@@YAXPBDFPBUGAMEPROTO_SC_REMOVECLIENT@@@Z 00403560 f   RWPMLog.obj
 0001:00002630       ?Log@rwpmlog@@YAXPBDFPBUGAMEPROTO_SC_SPY_CHANGE@@@Z 00403630 f   RWPMLog.obj
 0001:000026d0       ?Log@rwpmlog@@YAXPBDFPBUGAMEPROTO_SS_GAMEEND@@@Z 004036d0 f   RWPMLog.obj
 0001:00002940       ?Log@rwpmlog@@YAXPBDFPBUPROTOCOL_AI2_BONUSROUND_REWARD_REQ_tag@@@Z 00403940 f   RWPMLog.obj
 0001:000029f0       ?Log@rwpmlog@@YAXPBDFPBUPROTO_AI_EXTRA_REWARD_REQ@@@Z 004039f0 f   RWPMLog.obj
 0001:00002aa0       ?Log@rwpmlog@@YAXPBDFPBUPROTO_BAN_USER_tag@@@Z 00403aa0 f   RWPMLog.obj
 0001:00002b20       ?Log@rwpmlog@@YAXPBDFPBUPROTO_FINISHED_GAME_PREV_tag@@@Z 00403b20 f   RWPMLog.obj
 0001:00002bb0       ?Log@rwpmlog@@YAXPBDFPBUPROTO_GAMEGT_AUTO_SIDE_CHANGE_TEAM_INFO_NTY@@@Z 00403bb0 f   RWPMLog.obj
 0001:00002d00       ?Log@rwpmlog@@YAXPBDFPBUPROTO_GAMEGT_INGAME_AI3_BONUS_REWARD_ITEM_REQ@@@Z 00403d00 f   RWPMLog.obj
 0001:00002da0       ?Log@rwpmlog@@YAXPBDFPBUPROTO_GAMEGT_INGAME_AIGACHA_GROUP_RATE_RESULT@@@Z 00403da0 f   RWPMLog.obj
 0001:00002e60       ?Log@rwpmlog@@YAXPBDFPBUPROTO_GAMEGT_INGAME_AIGACHA_ITEM_INSERT@@@Z 00403e60 f   RWPMLog.obj
 0001:00002f30       ?Log@rwpmlog@@YAXPBDFPBUPROTO_GAMEGT_INGAME_AIGACHA_ITEM_INSERT_RESULT@@@Z 00403f30 f   RWPMLog.obj
 0001:00002ff0       ?Log@rwpmlog@@YAXPBDFPBUPROTO_GAMEGT_INGAME_FARMING_ITEM_REQ@@@Z 00403ff0 f   RWPMLog.obj
 0001:000030b0       ?Log@rwpmlog@@YAXPBDFPBUPROTO_GAMEGT_MAPLOADING_COMPLETE_NTY_tag@@@Z 004040b0 f   RWPMLog.obj
 0001:00003130       ?Log@rwpmlog@@YAXPBDFPBUPROTO_GAME_USER_INFO_tag@@@Z 00404130 f   RWPMLog.obj
 0001:00003280       ?Log@rwpmlog@@YAXPBDFPBUPROTO_GMGMT_BATTLE_USER_EXIT_NTY@@@Z 00404280 f   RWPMLog.obj
 0001:000033c0       ?Log@rwpmlog@@YAXPBDFPBUPROTO_INSERT_CHARACTER_RESULT_tag@@@Z 004043c0 f   RWPMLog.obj
 0001:00003440       ?Log@rwpmlog@@YAXPBDFPBUPROTO_SPEC_RECOMMENDROOM_INGAME_DATA@@@Z 00404440 f   RWPMLog.obj
 0001:00003560       ?Log@rwpmlog@@YAXPBDFPBUPROTO_START_HOST_tag@@@Z 00404560 f   RWPMLog.obj
 0001:00003660       ?_AppendInt@rwpmlog@@YA_NPADI_J@Z 00404660 f   RWPMLog.obj
 0001:00003700       ?_AppendStr@rwpmlog@@YA_NPADIPBD@Z 00404700 f   RWPMLog.obj
 0001:000037a0       __initialize_invalid_parameter_handler 004047a0 f i msvcrt:invalid_parameter_handler.obj
 0001:000037a0       ?__global_delete@@YAXPAXI@Z 004047a0 f i RWPMLog.obj
 0001:000037a0       ?__empty_global_delete@@YAXPAXI@Z 004047a0 f i RWPMLog.obj
 0001:000037a0       __initialize_denormal_control 004047a0 f i msvcrt:denormal_control.obj
 0001:000037a0       @_guard_check_icall_nop@4  004047a0 f i msvcrt:guard_support.obj
 0001:000037a0       ?AssertValid@CObject@@UBEXXZ 004047a0 f i ServerApp.obj
 0001:000037a0       ?LogBR@CHLogger@@SAXW4ELOG_LEVEL@1@PBDZZ 004047a0 f i ServerAppDlg.obj
 0001:000037b0       ??0?$database_list@VCAPIHolderBase@@@@QAE@XZ 004047b0 f i ltmodule.obj
 0001:000037b0       ??0?$database_list@VCInterfaceChooser@@@@QAE@XZ 004047b0 f i ltmodule.obj
 0001:000037b0       ??0?$database_array@VIBase@@PBD@@QAE@XZ 004047b0 f i ltmodule.obj
 0001:000037b0       ??0?$database_array@VCInterfaceNameMgr@@PBD@@QAE@XZ 004047b0 f i ltmodule.obj
 0001:000037e0       ??0CAPIHolderBase@@QAE@PBDH@Z 004047e0 f   ltmodule.obj
 0001:00003810       ??0CInterfaceDatabase@@QAE@XZ 00404810 f   ltmodule.obj
 0001:000038b0       ??0CInterfaceNameMgr@@QAE@PBDH@Z 004048b0 f   ltmodule.obj
 0001:000039c0       ??1?$CPointerTracked@VCInterfaceDatabase@@@@QAE@XZ 004049c0 f i ltmodule.obj
 0001:000039d0       ??1?$CPointerTrackedTarget@VCInterfaceDatabase@@@@QAE@XZ 004049d0 f i ltmodule.obj
 0001:000039e0       ??1?$database_array@VCInterfaceNameMgr@@PBD@@QAE@XZ 004049e0 f i ltmodule.obj
 0001:00003a30       ??1?$database_array@VIBase@@PBD@@QAE@XZ 00404a30 f i ltmodule.obj
 0001:00003a80       ??1?$database_list@VCInterfaceChooser@@@@QAE@XZ 00404a80 f i ltmodule.obj
 0001:00003a80       ??1?$database_list@VCAPIHolderBase@@@@QAE@XZ 00404a80 f i ltmodule.obj
 0001:00003aa0       ??1CAPIHolderBase@@UAE@XZ  00404aa0 f   ltmodule.obj
 0001:00003ab0       ??1CInterfaceDatabase@@QAE@XZ 00404ab0 f   ltmodule.obj
 0001:00003b00       ??1CInterfaceNameMgr@@UAE@XZ 00404b00 f   ltmodule.obj
 0001:00003b90       ??1_FILE_SHUTDOWN_class_ltmod_database_@@QAE@XZ 00404b90 f   ltmodule.obj
 0001:00003be0       ??_ECAPIHolderBase@@UAEPAXI@Z 00404be0 f i ltmodule.obj
 0001:00003be0       ??_GCAPIHolderBase@@UAEPAXI@Z 00404be0 f i ltmodule.obj
 0001:00003c10       ??_GCInterfaceNameMgr@@UAEPAXI@Z 00404c10 f i ltmodule.obj
 0001:00003c10       ??_ECInterfaceNameMgr@@UAEPAXI@Z 00404c10 f i ltmodule.obj
 0001:00003c40       ?Add@CInterfaceDatabase@@EAEXPAVCAPIHolderBase@@@Z 00404c40 f   ltmodule.obj
 0001:00003d10       ?Add@CInterfaceDatabase@@EAEXPAVCInterfaceChooser@@@Z 00404d10 f   ltmodule.obj
 0001:00003de0       ?Add@CInterfaceDatabase@@EAEXPAVIBase@@PBDH@Z 00404de0 f   ltmodule.obj
 0001:00003eb0       ?Add@CInterfaceNameMgr@@QAEXPAVCAPIHolderBase@@@Z 00404eb0 f   ltmodule.obj
 0001:00003ee0       ?Add@CInterfaceNameMgr@@QAEXPAVCInterfaceChooser@@@Z 00404ee0 f   ltmodule.obj
 0001:00003f10       ?Add@CInterfaceNameMgr@@QAEXPAVIBase@@@Z 00404f10 f   ltmodule.obj
 0001:00003f90       ?AddAPI@CInterfaceDatabase@@SAXPAVIBase@@PBDH@Z 00404f90 f   ltmodule.obj
 0001:00004050       ?AddChooser@CInterfaceDatabase@@SAXPAVCInterfaceChooser@@@Z 00405050 f   ltmodule.obj
 0001:00004100       ?AddHolder@CInterfaceDatabase@@SAXPAVCAPIHolderBase@@@Z 00405100 f   ltmodule.obj
 0001:000041b0       ?ConnectHolder@CInterfaceNameMgr@@IAEXPAVCAPIHolderBase@@@Z 004051b0 f   ltmodule.obj
 0001:000041d0       ?ConnectHolders@CInterfaceNameMgr@@IAEXPAVIBase@@@Z 004051d0 f   ltmodule.obj
 0001:00004220       ?DatabaseItemCountDec@CInterfaceDatabase@@SAXXZ 00405220 f   ltmodule.obj
 0001:00004270       ?DatabaseItemCountInc@CInterfaceDatabase@@SAXXZ 00405270 f   ltmodule.obj
 0001:000042c0       ?Destroy@CInterfaceDatabase@@UAEXXZ 004052c0 f   ltmodule.obj
 0001:000042e0       ?DisconnectHolders@CInterfaceNameMgr@@IAEXXZ 004052e0 f   ltmodule.obj
 0001:00004320       ?GetMasterDatabase@@YAPAVCInterfaceDatabase@@XZ 00405320 f   ltmodule.obj
 0001:000043f0       ?IsEmpty@CInterfaceDatabase@@EAE_NXZ 004053f0 f   ltmodule.obj
 0001:00004400       ?IsEmpty@CInterfaceNameMgr@@QAE_NXZ 00405400 f   ltmodule.obj
 0001:00004430       ?Num@?$database_list@VCAPIHolderBase@@@@QAEIXZ 00405430 f i ltmodule.obj
 0001:00004430       ?Num@?$database_array@VIBase@@PBD@@QAEIXZ 00405430 f i ltmodule.obj
 0001:00004430       ?Num@?$database_array@VCInterfaceNameMgr@@PBD@@QAEIXZ 00405430 f i ltmodule.obj
 0001:00004430       ?Num@?$database_list@VCInterfaceChooser@@@@QAEIXZ 00405430 f i ltmodule.obj
 0001:00004440       ?RedirectPointers@?$CPointerTrackedTarget@VCInterfaceDatabase@@@@QAEXPAVCInterfaceDatabase@@@Z 00405440 f i ltmodule.obj
 0001:00004480       ?Remove@CInterfaceDatabase@@EAEXPAVCAPIHolderBase@@@Z 00405480 f   ltmodule.obj
 0001:000044d0       ?Remove@CInterfaceDatabase@@EAEXPAVCInterfaceChooser@@@Z 004054d0 f   ltmodule.obj
 0001:00004520       ?Remove@CInterfaceDatabase@@EAEXPAVIBase@@PBD@Z 00405520 f   ltmodule.obj
 0001:00004570       ?Remove@CInterfaceNameMgr@@QAEXPAVCAPIHolderBase@@@Z 00405570 f   ltmodule.obj
 0001:00004590       ?Remove@CInterfaceNameMgr@@QAEXPAVCInterfaceChooser@@@Z 00405590 f   ltmodule.obj
 0001:000045b0       ?Remove@CInterfaceNameMgr@@QAEXPAVIBase@@@Z 004055b0 f   ltmodule.obj
 0001:00004630       ?RemoveHolder@CInterfaceDatabase@@SAXPAVCAPIHolderBase@@@Z 00405630 f   ltmodule.obj
 0001:00004690       ?Run@CInterfaceDatabase@@EAE?AW4EChooserRun@@PAVCInterfaceChooser@@@Z 00405690 f   ltmodule.obj
 0001:000046d0       ?Run@CInterfaceNameMgr@@QAE?AW4EChooserRun@@PAVCInterfaceChooser@@@Z 004056d0 f   ltmodule.obj
 0001:00004740       ?Set@?$CPointerTracked@VCInterfaceDatabase@@@@IAEXPAVCInterfaceDatabase@@@Z 00405740 f i ltmodule.obj
 0001:00004780       ?SortedArrayCompareIBase@@YA?AW4RELATION@@PAVIBase@@0@Z 00405780 f   ltmodule.obj
 0001:000047d0       ?SortedArrayCompareNameMgr@@YA?AW4RELATION@@PAVCInterfaceNameMgr@@0@Z 004057d0 f   ltmodule.obj
 0001:00004820       ?SortedArrayFindNameMgr@@YA?AW4RELATION@@PBDPAVCInterfaceNameMgr@@@Z 00405820 f   ltmodule.obj
 0001:00004870       ?TransferFrom@CInterfaceDatabase@@UAEXPAV1@@Z 00405870 f   ltmodule.obj
 0001:00004970       ?TransferFrom@CInterfaceNameMgr@@QAEXPAV1@@Z 00405970 f   ltmodule.obj
 0001:00004a30       ?Unset@?$CPointerTracked@VCInterfaceDatabase@@@@IAEXXZ 00405a30 f i ltmodule.obj
 0001:00004a70       ?VersionError@CInterfaceDatabase@@AAEXPBD@Z 00405a70 f   ltmodule.obj
 0001:00004ad0       ?add@?$database_array@VCInterfaceNameMgr@@PBD@@QAEXPAVCInterfaceNameMgr@@P6A?AW4RELATION@@00@Z@Z 00405ad0 f i ltmodule.obj
 0001:00004ad0       ?add@?$database_array@VIBase@@PBD@@QAEXPAVIBase@@P6A?AW4RELATION@@00@Z@Z 00405ad0 f i ltmodule.obj
 0001:00004ba0       ?add@?$database_list@VCInterfaceChooser@@@@QAEXPAVCInterfaceChooser@@@Z 00405ba0 f i ltmodule.obj
 0001:00004ba0       ?add@?$database_list@VCAPIHolderBase@@@@QAEXPAVCAPIHolderBase@@@Z 00405ba0 f i ltmodule.obj
 0001:00004bd0       ?get@?$database_array@VIBase@@PBD@@QAEPAVIBase@@I@Z 00405bd0 f i ltmodule.obj
 0001:00004bd0       ?get@?$database_list@VCInterfaceChooser@@@@QAEPAVCInterfaceChooser@@I@Z 00405bd0 f i ltmodule.obj
 0001:00004bd0       ?get@?$database_list@VCAPIHolderBase@@@@QAEPAVCAPIHolderBase@@I@Z 00405bd0 f i ltmodule.obj
 0001:00004bd0       ?get@?$database_array@VCInterfaceNameMgr@@PBD@@QAEPAVCInterfaceNameMgr@@I@Z 00405bd0 f i ltmodule.obj
 0001:00004bf0       ?get@?$database_array@VCInterfaceNameMgr@@PBD@@QAEPAVCInterfaceNameMgr@@PBDP6A?AW4RELATION@@0PAV2@@Z@Z 00405bf0 f i ltmodule.obj
 0001:00004c20       ?index@?$database_array@VCInterfaceNameMgr@@PBD@@IAEHPBDP6A?AW4RELATION@@0PAVCInterfaceNameMgr@@@Z@Z 00405c20 f i ltmodule.obj
 0001:00004cc0       ?insert@?$database_array@VIBase@@PBD@@IAEXPAVIBase@@I@Z 00405cc0 f i ltmodule.obj
 0001:00004cc0       ?insert@?$database_array@VCInterfaceNameMgr@@PBD@@IAEXPAVCInterfaceNameMgr@@I@Z 00405cc0 f i ltmodule.obj
 0001:00004d10       ?lengthen@?$database_array@VIBase@@PBD@@IAEXXZ 00405d10 f i ltmodule.obj
 0001:00004d10       ?lengthen@?$database_list@VCAPIHolderBase@@@@IAEXXZ 00405d10 f i ltmodule.obj
 0001:00004d10       ?lengthen@?$database_list@VCInterfaceChooser@@@@IAEXXZ 00405d10 f i ltmodule.obj
 0001:00004d10       ?lengthen@?$database_array@VCInterfaceNameMgr@@PBD@@IAEXXZ 00405d10 f i ltmodule.obj
 0001:00004d70       ?remove@?$database_array@VCInterfaceNameMgr@@PBD@@QAE_NPAVCInterfaceNameMgr@@@Z 00405d70 f i ltmodule.obj
 0001:00004d70       ?remove_shift@?$database_list@VCInterfaceChooser@@@@QAE_NPAVCInterfaceChooser@@@Z 00405d70 f i ltmodule.obj
 0001:00004d70       ?remove@?$database_array@VIBase@@PBD@@QAE_NPAVIBase@@@Z 00405d70 f i ltmodule.obj
 0001:00004dc0       ?remove@?$database_list@VCInterfaceChooser@@@@QAEPAVCInterfaceChooser@@I@Z 00405dc0 f i ltmodule.obj
 0001:00004dc0       ?remove@?$database_list@VCAPIHolderBase@@@@QAEPAVCAPIHolderBase@@I@Z 00405dc0 f i ltmodule.obj
 0001:00004e10       ?remove@?$database_list@VCAPIHolderBase@@@@QAE_NPAVCAPIHolderBase@@@Z 00405e10 f i ltmodule.obj
 0001:00004e50       ?remove_last@?$database_array@VIBase@@PBD@@QAEPAVIBase@@XZ 00405e50 f i ltmodule.obj
 0001:00004e70       _SetMasterDatabase         00405e70 f   ltmodule.obj
 0001:00004f20       ??_GCMustSyncObjectLog@@UAEPAXI@Z 00405f20 f i HostLogger.obj
 0001:00004f20       ??_ECMustSyncObjectLog@@UAEPAXI@Z 00405f20 f i HostLogger.obj
 0001:00004f50       ??1CSynchronizedLog@@QAE@XZ 00405f50 f i HostLogger.obj
 0001:00004f70       ?Init@CHLogger@@SAXPBD000@Z 00405f70 f   HostLogger.obj
 0001:00004fe0       ?Log@CHLogger@@SAXW4ELOG_LEVEL@1@PBDZZ 00405fe0 f   HostLogger.obj
 0001:00005020       ?LogEtc@CHLogger@@SAXPBDZZ 00406020 f   HostLogger.obj
 0001:000051d0       ?LogIPCMessage@CHLogger@@SAXPBDZZ 004061d0 f   HostLogger.obj
 0001:00005360       ?LogKernel@CHLogger@@SAXW4ELOG_LEVEL@1@PBDZZ 00406360 f   HostLogger.obj
 0001:000053a0       ?LogPacket@CHLogger@@SAXPBDZZ 004063a0 f   HostLogger.obj
 0001:000055a0       ?LogRWProcessMemory@CHLogger@@SAXPBDZZ 004065a0 f   HostLogger.obj
 0001:00005730       ?LogTimeOut@CHLogger@@SAXPBDZZ 00406730 f   HostLogger.obj
 0001:000058c0       ?_BuildDirectory@CHLogger@@CAXABU_SYSTEMTIME@@@Z 004068c0 f   HostLogger.obj
 0001:00005d90       ?_CheckLevel@CHLogger@@CA?B_NW4ELOG_LEVEL@1@@Z 00406d90 f   HostLogger.obj
 0001:00005da0       ?_DoLogWithLevel@CHLogger@@CAXPBDW4ELOG_LEVEL@1@0PAD@Z 00406da0 f   HostLogger.obj
 0001:00005ff0       ?_InitPathNameInfo@CHLogger@@CAXPBD000@Z 00406ff0 f   HostLogger.obj
 0001:00006380       ?_Xran@?$_String_val@U?$_Simple_types@D@std@@@std@@SAXXZ 00407380 f i HostLogger.obj
 0001:00006390       ?append@?$basic_string@DU?$char_traits@D@std@@V?$allocator@D@2@@std@@QAEAAV12@QBDI@Z 00407390 f i HostLogger.obj
 0001:000064f0       ??$_Emplace_reallocate@ABQAX@?$vector@PAXV?$allocator@PAX@std@@@std@@QAEPAPAXQAPAXABQAX@Z 004074f0 f i LogMsgManager.obj
 0001:00006650       ??$sprintf_s@$0CA@@cf@@YAHAAY0CA@DPBDZZ 00407650 f i LogMsgManager.obj
 0001:00006680       ?Destroy@CLogMsgManager@@SAXXZ 00407680 f   LogMsgManager.obj
 0001:00006700       ?GetString@CLogMsgManager@@SA?BV?$basic_string@DU?$char_traits@D@std@@V?$allocator@D@2@@std@@I@Z 00407700 f   LogMsgManager.obj
 0001:00006720       ?Init@CLogMsgManager@@SA_NW4ESHARED_MEM_USAGE_TYPE@1@@Z 00407720 f   LogMsgManager.obj
 0001:00006890       ?_DoesSharedMemAlreadyExist@CLogMsgManager@@CA_NXZ 00407890 f   LogMsgManager.obj
 0001:000068b0       ?_GetMessageFromXls@CLogMsgManager@@CA?BV?$basic_string@DU?$char_traits@D@std@@V?$allocator@D@2@@std@@I@Z 004078b0 f   LogMsgManager.obj
 0001:000069e0       ?_LoadXlsData@CLogMsgManager@@CA_NXZ 004079e0 f   LogMsgManager.obj
 0001:00006a10       ?_OpenSharedMemoryHandles@CLogMsgManager@@CA_NXZ 00407a10 f   LogMsgManager.obj
 0001:00006b60       ?_SetLastError@CLogMsgManager@@CAXW4EERROR_TYPE@1@@Z 00407b60 f   LogMsgManager.obj
 0001:00006b70       ?_WaitTillOpen@CLogMsgManager@@CA_NK@Z 00407b70 f   LogMsgManager.obj
 0001:00006be0       ?_WaitTillValid@CLogMsgManager@@CA_NPCIK@Z 00407be0 f   LogMsgManager.obj
 0001:00006c20       ?_WriteXlsDataToSharedMemory@CLogMsgManager@@CA_NXZ 00407c20 f   LogMsgManager.obj
 0001:00006e70       ?_Xlength@?$vector@PAXV?$allocator@PAX@std@@@std@@CAXXZ 00407e70 f i LogMsgManager.obj
 0001:00006e80       ??$_Buynode@ABUpiecewise_construct_t@std@@V?$tuple@AB_J@2@V?$tuple@$$V@2@@?$_Tree_comp_alloc@V?$_Tmap_traits@_JV?$basic_string@DU?$char_traits@D@std@@V?$allocator@D@2@@std@@U?$less@_J@2@V?$allocator@U?$pair@$$CB_JV?$basic_string@DU?$char_traits@D@std@@V?$allocator@D@2@@std@@@std@@@2@$0A@@std@@@std@@QAEPAU?$_Tree_node@U?$pair@$$CB_JV?$basic_string@DU?$char_traits@D@std@@V?$allocator@D@2@@std@@@std@@PAX@1@ABUpiecewise_construct_t@1@$$QAV?$tuple@AB_J@1@$$QAV?$tuple@$$V@1@@Z 00407e80 f i LoadXlsMsg.obj
 0001:00006ec0       ??$_Insert_at@AAU?$pair@$$CB_JV?$basic_string@DU?$char_traits@D@std@@V?$allocator@D@2@@std@@@std@@PAU?$_Tree_node@U?$pair@$$CB_JV?$basic_string@DU?$char_traits@D@std@@V?$allocator@D@2@@std@@@std@@PAX@2@@?$_Tree@V?$_Tmap_traits@_JV?$basic_string@DU?$char_traits@D@std@@V?$allocator@D@2@@std@@U?$less@_J@2@V?$allocator@U?$pair@$$CB_JV?$basic_string@DU?$char_traits@D@std@@V?$allocator@D@2@@std@@@std@@@2@$0A@@std@@@std@@IAE?AV?$_Tree_iterator@V?$_Tree_val@U?$_Tree_simple_types@U?$pair@$$CB_JV?$basic_string@DU?$char_traits@D@std@@V?$allocator@D@2@@std@@@std@@@std@@@std@@@1@_NPAU?$_Tree_node@U?$pair@$$CB_JV?$basic_string@DU?$char_traits@D@std@@V?$allocator@D@2@@std@@@std@@PAX@1@AAU?$pair@$$CB_JV?$basic_string@DU?$char_traits@D@std@@V?$allocator@D@2@@std@@@1@1@Z 00407ec0 f i LoadXlsMsg.obj
 0001:00007020       ??$_Insert_hint@AAU?$pair@$$CB_JV?$basic_string@DU?$char_traits@D@std@@V?$allocator@D@2@@std@@@std@@PAU?$_Tree_node@U?$pair@$$CB_JV?$basic_string@DU?$char_traits@D@std@@V?$allocator@D@2@@std@@@std@@PAX@2@@?$_Tree@V?$_Tmap_traits@_JV?$basic_string@DU?$char_traits@D@std@@V?$allocator@D@2@@std@@U?$less@_J@2@V?$allocator@U?$pair@$$CB_JV?$basic_string@DU?$char_traits@D@std@@V?$allocator@D@2@@std@@@std@@@2@$0A@@std@@@std@@IAE?AV?$_Tree_iterator@V?$_Tree_val@U?$_Tree_simple_types@U?$pair@$$CB_JV?$basic_string@DU?$char_traits@D@std@@V?$allocator@D@2@@std@@@std@@@std@@@std@@@1@V?$_Tree_const_iterator@V?$_Tree_val@U?$_Tree_simple_types@U?$pair@$$CB_JV?$basic_string@DU?$char_traits@D@std@@V?$allocator@D@2@@std@@@std@@@std@@@std@@@1@AAU?$pair@$$CB_JV?$basic_string@DU?$char_traits@D@std@@V?$allocator@D@2@@std@@@1@PAU?$_Tree_node@U?$pair@$$CB_JV?$basic_string@DU?$char_traits@D@std@@V?$allocator@D@2@@std@@@std@@PAX@1@@Z 00408020 f i LoadXlsMsg.obj
 0001:00007280       ??$_Insert_nohint@AAU?$pair@$$CB_JV?$basic_string@DU?$char_traits@D@std@@V?$allocator@D@2@@std@@@std@@PAU?$_Tree_node@U?$pair@$$CB_JV?$basic_string@DU?$char_traits@D@std@@V?$allocator@D@2@@std@@@std@@PAX@2@@?$_Tree@V?$_Tmap_traits@_JV?$basic_string@DU?$char_traits@D@std@@V?$allocator@D@2@@std@@U?$less@_J@2@V?$allocator@U?$pair@$$CB_JV?$basic_string@DU?$char_traits@D@std@@V?$allocator@D@2@@std@@@std@@@2@$0A@@std@@@std@@IAE?AU?$pair@V?$_Tree_iterator@V?$_Tree_val@U?$_Tree_simple_types@U?$pair@$$CB_JV?$basic_string@DU?$char_traits@D@std@@V?$allocator@D@2@@std@@@std@@@std@@@std@@@std@@_N@1@_NAAU?$pair@$$CB_JV?$basic_string@DU?$char_traits@D@std@@V?$allocator@D@2@@std@@@1@PAU?$_Tree_node@U?$pair@$$CB_JV?$basic_string@DU?$char_traits@D@std@@V?$allocator@D@2@@std@@@std@@PAX@1@@Z 00408280 f i LoadXlsMsg.obj
 0001:000073c0       ??0FindXlsMsg@@QAE@XZ      004083c0 f   LoadXlsMsg.obj
 0001:00007410       ??1FindXlsMsg@@UAE@XZ      00408410 f   LoadXlsMsg.obj
 0001:00007510       ??A?$map@_JV?$basic_string@DU?$char_traits@D@std@@V?$allocator@D@2@@std@@U?$less@_J@2@V?$allocator@U?$pair@$$CB_JV?$basic_string@DU?$char_traits@D@std@@V?$allocator@D@2@@std@@@std@@@2@@std@@QAEAAV?$basic_string@DU?$char_traits@D@std@@V?$allocator@D@2@@1@AB_J@Z 00408510 f i LoadXlsMsg.obj
 0001:000075b0       ??E?$_Tree_const_iterator@V?$_Tree_val@U?$_Tree_simple_types@U?$pair@$$CB_JV?$basic_string@DU?$char_traits@D@std@@V?$allocator@D@2@@std@@@std@@@std@@@std@@@std@@QAEAAV01@XZ 004085b0 f i LoadXlsMsg.obj
 0001:00007610       ??F?$_Tree_const_iterator@V?$_Tree_val@U?$_Tree_simple_types@U?$pair@$$CB_JV?$basic_string@DU?$char_traits@D@std@@V?$allocator@D@2@@std@@@std@@@std@@@std@@@std@@QAEAAV01@XZ 00408610 f i LoadXlsMsg.obj
 0001:000076a0       ??R?$less@_J@std@@QBE_NAB_J0@Z 004086a0 f i LoadXlsMsg.obj
 0001:000076d0       ??Y?$basic_string@DU?$char_traits@D@std@@V?$allocator@D@2@@std@@QAEAAV01@QBD@Z 004086d0 f i LoadXlsMsg.obj
 0001:00007830       ??_GFindXlsMsg@@UAEPAXI@Z  00408830 f i LoadXlsMsg.obj
 0001:00007830       ??_EFindXlsMsg@@UAEPAXI@Z  00408830 f i LoadXlsMsg.obj
 0001:00007860       ?CheckAndChangeNewLineCommand@FindXlsMsg@@AAEXPAD@Z 00408860 f   LoadXlsMsg.obj
 0001:000078a0       ?GetMessageByIndex@FindXlsMsg@@QAEPBD_JPAD@Z 004088a0 f   LoadXlsMsg.obj
 0001:000078c0       ?LoadWMszFile@FindXlsMsg@@QAE_NPAD@Z 004088c0 f   LoadXlsMsg.obj
 0001:00007cf0       ?_Buyheadnode@?$_Tree_comp_alloc@V?$_Tmap_traits@_JV?$basic_string@DU?$char_traits@D@std@@V?$allocator@D@2@@std@@U?$less@_J@2@V?$allocator@U?$pair@$$CB_JV?$basic_string@DU?$char_traits@D@std@@V?$allocator@D@2@@std@@@std@@@2@$0A@@std@@@std@@QAEPAU?$_Tree_node@U?$pair@$$CB_JV?$basic_string@DU?$char_traits@D@std@@V?$allocator@D@2@@std@@@std@@PAX@2@XZ 00408cf0 f i LoadXlsMsg.obj
 0001:00007d10       ?_Buynode0@?$_Tree_comp_alloc@V?$_Tmap_traits@_JV?$basic_string@DU?$char_traits@D@std@@V?$allocator@D@2@@std@@U?$less@_J@2@V?$allocator@U?$pair@$$CB_JV?$basic_string@DU?$char_traits@D@std@@V?$allocator@D@2@@std@@@std@@@2@$0A@@std@@@std@@QAEPAU?$_Tree_node@U?$pair@$$CB_JV?$basic_string@DU?$char_traits@D@std@@V?$allocator@D@2@@std@@@std@@PAX@2@XZ 00408d10 f i LoadXlsMsg.obj
 0001:00007d30       ?_Destroy_if_node@?$_Tree@V?$_Tmap_traits@_JV?$basic_string@DU?$char_traits@D@std@@V?$allocator@D@2@@std@@U?$less@_J@2@V?$allocator@U?$pair@$$CB_JV?$basic_string@DU?$char_traits@D@std@@V?$allocator@D@2@@std@@@std@@@2@$0A@@std@@@std@@IAEXPAU?$_Tree_node@U?$pair@$$CB_JV?$basic_string@DU?$char_traits@D@std@@V?$allocator@D@2@@std@@@std@@PAX@2@@Z 00408d30 f i LoadXlsMsg.obj
 0001:00007d90       ?_Erase@?$_Tree@V?$_Tmap_traits@_JV?$basic_string@DU?$char_traits@D@std@@V?$allocator@D@2@@std@@U?$less@_J@2@V?$allocator@U?$pair@$$CB_JV?$basic_string@DU?$char_traits@D@std@@V?$allocator@D@2@@std@@@std@@@2@$0A@@std@@@std@@IAEXPAU?$_Tree_node@U?$pair@$$CB_JV?$basic_string@DU?$char_traits@D@std@@V?$allocator@D@2@@std@@@std@@PAX@2@@Z 00408d90 f i LoadXlsMsg.obj
 0001:00007e20       ?_Lrotate@?$_Tree_val@U?$_Tree_simple_types@U?$pair@$$CB_JV?$basic_string@DU?$char_traits@D@std@@V?$allocator@D@2@@std@@@std@@@std@@@std@@QAEXPAU?$_Tree_node@U?$pair@$$CB_JV?$basic_string@DU?$char_traits@D@std@@V?$allocator@D@2@@std@@@std@@PAX@2@@Z 00408e20 f i LoadXlsMsg.obj
 0001:00007e80       ?_Rrotate@?$_Tree_val@U?$_Tree_simple_types@U?$pair@$$CB_JV?$basic_string@DU?$char_traits@D@std@@V?$allocator@D@2@@std@@@std@@@std@@@std@@QAEXPAU?$_Tree_node@U?$pair@$$CB_JV?$basic_string@DU?$char_traits@D@std@@V?$allocator@D@2@@std@@@std@@PAX@2@@Z 00408e80 f i LoadXlsMsg.obj
 0001:00007ee0       ??0CServerAppApp@@QAE@XZ   00408ee0 f   ServerApp.obj
 0001:00007f00       ??1CServerAppApp@@UAE@XZ   00408f00 f   ServerApp.obj
 0001:00007f10       ??_ECServerAppApp@@UAEPAXI@Z 00408f10 f i ServerApp.obj
 0001:00007f10       ??_GCServerAppApp@@UAEPAXI@Z 00408f10 f i ServerApp.obj
 0001:00007f50       ?Dump@CObject@@UBEXAAVCDumpContext@@@Z 00408f50 f i ServerApp.obj
 0001:00007f50       ?DoDataExchange@CWnd@@MAEXPAVCDataExchange@@@Z 00408f50 f i ServerAppDlg.obj
 0001:00007f50       ?Serialize@CObject@@UAEXAAVCArchive@@@Z 00408f50 f i ServerApp.obj
 0001:00007f60       __matherr                  00408f60 f i msvcrt:matherr.obj
 0001:00007f60       __get_startup_thread_locale_mode 00408f60 f i msvcrt:thread_locale.obj
 0001:00007f60       ?GetApplicationRestartFlags@CWinApp@@UAEKXZ 00408f60 f i ServerApp.obj
 0001:00007f60       ___scrt_exe_initialize_mta 00408f60 f i msvcrt:utility_desktop.obj
 0001:00007f60       __get_startup_new_mode     00408f60 f i msvcrt:new_mode.obj
 0001:00007f60       ___scrt_initialize_winrt   00408f60 f i msvcrt:utility_desktop.obj
 0001:00007f60       __get_startup_commit_mode  00408f60 f i msvcrt:commit_mode.obj
 0001:00007f60       ___scrt_stub_for_initialize_mta 00408f60 f i msvcrt:utility_desktop.obj
 0001:00007f60       ?GetApplicationRecoveryParameter@CWinApp@@UAEPAXXZ 00408f60 f i ServerApp.obj
 0001:00007f70       ?GetApplicationRecoveryPingInterval@CWinApp@@UAEKXZ 00408f70 f i ServerApp.obj
 0001:00007f80       ?GetMessageMap@CServerAppApp@@MBEPBUAFX_MSGMAP@@XZ 00408f80 f   ServerApp.obj
 0001:00007f90       ?GetThisMessageMap@CServerAppApp@@KGPBUAFX_MSGMAP@@XZ 00408f90 f   ServerApp.obj
 0001:00007fa0       ?InitInstance@CServerAppApp@@UAEHXZ 00408fa0 f   ServerApp.obj
 0001:00007fb0       ?ReopenPreviousFilesAtRestart@CWinApp@@UBEHXZ 00408fb0 f i ServerApp.obj
 0001:00007fc0       ?RestoreAutosavedFilesAtRestart@CWinApp@@UBEHXZ 00408fc0 f i ServerApp.obj
 0001:00007fd0       ?Run@CServerAppApp@@UAEHXZ 00408fd0 f   ServerApp.obj
 0001:00008050       ?SupportsApplicationRecovery@CWinApp@@UBEHXZ 00409050 f i ServerApp.obj
 0001:00008060       ?SupportsAutosaveAtInterval@CWinApp@@UBEHXZ 00409060 f i ServerApp.obj
 0001:00008070       ?SupportsAutosaveAtRestart@CWinApp@@UBEHXZ 00409070 f i ServerApp.obj
 0001:00008080       ?SupportsRestartManager@CWinApp@@UBEHXZ 00409080 f i ServerApp.obj
 0001:00008090       _IsDebugMode               00409090 f   ServerApp.obj
 0001:000080a0       ?APIRemoved@?$CAPIHolder@VILTCommon@@@@UAEXXZ 004090a0 f i ServerAppDlg.obj
 0001:000080b0       ?APIFound@?$CAPIHolder@VILTCommon@@@@UAEXPAVIBase@@@Z 004090b0 f i ServerAppDlg.obj
 0001:000080c0       ?Interface@?$CAPIHolder@VILTCommon@@@@UAEPAVIBase@@XZ 004090c0 f i ServerAppDlg.obj
 0001:000080d0       ??_G?$CAPIHolder@VILTCommon@@@@UAEPAXI@Z 004090d0 f i ServerAppDlg.obj
 0001:000080d0       ??_E?$CAPIHolder@VILTCommon@@@@UAEPAXI@Z 004090d0 f i ServerAppDlg.obj
 0001:00008100       ??$?HDU?$char_traits@D@std@@V?$allocator@D@1@@std@@YA?AV?$basic_string@DU?$char_traits@D@std@@V?$allocator@D@2@@0@ABV10@0@Z 00409100 f i ServerAppDlg.obj
 0001:000081b0       ??$_Traits_find@U?$char_traits@D@std@@@std@@YAIQBDII0I@Z 004091b0 f i ServerAppDlg.obj
 0001:000082a0       ??$sprintf_s@$0BAA@@cf@@YAHAAY0BAA@DPBDZZ 004092a0 f i ServerAppDlg.obj
 0001:000082d0       ??$sprintf_s@$0BAE@@cf@@YAHAAY0BAE@DPBDZZ 004092d0 f i ServerAppDlg.obj
 0001:00008300       ??$sprintf_s@$0IA@@cf@@YAHAAY0IA@DPBDZZ 00409300 f i ServerAppDlg.obj
 0001:00008330       ??$strcpy_s@$0L@@cf@@YAHAAY0L@DPBD@Z 00409330 f i ServerAppDlg.obj
 0001:00008350       ??$strncpy_s@$0BAAA@@cf@@YAHAAY0BAAA@DPBDI@Z 00409350 f i ServerAppDlg.obj
 0001:00008370       ??$strncpy_s@$0L@@cf@@YAHAAY0L@DPBDI@Z 00409370 f i ServerAppDlg.obj
 0001:00008390       ??0?$CAPIHolder@VILTCommon@@@@QAE@PBDAAPAVILTCommon@@H@Z 00409390 f i ServerAppDlg.obj
 0001:00008400       ??0?$basic_string@DU?$char_traits@D@std@@V?$allocator@D@2@@std@@QAE@ABV01@@Z 00409400 f i ServerAppDlg.obj
 0001:00008490       ??0BATTLE_ROYAL_RESULT_USER@@QAE@XZ 00409490 f i ServerAppDlg.obj
 0001:000084f0       ??0CServerAppDlg@@QAE@PAVCWnd@@@Z 004094f0 f   ServerAppDlg.obj
 0001:00008720       ??0PROTO_GAMEGT_MAPLOADING_COMPLETE_NTY_tag@@QAE@XZ 00409720 f i ServerAppDlg.obj
 0001:00008750       ??0PROTO_GAME_USER_INFO_tag@@QAE@XZ 00409750 f i ServerAppDlg.obj
 0001:00008920       ??0PROTO_SERVERAPPMSG_INIT@@QAE@XZ 00409920 f i ServerAppDlg.obj
 0001:00008960       ??0PROTO_START_HOST_tag@@QAE@XZ 00409960 f i ServerAppDlg.obj
 0001:000089c0       ??0exception@std@@QAE@ABV01@@Z 004099c0 f i ServerAppDlg.obj
 0001:000089f0       ??0exception@std@@QAE@QBD@Z 004099f0 f i ServerAppDlg.obj
 0001:00008a30       ??1?$CAPIHolder@VILTCommon@@@@UAE@XZ 00409a30 f i ServerAppDlg.obj
 0001:00008a90       ??1CServerAppDlg@@UAE@XZ   00409a90 f   ServerAppDlg.obj
 0001:00008bb0       ??1CWaitCursor@@QAE@XZ     00409bb0 f i ServerAppDlg.obj
 0001:00008cd0       ??1exception@std@@UAE@XZ   00409cd0 f i ServerAppDlg.obj
 0001:00008cf0       ??1tUCCGamePlayInfo@CServerAppDlg@@QAE@XZ 00409cf0 f i ServerAppDlg.obj
 0001:00008d40       ??4?$basic_string@DU?$char_traits@D@std@@V?$allocator@D@2@@std@@QAEAAV01@$$QAV01@@Z 00409d40 f i ServerAppDlg.obj
 0001:00008d80       ??_ECEdit@@UAEPAXI@Z       00409d80 f i ServerAppDlg.obj
 0001:00008d80       ??_GCEdit@@UAEPAXI@Z       00409d80 f i ServerAppDlg.obj
 0001:00008dc0       ??_GCListBox@@UAEPAXI@Z    00409dc0 f i ServerAppDlg.obj
 0001:00008dc0       ??_ECListBox@@UAEPAXI@Z    00409dc0 f i ServerAppDlg.obj
 0001:00008e00       ??_GCServerAppDlg@@UAEPAXI@Z 00409e00 f i ServerAppDlg.obj
 0001:00008e00       ??_ECServerAppDlg@@UAEPAXI@Z 00409e00 f i ServerAppDlg.obj
 0001:00008e40       ??_Eexception@std@@UAEPAXI@Z 00409e40 f i ServerAppDlg.obj
 0001:00008e40       ??_Gexception@std@@UAEPAXI@Z 00409e40 f i ServerAppDlg.obj
 0001:00008e70       ?AddResources@CServerAppDlg@@QAE_NXZ 00409e70 f   ServerAppDlg.obj
 0001:00009110       ?AddServerMsg@CServerAppDlg@@QAEXPBDH@Z 0040a110 f   ServerAppDlg.obj
 0001:00009270       ?BeginModalState@CWnd@@UAEXXZ 0040a270 f i ServerAppDlg.obj
 0001:00009280       ?ConsoleOutputFn@CGameServerAppHandler@@UAEIHHPBD@Z 0040a280 f   ServerAppDlg.obj
 0001:000094c0       ?ConsoleOutputFn@CGameServerAppHandler@@UAEIPBD@Z 0040a4c0 f   ServerAppDlg.obj
 0001:000094e0       ?Create@CDialog@@UAEHIPAVCWnd@@@Z 0040a4e0 f i ServerAppDlg.obj
 0001:000094f0       ?Destroy@CServerAppDlg@@QAEXXZ 0040a4f0 f   ServerAppDlg.obj
 0001:00009530       ?DoDataExchange@CServerAppDlg@@MAEXPAVCDataExchange@@@Z 0040a530 f   ServerAppDlg.obj
 0001:00009570       ?DoHost@CServerAppDlg@@QAE_NXZ 0040a570 f   ServerAppDlg.obj
 0001:000096b0       ?DownloadUCCMapFile_HTTP@CServerAppDlg@@AAE?AW4UCCMAPDOWNLOADREAULT@@V?$basic_string@DU?$char_traits@D@std@@V?$allocator@D@2@@std@@@Z 0040a6b0 f   ServerAppDlg.obj
 0001:00009d60       ?EndModalState@CWnd@@UAEXXZ 0040ad60 f i ServerAppDlg.obj
 0001:00009d70       ?GetCPUUtilization@ServerAppHandler@@UAEMXZ 0040ad70 f i ServerAppDlg.obj
 0001:00009d80       ?GetDownloadPath@CServerAppDlg@@AAE?AV?$basic_string@DU?$char_traits@D@std@@V?$allocator@D@2@@std@@XZ 0040ad80 f   ServerAppDlg.obj
 0001:00009e80       ?GetLogFileDir@ServerAppHandler@@UAE_NPADH@Z 0040ae80 f i ServerAppDlg.obj
 0001:00009e90       ?GetMessageMap@CServerAppDlg@@MBEPBUAFX_MSGMAP@@XZ 0040ae90 f   ServerAppDlg.obj
 0001:00009ea0       ?GetOptionValueString@CServerAppDlg@@IAE?AV?$basic_string@DU?$char_traits@D@std@@V?$allocator@D@2@@std@@V23@00@Z 0040aea0 f   ServerAppDlg.obj
 0001:0000a2b0       ?GetProcessMemoryUsage@CGameServerAppHandler@@UAEKXZ 0040b2b0 f   ServerAppDlg.obj
 0001:0000a3c0       ?GetThisMessageMap@CServerAppDlg@@KGPBUAFX_MSGMAP@@XZ 0040b3c0 f   ServerAppDlg.obj
 0001:0000a3d0       ?GetUpdateInterval@@YAJFW4ROUNDTYPE@@W4DEATHMATCHTYPE@@@Z 0040b3d0 f   ServerAppDlg.obj
 0001:0000a420       ?HaveFile@CServerAppDlg@@AAE_NV?$basic_string@DU?$char_traits@D@std@@V?$allocator@D@2@@std@@@Z 0040b420 f   ServerAppDlg.obj
 0001:0000a4a0       ?IsGameEnded@CGameServerAppHandler@@UAE_NXZ 0040b4a0 f i ServerAppDlg.obj
 0001:0000a4b0       ?IsReadProcessMemory@CServerAppDlg@@QAE_NXZ 0040b4b0 f   ServerAppDlg.obj
 0001:0000a4c0       ?IsWriteProcessMemory@CServerAppDlg@@QAE_NXZ 0040b4c0 f   ServerAppDlg.obj
 0001:0000a4d0       ?LoadHostGameInfo@CServerAppDlg@@IAEXXZ 0040b4d0 f   ServerAppDlg.obj
 0001:0000a830       ?LoadServer@CServerAppDlg@@QAE_NXZ 0040b830 f   ServerAppDlg.obj
 0001:0000aa10       ?NetworkDelayCount@CGameServerAppHandler@@UAEIXZ 0040ba10 f   ServerAppDlg.obj
 0001:0000aa20       ?NetworkDelayCount@CServerAppDlg@@QAEXXZ 0040ba20 f   ServerAppDlg.obj
 0001:0000aa50       ?OnBnClickedButtonGo@CServerAppDlg@@QAEXXZ 0040ba50 f   ServerAppDlg.obj
 0001:0000ab10       ?OnButtonStartServer@CServerAppDlg@@QAEHXZ 0040bb10 f   ServerAppDlg.obj
 0001:0000ac10       ?OnCopyData@CServerAppDlg@@IAEHPAVCWnd@@PAUtagCOPYDATASTRUCT@@@Z 0040bc10 f   ServerAppDlg.obj
 0001:0000b720       ?OnGameServerMsg@CServerAppDlg@@IAEJIJ@Z 0040c720 f   ServerAppDlg.obj
 0001:0000bc70       ?OnInitDialog@CServerAppDlg@@MAEHXZ 0040cc70 f   ServerAppDlg.obj
 0001:0000c3b0       ?OnPaint@CServerAppDlg@@IAEXXZ 0040d3b0 f   ServerAppDlg.obj
 0001:0000c3c0       ?OnQueryDragIcon@CServerAppDlg@@IAEPAUHICON__@@XZ 0040d3c0 f   ServerAppDlg.obj
 0001:0000c3d0       ?OnShellMessage@CServerAppDlg@@QAEXAAVILTMessage_Read@@@Z 0040d3d0 f   ServerAppDlg.obj
 0001:0000e930       ?OnTimer@CServerAppDlg@@QAEXI@Z 0040f930 f   ServerAppDlg.obj
 0001:0000ead0       ?OutOfMemory@CGameServerAppHandler@@UAEIXZ 0040fad0 f   ServerAppDlg.obj
 0001:0000eb80       ?PostMessageToWriteLogFile@CServerAppDlg@@AAE_NIW4GAMESERVERMSG@@JPAX@Z 0040fb80 f   ServerAppDlg.obj
 0001:0000ec60       ?PostReadData@GAMEPROTO_SC_COMMON@@UAE_NPAVILTMessage_Read@@@Z 0040fc60 f i ServerAppDlg.obj
 0001:0000ece0       ?PostWriteData@GAMEPROTO_SC_COMMON@@UAE_NPAVILTMessage_Write@@@Z 0040fce0 f i ServerAppDlg.obj
 0001:0000ed30       ?PreWriteData@GAMEPROTO_SC_COMMON@@UAE_NPAVILTMessage_Write@@@Z 0040fd30 f i ServerAppDlg.obj
 0001:0000ed30       ?PreReadData@GAMEPROTO_SC_COMMON@@UAE_NPAVILTMessage_Read@@@Z 0040fd30 f i ServerAppDlg.obj
 0001:0000ed40       ?ProcessPacket@ServerAppHandler@@UAEIAAVILTMessage_Read@@QAEG@Z 0040fd40 f i ServerAppDlg.obj
 0001:0000ed50       ?RECV_MSG_AIITEM_DEC@CServerAppDlg@@AAEXJ@Z 0040fd50 f   ServerAppDlg.obj
 0001:0000ef50       ?RECV_MSG_AIITEM_GROUP_RATE_RESULT@CServerAppDlg@@AAEXJ@Z 0040ff50 f   ServerAppDlg.obj
 0001:0000f160       ?RECV_MSG_INSERTCHARACTER@CServerAppDlg@@AAEXJ@Z 00410160 f   ServerAppDlg.obj
 0001:0000f330       ?RECV_MSG_ROOMINFO@CServerAppDlg@@AAEXJ@Z 00410330 f   ServerAppDlg.obj
 0001:0000f450       ?RECV_MSG_RPM_ADDRESS@CServerAppDlg@@AAEXJ@Z 00410450 f   ServerAppDlg.obj
 0001:0000f4e0       ?RECV_MSG_USER_DISCONNECTED@CServerAppDlg@@AAEXJ@Z 004104e0 f   ServerAppDlg.obj
 0001:0000f7c0       ?ReadData@PROTO_SERVERAPPMSG_INIT@@UAE_NPAVILTMessage_Read@@@Z 004107c0 f i ServerAppDlg.obj
 0001:0000f830       ?ReadGSMMemory@CServerAppDlg@@QAE_NPAX0K@Z 00410830 f   ServerAppDlg.obj
 0001:0000f970       ?Readint32@ILTMessage_Read@@QAEHXZ 00410970 f i ServerAppDlg.obj
 0001:0000f970       ?Readuint32@ILTMessage_Read@@QAEIXZ 00410970 f i ServerAppDlg.obj
 0001:0000f9b0       ?RunServer@CServerAppDlg@@QAE_NXZ 004109b0 f   ServerAppDlg.obj
 0001:0000fb10       ?SaveHostGameInfo@CServerAppDlg@@IAEXXZ 00410b10 f   ServerAppDlg.obj
 0001:0000fcf0       ?SendMessageToWriteLogFile@CServerAppDlg@@QAEXPAUHWND__@@0AAUtagCOPYDATASTRUCT@@@Z 00410cf0 f   ServerAppDlg.obj
 0001:0000fd10       ?SendServerAppInit@CServerAppDlg@@AAEXXZ 00410d10 f   ServerAppDlg.obj
 0001:0000fe70       ?SendServerAppInitFail@CServerAppDlg@@AAEXHH@Z 00410e70 f   ServerAppDlg.obj
 0001:0000ff90       ?ServerUpdate@CServerAppDlg@@QAEXXZ 00410f90 f   ServerAppDlg.obj
 0001:00010170       ?SetService@CServerAppDlg@@QAE_NXZ 00411170 f   ServerAppDlg.obj
 0001:00010200       ?ShellMessageFn@CGameServerAppHandler@@UAEIAAVILTMessage_Read@@@Z 00411200 f   ServerAppDlg.obj
 0001:00010220       ?StopServer@CServerAppDlg@@QAE_NXZ 00411220 f   ServerAppDlg.obj
 0001:00010390       ?ThreadUpdate@CServerAppDlg@@SAXPAX@Z 00411390 f   ServerAppDlg.obj
 0001:00010840       ?Thread_SendGameInfo@@YAXPAVCServerAppDlg@@AAUPROTO_START_HOST_tag@@@Z 00411840 f   ServerAppDlg.obj
 0001:00011840       ?Thread_SendUserInfo@@YAXPAVCServerAppDlg@@AAUPROTO_GAME_USER_INFO_tag@@@Z 00412840 f   ServerAppDlg.obj
 0001:000122a0       ?UpdateLocalHostGameInfo@CServerAppDlg@@IAEXXZ 004132a0 f   ServerAppDlg.obj
 0001:000122b0       ?WriteData@PROTO_SERVERAPPMSG_INIT@@UAE_NPAVILTMessage_Write@@@Z 004132b0 f i ServerAppDlg.obj
 0001:00012350       ?WriteGSMMemory@CServerAppDlg@@QAE_NW4GAMESERVERMSG@@HPAXK@Z 00413350 f   ServerAppDlg.obj
 0001:00012480       ?_HLOG_MSG_Init@CServerAppDlg@@IAEHXZ 00413480 f   ServerAppDlg.obj
 0001:00012550       ?reserve@?$basic_string@DU?$char_traits@D@std@@V?$allocator@D@2@@std@@QAEXI@Z 00413550 f i ServerAppDlg.obj
 0001:000126b0       ?what@exception@std@@UBEPBDXZ 004136b0 f i ServerAppDlg.obj
 0001:000126c0       ___local_stdio_scanf_options 004136c0 f i ServerAppDlg.obj
 0001:000126d0       _fscanf_s                  004136d0 f i ServerAppDlg.obj
 0001:00012700       ??$sprintf_s@$0BE@@cf@@YAHAAY0BE@DPBDZZ 00413700 f i BugReporter1.obj
 0001:00012730       ??$sprintf_s@$0BJB@@cf@@YAHAAY0BJB@DPBDZZ 00413730 f i BugReporter1.obj
 0001:00012760       ??$sprintf_s@$0DOJ@@cf@@YAHAAY0DOJ@DPBDZZ 00413760 f i BugReporter1.obj
 0001:00012790       ??$strcpy_s@$0GF@@cf@@YAHAAY0GF@DPBD@Z 00413790 f i BugReporter1.obj
 0001:00012820       ?CrashExceptionDump@@YGJPAU_EXCEPTION_POINTERS@@@Z 00413820 f   BugReporter1.obj
 0001:00012870       ?CrashExceptionNoneDump@@YGJPAU_EXCEPTION_POINTERS@@@Z 00413870 f   BugReporter1.obj
 0001:00012890       ?InitBugReporter@@YAXPAD0000@Z 00413890 f   BugReporter1.obj
 0001:00012b80       ?InvalidParameterHandler@@YAXPB_W00II@Z 00413b80 f   BugReporter1.obj
 0001:00012ba0       ?ResetBugReporter@@YAXXZ   00413ba0 f   BugReporter1.obj
 0001:00012bb0       ?SetLogFolder@@YAXPAD@Z    00413bb0 f   BugReporter1.obj
 0001:00012ce0       ?threadCreateDumpFile@@YGKPAX@Z 00413ce0 f   BugReporter1.obj
 0001:00012f50       __snprintf_s               00413f50 f i BugReporter1.obj
 0001:00012f90       ??$_snprintf_s@$0IA@@@YAHAAY0IA@DIPBDZZ 00413f90 f i crs_uploader1.obj
 0001:00012fd0       ??$makeFilename@$0BAE@@Uploader@crs@@AAEXAAU_SYSTEMTIME@@PA_WAAY0BAE@_W@Z 00413fd0 f i crs_uploader1.obj
 0001:00013040       ??0Uploader@crs@@QAE@XZ    00414040 f   crs_uploader1.obj
 0001:00013190       ??1?$auto_ptr@VUrl@crs@@@std@@QAE@XZ 00414190 f i crs_uploader1.obj
 0001:00013200       ??1?$basic_string@_WU?$char_traits@_W@std@@V?$allocator@_W@2@@std@@QAE@XZ 00414200 f i crs_uploader1.obj
 0001:00013210       ?close@FileHandle@crs@@QAEXXZ 00414210 f i crs_uploader1.obj
 0001:00013210       ??1FileHandle@crs@@QAE@XZ  00414210 f i crs_uploader1.obj
 0001:00013230       ??1Uploader@crs@@QAE@XZ    00414230 f   crs_uploader1.obj
 0001:00013390       ?_Tidy_deallocate@?$basic_string@_WU?$char_traits@_W@std@@V?$allocator@_W@2@@std@@QAEXXZ 00414390 f i crs_uploader1.obj
 0001:000133f0       ?allocate@?$allocator@_W@std@@QAEPA_WI@Z 004143f0 f i crs_uploader1.obj
 0001:00013460       ?append@?$basic_string@_WU?$char_traits@_W@std@@V?$allocator@_W@2@@std@@QAEAAV12@QB_WI@Z 00414460 f i crs_uploader1.obj
 0001:000135e0       ?assign@?$basic_string@_WU?$char_traits@_W@std@@V?$allocator@_W@2@@std@@QAEAAV12@QB_WI@Z 004145e0 f i crs_uploader1.obj
 0001:000136f0       ?disabled@Uploader@crs@@AAE_NXZ 004146f0 f   crs_uploader1.obj
 0001:00013700       ?error@Uploader@crs@@AAA_NPBDZZ 00414700 f i crs_uploader1.obj
 0001:00013730       ?init@Uploader@crs@@QAE_N_NPAD1@Z 00414730 f   crs_uploader1.obj
 0001:00013af0       ?makeBaseInfo@Uploader@crs@@AAEXPAD0@Z 00414af0 f i crs_uploader1.obj
 0001:00013d10       ?makeExceptionLog@Uploader@crs@@QAEXPAU_EXCEPTION_POINTERS@@AAVLogBuffer@2@@Z 00414d10 f   crs_uploader1.obj
 0001:00013f80       ?prepare@Uploader@crs@@AAE_NAAVHttpHandles@2@@Z 00414f80 f   crs_uploader1.obj
 0001:00014050       ?readURL@Uploader@crs@@AAEXAAV?$basic_string@_WU?$char_traits@_W@std@@V?$allocator@_W@2@@std@@@Z 00415050 f i crs_uploader1.obj
 0001:000143d0       ?recordExceptionLog@Uploader@crs@@QAAXAAVLogBuffer@2@PBDZZ 004153d0 f i crs_uploader1.obj
 0001:000144a0       ?set@Url@crs@@QAEKABV?$basic_string@_WU?$char_traits@_W@std@@V?$allocator@_W@2@@std@@@Z 004154a0 f i crs_uploader1.obj
 0001:00014750       ?success@Uploader@crs@@AAE_NPBDAAVHttpHandle@2@@Z 00415750 f   crs_uploader1.obj
 0001:00014830       ?upload@Uploader@crs@@QAE_N_NABV?$basic_string@DU?$char_traits@D@std@@V?$allocator@D@2@@std@@AAVLogBuffer@2@@Z 00415830 f   crs_uploader1.obj
 0001:00014ab0       ?uploadHTTP@Uploader@crs@@AAE_NAAVHttpHandle@2@PBDPB_W2@Z 00415ab0 f   crs_uploader1.obj
 0001:00014e40       ?uploadLOG@Uploader@crs@@AAE_NAAVHttpHandle@2@AAU_SYSTEMTIME@@AAVLogBuffer@2@@Z 00415e40 f   crs_uploader1.obj
 0001:00015060       ?uploadVersion@Uploader@crs@@QAE_NXZ 00416060 f   crs_uploader1.obj
 0001:00015180       ?urlChar@Uploader@crs@@QAEPBDXZ 00416180 f   crs_uploader1.obj
 0001:00015190       __snwprintf_s              00416190 f i crs_uploader1.obj
 0001:000151d0       ??0CServerLog@@QAE@H@Z     004161d0 f   LogMgmt1.obj
 0001:000152d0       ??1CServerLog@@UAE@XZ      004162d0 f   LogMgmt1.obj
 0001:00015390       ??_ECServerLog@@UAEPAXI@Z  00416390 f i LogMgmt1.obj
 0001:00015390       ??_GCServerLog@@UAEPAXI@Z  00416390 f i LogMgmt1.obj
 0001:000153b6       _GetProcessMemoryInfo@12   004163b6 f   Psapi:PSAPI.DLL
 0001:000153bc       ??3@YAXPAX@Z               004163bc f   mfc140:mfc140.dll
 0001:000153c2       ??2@YAPAXI@Z               004163c2 f   mfc140:mfc140.dll
 0001:000153c8       ??_U@YAPAXI@Z              004163c8 f   mfc140:mfc140.dll
 0001:000153ce       ??_V@YAXPAX@Z              004163ce f   mfc140:mfc140.dll
 0001:000153d4       ?OnCmdMsg@CCmdTarget@@UAEHIHPAXPAUAFX_CMDHANDLERINFO@@@Z 004163d4 f   mfc140:mfc140.dll
 0001:000153da       ?OnFinalRelease@CCmdTarget@@UAEXXZ 004163da f   mfc140:mfc140.dll
 0001:000153e0       ?IsInvokeAllowed@CCmdTarget@@UAEHJ@Z 004163e0 f   mfc140:mfc140.dll
 0001:000153e6       ?GetDispatchIID@CCmdTarget@@UAEHPAU_GUID@@@Z 004163e6 f   mfc140:mfc140.dll
 0001:000153ec       ?GetTypeInfoCount@CCmdTarget@@UAEIXZ 004163ec f   mfc140:mfc140.dll
 0001:000153f2       ?GetTypeLibCache@CCmdTarget@@UAEPAVCTypeLibCache@@XZ 004163f2 f   mfc140:mfc140.dll
 0001:000153f8       ?GetTypeLib@CCmdTarget@@UAEJKPAPAUITypeLib@@@Z 004163f8 f   mfc140:mfc140.dll
 0001:000153fe       ?GetCommandMap@CCmdTarget@@MBEPBUAFX_OLECMDMAP@@XZ 004163fe f   mfc140:mfc140.dll
 0001:00015404       ?GetDispatchMap@CCmdTarget@@MBEPBUAFX_DISPMAP@@XZ 00416404 f   mfc140:mfc140.dll
 0001:0001540a       ?GetConnectionMap@CCmdTarget@@MBEPBUAFX_CONNECTIONMAP@@XZ 0041640a f   mfc140:mfc140.dll
 0001:00015410       ?GetInterfaceMap@CCmdTarget@@MBEPBUAFX_INTERFACEMAP@@XZ 00416410 f   mfc140:mfc140.dll
 0001:00015416       ?GetEventSinkMap@CCmdTarget@@MBEPBUAFX_EVENTSINKMAP@@XZ 00416416 f   mfc140:mfc140.dll
 0001:0001541c       ?OnCreateAggregates@CCmdTarget@@UAEHXZ 0041641c f   mfc140:mfc140.dll
 0001:00015422       ?GetInterfaceHook@CCmdTarget@@UAEPAUIUnknown@@PBX@Z 00416422 f   mfc140:mfc140.dll
 0001:00015428       ?GetExtraConnectionPoints@CCmdTarget@@MAEHPAVCPtrArray@@@Z 00416428 f   mfc140:mfc140.dll
 0001:0001542e       ?GetConnectionHook@CCmdTarget@@MAEPAUIConnectionPoint@@ABU_GUID@@@Z 0041642e f   mfc140:mfc140.dll
 0001:00015434       ?DoModal@CDialog@@UAEHXZ   00416434 f   mfc140:mfc140.dll
 0001:0001543a       ?PreTranslateMessage@CWinThread@@UAEHPAUtagMSG@@@Z 0041643a f   mfc140:mfc140.dll
 0001:00015440       ?PumpMessage@CWinThread@@UAEHXZ 00416440 f   mfc140:mfc140.dll
 0001:00015446       ?IsIdleMessage@CWinThread@@UAEHPAUtagMSG@@@Z 00416446 f   mfc140:mfc140.dll
 0001:0001544c       ?ProcessMessageFilter@CWinThread@@UAEHHPAUtagMSG@@@Z 0041644c f   mfc140:mfc140.dll
 0001:00015452       ?GetMainWnd@CWinThread@@UAEPAVCWnd@@XZ 00416452 f   mfc140:mfc140.dll
 0001:00015458       ?Delete@CWinThread@@UAEXXZ 00416458 f   mfc140:mfc140.dll
 0001:0001545e       ?GetRuntimeClass@CWinApp@@UBEPAUCRuntimeClass@@XZ 0041645e f   mfc140:mfc140.dll
 0001:00015464       ??0CWinApp@@QAE@PBD@Z      00416464 f   mfc140:mfc140.dll
 0001:0001546a       ?GetProfileIntA@CWinApp@@UAEIPBD0H@Z 0041646a f   mfc140:mfc140.dll
 0001:00015470       ?WriteProfileInt@CWinApp@@UAEHPBD0H@Z 00416470 f   mfc140:mfc140.dll
 0001:00015476       ?GetProfileStringA@CWinApp@@UAE?AV?$CStringT@DV?$StrTraitMFC_DLL@DV?$ChTraitsCRT@D@ATL@@@@@ATL@@PBD00@Z 00416476 f   mfc140:mfc140.dll
 0001:0001547c       ?WriteProfileStringA@CWinApp@@UAEHPBD00@Z 0041647c f   mfc140:mfc140.dll
 0001:00015482       ?GetProfileBinary@CWinApp@@UAEHPBD0PAPAEPAI@Z 00416482 f   mfc140:mfc140.dll
 0001:00015488       ?WriteProfileBinary@CWinApp@@UAEHPBD0PAEI@Z 00416488 f   mfc140:mfc140.dll
 0001:0001548e       ?InitLibId@CWinApp@@UAEXXZ 0041648e f   mfc140:mfc140.dll
 0001:00015494       ?Register@CWinApp@@UAEHXZ  00416494 f   mfc140:mfc140.dll
 0001:0001549a       ?Unregister@CWinApp@@UAEHXZ 0041649a f   mfc140:mfc140.dll
 0001:000154a0       ?OpenDocumentFile@CWinApp@@UAEPAVCDocument@@PBD@Z 004164a0 f   mfc140:mfc140.dll
 0001:000154a6       ?OpenDocumentFile@CWinApp@@UAEPAVCDocument@@PBDH@Z 004164a6 f   mfc140:mfc140.dll
 0001:000154ac       ?AddToRecentFileList@CWinApp@@UAEXPBD@Z 004164ac f   mfc140:mfc140.dll
 0001:000154b2       ?InitApplication@CWinApp@@UAEHXZ 004164b2 f   mfc140:mfc140.dll
 0001:000154b8       ?SaveAllModified@CWinApp@@UAEHXZ 004164b8 f   mfc140:mfc140.dll
 0001:000154be       ?DoMessageBox@CWinApp@@UAEHPBDII@Z 004164be f   mfc140:mfc140.dll
 0001:000154c4       ?DoWaitCursor@CWinApp@@UAEXH@Z 004164c4 f   mfc140:mfc140.dll
 0001:000154ca       ?OnDDECommand@CWinApp@@UAEHPAD@Z 004164ca f   mfc140:mfc140.dll
 0001:000154d0       ?WinHelpA@CWinApp@@UAEXKI@Z 004164d0 f   mfc140:mfc140.dll
 0001:000154d6       ?HtmlHelpA@CWinApp@@UAEXKI@Z 004164d6 f   mfc140:mfc140.dll
 0001:000154dc       ?WinHelpInternal@CWinApp@@UAEXKI@Z 004164dc f   mfc140:mfc140.dll
 0001:000154e2       ?RegisterWithRestartManager@CWinApp@@UAEJHABV?$CStringT@DV?$StrTraitMFC_DLL@DV?$ChTraitsCRT@D@ATL@@@@@ATL@@@Z 004164e2 f   mfc140:mfc140.dll
 0001:000154e8       ?RegisterWithRestartManager@CWinApp@@UAEJPB_WKP6GKPAX@Z1KK@Z 004164e8 f   mfc140:mfc140.dll
 0001:000154ee       ?ApplicationRecoveryCallback@CWinApp@@UAEKPAX@Z 004164ee f   mfc140:mfc140.dll
 0001:000154f4       ?OnHelp@CWinApp@@IAEXXZ    004164f4 f   mfc140:mfc140.dll
 0001:000154fa       ?GetDataRecoveryHandler@CWinApp@@UAEPAVCDataRecoveryHandler@@XZ 004164fa f   mfc140:mfc140.dll
 0001:00015500       ?IsTaskbarInteractionEnabled@CWinApp@@UAEHXZ 00416500 f   mfc140:mfc140.dll
 0001:00015506       ?ExitInstance@CWinApp@@UAEHXZ 00416506 f   mfc140:mfc140.dll
 0001:0001550c       ?RestartInstance@CWinApp@@UAEHXZ 0041650c f   mfc140:mfc140.dll
 0001:00015512       ?OnIdle@CWinApp@@UAEHJ@Z   00416512 f   mfc140:mfc140.dll
 0001:00015518       ?ProcessWndProcException@CWinApp@@UAEJPAVCException@@PBUtagMSG@@@Z 00416518 f   mfc140:mfc140.dll
 0001:0001551e       ?LoadAppLangResourceDLL@CWinApp@@UAEPAUHINSTANCE__@@XZ 0041651e f   mfc140:mfc140.dll
 0001:00015524       ??1CWinApp@@UAE@XZ         00416524 f   mfc140:mfc140.dll
 0001:0001552a       ?GetThisMessageMap@CWinApp@@KGPBUAFX_MSGMAP@@XZ 0041652a f   mfc140:mfc140.dll
 0001:00015530       ?LoadSysPolicies@CWinApp@@UAEHXZ 00416530 f   mfc140:mfc140.dll
 0001:00015536       ?AfxThrowInvalidArgException@@YGXXZ 00416536 f   mfc140:mfc140.dll
 0001:0001553c       ??0CFileFind@@QAE@XZ       0041653c f   mfc140:mfc140.dll
 0001:00015542       ??1CFileFind@@UAE@XZ       00416542 f   mfc140:mfc140.dll
 0001:00015548       ?GetFileName@CFileFind@@UBE?AV?$CStringT@DV?$StrTraitMFC_DLL@DV?$ChTraitsCRT@D@ATL@@@@@ATL@@XZ 00416548 f   mfc140:mfc140.dll
 0001:0001554e       ?IsDots@CFileFind@@UBEHXZ  0041654e f   mfc140:mfc140.dll
 0001:00015554       ?Close@CFileFind@@QAEXXZ   00416554 f   mfc140:mfc140.dll
 0001:0001555a       ?FindFile@CFileFind@@UAEHPBDK@Z 0041655a f   mfc140:mfc140.dll
 0001:00015560       ?FindNextFileA@CFileFind@@UAEHXZ 00416560 f   mfc140:mfc140.dll
 0001:00015566       ??0CStringList@@QAE@H@Z    00416566 f   mfc140:mfc140.dll
 0001:0001556c       ?AddTail@CStringList@@QAEPAU__POSITION@@ABV?$CStringT@DV?$StrTraitMFC_DLL@DV?$ChTraitsCRT@D@ATL@@@@@ATL@@@Z 0041656c f   mfc140:mfc140.dll
 0001:00015572       ??1CStringList@@UAE@XZ     00416572 f   mfc140:mfc140.dll
 0001:00015578       ?AfxGetModuleState@@YGPAVAFX_MODULE_STATE@@XZ 00416578 f   mfc140:mfc140.dll
 0001:0001557e       ?DDX_Control@@YGXPAVCDataExchange@@HAAVCWnd@@@Z 0041657e f   mfc140:mfc140.dll
 0001:00015584       ?BeginWaitCursor@CCmdTarget@@QAEXXZ 00416584 f   mfc140:mfc140.dll
 0001:0001558a       ?EndWaitCursor@CCmdTarget@@QAEXXZ 0041658a f   mfc140:mfc140.dll
 0001:00015590       ??0CWnd@@QAE@XZ            00416590 f   mfc140:mfc140.dll
 0001:00015596       ?PreSubclassWindow@CWnd@@UAEXXZ 00416596 f   mfc140:mfc140.dll
 0001:0001559c       ?Create@CWnd@@UAEHPBD0KABUtagRECT@@PAV1@IPAUCCreateContext@@@Z 0041659c f   mfc140:mfc140.dll
 0001:000155a2       ?CreateEx@CWnd@@UAEHKPBD0KHHHHPAUHWND__@@PAUHMENU__@@PAX@Z 004165a2 f   mfc140:mfc140.dll
 0001:000155a8       ?CreateEx@CWnd@@UAEHKPBD0KABUtagRECT@@PAV1@IPAX@Z 004165a8 f   mfc140:mfc140.dll
 0001:000155ae       ?DestroyWindow@CWnd@@UAEHXZ 004165ae f   mfc140:mfc140.dll
 0001:000155b4       ?PreCreateWindow@CWnd@@UAEHAAUtagCREATESTRUCTA@@@Z 004165b4 f   mfc140:mfc140.dll
 0001:000155ba       ?CalcWindowRect@CWnd@@UAEXPAUtagRECT@@I@Z 004165ba f   mfc140:mfc140.dll
 0001:000155c0       ?GetDlgItem@CWnd@@QBEPAV1@H@Z 004165c0 f   mfc140:mfc140.dll
 0001:000155c6       ?SetWindowTextA@CWnd@@QAEXPBD@Z 004165c6 f   mfc140:mfc140.dll
 0001:000155cc       ?GetWindowTextA@CWnd@@QBEHPADH@Z 004165cc f   mfc140:mfc140.dll
 0001:000155d2       ?GetMenu@CWnd@@UBEPAVCMenu@@XZ 004165d2 f   mfc140:mfc140.dll
 0001:000155d8       ?SetMenu@CWnd@@UAEHPAVCMenu@@@Z 004165d8 f   mfc140:mfc140.dll
 0001:000155de       ?OnToolHitTest@CWnd@@UBEHVCPoint@@PAUtagTOOLINFOA@@@Z 004165de f   mfc140:mfc140.dll
 0001:000155e4       ?SetFocus@CWnd@@QAEPAV1@XZ 004165e4 f   mfc140:mfc140.dll
 0001:000155ea       ?GetScrollBarCtrl@CWnd@@UBEPAVCScrollBar@@H@Z 004165ea f   mfc140:mfc140.dll
 0001:000155f0       ?MessageBoxA@CWnd@@QAEHPBD0I@Z 004165f0 f   mfc140:mfc140.dll
 0001:000155f6       ?WinHelpA@CWnd@@UAEXKI@Z   004165f6 f   mfc140:mfc140.dll
 0001:000155fc       ?HtmlHelpA@CWnd@@UAEXKI@Z  004165fc f   mfc140:mfc140.dll
 0001:00015602       ?WinHelpInternal@CWnd@@UAEXKI@Z 00416602 f   mfc140:mfc140.dll
 0001:00015608       ?ContinueModal@CWnd@@UAEHXZ 00416608 f   mfc140:mfc140.dll
 0001:0001560e       ?EndModalLoop@CWnd@@UAEXH@Z 0041660e f   mfc140:mfc140.dll
 0001:00015614       ?OnDrawIconicThumbnailOrLivePreview@CWnd@@UAEXAAVCDC@@VCRect@@VCSize@@HAAH@Z 00416614 f   mfc140:mfc140.dll
 0001:0001561a       ?GetInterfaceMap@CWnd@@MBEPBUAFX_INTERFACEMAP@@XZ 0041661a f   mfc140:mfc140.dll
 0001:00015620       ?EnsureStdObj@CWnd@@UAEJXZ 00416620 f   mfc140:mfc140.dll
 0001:00015626       ?get_accParent@CWnd@@UAEJPAPAUIDispatch@@@Z 00416626 f   mfc140:mfc140.dll
 0001:0001562c       ?get_accChildCount@CWnd@@UAEJPAJ@Z 0041662c f   mfc140:mfc140.dll
 0001:00015632       ?get_accChild@CWnd@@UAEJUtagVARIANT@@PAPAUIDispatch@@@Z 00416632 f   mfc140:mfc140.dll
 0001:00015638       ?get_accName@CWnd@@UAEJUtagVARIANT@@PAPA_W@Z 00416638 f   mfc140:mfc140.dll
 0001:0001563e       ?get_accValue@CWnd@@UAEJUtagVARIANT@@PAPA_W@Z 0041663e f   mfc140:mfc140.dll
 0001:00015644       ?get_accDescription@CWnd@@UAEJUtagVARIANT@@PAPA_W@Z 00416644 f   mfc140:mfc140.dll
 0001:0001564a       ?get_accRole@CWnd@@UAEJUtagVARIANT@@PAU2@@Z 0041664a f   mfc140:mfc140.dll
 0001:00015650       ?get_accState@CWnd@@UAEJUtagVARIANT@@PAU2@@Z 00416650 f   mfc140:mfc140.dll
 0001:00015656       ?get_accHelp@CWnd@@UAEJUtagVARIANT@@PAPA_W@Z 00416656 f   mfc140:mfc140.dll
 0001:0001565c       ?get_accHelpTopic@CWnd@@UAEJPAPA_WUtagVARIANT@@PAJ@Z 0041665c f   mfc140:mfc140.dll
 0001:00015662       ?get_accKeyboardShortcut@CWnd@@UAEJUtagVARIANT@@PAPA_W@Z 00416662 f   mfc140:mfc140.dll
 0001:00015668       ?get_accFocus@CWnd@@UAEJPAUtagVARIANT@@@Z 00416668 f   mfc140:mfc140.dll
 0001:0001566e       ?get_accSelection@CWnd@@UAEJPAUtagVARIANT@@@Z 0041666e f   mfc140:mfc140.dll
 0001:00015674       ?get_accDefaultAction@CWnd@@UAEJUtagVARIANT@@PAPA_W@Z 00416674 f   mfc140:mfc140.dll
 0001:0001567a       ?accSelect@CWnd@@UAEJJUtagVARIANT@@@Z 0041667a f   mfc140:mfc140.dll
 0001:00015680       ?accLocation@CWnd@@UAEJPAJ000UtagVARIANT@@@Z 00416680 f   mfc140:mfc140.dll
 0001:00015686       ?accNavigate@CWnd@@UAEJJUtagVARIANT@@PAU2@@Z 00416686 f   mfc140:mfc140.dll
 0001:0001568c       ?accHitTest@CWnd@@UAEJJJPAUtagVARIANT@@@Z 0041668c f   mfc140:mfc140.dll
 0001:00015692       ?accDoDefaultAction@CWnd@@UAEJUtagVARIANT@@@Z 00416692 f   mfc140:mfc140.dll
 0001:00015698       ?put_accName@CWnd@@UAEJUtagVARIANT@@PA_W@Z 00416698 f   mfc140:mfc140.dll
 0001:0001569e       ?put_accValue@CWnd@@UAEJUtagVARIANT@@PA_W@Z 0041669e f   mfc140:mfc140.dll
 0001:000156a4       ?SetProxy@CWnd@@UAEJPAUIAccessibleProxy@@@Z 004166a4 f   mfc140:mfc140.dll
 0001:000156aa       ?CreateAccessibleProxy@CWnd@@UAEJIJPAJ@Z 004166aa f   mfc140:mfc140.dll
 0001:000156b0       ?OnCommand@CWnd@@MAEHIJ@Z  004166b0 f   mfc140:mfc140.dll
 0001:000156b6       ?OnNotify@CWnd@@MAEHIJPAJ@Z 004166b6 f   mfc140:mfc140.dll
 0001:000156bc       ?GetSuperWndProcAddr@CWnd@@MAEPAP6GJPAUHWND__@@IIJ@ZXZ 004166bc f   mfc140:mfc140.dll
 0001:000156c2       ?PreTranslateMessage@CWnd@@UAEHPAUtagMSG@@@Z 004166c2 f   mfc140:mfc140.dll
 0001:000156c8       ?OnAmbientProperty@CWnd@@UAEHPAVCOleControlSite@@JPAUtagVARIANT@@@Z 004166c8 f   mfc140:mfc140.dll
 0001:000156ce       ?WindowProc@CWnd@@MAEJIIJ@Z 004166ce f   mfc140:mfc140.dll
 0001:000156d4       ?OnWndMsg@CWnd@@MAEHIIJPAJ@Z 004166d4 f   mfc140:mfc140.dll
 0001:000156da       ?Default@CWnd@@IAEJXZ      004166da f   mfc140:mfc140.dll
 0001:000156e0       ?DefWindowProcA@CWnd@@MAEJIIJ@Z 004166e0 f   mfc140:mfc140.dll
 0001:000156e6       ?PostNcDestroy@CWnd@@MAEXXZ 004166e6 f   mfc140:mfc140.dll
 0001:000156ec       ?OnChildNotify@CWnd@@MAEHIIJPAJ@Z 004166ec f   mfc140:mfc140.dll
 0001:000156f2       ?OnTouchInputs@CWnd@@MAEHIPAUtagTOUCHINPUT@@@Z 004166f2 f   mfc140:mfc140.dll
 0001:000156f8       ?OnTouchInput@CWnd@@MAEHVCPoint@@HHPAUtagTOUCHINPUT@@@Z 004166f8 f   mfc140:mfc140.dll
 0001:000156fe       ?GetGestureStatus@CWnd@@MAEKVCPoint@@@Z 004166fe f   mfc140:mfc140.dll
 0001:00015704       ?OnGestureZoom@CWnd@@MAEHVCPoint@@J@Z 00416704 f   mfc140:mfc140.dll
 0001:0001570a       ?OnGesturePan@CWnd@@MAEHVCPoint@@0@Z 0041670a f   mfc140:mfc140.dll
 0001:00015710       ?OnGestureRotate@CWnd@@MAEHVCPoint@@N@Z 00416710 f   mfc140:mfc140.dll
 0001:00015716       ?OnGestureTwoFingerTap@CWnd@@MAEHVCPoint@@@Z 00416716 f   mfc140:mfc140.dll
 0001:0001571c       ?OnGesturePressAndTap@CWnd@@MAEHVCPoint@@J@Z 0041671c f   mfc140:mfc140.dll
 0001:00015722       ?ResizeDynamicLayout@CWnd@@MAEXXZ 00416722 f   mfc140:mfc140.dll
 0001:00015728       ?CheckAutoCenter@CWnd@@UAEHXZ 00416728 f   mfc140:mfc140.dll
 0001:0001572e       ?IsFrameWnd@CWnd@@UBEHXZ   0041672e f   mfc140:mfc140.dll
 0001:00015734       ?OnFinalRelease@CWnd@@UAEXXZ 00416734 f   mfc140:mfc140.dll
 0001:0001573a       ?CreateControlContainer@CWnd@@MAEHPAPAVCOleControlContainer@@@Z 0041673a f   mfc140:mfc140.dll
 0001:00015740       ?CreateControlSite@CWnd@@MAEHPAVCOleControlContainer@@PAPAVCOleControlSite@@IABU_GUID@@@Z 00416740 f   mfc140:mfc140.dll
 0001:00015746       ?SetOccDialogInfo@CWnd@@MAEHPAU_AFX_OCC_DIALOG_INFO@@@Z 00416746 f   mfc140:mfc140.dll
 0001:0001574c       ?GetOccDialogInfo@CWnd@@MAEPAU_AFX_OCC_DIALOG_INFO@@XZ 0041674c f   mfc140:mfc140.dll
 0001:00015752       ?GetMessageMap@CWnd@@MBEPBUAFX_MSGMAP@@XZ 00416752 f   mfc140:mfc140.dll
 0001:00015758       ?GetRuntimeClass@CDialog@@UBEPAUCRuntimeClass@@XZ 00416758 f   mfc140:mfc140.dll
 0001:0001575e       ?Create@CDialog@@UAEHPBDPAVCWnd@@@Z 0041675e f   mfc140:mfc140.dll
 0001:00015764       ?CreateIndirect@CDialog@@UAEHPBUDLGTEMPLATE@@PAVCWnd@@PAX@Z 00416764 f   mfc140:mfc140.dll
 0001:0001576a       ?CreateIndirect@CDialog@@UAEHPAXPAVCWnd@@@Z 0041676a f   mfc140:mfc140.dll
 0001:00015770       ??0CDialog@@QAE@IPAVCWnd@@@Z 00416770 f   mfc140:mfc140.dll
 0001:00015776       ?OnInitDialog@CDialog@@UAEHXZ 00416776 f   mfc140:mfc140.dll
 0001:0001577c       ?OnSetFont@CDialog@@UAEXPAVCFont@@@Z 0041677c f   mfc140:mfc140.dll
 0001:00015782       ?OnOK@CDialog@@MAEXXZ      00416782 f   mfc140:mfc140.dll
 0001:00015788       ?OnCancel@CDialog@@MAEXXZ  00416788 f   mfc140:mfc140.dll
 0001:0001578e       ??1CDialog@@UAE@XZ         0041678e f   mfc140:mfc140.dll
 0001:00015794       ?PreTranslateMessage@CDialog@@UAEHPAUtagMSG@@@Z 00416794 f   mfc140:mfc140.dll
 0001:0001579a       ?OnCmdMsg@CDialog@@UAEHIHPAXPAUAFX_CMDHANDLERINFO@@@Z 0041679a f   mfc140:mfc140.dll
 0001:000157a0       ?CheckAutoCenter@CDialog@@UAEHXZ 004167a0 f   mfc140:mfc140.dll
 0001:000157a6       ?SetOccDialogInfo@CDialog@@MAEHPAU_AFX_OCC_DIALOG_INFO@@@Z 004167a6 f   mfc140:mfc140.dll
 0001:000157ac       ?GetOccDialogInfo@CDialog@@MAEPAU_AFX_OCC_DIALOG_INFO@@XZ 004167ac f   mfc140:mfc140.dll
 0001:000157b2       ?PreInitDialog@CDialog@@MAEXXZ 004167b2 f   mfc140:mfc140.dll
 0001:000157b8       ?OnPaint@CDialog@@IAEXXZ   004167b8 f   mfc140:mfc140.dll
 0001:000157be       ?GetThisMessageMap@CDialog@@KGPBUAFX_MSGMAP@@XZ 004167be f   mfc140:mfc140.dll
 0001:000157c4       ?GetRuntimeClass@CListBox@@UBEPAUCRuntimeClass@@XZ 004167c4 f   mfc140:mfc140.dll
 0001:000157ca       ?Create@CListBox@@UAEHKABUtagRECT@@PAVCWnd@@I@Z 004167ca f   mfc140:mfc140.dll
 0001:000157d0       ?DrawItem@CListBox@@UAEXPAUtagDRAWITEMSTRUCT@@@Z 004167d0 f   mfc140:mfc140.dll
 0001:000157d6       ?MeasureItem@CListBox@@UAEXPAUtagMEASUREITEMSTRUCT@@@Z 004167d6 f   mfc140:mfc140.dll
 0001:000157dc       ?CompareItem@CListBox@@UAEHPAUtagCOMPAREITEMSTRUCT@@@Z 004167dc f   mfc140:mfc140.dll
 0001:000157e2       ?DeleteItem@CListBox@@UAEXPAUtagDELETEITEMSTRUCT@@@Z 004167e2 f   mfc140:mfc140.dll
 0001:000157e8       ?VKeyToItem@CListBox@@UAEHII@Z 004167e8 f   mfc140:mfc140.dll
 0001:000157ee       ?CharToItem@CListBox@@UAEHII@Z 004167ee f   mfc140:mfc140.dll
 0001:000157f4       ??1CListBox@@UAE@XZ        004167f4 f   mfc140:mfc140.dll
 0001:000157fa       ?OnChildNotify@CListBox@@MAEHIIJPAJ@Z 004167fa f   mfc140:mfc140.dll
 0001:00015800       ?GetRuntimeClass@CEdit@@UBEPAUCRuntimeClass@@XZ 00416800 f   mfc140:mfc140.dll
 0001:00015806       ??1CEdit@@UAE@XZ           00416806 f   mfc140:mfc140.dll
 0001:0001580c       ?AfxFindResourceHandle@@YGPAUHINSTANCE__@@PBD0@Z 0041680c f   mfc140:mfc140.dll
 0001:00015812       ?AfxMessageBox@@YGHPBDII@Z 00416812 f   mfc140:mfc140.dll
 0001:00015818       ?AfxLoadLibrary@@YGPAUHINSTANCE__@@PBD@Z 00416818 f   mfc140:mfc140.dll
 0001:0001581e       ?AfxFreeLibrary@@YGHPAUHINSTANCE__@@@Z 0041681e f   mfc140:mfc140.dll
 0001:00015824       ?Init@CComCriticalSection@ATL@@QAEJXZ 00416824 f i mfcs140:nolib.obj
 0001:0001584c       @__security_check_cookie@4 0041684c f   msvcrt:secchk.obj
 0001:0001585d       ??3@YAXPAXI@Z              0041685d f   msvcrt:delete_scalar_size.obj
 0001:000158af       ___scrt_acquire_startup_lock 004168af f   msvcrt:utility.obj
 0001:000158e1       ___scrt_initialize_crt     004168e1 f   msvcrt:utility.obj
 0001:0001591a       ___scrt_initialize_onexit_tables 0041691a f   msvcrt:utility.obj
 0001:000159bf       ___scrt_is_nonwritable_in_current_image 004169bf f   msvcrt:utility.obj
 0001:00015a53       ___scrt_release_startup_lock 00416a53 f   msvcrt:utility.obj
 0001:00015a70       ___scrt_uninitialize_crt   00416a70 f   msvcrt:utility.obj
 0001:00015a98       __onexit                   00416a98 f   msvcrt:utility.obj
 0001:00015ad3       _atexit                    00416ad3 f   msvcrt:utility.obj
 0001:00015ae8       ??_Gtype_info@@UAEPAXI@Z   00416ae8 f i msvcrt:std_type_info_static.obj
 0001:00015ae8       ??_Etype_info@@UAEPAXI@Z   00416ae8 f i msvcrt:std_type_info_static.obj
 0001:00015b10       __alloca_probe             00416b10 f   msvcrt:chkstk.obj
 0001:00015b10       __chkstk                   00416b10 f   msvcrt:chkstk.obj
 0001:00015d7e       _WinMainCRTStartup         00416d7e f   msvcrt:exe_winmain.obj
 0001:00015d90       __SEH_prolog4              00416d90 f   msvcrt:sehprolg4.obj
 0001:00015dd6       __SEH_epilog4              00416dd6 f   msvcrt:sehprolg4.obj
 0001:00015df0       __SEH_prolog4_GS           00416df0 f   msvcrt:sehprolg4gs.obj
 0001:00015e39       __SEH_epilog4_GS           00416e39 f   msvcrt:sehprolg4gs.obj
 0001:00015e4a       __except_handler4          00416e4a f   msvcrt:chandler4gs.obj
 0001:00015e6d       ___raise_securityfailure   00416e6d f   msvcrt:gs_report.obj
 0001:00015e95       ___report_gsfailure        00416e95 f   msvcrt:gs_report.obj
 0001:00015f8e       ___isa_available_init      00416f8e f   msvcrt:cpu_disp.obj
 0001:00016125       __get_startup_argv_mode    00417125 f   msvcrt:argv_mode.obj
 0001:00016129       ___scrt_is_ucrt_dll_in_use 00417129 f   msvcrt:ucrt_detection.obj
 0001:00016135       ___scrt_fastfail           00417135 f   msvcrt:utility_desktop.obj
 0001:0001624f       ___scrt_get_show_window_mode 0041724f f   msvcrt:utility_desktop.obj
 0001:00016280       ___scrt_initialize_mta     00417280 f   msvcrt:utility_desktop.obj
 0001:00016285       ___scrt_is_managed_app     00417285 f   msvcrt:utility_desktop.obj
 0001:000162c8       ___scrt_set_unhandled_exception_filter 004172c8 f   msvcrt:utility_desktop.obj
 0001:000162d4       ___scrt_unhandled_exception_filter@4 004172d4 f   msvcrt:utility_desktop.obj
 0001:00016315       __crt_debugger_hook        00417315 f   msvcrt:utility_desktop.obj
 0001:0001636a       ___security_init_cookie    0041736a f   msvcrt:gs_support.obj
 0001:000163b5       __get_startup_file_mode    004173b5 f   msvcrt:file_mode.obj
 0001:000163bb       ?__scrt_initialize_type_info@@YAXXZ 004173bb f   msvcrt:tncleanup.obj
 0001:000163c7       ___acrt_initialize         004173c7 f   msvcrt:ucrt_stubs.obj
 0001:000163c7       __should_initialize_environment 004173c7 f   msvcrt:env_mode.obj
 0001:000163c7       ___vcrt_uninitialize       004173c7 f   msvcrt:ucrt_stubs.obj
 0001:000163c7       ___scrt_stub_for_acrt_uninitialize 004173c7 f   msvcrt:ucrt_stubs.obj
 0001:000163c7       ___vcrt_initialize         004173c7 f   msvcrt:ucrt_stubs.obj
 0001:000163c7       ___acrt_uninitialize       004173c7 f   msvcrt:ucrt_stubs.obj
 0001:000163c7       ___scrt_stub_for_acrt_initialize 004173c7 f   msvcrt:ucrt_stubs.obj
 0001:000163ca       __initialize_default_precision 004173ca f   msvcrt:default_precision.obj
 0001:000163eb       ___scrt_initialize_default_local_stdio_options 004173eb f   msvcrt:default_local_stdio_options.obj
 0001:00016408       ___scrt_is_user_matherr_present 00417408 f   msvcrt:matherr_detection.obj
 0001:00016414       ___scrt_get_dyn_tls_init_callback 00417414 f   msvcrt:dyn_tls_init.obj
 0001:0001641a       ___scrt_get_dyn_tls_dtor_callback 0041741a f   msvcrt:dyn_tls_dtor.obj
 0001:00016420       __RTC_Initialize           00417420 f   msvcrt:initsect.obj
 0001:0001644c       __RTC_Terminate            0041744c f   msvcrt:initsect.obj
 0001:00016478       _IsProcessorFeaturePresent@4 00417478 f   kernel32:KERNEL32.dll
 0001:0001647e       ??0CAtlBaseModule@ATL@@QAE@XZ 0041747e f   atls:atlbase.obj
 0001:000164d1       ??0_ATL_BASE_MODULE70@ATL@@QAE@XZ 004174d1 f i atls:atlbase.obj
 0001:000164f4       ??1CAtlBaseModule@ATL@@QAE@XZ 004174f4 f   atls:atlbase.obj
 0001:0001650a       ?RemoveAll@?$CSimpleArray@PAUHINSTANCE__@@V?$CSimpleArrayEqualHelper@PAUHINSTANCE__@@@ATL@@@ATL@@QAEXXZ 0041750a f i atls:atlbase.obj
 0001:00016527       ?_Xlength_error@std@@YAXPBD@Z 00417527 f   msvcprt:MSVCP140.dll
 0001:0001652d       ?_Xout_of_range@std@@YAXPBD@Z 0041752d f   msvcprt:MSVCP140.dll
 0001:00016533       _MiniDumpWriteDump@28      00417533 f   DbgHelp:dbghelp.dll
 0001:00016539       _memset                    00417539 f   vcruntime:VCRUNTIME140.dll
 0001:0001653f       __purecall                 0041753f f   vcruntime:VCRUNTIME140.dll
 0001:00016545       ___CxxFrameHandler3        00417545 f   vcruntime:VCRUNTIME140.dll
 0001:0001654b       _memchr                    0041754b f   vcruntime:VCRUNTIME140.dll
 0001:00016551       _memcpy                    00417551 f   vcruntime:VCRUNTIME140.dll
 0001:00016557       _memmove                   00417557 f   vcruntime:VCRUNTIME140.dll
 0001:0001655d       __CxxThrowException@8      0041755d f   vcruntime:VCRUNTIME140.dll
 0001:00016563       ___std_terminate           00417563 f   vcruntime:VCRUNTIME140.dll
 0001:00016569       _strstr                    00417569 f   vcruntime:VCRUNTIME140.dll
 0001:0001656f       ___std_exception_copy      0041756f f   vcruntime:VCRUNTIME140.dll
 0001:00016575       ___std_exception_destroy   00417575 f   vcruntime:VCRUNTIME140.dll
 0001:0001657b       ___RTDynamicCast           0041757b f   vcruntime:VCRUNTIME140.dll
 0001:00016581       _wcsrchr                   00417581 f   vcruntime:VCRUNTIME140.dll
 0001:00016587       __except_handler4_common   00417587 f   vcruntime:VCRUNTIME140.dll
 0001:0001658d       __libm_sse2_atan_precise   0041758d f   ucrt:api-ms-win-crt-math-l1-1-0.dll
 0001:00016593       __libm_sse2_sqrt_precise   00417593 f   ucrt:api-ms-win-crt-math-l1-1-0.dll
 0001:00016599       _free                      00417599 f   ucrt:api-ms-win-crt-heap-l1-1-0.dll
 0001:0001659f       __configure_narrow_argv    0041759f f   ucrt:api-ms-win-crt-runtime-l1-1-0.dll
 0001:000165a5       __initialize_narrow_environment 004175a5 f   ucrt:api-ms-win-crt-runtime-l1-1-0.dll
 0001:000165ab       __initialize_onexit_table  004175ab f   ucrt:api-ms-win-crt-runtime-l1-1-0.dll
 0001:000165b1       __register_onexit_function 004175b1 f   ucrt:api-ms-win-crt-runtime-l1-1-0.dll
 0001:000165b7       __crt_atexit               004175b7 f   ucrt:api-ms-win-crt-runtime-l1-1-0.dll
 0001:000165bd       __cexit                    004175bd f   ucrt:api-ms-win-crt-runtime-l1-1-0.dll
 0001:000165c3       __seh_filter_exe           004175c3 f   ucrt:api-ms-win-crt-runtime-l1-1-0.dll
 0001:000165c9       __set_app_type             004175c9 f   ucrt:api-ms-win-crt-runtime-l1-1-0.dll
 0001:000165cf       ___setusermatherr          004175cf f   ucrt:api-ms-win-crt-math-l1-1-0.dll
 0001:000165d5       __get_narrow_winmain_command_line 004175d5 f   ucrt:api-ms-win-crt-runtime-l1-1-0.dll
 0001:000165db       __initterm                 004175db f   ucrt:api-ms-win-crt-runtime-l1-1-0.dll
 0001:000165e1       __initterm_e               004175e1 f   ucrt:api-ms-win-crt-runtime-l1-1-0.dll
 0001:000165e7       _exit                      004175e7 f   ucrt:api-ms-win-crt-runtime-l1-1-0.dll
 0001:000165ed       __exit                     004175ed f   ucrt:api-ms-win-crt-runtime-l1-1-0.dll
 0001:000165f3       __set_fmode                004175f3 f   ucrt:api-ms-win-crt-stdio-l1-1-0.dll
 0001:000165f9       __c_exit                   004175f9 f   ucrt:api-ms-win-crt-runtime-l1-1-0.dll
 0001:000165ff       __register_thread_local_exe_atexit_callback 004175ff f   ucrt:api-ms-win-crt-runtime-l1-1-0.dll
 0001:00016605       __configthreadlocale       00417605 f   ucrt:api-ms-win-crt-locale-l1-1-0.dll
 0001:0001660b       __set_new_mode             0041760b f   ucrt:api-ms-win-crt-heap-l1-1-0.dll
 0001:00016611       ___p__commode              00417611 f   ucrt:api-ms-win-crt-stdio-l1-1-0.dll
 0001:00016617       _terminate                 00417617 f   ucrt:api-ms-win-crt-runtime-l1-1-0.dll
 0001:0001661d       __controlfp_s              0041761d f   ucrt:api-ms-win-crt-runtime-l1-1-0.dll
 0001:00016623       ?AfxInitialize@@YGHHK@Z    00417623 f   mfcs140:appmodul.obj
 0001:0001664b       _WinMain@16                0041764b f   mfcs140:appmodul.obj
 0001:00016654       ?_Lock@?$basic_streambuf@DU?$char_traits@D@std@@@std@@UAEXXZ 00417654 f   msvcprt:MSVCP140.dll
 0001:0001665a       ?_Unlock@?$basic_streambuf@DU?$char_traits@D@std@@@std@@UAEXXZ 0041765a f   msvcprt:MSVCP140.dll
 0001:00016660       ?showmanyc@?$basic_streambuf@DU?$char_traits@D@std@@@std@@MAE_JXZ 00417660 f   msvcprt:MSVCP140.dll
 0001:00016666       ?uflow@?$basic_streambuf@DU?$char_traits@D@std@@@std@@MAEHXZ 00417666 f   msvcprt:MSVCP140.dll
 0001:0001666c       ?xsgetn@?$basic_streambuf@DU?$char_traits@D@std@@@std@@MAE_JPAD_J@Z 0041766c f   msvcprt:MSVCP140.dll
 0001:00016672       ?xsputn@?$basic_streambuf@DU?$char_traits@D@std@@@std@@MAE_JPBD_J@Z 00417672 f   msvcprt:MSVCP140.dll
 0001:00016678       ?setbuf@?$basic_streambuf@DU?$char_traits@D@std@@@std@@MAEPAV12@PAD_J@Z 00417678 f   msvcprt:MSVCP140.dll
 0001:0001667e       ?sync@?$basic_streambuf@DU?$char_traits@D@std@@@std@@MAEHXZ 0041767e f   msvcprt:MSVCP140.dll
 0001:00016684       ?imbue@?$basic_streambuf@DU?$char_traits@D@std@@@std@@MAEXABVlocale@2@@Z 00417684 f   msvcprt:MSVCP140.dll
 0001:0001668a       ?AfxWinMain@@YGHPAUHINSTANCE__@@0PADH@Z 0041768a f   mfc140:mfc140.dll
 0002:00000000       __imp__WaitForSingleObject@8 00419000     kernel32:KERNEL32.dll
 0002:00000004       __imp__EnterCriticalSection@4 00419004     kernel32:KERNEL32.dll
 0002:00000008       __imp__LeaveCriticalSection@4 00419008     kernel32:KERNEL32.dll
 0002:0000000c       __imp__DeleteCriticalSection@4 0041900c     kernel32:KERNEL32.dll
 0002:00000010       __imp__GetLocalTime@4      00419010     kernel32:KERNEL32.dll
 0002:00000014       __imp__GetPrivateProfileIntA@16 00419014     kernel32:KERNEL32.dll
 0002:00000018       __imp__SetCurrentDirectoryA@4 00419018     kernel32:KERNEL32.dll
 0002:0000001c       __imp__GetCurrentDirectoryA@8 0041901c     kernel32:KERNEL32.dll
 0002:00000020       __imp__Sleep@4             00419020     kernel32:KERNEL32.dll
 0002:00000024       __imp__CloseHandle@4       00419024     kernel32:KERNEL32.dll
 0002:00000028       __imp__GetTickCount@0      00419028     kernel32:KERNEL32.dll
 0002:0000002c       __imp__MapViewOfFile@20    0041902c     kernel32:KERNEL32.dll
 0002:00000030       __imp__UnmapViewOfFile@4   00419030     kernel32:KERNEL32.dll
 0002:00000034       __imp__CreateFileMappingA@24 00419034     kernel32:KERNEL32.dll
 0002:00000038       __imp__OpenFileMappingA@12 00419038     kernel32:KERNEL32.dll
 0002:0000003c       __imp__ReadFile@20         0041903c     kernel32:KERNEL32.dll
 0002:00000040       __imp__CreateFileA@28      00419040     kernel32:KERNEL32.dll
 0002:00000044       __imp__WideCharToMultiByte@32 00419044     kernel32:KERNEL32.dll
 0002:00000048       __imp__InterlockedExchange@8 00419048     kernel32:KERNEL32.dll
 0002:0000004c       __imp__InterlockedCompareExchange@12 0041904c     kernel32:KERNEL32.dll
 0002:00000050       __imp__GetProcAddress@8    00419050     kernel32:KERNEL32.dll
 0002:00000054       __imp__OpenProcess@12      00419054     kernel32:KERNEL32.dll
 0002:00000058       __imp__GetCurrentProcessId@0 00419058     kernel32:KERNEL32.dll
 0002:0000005c       __imp__TerminateThread@8   0041905c     kernel32:KERNEL32.dll
 0002:00000060       __imp__GetLastError@0      00419060     kernel32:KERNEL32.dll
 0002:00000064       __imp__ReadProcessMemory@20 00419064     kernel32:KERNEL32.dll
 0002:00000068       __imp__WriteProcessMemory@20 00419068     kernel32:KERNEL32.dll
 0002:0000006c       __imp__SetEvent@4          0041906c     kernel32:KERNEL32.dll
 0002:00000070       __imp__ResetEvent@4        00419070     kernel32:KERNEL32.dll
 0002:00000074       __imp__CreateEventA@16     00419074     kernel32:KERNEL32.dll
 0002:00000078       __imp__GetModuleHandleA@4  00419078     kernel32:KERNEL32.dll
 0002:0000007c       __imp__GetPrivateProfileStringA@24 0041907c     kernel32:KERNEL32.dll
 0002:00000080       __imp__FindFirstFileA@8    00419080     kernel32:KERNEL32.dll
 0002:00000084       __imp__RaiseException@16   00419084     kernel32:KERNEL32.dll
 0002:00000088       __imp__InitializeCriticalSectionAndSpinCount@8 00419088     kernel32:KERNEL32.dll
 0002:0000008c       __imp__GetCurrentProcess@0 0041908c     kernel32:KERNEL32.dll
 0002:00000090       __imp__SetUnhandledExceptionFilter@4 00419090     kernel32:KERNEL32.dll
 0002:00000094       __imp__OutputDebugStringW@4 00419094     kernel32:KERNEL32.dll
 0002:00000098       __imp__CreateThread@24     00419098     kernel32:KERNEL32.dll
 0002:0000009c       __imp__GetCurrentThreadId@0 0041909c     kernel32:KERNEL32.dll
 0002:000000a0       __imp__GetCurrentThread@0  004190a0     kernel32:KERNEL32.dll
 0002:000000a4       __imp__GetFileSize@8       004190a4     kernel32:KERNEL32.dll
 0002:000000a8       __imp__GetModuleFileNameW@12 004190a8     kernel32:KERNEL32.dll
 0002:000000ac       __imp__InitializeSListHead@4 004190ac     kernel32:KERNEL32.dll
 0002:000000b0       __imp__GetSystemTimeAsFileTime@4 004190b0     kernel32:KERNEL32.dll
 0002:000000b4       __imp__QueryPerformanceCounter@4 004190b4     kernel32:KERNEL32.dll
 0002:000000b8       __imp__GetStartupInfoW@4   004190b8     kernel32:KERNEL32.dll
 0002:000000bc       __imp__IsDebuggerPresent@0 004190bc     kernel32:KERNEL32.dll
 0002:000000c0       __imp__IsProcessorFeaturePresent@4 004190c0     kernel32:KERNEL32.dll
 0002:000000c4       __imp__TerminateProcess@8  004190c4     kernel32:KERNEL32.dll
 0002:000000c8       __imp__UnhandledExceptionFilter@4 004190c8     kernel32:KERNEL32.dll
 0002:000000cc       __imp__GetModuleHandleW@4  004190cc     kernel32:KERNEL32.dll
 0002:000000d0       __imp__MultiByteToWideChar@24 004190d0     kernel32:KERNEL32.dll
 0002:000000d4       __imp__GetComputerNameW@8  004190d4     kernel32:KERNEL32.dll
 0002:000000d8       __imp__CreateFileW@28      004190d8     kernel32:KERNEL32.dll
 0002:000000dc       __imp__GetPrivateProfileStringW@24 004190dc     kernel32:KERNEL32.dll
 0002:000000e0       __imp__InitializeCriticalSection@4 004190e0     kernel32:KERNEL32.dll
 0002:000000e4       \177KERNEL32_NULL_THUNK_DATA 004190e4     kernel32:KERNEL32.dll
 0002:000000e8       __imp_?_Xlength_error@std@@YAXPBD@Z 004190e8     msvcprt:MSVCP140.dll
 0002:000000ec       __imp_?_Xout_of_range@std@@YAXPBD@Z 004190ec     msvcprt:MSVCP140.dll
 0002:000000f0       __imp_?uncaught_exception@std@@YA_NXZ 004190f0     msvcprt:MSVCP140.dll
 0002:000000f4       __imp_?sputn@?$basic_streambuf@DU?$char_traits@D@std@@@std@@QAE_JPBD_J@Z 004190f4     msvcprt:MSVCP140.dll
 0002:000000f8       __imp_?put@?$basic_ostream@DU?$char_traits@D@std@@@std@@QAEAAV12@D@Z 004190f8     msvcprt:MSVCP140.dll
 0002:000000fc       __imp_?widen@?$basic_ios@DU?$char_traits@D@std@@@std@@QBEDD@Z 004190fc     msvcprt:MSVCP140.dll
 0002:00000100       __imp_?sputc@?$basic_streambuf@DU?$char_traits@D@std@@@std@@QAEHD@Z 00419100     msvcprt:MSVCP140.dll
 0002:00000104       __imp_??0?$basic_streambuf@DU?$char_traits@D@std@@@std@@IAE@XZ 00419104     msvcprt:MSVCP140.dll
 0002:00000108       __imp_?_Osfx@?$basic_ostream@DU?$char_traits@D@std@@@std@@QAEXXZ 00419108     msvcprt:MSVCP140.dll
 0002:0000010c       __imp_?flush@?$basic_ostream@DU?$char_traits@D@std@@@std@@QAEAAV12@XZ 0041910c     msvcprt:MSVCP140.dll
 0002:00000110       __imp_?setstate@?$basic_ios@DU?$char_traits@D@std@@@std@@QAEXH_N@Z 00419110     msvcprt:MSVCP140.dll
 0002:00000114       __imp_??0?$basic_ios@DU?$char_traits@D@std@@@std@@IAE@XZ 00419114     msvcprt:MSVCP140.dll
 0002:00000118       __imp_?_Pninc@?$basic_streambuf@DU?$char_traits@D@std@@@std@@IAEPADXZ 00419118     msvcprt:MSVCP140.dll
 0002:0000011c       __imp_??0?$basic_iostream@DU?$char_traits@D@std@@@std@@QAE@PAV?$basic_streambuf@DU?$char_traits@D@std@@@1@@Z 0041911c     msvcprt:MSVCP140.dll
 0002:00000120       __imp_??1?$basic_ios@DU?$char_traits@D@std@@@std@@UAE@XZ 00419120     msvcprt:MSVCP140.dll
 0002:00000124       __imp_??1?$basic_streambuf@DU?$char_traits@D@std@@@std@@UAE@XZ 00419124     msvcprt:MSVCP140.dll
 0002:00000128       __imp_?_Lock@?$basic_streambuf@DU?$char_traits@D@std@@@std@@UAEXXZ 00419128     msvcprt:MSVCP140.dll
 0002:0000012c       __imp_?_Unlock@?$basic_streambuf@DU?$char_traits@D@std@@@std@@UAEXXZ 0041912c     msvcprt:MSVCP140.dll
 0002:00000130       __imp_?showmanyc@?$basic_streambuf@DU?$char_traits@D@std@@@std@@MAE_JXZ 00419130     msvcprt:MSVCP140.dll
 0002:00000134       __imp_?uflow@?$basic_streambuf@DU?$char_traits@D@std@@@std@@MAEHXZ 00419134     msvcprt:MSVCP140.dll
 0002:00000138       __imp_?xsgetn@?$basic_streambuf@DU?$char_traits@D@std@@@std@@MAE_JPAD_J@Z 00419138     msvcprt:MSVCP140.dll
 0002:0000013c       __imp_?xsputn@?$basic_streambuf@DU?$char_traits@D@std@@@std@@MAE_JPBD_J@Z 0041913c     msvcprt:MSVCP140.dll
 0002:00000140       __imp_?setbuf@?$basic_streambuf@DU?$char_traits@D@std@@@std@@MAEPAV12@PAD_J@Z 00419140     msvcprt:MSVCP140.dll
 0002:00000144       __imp_?sync@?$basic_streambuf@DU?$char_traits@D@std@@@std@@MAEHXZ 00419144     msvcprt:MSVCP140.dll
 0002:00000148       __imp_?imbue@?$basic_streambuf@DU?$char_traits@D@std@@@std@@MAEXABVlocale@2@@Z 00419148     msvcprt:MSVCP140.dll
 0002:0000014c       __imp_??6?$basic_ostream@DU?$char_traits@D@std@@@std@@QAEAAV01@P6AAAV01@AAV01@@Z@Z 0041914c     msvcprt:MSVCP140.dll
 0002:00000150       __imp_??6?$basic_ostream@DU?$char_traits@D@std@@@std@@QAEAAV01@I@Z 00419150     msvcprt:MSVCP140.dll
 0002:00000154       __imp_??1?$basic_iostream@DU?$char_traits@D@std@@@std@@UAE@XZ 00419154     msvcprt:MSVCP140.dll
 0002:00000158       \177MSVCP140_NULL_THUNK_DATA 00419158     msvcprt:MSVCP140.dll
 0002:0000015c       __imp__GetProcessMemoryInfo@12 0041915c     Psapi:PSAPI.DLL
 0002:00000160       \177PSAPI_NULL_THUNK_DATA  00419160     Psapi:PSAPI.DLL
 0002:00000164       __imp__SHCreateDirectoryExA@12 00419164     shell32:SHELL32.dll
 0002:00000168       \177SHELL32_NULL_THUNK_DATA 00419168     shell32:SHELL32.dll
 0002:0000016c       __imp__PathFileExistsW@4   0041916c     shlwapi:SHLWAPI.dll
 0002:00000170       \177SHLWAPI_NULL_THUNK_DATA 00419170     shlwapi:SHLWAPI.dll
 0002:00000174       __imp__KillTimer@8         00419174     user32:USER32.dll
 0002:00000178       __imp__LoadIconW@8         00419178     user32:USER32.dll
 0002:0000017c       __imp__IsWindow@4          0041917c     user32:USER32.dll
 0002:00000180       __imp__PostMessageA@16     00419180     user32:USER32.dll
 0002:00000184       __imp__SendMessageA@16     00419184     user32:USER32.dll
 0002:00000188       __imp__GetWindowThreadProcessId@8 00419188     user32:USER32.dll
 0002:0000018c       __imp__EnableWindow@8      0041918c     user32:USER32.dll
 0002:00000190       __imp__wsprintfA           00419190     user32:USER32.dll
 0002:00000194       \177USER32_NULL_THUNK_DATA 00419194     user32:USER32.dll
 0002:00000198       __imp___purecall           00419198     vcruntime:VCRUNTIME140.dll
 0002:0000019c       __imp__memset              0041919c     vcruntime:VCRUNTIME140.dll
 0002:000001a0       __imp____std_terminate     004191a0     vcruntime:VCRUNTIME140.dll
 0002:000001a4       __imp___CxxThrowException@8 004191a4     vcruntime:VCRUNTIME140.dll
 0002:000001a8       __imp__memmove             004191a8     vcruntime:VCRUNTIME140.dll
 0002:000001ac       __imp__memcpy              004191ac     vcruntime:VCRUNTIME140.dll
 0002:000001b0       __imp__strstr              004191b0     vcruntime:VCRUNTIME140.dll
 0002:000001b4       __imp____std_exception_copy 004191b4     vcruntime:VCRUNTIME140.dll
 0002:000001b8       __imp____std_exception_destroy 004191b8     vcruntime:VCRUNTIME140.dll
 0002:000001bc       __imp__memchr              004191bc     vcruntime:VCRUNTIME140.dll
 0002:000001c0       __imp____RTDynamicCast     004191c0     vcruntime:VCRUNTIME140.dll
 0002:000001c4       __imp__wcsrchr             004191c4     vcruntime:VCRUNTIME140.dll
 0002:000001c8       __imp___except_handler4_common 004191c8     vcruntime:VCRUNTIME140.dll
 0002:000001cc       __imp____CxxFrameHandler3  004191cc     vcruntime:VCRUNTIME140.dll
 0002:000001d0       \177VCRUNTIME140_NULL_THUNK_DATA 004191d0     vcruntime:VCRUNTIME140.dll
 0002:000001d4       __imp__WinHttpConnect@16   004191d4     winhttp:WINHTTP.dll
 0002:000001d8       __imp__WinHttpWriteData@16 004191d8     winhttp:WINHTTP.dll
 0002:000001dc       __imp__WinHttpOpen@20      004191dc     winhttp:WINHTTP.dll
 0002:000001e0       __imp__WinHttpSendRequest@28 004191e0     winhttp:WINHTTP.dll
 0002:000001e4       __imp__WinHttpReceiveResponse@8 004191e4     winhttp:WINHTTP.dll
 0002:000001e8       __imp__WinHttpQueryHeaders@24 004191e8     winhttp:WINHTTP.dll
 0002:000001ec       __imp__WinHttpOpenRequest@28 004191ec     winhttp:WINHTTP.dll
 0002:000001f0       __imp__WinHttpCloseHandle@4 004191f0     winhttp:WINHTTP.dll
 0002:000001f4       __imp__WinHttpCrackUrl@16  004191f4     winhttp:WINHTTP.dll
 0002:000001f8       \177WINHTTP_NULL_THUNK_DATA 004191f8     winhttp:WINHTTP.dll
 0002:000001fc       __imp__InternetReadFile@16 004191fc     wininet:WININET.dll
 0002:00000200       __imp__InternetCloseHandle@4 00419200     wininet:WININET.dll
 0002:00000204       __imp__InternetOpenA@20    00419204     wininet:WININET.dll
 0002:00000208       __imp__InternetOpenUrlA@24 00419208     wininet:WININET.dll
 0002:0000020c       \177WININET_NULL_THUNK_DATA 0041920c     wininet:WININET.dll
 0002:00000210       __imp__timeGetTime@0       00419210     winmm:WINMM.dll
 0002:00000214       \177WINMM_NULL_THUNK_DATA  00419214     winmm:WINMM.dll
 0002:00000218       __imp__WSACleanup@0        00419218     ws2_32:WS2_32.dll
 0002:0000021c       __imp__WSAStartup@8        0041921c     ws2_32:WS2_32.dll
 0002:00000220       __imp__gethostname@8       00419220     ws2_32:WS2_32.dll
 0002:00000224       \177WS2_32_NULL_THUNK_DATA 00419224     ws2_32:WS2_32.dll
 0002:00000228       __imp__mbstowcs            00419228     ucrt:api-ms-win-crt-convert-l1-1-0.dll
 0002:0000022c       __imp__atoi                0041922c     ucrt:api-ms-win-crt-convert-l1-1-0.dll
 0002:00000230       __imp__atol                00419230     ucrt:api-ms-win-crt-convert-l1-1-0.dll
 0002:00000234       \177api-ms-win-crt-convert-l1-1-0_NULL_THUNK_DATA 00419234     ucrt:api-ms-win-crt-convert-l1-1-0.dll
 0002:00000238       __imp__remove              00419238     ucrt:api-ms-win-crt-filesystem-l1-1-0.dll
 0002:0000023c       __imp___mkdir              0041923c     ucrt:api-ms-win-crt-filesystem-l1-1-0.dll
 0002:00000240       __imp___splitpath_s        00419240     ucrt:api-ms-win-crt-filesystem-l1-1-0.dll
 0002:00000244       __imp__rename              00419244     ucrt:api-ms-win-crt-filesystem-l1-1-0.dll
 0002:00000248       \177api-ms-win-crt-filesystem-l1-1-0_NULL_THUNK_DATA 00419248     ucrt:api-ms-win-crt-filesystem-l1-1-0.dll
 0002:0000024c       __imp___set_new_mode       0041924c     ucrt:api-ms-win-crt-heap-l1-1-0.dll
 0002:00000250       __imp__free                00419250     ucrt:api-ms-win-crt-heap-l1-1-0.dll
 0002:00000254       \177api-ms-win-crt-heap-l1-1-0_NULL_THUNK_DATA 00419254     ucrt:api-ms-win-crt-heap-l1-1-0.dll
 0002:00000258       __imp___setmbcp            00419258     ucrt:api-ms-win-crt-locale-l1-1-0.dll
 0002:0000025c       __imp___configthreadlocale 0041925c     ucrt:api-ms-win-crt-locale-l1-1-0.dll
 0002:00000260       \177api-ms-win-crt-locale-l1-1-0_NULL_THUNK_DATA 00419260     ucrt:api-ms-win-crt-locale-l1-1-0.dll
 0002:00000264       __imp___libm_sse2_sqrt_precise 00419264     ucrt:api-ms-win-crt-math-l1-1-0.dll
 0002:00000268       __imp___libm_sse2_atan_precise 00419268     ucrt:api-ms-win-crt-math-l1-1-0.dll
 0002:0000026c       __imp____setusermatherr    0041926c     ucrt:api-ms-win-crt-math-l1-1-0.dll
 0002:00000270       \177api-ms-win-crt-math-l1-1-0_NULL_THUNK_DATA 00419270     ucrt:api-ms-win-crt-math-l1-1-0.dll
 0002:00000274       __imp____p___argv          00419274     ucrt:api-ms-win-crt-runtime-l1-1-0.dll
 0002:00000278       __imp____p___argc          00419278     ucrt:api-ms-win-crt-runtime-l1-1-0.dll
 0002:0000027c       __imp___invalid_parameter_noinfo_noreturn 0041927c     ucrt:api-ms-win-crt-runtime-l1-1-0.dll
 0002:00000280       __imp___beginthread        00419280     ucrt:api-ms-win-crt-runtime-l1-1-0.dll
 0002:00000284       __imp___controlfp_s        00419284     ucrt:api-ms-win-crt-runtime-l1-1-0.dll
 0002:00000288       __imp__terminate           00419288     ucrt:api-ms-win-crt-runtime-l1-1-0.dll
 0002:0000028c       __imp___endthread          0041928c     ucrt:api-ms-win-crt-runtime-l1-1-0.dll
 0002:00000290       __imp___register_thread_local_exe_atexit_callback 00419290     ucrt:api-ms-win-crt-runtime-l1-1-0.dll
 0002:00000294       __imp___c_exit             00419294     ucrt:api-ms-win-crt-runtime-l1-1-0.dll
 0002:00000298       __imp___set_invalid_parameter_handler 00419298     ucrt:api-ms-win-crt-runtime-l1-1-0.dll
 0002:0000029c       __imp___exit               0041929c     ucrt:api-ms-win-crt-runtime-l1-1-0.dll
 0002:000002a0       __imp__exit                004192a0     ucrt:api-ms-win-crt-runtime-l1-1-0.dll
 0002:000002a4       __imp___initterm_e         004192a4     ucrt:api-ms-win-crt-runtime-l1-1-0.dll
 0002:000002a8       __imp___initterm           004192a8     ucrt:api-ms-win-crt-runtime-l1-1-0.dll
 0002:000002ac       __imp___get_narrow_winmain_command_line 004192ac     ucrt:api-ms-win-crt-runtime-l1-1-0.dll
 0002:000002b0       __imp___initialize_onexit_table 004192b0     ucrt:api-ms-win-crt-runtime-l1-1-0.dll
 0002:000002b4       __imp___set_app_type       004192b4     ucrt:api-ms-win-crt-runtime-l1-1-0.dll
 0002:000002b8       __imp___seh_filter_exe     004192b8     ucrt:api-ms-win-crt-runtime-l1-1-0.dll
 0002:000002bc       __imp___cexit              004192bc     ucrt:api-ms-win-crt-runtime-l1-1-0.dll
 0002:000002c0       __imp___crt_atexit         004192c0     ucrt:api-ms-win-crt-runtime-l1-1-0.dll
 0002:000002c4       __imp___register_onexit_function 004192c4     ucrt:api-ms-win-crt-runtime-l1-1-0.dll
 0002:000002c8       __imp___initialize_narrow_environment 004192c8     ucrt:api-ms-win-crt-runtime-l1-1-0.dll
 0002:000002cc       __imp___configure_narrow_argv 004192cc     ucrt:api-ms-win-crt-runtime-l1-1-0.dll
 0002:000002d0       \177api-ms-win-crt-runtime-l1-1-0_NULL_THUNK_DATA 004192d0     ucrt:api-ms-win-crt-runtime-l1-1-0.dll
 0002:000002d4       __imp____stdio_common_vsprintf 004192d4     ucrt:api-ms-win-crt-stdio-l1-1-0.dll
 0002:000002d8       __imp____stdio_common_vsnwprintf_s 004192d8     ucrt:api-ms-win-crt-stdio-l1-1-0.dll
 0002:000002dc       __imp__fclose              004192dc     ucrt:api-ms-win-crt-stdio-l1-1-0.dll
 0002:000002e0       __imp____stdio_common_vfprintf 004192e0     ucrt:api-ms-win-crt-stdio-l1-1-0.dll
 0002:000002e4       __imp___set_fmode          004192e4     ucrt:api-ms-win-crt-stdio-l1-1-0.dll
 0002:000002e8       __imp____stdio_common_vsnprintf_s 004192e8     ucrt:api-ms-win-crt-stdio-l1-1-0.dll
 0002:000002ec       __imp____p__commode        004192ec     ucrt:api-ms-win-crt-stdio-l1-1-0.dll
 0002:000002f0       __imp__fwrite              004192f0     ucrt:api-ms-win-crt-stdio-l1-1-0.dll
 0002:000002f4       __imp__fopen_s             004192f4     ucrt:api-ms-win-crt-stdio-l1-1-0.dll
 0002:000002f8       __imp___setmaxstdio        004192f8     ucrt:api-ms-win-crt-stdio-l1-1-0.dll
 0002:000002fc       __imp____stdio_common_vsprintf_s 004192fc     ucrt:api-ms-win-crt-stdio-l1-1-0.dll
 0002:00000300       __imp____stdio_common_vfscanf 00419300     ucrt:api-ms-win-crt-stdio-l1-1-0.dll
 0002:00000304       \177api-ms-win-crt-stdio-l1-1-0_NULL_THUNK_DATA 00419304     ucrt:api-ms-win-crt-stdio-l1-1-0.dll
 0002:00000308       __imp__strncpy_s           00419308     ucrt:api-ms-win-crt-string-l1-1-0.dll
 0002:0000030c       __imp__tolower             0041930c     ucrt:api-ms-win-crt-string-l1-1-0.dll
 0002:00000310       __imp__wcscpy_s            00419310     ucrt:api-ms-win-crt-string-l1-1-0.dll
 0002:00000314       __imp___wcsicmp            00419314     ucrt:api-ms-win-crt-string-l1-1-0.dll
 0002:00000318       __imp__strcat_s            00419318     ucrt:api-ms-win-crt-string-l1-1-0.dll
 0002:0000031c       __imp__strcpy_s            0041931c     ucrt:api-ms-win-crt-string-l1-1-0.dll
 0002:00000320       \177api-ms-win-crt-string-l1-1-0_NULL_THUNK_DATA 00419320     ucrt:api-ms-win-crt-string-l1-1-0.dll
 0002:00000324       __imp___time32             00419324     ucrt:api-ms-win-crt-time-l1-1-0.dll
 0002:00000328       \177api-ms-win-crt-time-l1-1-0_NULL_THUNK_DATA 00419328     ucrt:api-ms-win-crt-time-l1-1-0.dll
 0002:0000032c       __imp__srand               0041932c     ucrt:api-ms-win-crt-utility-l1-1-0.dll
 0002:00000330       \177api-ms-win-crt-utility-l1-1-0_NULL_THUNK_DATA 00419330     ucrt:api-ms-win-crt-utility-l1-1-0.dll
 0002:00000334       __imp__SymGetModuleBase64@12 00419334     DbgHelp:dbghelp.dll
 0002:00000338       __imp__SymFunctionTableAccess64@12 00419338     DbgHelp:dbghelp.dll
 0002:0000033c       __imp__EnumerateLoadedModules64@12 0041933c     DbgHelp:dbghelp.dll
 0002:00000340       __imp__SymCleanup@4        00419340     DbgHelp:dbghelp.dll
 0002:00000344       __imp__SymSetOptions@4     00419344     DbgHelp:dbghelp.dll
 0002:00000348       __imp__StackWalk64@36      00419348     DbgHelp:dbghelp.dll
 0002:0000034c       __imp__MiniDumpWriteDump@28 0041934c     DbgHelp:dbghelp.dll
 0002:00000350       __imp__SymInitialize@12    00419350     DbgHelp:dbghelp.dll
 0002:00000354       \177dbghelp_NULL_THUNK_DATA 00419354     DbgHelp:dbghelp.dll
 0002:00000358       __imp_?LoadAppLangResourceDLL@CWinApp@@UAEPAUHINSTANCE__@@XZ 00419358     mfc140:mfc140.dll
 0002:0000035c       __imp_?ProcessWndProcException@CWinApp@@UAEJPAVCException@@PBUtagMSG@@@Z 0041935c     mfc140:mfc140.dll
 0002:00000360       __imp_?OnIdle@CWinApp@@UAEHJ@Z 00419360     mfc140:mfc140.dll
 0002:00000364       __imp_?RestartInstance@CWinApp@@UAEHXZ 00419364     mfc140:mfc140.dll
 0002:00000368       __imp_?ExitInstance@CWinApp@@UAEHXZ 00419368     mfc140:mfc140.dll
 0002:0000036c       __imp_?IsTaskbarInteractionEnabled@CWinApp@@UAEHXZ 0041936c     mfc140:mfc140.dll
 0002:00000370       __imp_?GetDataRecoveryHandler@CWinApp@@UAEPAVCDataRecoveryHandler@@XZ 00419370     mfc140:mfc140.dll
 0002:00000374       __imp_?OnHelp@CWinApp@@IAEXXZ 00419374     mfc140:mfc140.dll
 0002:00000378       __imp_?ApplicationRecoveryCallback@CWinApp@@UAEKPAX@Z 00419378     mfc140:mfc140.dll
 0002:0000037c       __imp_?RegisterWithRestartManager@CWinApp@@UAEJPB_WKP6GKPAX@Z1KK@Z 0041937c     mfc140:mfc140.dll
 0002:00000380       __imp_?RegisterWithRestartManager@CWinApp@@UAEJHABV?$CStringT@DV?$StrTraitMFC_DLL@DV?$ChTraitsCRT@D@ATL@@@@@ATL@@@Z 00419380     mfc140:mfc140.dll
 0002:00000384       __imp_?OnInitDialog@CDialog@@UAEHXZ 00419384     mfc140:mfc140.dll
 0002:00000388       __imp_??0CDialog@@QAE@IPAVCWnd@@@Z 00419388     mfc140:mfc140.dll
 0002:0000038c       __imp_?CreateIndirect@CDialog@@UAEHPAXPAVCWnd@@@Z 0041938c     mfc140:mfc140.dll
 0002:00000390       __imp_?CreateIndirect@CDialog@@UAEHPBUDLGTEMPLATE@@PAVCWnd@@PAX@Z 00419390     mfc140:mfc140.dll
 0002:00000394       __imp_?Create@CDialog@@UAEHPBDPAVCWnd@@@Z 00419394     mfc140:mfc140.dll
 0002:00000398       __imp_?GetRuntimeClass@CDialog@@UBEPAUCRuntimeClass@@XZ 00419398     mfc140:mfc140.dll
 0002:0000039c       __imp_?GetMessageMap@CWnd@@MBEPBUAFX_MSGMAP@@XZ 0041939c     mfc140:mfc140.dll
 0002:000003a0       __imp_?GetOccDialogInfo@CWnd@@MAEPAU_AFX_OCC_DIALOG_INFO@@XZ 004193a0     mfc140:mfc140.dll
 0002:000003a4       __imp_?SetOccDialogInfo@CWnd@@MAEHPAU_AFX_OCC_DIALOG_INFO@@@Z 004193a4     mfc140:mfc140.dll
 0002:000003a8       __imp_?CreateControlSite@CWnd@@MAEHPAVCOleControlContainer@@PAPAVCOleControlSite@@IABU_GUID@@@Z 004193a8     mfc140:mfc140.dll
 0002:000003ac       __imp_??1CWinApp@@UAE@XZ   004193ac     mfc140:mfc140.dll
 0002:000003b0       __imp_?OnFinalRelease@CWnd@@UAEXXZ 004193b0     mfc140:mfc140.dll
 0002:000003b4       __imp_?IsFrameWnd@CWnd@@UBEHXZ 004193b4     mfc140:mfc140.dll
 0002:000003b8       __imp_?CheckAutoCenter@CWnd@@UAEHXZ 004193b8     mfc140:mfc140.dll
 0002:000003bc       __imp_?WinHelpInternal@CWinApp@@UAEXKI@Z 004193bc     mfc140:mfc140.dll
 0002:000003c0       __imp_?HtmlHelpA@CWinApp@@UAEXKI@Z 004193c0     mfc140:mfc140.dll
 0002:000003c4       __imp_?WinHelpA@CWinApp@@UAEXKI@Z 004193c4     mfc140:mfc140.dll
 0002:000003c8       __imp_?OnDDECommand@CWinApp@@UAEHPAD@Z 004193c8     mfc140:mfc140.dll
 0002:000003cc       __imp_?ResizeDynamicLayout@CWnd@@MAEXXZ 004193cc     mfc140:mfc140.dll
 0002:000003d0       __imp_?get_accHelp@CWnd@@UAEJUtagVARIANT@@PAPA_W@Z 004193d0     mfc140:mfc140.dll
 0002:000003d4       __imp_?OnChildNotify@CListBox@@MAEHIIJPAJ@Z 004193d4     mfc140:mfc140.dll
 0002:000003d8       __imp_?OnGestureTwoFingerTap@CWnd@@MAEHVCPoint@@@Z 004193d8     mfc140:mfc140.dll
 0002:000003dc       __imp_?OnGestureRotate@CWnd@@MAEHVCPoint@@N@Z 004193dc     mfc140:mfc140.dll
 0002:000003e0       __imp_?OnGesturePan@CWnd@@MAEHVCPoint@@0@Z 004193e0     mfc140:mfc140.dll
 0002:000003e4       __imp_?OnGestureZoom@CWnd@@MAEHVCPoint@@J@Z 004193e4     mfc140:mfc140.dll
 0002:000003e8       __imp_?GetGestureStatus@CWnd@@MAEKVCPoint@@@Z 004193e8     mfc140:mfc140.dll
 0002:000003ec       __imp_?OnTouchInput@CWnd@@MAEHVCPoint@@HHPAUtagTOUCHINPUT@@@Z 004193ec     mfc140:mfc140.dll
 0002:000003f0       __imp_??1CListBox@@UAE@XZ  004193f0     mfc140:mfc140.dll
 0002:000003f4       __imp_?CharToItem@CListBox@@UAEHII@Z 004193f4     mfc140:mfc140.dll
 0002:000003f8       __imp_?VKeyToItem@CListBox@@UAEHII@Z 004193f8     mfc140:mfc140.dll
 0002:000003fc       __imp_??4?$CStringT@DV?$StrTraitMFC_DLL@DV?$ChTraitsCRT@D@ATL@@@@@ATL@@QAEAAV01@PBD@Z 004193fc     mfc140:mfc140.dll
 0002:00000400       __imp_?CompareItem@CListBox@@UAEHPAUtagCOMPAREITEMSTRUCT@@@Z 00419400     mfc140:mfc140.dll
 0002:00000404       __imp_?GetThisMessageMap@CWinApp@@KGPBUAFX_MSGMAP@@XZ 00419404     mfc140:mfc140.dll
 0002:00000408       __imp_?LoadSysPolicies@CWinApp@@UAEHXZ 00419408     mfc140:mfc140.dll
 0002:0000040c       __imp_?AfxThrowInvalidArgException@@YGXXZ 0041940c     mfc140:mfc140.dll
 0002:00000410       __imp_??B?$CSimpleStringT@D$00@ATL@@QBEPBDXZ 00419410     mfc140:mfc140.dll
 0002:00000414       __imp_?Empty@?$CSimpleStringT@D$00@ATL@@QAEXXZ 00419414     mfc140:mfc140.dll
 0002:00000418       __imp_?GetString@?$CSimpleStringT@D$00@ATL@@QBEPBDXZ 00419418     mfc140:mfc140.dll
 0002:0000041c       __imp_??0?$CStringT@DV?$StrTraitMFC_DLL@DV?$ChTraitsCRT@D@ATL@@@@@ATL@@QAE@XZ 0041941c     mfc140:mfc140.dll
 0002:00000420       __imp_?CreateControlContainer@CWnd@@MAEHPAPAVCOleControlContainer@@@Z 00419420     mfc140:mfc140.dll
 0002:00000424       __imp_??1?$CStringT@DV?$StrTraitMFC_DLL@DV?$ChTraitsCRT@D@ATL@@@@@ATL@@QAE@XZ 00419424     mfc140:mfc140.dll
 0002:00000428       __imp_?MeasureItem@CListBox@@UAEXPAUtagMEASUREITEMSTRUCT@@@Z 00419428     mfc140:mfc140.dll
 0002:0000042c       __imp_?DrawItem@CListBox@@UAEXPAUtagDRAWITEMSTRUCT@@@Z 0041942c     mfc140:mfc140.dll
 0002:00000430       __imp_?OnTouchInputs@CWnd@@MAEHIPAUtagTOUCHINPUT@@@Z 00419430     mfc140:mfc140.dll
 0002:00000434       __imp_?OnChildNotify@CWnd@@MAEHIIJPAJ@Z 00419434     mfc140:mfc140.dll
 0002:00000438       __imp_?PostNcDestroy@CWnd@@MAEXXZ 00419438     mfc140:mfc140.dll
 0002:0000043c       __imp_?DefWindowProcA@CWnd@@MAEJIIJ@Z 0041943c     mfc140:mfc140.dll
 0002:00000440       __imp_?Default@CWnd@@IAEJXZ 00419440     mfc140:mfc140.dll
 0002:00000444       __imp_?OnWndMsg@CWnd@@MAEHIIJPAJ@Z 00419444     mfc140:mfc140.dll
 0002:00000448       __imp_?WindowProc@CWnd@@MAEJIIJ@Z 00419448     mfc140:mfc140.dll
 0002:0000044c       __imp_?OnAmbientProperty@CWnd@@UAEHPAVCOleControlSite@@JPAUtagVARIANT@@@Z 0041944c     mfc140:mfc140.dll
 0002:00000450       __imp_?PreTranslateMessage@CWnd@@UAEHPAUtagMSG@@@Z 00419450     mfc140:mfc140.dll
 0002:00000454       __imp_?GetSuperWndProcAddr@CWnd@@MAEPAP6GJPAUHWND__@@IIJ@ZXZ 00419454     mfc140:mfc140.dll
 0002:00000458       __imp_?OnNotify@CWnd@@MAEHIJPAJ@Z 00419458     mfc140:mfc140.dll
 0002:0000045c       __imp_?OnCommand@CWnd@@MAEHIJ@Z 0041945c     mfc140:mfc140.dll
 0002:00000460       __imp_?CreateAccessibleProxy@CWnd@@UAEJIJPAJ@Z 00419460     mfc140:mfc140.dll
 0002:00000464       __imp_?SetProxy@CWnd@@UAEJPAUIAccessibleProxy@@@Z 00419464     mfc140:mfc140.dll
 0002:00000468       __imp_?put_accValue@CWnd@@UAEJUtagVARIANT@@PA_W@Z 00419468     mfc140:mfc140.dll
 0002:0000046c       __imp_?put_accName@CWnd@@UAEJUtagVARIANT@@PA_W@Z 0041946c     mfc140:mfc140.dll
 0002:00000470       __imp_?accDoDefaultAction@CWnd@@UAEJUtagVARIANT@@@Z 00419470     mfc140:mfc140.dll
 0002:00000474       __imp_?accHitTest@CWnd@@UAEJJJPAUtagVARIANT@@@Z 00419474     mfc140:mfc140.dll
 0002:00000478       __imp_?accNavigate@CWnd@@UAEJJUtagVARIANT@@PAU2@@Z 00419478     mfc140:mfc140.dll
 0002:0000047c       __imp_?accLocation@CWnd@@UAEJPAJ000UtagVARIANT@@@Z 0041947c     mfc140:mfc140.dll
 0002:00000480       __imp_?accSelect@CWnd@@UAEJJUtagVARIANT@@@Z 00419480     mfc140:mfc140.dll
 0002:00000484       __imp_?get_accDefaultAction@CWnd@@UAEJUtagVARIANT@@PAPA_W@Z 00419484     mfc140:mfc140.dll
 0002:00000488       __imp_?get_accSelection@CWnd@@UAEJPAUtagVARIANT@@@Z 00419488     mfc140:mfc140.dll
 0002:0000048c       __imp_?get_accFocus@CWnd@@UAEJPAUtagVARIANT@@@Z 0041948c     mfc140:mfc140.dll
 0002:00000490       __imp_?get_accKeyboardShortcut@CWnd@@UAEJUtagVARIANT@@PAPA_W@Z 00419490     mfc140:mfc140.dll
 0002:00000494       __imp_?get_accHelpTopic@CWnd@@UAEJPAPA_WUtagVARIANT@@PAJ@Z 00419494     mfc140:mfc140.dll
 0002:00000498       __imp_??Y?$CStringT@DV?$StrTraitMFC_DLL@DV?$ChTraitsCRT@D@ATL@@@@@ATL@@QAEAAV01@ABV?$CSimpleStringT@D$00@1@@Z 00419498     mfc140:mfc140.dll
 0002:0000049c       __imp_??Y?$CStringT@DV?$StrTraitMFC_DLL@DV?$ChTraitsCRT@D@ATL@@@@@ATL@@QAEAAV01@PBD@Z 0041949c     mfc140:mfc140.dll
 0002:000004a0       __imp_?Compare@?$CStringT@DV?$StrTraitMFC_DLL@DV?$ChTraitsCRT@D@ATL@@@@@ATL@@QBEHPBD@Z 004194a0     mfc140:mfc140.dll
 0002:000004a4       __imp_?FindOneOf@?$CStringT@DV?$StrTraitMFC_DLL@DV?$ChTraitsCRT@D@ATL@@@@@ATL@@QBEHPBD@Z 004194a4     mfc140:mfc140.dll
 0002:000004a8       __imp_?Format@?$CStringT@DV?$StrTraitMFC_DLL@DV?$ChTraitsCRT@D@ATL@@@@@ATL@@QAAXPBDZZ 004194a8     mfc140:mfc140.dll
 0002:000004ac       __imp_??0CFileFind@@QAE@XZ 004194ac     mfc140:mfc140.dll
 0002:000004b0       __imp_??1CFileFind@@UAE@XZ 004194b0     mfc140:mfc140.dll
 0002:000004b4       __imp_?Create@CListBox@@UAEHKABUtagRECT@@PAVCWnd@@I@Z 004194b4     mfc140:mfc140.dll
 0002:000004b8       __imp_?GetFileName@CFileFind@@UBE?AV?$CStringT@DV?$StrTraitMFC_DLL@DV?$ChTraitsCRT@D@ATL@@@@@ATL@@XZ 004194b8     mfc140:mfc140.dll
 0002:000004bc       __imp_?IsDots@CFileFind@@UBEHXZ 004194bc     mfc140:mfc140.dll
 0002:000004c0       __imp_?GetRuntimeClass@CListBox@@UBEPAUCRuntimeClass@@XZ 004194c0     mfc140:mfc140.dll
 0002:000004c4       __imp_?GetThisMessageMap@CDialog@@KGPBUAFX_MSGMAP@@XZ 004194c4     mfc140:mfc140.dll
 0002:000004c8       __imp_?Close@CFileFind@@QAEXXZ 004194c8     mfc140:mfc140.dll
 0002:000004cc       __imp_?FindFile@CFileFind@@UAEHPBDK@Z 004194cc     mfc140:mfc140.dll
 0002:000004d0       __imp_?FindNextFileA@CFileFind@@UAEHXZ 004194d0     mfc140:mfc140.dll
 0002:000004d4       __imp_?OnPaint@CDialog@@IAEXXZ 004194d4     mfc140:mfc140.dll
 0002:000004d8       __imp_?PreInitDialog@CDialog@@MAEXXZ 004194d8     mfc140:mfc140.dll
 0002:000004dc       __imp_??0CStringList@@QAE@H@Z 004194dc     mfc140:mfc140.dll
 0002:000004e0       __imp_?AddTail@CStringList@@QAEPAU__POSITION@@ABV?$CStringT@DV?$StrTraitMFC_DLL@DV?$ChTraitsCRT@D@ATL@@@@@ATL@@@Z 004194e0     mfc140:mfc140.dll
 0002:000004e4       __imp_??1CStringList@@UAE@XZ 004194e4     mfc140:mfc140.dll
 0002:000004e8       __imp_?AfxGetModuleState@@YGPAVAFX_MODULE_STATE@@XZ 004194e8     mfc140:mfc140.dll
 0002:000004ec       __imp_?DDX_Control@@YGXPAVCDataExchange@@HAAVCWnd@@@Z 004194ec     mfc140:mfc140.dll
 0002:000004f0       __imp_?GetOccDialogInfo@CDialog@@MAEPAU_AFX_OCC_DIALOG_INFO@@XZ 004194f0     mfc140:mfc140.dll
 0002:000004f4       __imp_?BeginWaitCursor@CCmdTarget@@QAEXXZ 004194f4     mfc140:mfc140.dll
 0002:000004f8       __imp_?EndWaitCursor@CCmdTarget@@QAEXXZ 004194f8     mfc140:mfc140.dll
 0002:000004fc       __imp_?SetOccDialogInfo@CDialog@@MAEHPAU_AFX_OCC_DIALOG_INFO@@@Z 004194fc     mfc140:mfc140.dll
 0002:00000500       __imp_??0CWnd@@QAE@XZ      00419500     mfc140:mfc140.dll
 0002:00000504       __imp_?PreSubclassWindow@CWnd@@UAEXXZ 00419504     mfc140:mfc140.dll
 0002:00000508       __imp_?Create@CWnd@@UAEHPBD0KABUtagRECT@@PAV1@IPAUCCreateContext@@@Z 00419508     mfc140:mfc140.dll
 0002:0000050c       __imp_?CheckAutoCenter@CDialog@@UAEHXZ 0041950c     mfc140:mfc140.dll
 0002:00000510       __imp_?CreateEx@CWnd@@UAEHKPBD0KHHHHPAUHWND__@@PAUHMENU__@@PAX@Z 00419510     mfc140:mfc140.dll
 0002:00000514       __imp_?CreateEx@CWnd@@UAEHKPBD0KABUtagRECT@@PAV1@IPAX@Z 00419514     mfc140:mfc140.dll
 0002:00000518       __imp_?DestroyWindow@CWnd@@UAEHXZ 00419518     mfc140:mfc140.dll
 0002:0000051c       __imp_?PreCreateWindow@CWnd@@UAEHAAUtagCREATESTRUCTA@@@Z 0041951c     mfc140:mfc140.dll
 0002:00000520       __imp_?CalcWindowRect@CWnd@@UAEXPAUtagRECT@@I@Z 00419520     mfc140:mfc140.dll
 0002:00000524       __imp_?GetDlgItem@CWnd@@QBEPAV1@H@Z 00419524     mfc140:mfc140.dll
 0002:00000528       __imp_?SetWindowTextA@CWnd@@QAEXPBD@Z 00419528     mfc140:mfc140.dll
 0002:0000052c       __imp_?GetWindowTextA@CWnd@@QBEHPADH@Z 0041952c     mfc140:mfc140.dll
 0002:00000530       __imp_?GetMenu@CWnd@@UBEPAVCMenu@@XZ 00419530     mfc140:mfc140.dll
 0002:00000534       __imp_?SetMenu@CWnd@@UAEHPAVCMenu@@@Z 00419534     mfc140:mfc140.dll
 0002:00000538       __imp_?OnToolHitTest@CWnd@@UBEHVCPoint@@PAUtagTOOLINFOA@@@Z 00419538     mfc140:mfc140.dll
 0002:0000053c       __imp_?SetFocus@CWnd@@QAEPAV1@XZ 0041953c     mfc140:mfc140.dll
 0002:00000540       __imp_?GetScrollBarCtrl@CWnd@@UBEPAVCScrollBar@@H@Z 00419540     mfc140:mfc140.dll
 0002:00000544       __imp_?MessageBoxA@CWnd@@QAEHPBD0I@Z 00419544     mfc140:mfc140.dll
 0002:00000548       __imp_?WinHelpA@CWnd@@UAEXKI@Z 00419548     mfc140:mfc140.dll
 0002:0000054c       __imp_?HtmlHelpA@CWnd@@UAEXKI@Z 0041954c     mfc140:mfc140.dll
 0002:00000550       __imp_?WinHelpInternal@CWnd@@UAEXKI@Z 00419550     mfc140:mfc140.dll
 0002:00000554       __imp_?ContinueModal@CWnd@@UAEHXZ 00419554     mfc140:mfc140.dll
 0002:00000558       __imp_?EndModalLoop@CWnd@@UAEXH@Z 00419558     mfc140:mfc140.dll
 0002:0000055c       __imp_?OnDrawIconicThumbnailOrLivePreview@CWnd@@UAEXAAVCDC@@VCRect@@VCSize@@HAAH@Z 0041955c     mfc140:mfc140.dll
 0002:00000560       __imp_?GetInterfaceMap@CWnd@@MBEPBUAFX_INTERFACEMAP@@XZ 00419560     mfc140:mfc140.dll
 0002:00000564       __imp_?EnsureStdObj@CWnd@@UAEJXZ 00419564     mfc140:mfc140.dll
 0002:00000568       __imp_?get_accParent@CWnd@@UAEJPAPAUIDispatch@@@Z 00419568     mfc140:mfc140.dll
 0002:0000056c       __imp_?OnCmdMsg@CDialog@@UAEHIHPAXPAUAFX_CMDHANDLERINFO@@@Z 0041956c     mfc140:mfc140.dll
 0002:00000570       __imp_?PreTranslateMessage@CDialog@@UAEHPAUtagMSG@@@Z 00419570     mfc140:mfc140.dll
 0002:00000574       __imp_?get_accChildCount@CWnd@@UAEJPAJ@Z 00419574     mfc140:mfc140.dll
 0002:00000578       __imp_?get_accChild@CWnd@@UAEJUtagVARIANT@@PAPAUIDispatch@@@Z 00419578     mfc140:mfc140.dll
 0002:0000057c       __imp_?get_accName@CWnd@@UAEJUtagVARIANT@@PAPA_W@Z 0041957c     mfc140:mfc140.dll
 0002:00000580       __imp_?get_accValue@CWnd@@UAEJUtagVARIANT@@PAPA_W@Z 00419580     mfc140:mfc140.dll
 0002:00000584       __imp_?get_accDescription@CWnd@@UAEJUtagVARIANT@@PAPA_W@Z 00419584     mfc140:mfc140.dll
 0002:00000588       __imp_??1CDialog@@UAE@XZ   00419588     mfc140:mfc140.dll
 0002:0000058c       __imp_?get_accRole@CWnd@@UAEJUtagVARIANT@@PAU2@@Z 0041958c     mfc140:mfc140.dll
 0002:00000590       __imp_?get_accState@CWnd@@UAEJUtagVARIANT@@PAU2@@Z 00419590     mfc140:mfc140.dll
 0002:00000594       __imp_?GetRuntimeClass@CEdit@@UBEPAUCRuntimeClass@@XZ 00419594     mfc140:mfc140.dll
 0002:00000598       __imp_?AfxFreeLibrary@@YGHPAUHINSTANCE__@@@Z 00419598     mfc140:mfc140.dll
 0002:0000059c       __imp_?AfxLoadLibrary@@YGPAUHINSTANCE__@@PBD@Z 0041959c     mfc140:mfc140.dll
 0002:000005a0       __imp_?AfxMessageBox@@YGHPBDII@Z 004195a0     mfc140:mfc140.dll
 0002:000005a4       __imp_?AfxFindResourceHandle@@YGPAUHINSTANCE__@@PBD0@Z 004195a4     mfc140:mfc140.dll
 0002:000005a8       __imp_?OnCancel@CDialog@@MAEXXZ 004195a8     mfc140:mfc140.dll
 0002:000005ac       __imp_?DeleteItem@CListBox@@UAEXPAUtagDELETEITEMSTRUCT@@@Z 004195ac     mfc140:mfc140.dll
 0002:000005b0       __imp_?OnOK@CDialog@@MAEXXZ 004195b0     mfc140:mfc140.dll
 0002:000005b4       __imp_??1CEdit@@UAE@XZ     004195b4     mfc140:mfc140.dll
 0002:000005b8       __imp_?OnGesturePressAndTap@CWnd@@MAEHVCPoint@@J@Z 004195b8     mfc140:mfc140.dll
 0002:000005bc       __imp_?OnSetFont@CDialog@@UAEXPAVCFont@@@Z 004195bc     mfc140:mfc140.dll
 0002:000005c0       __imp_?DoMessageBox@CWinApp@@UAEHPBDII@Z 004195c0     mfc140:mfc140.dll
 0002:000005c4       __imp_?SaveAllModified@CWinApp@@UAEHXZ 004195c4     mfc140:mfc140.dll
 0002:000005c8       __imp_?InitApplication@CWinApp@@UAEHXZ 004195c8     mfc140:mfc140.dll
 0002:000005cc       __imp_?AddToRecentFileList@CWinApp@@UAEXPBD@Z 004195cc     mfc140:mfc140.dll
 0002:000005d0       __imp_?OpenDocumentFile@CWinApp@@UAEPAVCDocument@@PBDH@Z 004195d0     mfc140:mfc140.dll
 0002:000005d4       __imp_?OpenDocumentFile@CWinApp@@UAEPAVCDocument@@PBD@Z 004195d4     mfc140:mfc140.dll
 0002:000005d8       __imp_?Unregister@CWinApp@@UAEHXZ 004195d8     mfc140:mfc140.dll
 0002:000005dc       __imp_?Register@CWinApp@@UAEHXZ 004195dc     mfc140:mfc140.dll
 0002:000005e0       __imp_?InitLibId@CWinApp@@UAEXXZ 004195e0     mfc140:mfc140.dll
 0002:000005e4       __imp_?WriteProfileBinary@CWinApp@@UAEHPBD0PAEI@Z 004195e4     mfc140:mfc140.dll
 0002:000005e8       __imp_?GetProfileBinary@CWinApp@@UAEHPBD0PAPAEPAI@Z 004195e8     mfc140:mfc140.dll
 0002:000005ec       __imp_?WriteProfileStringA@CWinApp@@UAEHPBD00@Z 004195ec     mfc140:mfc140.dll
 0002:000005f0       __imp_?GetProfileStringA@CWinApp@@UAE?AV?$CStringT@DV?$StrTraitMFC_DLL@DV?$ChTraitsCRT@D@ATL@@@@@ATL@@PBD00@Z 004195f0     mfc140:mfc140.dll
 0002:000005f4       __imp_?WriteProfileInt@CWinApp@@UAEHPBD0H@Z 004195f4     mfc140:mfc140.dll
 0002:000005f8       __imp_?GetProfileIntA@CWinApp@@UAEIPBD0H@Z 004195f8     mfc140:mfc140.dll
 0002:000005fc       __imp_??0CWinApp@@QAE@PBD@Z 004195fc     mfc140:mfc140.dll
 0002:00000600       __imp_?GetRuntimeClass@CWinApp@@UBEPAUCRuntimeClass@@XZ 00419600     mfc140:mfc140.dll
 0002:00000604       __imp_?Delete@CWinThread@@UAEXXZ 00419604     mfc140:mfc140.dll
 0002:00000608       __imp_?GetMainWnd@CWinThread@@UAEPAVCWnd@@XZ 00419608     mfc140:mfc140.dll
 0002:0000060c       __imp_?ProcessMessageFilter@CWinThread@@UAEHHPAUtagMSG@@@Z 0041960c     mfc140:mfc140.dll
 0002:00000610       __imp_?IsIdleMessage@CWinThread@@UAEHPAUtagMSG@@@Z 00419610     mfc140:mfc140.dll
 0002:00000614       __imp_?PumpMessage@CWinThread@@UAEHXZ 00419614     mfc140:mfc140.dll
 0002:00000618       __imp_?PreTranslateMessage@CWinThread@@UAEHPAUtagMSG@@@Z 00419618     mfc140:mfc140.dll
 0002:0000061c       __imp_?DoModal@CDialog@@UAEHXZ 0041961c     mfc140:mfc140.dll
 0002:00000620       __imp_?GetConnectionHook@CCmdTarget@@MAEPAUIConnectionPoint@@ABU_GUID@@@Z 00419620     mfc140:mfc140.dll
 0002:00000624       __imp_?GetExtraConnectionPoints@CCmdTarget@@MAEHPAVCPtrArray@@@Z 00419624     mfc140:mfc140.dll
 0002:00000628       __imp_?GetInterfaceHook@CCmdTarget@@UAEPAUIUnknown@@PBX@Z 00419628     mfc140:mfc140.dll
 0002:0000062c       __imp_?OnCreateAggregates@CCmdTarget@@UAEHXZ 0041962c     mfc140:mfc140.dll
 0002:00000630       __imp_?GetEventSinkMap@CCmdTarget@@MBEPBUAFX_EVENTSINKMAP@@XZ 00419630     mfc140:mfc140.dll
 0002:00000634       __imp_?GetInterfaceMap@CCmdTarget@@MBEPBUAFX_INTERFACEMAP@@XZ 00419634     mfc140:mfc140.dll
 0002:00000638       __imp_?GetConnectionMap@CCmdTarget@@MBEPBUAFX_CONNECTIONMAP@@XZ 00419638     mfc140:mfc140.dll
 0002:0000063c       __imp_?GetDispatchMap@CCmdTarget@@MBEPBUAFX_DISPMAP@@XZ 0041963c     mfc140:mfc140.dll
 0002:00000640       __imp_?GetCommandMap@CCmdTarget@@MBEPBUAFX_OLECMDMAP@@XZ 00419640     mfc140:mfc140.dll
 0002:00000644       __imp_?GetTypeLib@CCmdTarget@@UAEJKPAPAUITypeLib@@@Z 00419644     mfc140:mfc140.dll
 0002:00000648       __imp_?GetTypeLibCache@CCmdTarget@@UAEPAVCTypeLibCache@@XZ 00419648     mfc140:mfc140.dll
 0002:0000064c       __imp_?GetTypeInfoCount@CCmdTarget@@UAEIXZ 0041964c     mfc140:mfc140.dll
 0002:00000650       __imp_?GetDispatchIID@CCmdTarget@@UAEHPAU_GUID@@@Z 00419650     mfc140:mfc140.dll
 0002:00000654       __imp_?IsInvokeAllowed@CCmdTarget@@UAEHJ@Z 00419654     mfc140:mfc140.dll
 0002:00000658       __imp_?OnFinalRelease@CCmdTarget@@UAEXXZ 00419658     mfc140:mfc140.dll
 0002:0000065c       __imp_?OnCmdMsg@CCmdTarget@@UAEHIHPAXPAUAFX_CMDHANDLERINFO@@@Z 0041965c     mfc140:mfc140.dll
 0002:00000660       __imp_??_V@YAXPAX@Z        00419660     mfc140:mfc140.dll
 0002:00000664       __imp_??_U@YAPAXI@Z        00419664     mfc140:mfc140.dll
 0002:00000668       __imp_??2@YAPAXI@Z         00419668     mfc140:mfc140.dll
 0002:0000066c       __imp_??3@YAXPAX@Z         0041966c     mfc140:mfc140.dll
 0002:00000670       __imp_?DoWaitCursor@CWinApp@@UAEXH@Z 00419670     mfc140:mfc140.dll
 0002:00000674       __imp_?AfxWinMain@@YGHPAUHINSTANCE__@@0PADH@Z 00419674     mfc140:mfc140.dll
 0002:00000678       \177mfc140_NULL_THUNK_DATA 00419678     mfc140:mfc140.dll
 0002:0000067c       ___guard_check_icall_fptr  0041967c     msvcrt:guard_support.obj
 0002:00000680       ___xc_a                    00419680     msvcrt:initializers.obj
 0002:000008a0       ___xc_z                    004198a0     msvcrt:initializers.obj
 0002:000008a4       ___xi_a                    004198a4     msvcrt:initializers.obj
 0002:000008b0       ___xi_z                    004198b0     msvcrt:initializers.obj
 0002:000008b4       ___xp_a                    004198b4     msvcrt:initializers.obj
 0002:000008b8       ___xp_z                    004198b8     msvcrt:initializers.obj
 0002:000008bc       ___xt_a                    004198bc     msvcrt:initializers.obj
 0002:000008c0       ___xt_z                    004198c0     msvcrt:initializers.obj
 0002:000008d0       ??_C@_0BE@OHABKPEK@C?3?2log?2crossfire?2?$CFs@ 004198d0     RWPMLog.obj
 0002:000008e4       ??_C@_0BC@OFAGFEDM@?$CFs?2?$CFsdmp_?$CFs_?$CFs_?$CFs@ 004198e4     RWPMLog.obj
 0002:000008f8       ??_C@_0CC@FCEOPKOK@?$CF04d?$CF02d?$CF02d?9?$CF02d?$CF02d?$CF02d?$CF03d?4d@ 004198f8     RWPMLog.obj
 0002:0000091c       ??_C@_0BF@PAFLOJOC@?$CFs?2?$CFs?2error_?$CFs_?$CFs_?$CFs@ 0041991c     RWPMLog.obj
 0002:00000934       ??_C@_0BH@BGKMKGAL@?$CFs?2?$CFs?2etcinfo_?$CFs_?$CFs_?$CFs@ 00419934     RWPMLog.obj
 0002:0000094c       ??_C@_0BI@MAFDGCG@?$CFs?2?$CFs?2timeinfo_?$CFs_?$CFs_?$CFs@ 0041994c     RWPMLog.obj
 0002:00000964       ??_C@_0BE@DLJIFIGP@?$CFs?2timeout_?$CFs_?$CFs_?$CFs@ 00419964     RWPMLog.obj
 0002:00000978       ??_C@_0BI@BFLOLCHE@?$CFs?2?$CFs?2hackinfo_?$CFs_?$CFs_?$CFs@ 00419978     RWPMLog.obj
 0002:00000990       ??_C@_0BF@NIKPBFD@?$CFs?2?$CFs?2count_?$CFs_?$CFs_?$CFs@ 00419990     RWPMLog.obj
 0002:000009a8       ??_C@_0BE@NIBECFME@?$CFs?2?$CFs?2cash_?$CFs_?$CFs_?$CFs@ 004199a8     RWPMLog.obj
 0002:000009bc       ??_C@_0BL@JIHHBEMK@?$CFs?2?$CFs?2UnknownData_?$CFs_?$CFs_?$CFs@ 004199bc     RWPMLog.obj
 0002:000009d8       ??_C@_0BJ@GPOCOIKE@?$CFs?2?$CFs?2Megaphone_?$CFs_?$CFs_?$CFs@ 004199d8     RWPMLog.obj
 0002:000009f4       ??_C@_0BM@OINMANIA@?$CFs?2?$CFs?2ConnectCheck_?$CFs_?$CFs_?$CFs@ 004199f4     RWPMLog.obj
 0002:00000a10       ??_C@_0BO@OHCBCKHH@?$CFs?2?$CFs?2EmergencyState_?$CFs_?$CFs_?$CFs@ 00419a10     RWPMLog.obj
 0002:00000a30       ??_C@_0BH@JGBNIBCF@?$CFs?2?$CFs?2Hacking_?$CFs_?$CFs_?$CFs@ 00419a30     RWPMLog.obj
 0002:00000a48       ??_C@_0BI@CEJKNALJ@?$CFs?2?$CFs?2KickUser_?$CFs_?$CFs_?$CFs@ 00419a48     RWPMLog.obj
 0002:00000a60       ??_C@_0BC@BCEHJAGO@?$CFs?2error_?$CFs_?$CFs_?$CFs@ 00419a60     RWPMLog.obj
 0002:00000a74       ??_C@_0BE@KIEDFKMI@?$CFs?2etcinfo_?$CFs_?$CFs_?$CFs@ 00419a74     RWPMLog.obj
 0002:00000a88       ??_C@_0BM@JIDBDENL@?$CFs?2?$CFs?2SettingCheck_?$CFs_?$CFs_?$CFs@ 00419a88     RWPMLog.obj
 0002:00000aa4       ??_C@_0BH@DNCJAHH@?$CFs?2?$CFs?2MgrData_?$CFs_?$CFs_?$CFs@ 00419aa4     RWPMLog.obj
 0002:00000abc       ??_C@_0BJ@BDENKDK@?$CFs?2?$CFs?2GachaData_?$CFs_?$CFs_?$CFs@ 00419abc     RWPMLog.obj
 0002:00000ad8       ??_C@_0BG@HJJFNLNJ@?$CFs?2?$CFs?2mailer_?$CFs_?$CFs_?$CFs@ 00419ad8     RWPMLog.obj
 0002:00000af0       ??_C@_0BN@CGPMEGO@?$CFs?2?$CFs?2TryWeaponItem_?$CFs_?$CFs_?$CFs@ 00419af0     RWPMLog.obj
 0002:00000b10       ??_C@_04LIFAFMCE@?$FL?$CFs?$FN@ 00419b10     RWPMLog.obj
 0002:00000b18       ??_C@_06HJNJJLFL@?$FL?$CFlld?$FN@ 00419b18     RWPMLog.obj
 0002:00000b20       ??_C@_0BP@BMCLPMN@?$CFs?0?5?$CFd?0?5MEMORY_ADDRESS?$FL?$CFd?$FN?0?5?$CFs@ 00419b20     RWPMLog.obj
 0002:00000b40       ??_C@_0BN@OCKGOCDF@?$CFs?0?5?$CFd?0?5PROTO_START_HOST?0?5?$CFs@ 00419b40     RWPMLog.obj
 0002:00000b60       ??_C@_0CB@GNMPLMEI@?$CFs?0?5?$CFd?0?5PROTO_GAME_USER_INFO?0?5?$CF@ 00419b60     RWPMLog.obj
 0002:00000b84       ??_C@_0DK@MGKONJKE@?$CFs?0?5?$CFd?0?5PROTO_GAMEGT_INGAME_AIG@ 00419b84     RWPMLog.obj
 0002:00000bc0       ??_C@_0P@IEFPNEK@?$CFs?0?5?$CFd?0?5?$CFs?0?5?$CFs@ 00419bc0     RWPMLog.obj
 0002:00000bd0       ??_C@_0CG@MCFHKALN@?$CFs?0?5?$CFd?0?5GAMEPROTO_SC_REMOVECLIE@ 00419bd0     RWPMLog.obj
 0002:00000bf8       ??_C@_0CB@GMLIEFM@?$CFs?0?5?$CFd?0?5GAMEPROTO_SS_GAMEEND?0?5?$CF@ 00419bf8     RWPMLog.obj
 0002:00000c1c       ??_C@_0CI@FMLCGOEC@?$CFs?0?5?$CFd?0?5GAMEPROTO_SC_HOST_USER_@ 00419c1c     RWPMLog.obj
 0002:00000c44       ??_C@_0BP@FHPFEAAB@?$CFs?0?5?$CFd?0?5CLANSTATREPORTDATA?0?5?$CFs@ 00419c44     RWPMLog.obj
 0002:00000c64       ??_C@_0BL@NGCIOLCH@?$CFs?0?5?$CFd?0?5PROTO_BAN_USER?0?5?$CFs@ 00419c64     RWPMLog.obj
 0002:00000c80       ??_C@_0DE@DCEKNMHJ@?$CFs?0?5?$CFd?0?5PROTO_GAMEGT_INGAME_AIG@ 00419c80     RWPMLog.obj
 0002:00000cb4       ??_C@_0DB@KKCKHLAM@?$CFs?0?5?$CFd?0?5PROTO_GAMEGT_MAPLOADING@ 00419cb4     RWPMLog.obj
 0002:00000ce8       ??_C@_0CE@NNGOJKJJ@?$CFs?0?5?$CFd?0?5GAMEPROTO_SC_SPY_CHANGE@ 00419ce8     RWPMLog.obj
 0002:00000d0c       ??_C@_0DB@CHJEFLPF@?$CFs?0?5?$CFd?0?5PROTO_GAMEGT_INGAME_FAR@ 00419d0c     RWPMLog.obj
 0002:00000d40       ??_C@_0CM@HCGEFML@?$CFs?0?5?$CFd?0?5PROTO_AI2_BONUSROUND_RE@ 00419d40     RWPMLog.obj
 0002:00000d6c       ??_C@_0DK@CBOHEJM@?$CFs?0?5?$CFd?0?5PROTO_GAMEGT_INGAME_AI3@ 00419d6c     RWPMLog.obj
 0002:00000da8       ??_C@_0CK@BAHPFFKB@?$CFs?0?5?$CFd?0?5PROTO_INSERT_CHARACTER_@ 00419da8     RWPMLog.obj
 0002:00000dd4       ??_C@_0CG@MMMIDGFA@?$CFs?0?5?$CFd?0?5PROTO_AI_EXTRA_REWARD_R@ 00419dd4     RWPMLog.obj
 0002:00000dfc       ??_C@_0CF@MEMHOFAF@?$CFs?0?5?$CFd?0?5PROTO_FINISHED_GAME_PRE@ 00419dfc     RWPMLog.obj
 0002:00000e24       ??_C@_0DB@LMMMOHOA@?$CFs?0?5?$CFd?0?5PROTO_SPEC_RECOMMENDROO@ 00419e24     RWPMLog.obj
 0002:00000e58       ??_C@_0DI@NJDEIFAK@?$CFs?0?5?$CFd?0?5PROTO_GAMEGT_AUTO_SIDE_@ 00419e58     RWPMLog.obj
 0002:00000e90       ??_C@_0CN@ICDKOKLE@?$CFs?0?5?$CFd?0?5PROTO_GMGMT_BATTLE_USER@ 00419e90     RWPMLog.obj
 0002:00000ec0       ??_C@_0CA@KKGOCMBD@?$CFs?0?5?$CFd?0?5BATTLE_ROYAL_RESULT?0?5?$CFs@ 00419ec0     RWPMLog.obj
 0002:00000ee4       ??_C@_00CNPNBAHC@@         00419ee4     ltmodule.obj
 0002:00000eec       ??_7CAPIHolderBase@@6B@    00419eec     ltmodule.obj
 0002:00000f00       ??_7CInterfaceDatabase@@6B@ 00419f00     ltmodule.obj
 0002:00000f2c       ??_7CInterfaceNameMgr@@6B@ 00419f2c     ltmodule.obj
 0002:00000f30       __real@3e800000            00419f30     ltmodule.obj
 0002:00000f34       __real@3f000000            00419f34     ltmodule.obj
 0002:00000f38       __real@3fccccccc0000000    00419f38     ltmodule.obj
 0002:00000f40       __real@3fe8ccccc0000000    00419f40     ltmodule.obj
 0002:00000f48       __real@3ff0000000000000    00419f48     ltmodule.obj
 0002:00000f50       __real@4010000000000000    00419f50     ltmodule.obj
 0002:00000f58       __real@4030000000000000    00419f58     ltmodule.obj
 0002:00000f60       __real@40400000            00419f60     ltmodule.obj
 0002:00000f64       __real@43340000            00419f64     ltmodule.obj
 0002:00000f70       __xmm@00000000ffffffffffffffffffffffff 00419f70     ltmodule.obj
 0002:00000f80       __xmm@00000001000000010000000100000001 00419f80     ltmodule.obj
 0002:00000f90       __xmm@322bcc77322bcc77322bcc77322bcc77 00419f90     ltmodule.obj
 0002:00000fa0       __xmm@38d1b71738d1b71738d1b71738d1b717 00419fa0     ltmodule.obj
 0002:00000fb0       __xmm@3c0efa353c0efa353c0efa353c0efa35 00419fb0     ltmodule.obj
 0002:00000fc0       __xmm@3c23d70a3c23d70a3c23d70a3c23d70a 00419fc0     ltmodule.obj
 0002:00000fd0       __xmm@3c8efa353c8efa353c8efa353c8efa35 00419fd0     ltmodule.obj
 0002:00000fe0       __xmm@3e22f9833e22f9833e22f9833e22f983 00419fe0     ltmodule.obj
 0002:00000ff0       __xmm@3ea2f9833ea2f9833ea2f9833ea2f983 00419ff0     ltmodule.obj
 0002:00001000       __xmm@3f0000003f0000003f0000003f000000 0041a000     ltmodule.obj
 0002:00001010       __xmm@3f490fdb3f490fdb3f490fdb3f490fdb 0041a010     ltmodule.obj
 0002:00001020       __xmm@3f800000000000000000000000000000 0041a020     ltmodule.obj
 0002:00001030       __xmm@3f8000003f8000003f8000003f800000 0041a030     ltmodule.obj
 0002:00001040       __xmm@3f8000003f8000003f800000bf800000 0041a040     ltmodule.obj
 0002:00001050       __xmm@3f800000bf800000bf800000bf800000 0041a050     ltmodule.obj
 0002:00001060       __xmm@3fc90fdb3fc90fdb3fc90fdb3fc90fdb 0041a060     ltmodule.obj
 0002:00001070       __xmm@3fffffff3fffffff3fffffff3fffffff 0041a070     ltmodule.obj
 0002:00001080       __xmm@40000000400000004000000040000000 0041a080     ltmodule.obj
 0002:00001090       __xmm@40490fdb40490fdb40490fdb40490fdb 0041a090     ltmodule.obj
 0002:000010a0       __xmm@40c90fdb40c90fdb40c90fdb40c90fdb 0041a0a0     ltmodule.obj
 0002:000010b0       __xmm@42652ee042652ee042652ee042652ee0 0041a0b0     ltmodule.obj
 0002:000010c0       __xmm@42fe000042fe000042fe000042fe0000 0041a0c0     ltmodule.obj
 0002:000010d0       __xmm@43340000433400004334000043340000 0041a0d0     ltmodule.obj
 0002:000010e0       __xmm@437f0000437f0000437f0000437f0000 0041a0e0     ltmodule.obj
 0002:000010f0       __xmm@43b4000043b4000043b4000043b40000 0041a0f0     ltmodule.obj
 0002:00001100       __xmm@7f7fc99e7f7fc99e7f7fc99e7f7fc99e 0041a100     ltmodule.obj
 0002:00001110       __xmm@7f8000007f8000007f8000007f800000 0041a110     ltmodule.obj
 0002:00001120       __xmm@7fffffff7fffffff7fffffff7fffffff 0041a120     ltmodule.obj
 0002:00001130       __xmm@80000000800000008000000080000000 0041a130     ltmodule.obj
 0002:00001140       __xmm@bf000000bf000000bf000000bf000000 0041a140     ltmodule.obj
 0002:00001150       __xmm@bf8000003f8000003f8000003f800000 0041a150     ltmodule.obj
 0002:00001160       __xmm@bf8000003f8000003f800000bf800000 0041a160     ltmodule.obj
 0002:00001170       __xmm@bf8000003f800000bf8000003f800000 0041a170     ltmodule.obj
 0002:00001180       __xmm@bf800000bf8000003f8000003f800000 0041a180     ltmodule.obj
 0002:00001190       __xmm@bf800000bf800000bf800000bf800000 0041a190     ltmodule.obj
 0002:000011a0       __xmm@c2fe0000c2fe0000c2fe0000c2fe0000 0041a1a0     ltmodule.obj
 0002:000011b0       __xmm@ffffffffffffffffffffffffffffffff 0041a1b0     ltmodule.obj
 0002:000011c4       ??_7CMustSyncObjectLog@@6B@ 0041a1c4     HostLogger.obj
 0002:000011c8       ??_C@_0BI@CFPLBAOH@invalid?5string?5position@ 0041a1c8     HostLogger.obj
 0002:000011e0       ??_C@_0O@EMHFIMLF@?4?2Setting?4ini@ 0041a1e0     HostLogger.obj
 0002:000011f0       ??_C@_08IGMCDLDE@LogLevel@ 0041a1f0     HostLogger.obj
 0002:000011fc       ??_C@_07KMMFIOCI@LogInfo@  0041a1fc     HostLogger.obj
 0002:00001204       ??_C@_06LFKIJBMM@IPCMsg@   0041a204     HostLogger.obj
 0002:0000120c       ??_C@_09HNBAJPOD@IPCMemory@ 0041a20c     HostLogger.obj
 0002:00001218       ??_C@_0N@MJMCCHJI@?2?$CFd?$CF02d?$CF02d?2@ 0041a218     HostLogger.obj
 0002:00001228       ??_C@_0BG@NJNBAHKK@?$CF04d?$CF02d?$CF02d_?$CF02d?4log@ 0041a228     HostLogger.obj
 0002:00001240       ??_C@_0BI@PDBNHNN@?$CFs?2BattleRoyal_?$CFs_?$CFs_?$CFs@ 0041a240     HostLogger.obj
 0002:00001258       ??_C@_0BD@PBMCFJCL@?$CFs?2kernel_?$CFs_?$CFs_?$CFs@ 0041a258     HostLogger.obj
 0002:0000126c       ??_C@_0BB@FLNJAMGH@?$CF04d?$CF02d?$CF02d?4log@ 0041a26c     HostLogger.obj
 0002:00001280       ??_C@_0BD@DFOFGCOM@?$CFs?2packet_?$CFs_?$CFs_?$CFs@ 0041a280     HostLogger.obj
 0002:00001294       ??_C@_0BM@EPJGHEGG@?$CFs?2mode_user_count_?$CFs_?$CFs_?$CFs@ 0041a294     HostLogger.obj
 0002:000012b0       ??_C@_0CA@HLCLJLLN@?$CFs?2serverapp_use_count_?$CFs_?$CFs_?$CFs@ 0041a2b0     HostLogger.obj
 0002:000012d0       ??_C@_0BB@HFDGAAKA@?$CFs?2RWPM_?$CFs_?$CFs_?$CFs@ 0041a2d0     HostLogger.obj
 0002:000012e4       ??_C@_0BD@PILJABOB@?$CFs?2IPCMSG_?$CFs_?$CFs_?$CFs@ 0041a2e4     HostLogger.obj
 0002:000012f8       ??_C@_02DPNLHKJD@a?$CL@    0041a2f8     HostLogger.obj
 0002:000012fc       ??_C@_0DE@LGCHENKA@?$CFs?0?$CFs?0?$CF04d?4?$CF02d?4?$CF02d?5?$CF02d?3?$CF02d?3@ 0041a2fc     HostLogger.obj
 0002:00001330       ??_C@_0CJ@NOHHCMFI@?$CF04d?9?$CF02d?9?$CF02d?9?$CF02d?3?$CF02d?3?$CF02d?4?$CF@ 0041a330     HostLogger.obj
 0002:0000135c       ??_C@_01KICIPPFI@?2@       0041a35c     HostLogger.obj
 0002:00001360       ??_C@_0BE@MNIJIMLO@?$CF02d?3?$CF02d?3?$CF02d?4?$CF03d@ 0041a360     HostLogger.obj
 0002:00001374       ??_C@_0L@PIHNNPCB@?$CFs?5?$FLLOW__?$FN@ 0041a374     HostLogger.obj
 0002:00001380       ??_C@_0L@GMIAMKIO@?$CFs?5?$FLINFO_?$FN@ 0041a380     HostLogger.obj
 0002:0000138c       ??_C@_0L@IHOLMJOP@?$CFs?5?$FLWARN_?$FN@ 0041a38c     HostLogger.obj
 0002:00001398       ??_C@_0L@ECIMMAAL@?$CFs?5?$FLERROR?$FN@ 0041a398     HostLogger.obj
 0002:000013a4       ??_C@_0L@IPABKGEK@?$CFs?5?$FLFATAL?$FN@ 0041a3a4     HostLogger.obj
 0002:000013b0       ??_C@_08IHOEFJCP@?$CFs?5?$CFs?5?$AN?6@ 0041a3b0     HostLogger.obj
 0002:000013bc       ??_C@_0CN@PIILFGPG@?4?1rez?1NationMsz?1MSG_DEFINE_Serv@ 0041a3bc     LogMsgManager.obj
 0002:000013ec       ??_C@_0BA@KICEHKPF@App_LogDataSize@ 0041a3ec     LogMsgManager.obj
 0002:000013fc       ??_C@_0BA@CGBPPCJP@App_LogData?9?$CFzd@ 0041a3fc     LogMsgManager.obj
 0002:0000140c       ??_C@_02DKCKIIND@?$CFs@    0041a40c     LogMsgManager.obj
 0002:00001410       ??_C@_0BD@OLBABOEK@vector?$DMT?$DO?5too?5long@ 0041a410     LogMsgManager.obj
 0002:00001428       ??_7FindXlsMsg@@6B@        0041a428     LoadXlsMsg.obj
 0002:0000142c       ??_C@_0BE@JONHPENG@map?1set?$DMT?$DO?5too?5long@ 0041a42c     LoadXlsMsg.obj
 0002:00001444       ??_7CServerAppApp@@6B@     0041a444     ServerApp.obj
 0002:00001598       ??_7?$CAPIHolder@VILTCommon@@@@6B@ 0041a598     ServerAppDlg.obj
 0002:000015a8       ??_C@_0BB@DCFJGGKM@ILTCommon?4Server@ 0041a5a8     ServerAppDlg.obj
 0002:000015c0       ??_7CListBox@@6B@          0041a5c0     ServerAppDlg.obj
 0002:0000174c       ??_7CEdit@@6B@             0041a74c     ServerAppDlg.obj
 0002:000018b8       ??_C@_0BP@OIEOKIDM@Exception?5thrown?5in?5destructor@ 0041a8b8     ServerAppDlg.obj
 0002:000018d8       ??_C@_0BB@HBOOMJBF@?$CFTs?5?$CI?$CFTs?3?$CFd?$CJ?6?$CFTs@ 0041a8d8     ServerAppDlg.obj
 0002:000018ec       ??_C@_0N@OMEMOKLE@?$CFTs?5?$CI?$CFTs?3?$CFd?$CJ@ 0041a8ec     ServerAppDlg.obj
 0002:00001900       ??_C@_0HG@IFNAKGBH@c?3?2program?5files?5?$CIx86?$CJ?2microsof@ 0041a900     ServerAppDlg.obj
 0002:0000197c       ??_7exception@std@@6B@     0041a97c     ServerAppDlg.obj
 0002:00001984       ??_C@_0BC@EOODALEL@Unknown?5exception@ 0041a984     ServerAppDlg.obj
 0002:00001998       ??_C@_0L@JBGDLKBH@read?5error@ 0041a998     ServerAppDlg.obj
 0002:000019a8       ??_7PROTO_SERVERAPPMSG_INIT@@6B@ 0041a9a8     ServerAppDlg.obj
 0002:000019c0       ??_C@_04BFAHMMK@?$CFlld@   0041a9c0     ServerAppDlg.obj
 0002:000019c8       ??_C@_0L@JODCLDGE@RTID?3?$CFs?3?$CFd@ 0041a9c8     ServerAppDlg.obj
 0002:000019d8       ??_7CGameServerAppHandler@@6B@ 0041a9d8     ServerAppDlg.obj
 0002:00001a04       ??_7CServerAppDlg@@6B@     0041aa04     ServerAppDlg.obj
 0002:00001b98       ??_C@_0BO@KPHFACMM@ServerappIndex?$CI?$CFd?$CJ?0?5Port?$CI?$CFd?$CJ?5@ 0041ab98     ServerAppDlg.obj
 0002:00001bb8       ??_C@_0EM@HPPCGKPO@GetProcessMemoryUsage?$CI?$CJ?5Get?5pid@ 0041abb8     ServerAppDlg.obj
 0002:00001c08       ??_C@_0FB@MCFDPFPL@GetProcessMemoryUsage?$CI?$CJ?5Open?5pr@ 0041ac08     ServerAppDlg.obj
 0002:00001c60       ??_C@_0FJ@NOKGHOF@GetProcessMemoryUsage?$CI?$CJ?5GetProc@ 0041ac60     ServerAppDlg.obj
 0002:00001d70       ??_C@_09BJIIPNM@LocalHost@ 0041ad70     ServerAppDlg.obj
 0002:00001d7c       ??_C@_0DB@MCLBLGGG@Number?5of?5parameters?5is?5invalid@ 0041ad7c     ServerAppDlg.obj
 0002:00001db0       ??_C@_0DP@PDKDOPFG@ServerApp?5Init?5GSM_WND_HANDLE?5?3@ 0041adb0     ServerAppDlg.obj
 0002:00001df0       ??_C@_0DF@FJFGJCKG@Invalid?5manager?5window?5handle?5f@ 0041adf0     ServerAppDlg.obj
 0002:00001e28       ??_C@_0CM@IIIDOGJI@Invalid?5server?5index?5found?4?5Ter@ 0041ae28     ServerAppDlg.obj
 0002:00001e54       ??_C@_06EAOLBNEK@?$CFld_?$CFd@ 0041ae54     ServerAppDlg.obj
 0002:00001e5c       ??_C@_09LKCCBOGN@ServerApp@ 0041ae5c     ServerAppDlg.obj
 0002:00001e68       ??_C@_0BC@LFNIPHGA@ReadProcessMemory@ 0041ae68     ServerAppDlg.obj
 0002:00001e7c       ??_C@_08NCCBLF@GameMgmt@   0041ae7c     ServerAppDlg.obj
 0002:00001e88       ??_C@_0BD@PBGEEFCK@WriteProcessMemory@ 0041ae88     ServerAppDlg.obj
 0002:00001e9c       ??_C@_0CM@GMMNNKDE@ReadProcessMemory?$DN?$CFd?0?5WriteProc@ 0041ae9c     ServerAppDlg.obj
 0002:00001ec8       ??_C@_0HI@HCIAJJJC@GAMESERVERMSG_REPORT_HWND?5PostM@ 0041aec8     ServerAppDlg.obj
 0002:00001f40       ??_C@_0CO@GKLAPNMD@GAMESERVERMSG_LOADING_COMPLETE?5@ 0041af40     ServerAppDlg.obj
 0002:00001f70       ??_C@_0CF@FEDDMDMI@Recv?5SERVERAPPMSG_ADDCLIENT?5?9?5U@ 0041af70     ServerAppDlg.obj
 0002:00001f98       ??_C@_06FKAFBJKH@?$FLSEND?$FN@ 0041af98     ServerAppDlg.obj
 0002:00001fa0       ??_C@_0EG@BLGLGGEG@CServerAppDlg?3?3OnShellMessage?3?3@ 0041afa0     ServerAppDlg.obj
 0002:00001fe8       ??_C@_0CF@INADFEIB@?7usn?5?$DN?5?$CFs?0?5Index?5?$DN?5?$CFd?0?5IsReward@ 0041afe8     ServerAppDlg.obj
 0002:00002010       ??_C@_0DP@HJDGIELG@CServerAppDlg?9OnShellMessage?3?3S@ 0041b010     ServerAppDlg.obj
 0002:00002050       ??_C@_0DJ@LJHNNKOC@?7usn?5?$DN?5?$CFs?0?5loop?5?$DN?5?$CFd?0?5IsReward?5@ 0041b050     ServerAppDlg.obj
 0002:00002090       ??_C@_0EG@LLNDFMKB@CServerAppDlg?3?3OnShellMessage?3?3@ 0041b090     ServerAppDlg.obj
 0002:000020d8       ??_C@_0EA@FGCLOCKG@CServerAppDlg?3?3OnShellMessage?3?3@ 0041b0d8     ServerAppDlg.obj
 0002:00002118       ??_C@_0EJ@KIIACGNL@CServerAppDlg?3?3OnShellMessage?3?3@ 0041b118     ServerAppDlg.obj
 0002:00002164       ??_C@_0BC@JEAOIFOC@?7usn?5?$DN?5?$CFs?0?5i?5?$DN?5?$CFd@ 0041b164     ServerAppDlg.obj
 0002:00002178       ??_C@_05GAPFHKKC@?$CBerr?3@ 0041b178     ServerAppDlg.obj
 0002:00002180       ??_C@_06DBEGDDG@?$CBhack?3@ 0041b180     ServerAppDlg.obj
 0002:00002188       ??_C@_0L@KNEIOOMH@server?4dll@ 0041b188     ServerAppDlg.obj
 0002:00002194       ??_C@_0N@MGAIABNC@CreateServer@ 0041b194     ServerAppDlg.obj
 0002:000021a8       ??_C@_0FP@EDNMACCM@CServerAppDlg?3?3LoadServer?$CI?$CJ?0?5Fa@ 0041b1a8     ServerAppDlg.obj
 0002:00002208       ??_C@_0BC@NENPAAMN@SetMasterDatabase@ 0041b208     ServerAppDlg.obj
 0002:0000221c       ??_C@_0BF@HFLCBNHD@Resource?5Load?5Failed@ 0041b21c     ServerAppDlg.obj
 0002:00002234       ??_C@_0N@LBFNJNAG@DeleteServer@ 0041b234     ServerAppDlg.obj
 0002:00002244       ??_C@_06NLDEMLK@HAHAHA@    0041b244     ServerAppDlg.obj
 0002:00002250       ??_C@_0GG@JJILFGJG@?$FLBossBattle?$FN?5Send?5SERVERAPPMSG_@ 0041b250     ServerAppDlg.obj
 0002:000022b8       ??_C@_0FN@INOHFAIE@Thread_SendGameInfo?$CI?$CJ?5SlotIndex@ 0041b2b8     ServerAppDlg.obj
 0002:00002318       ??_C@_0FN@JIPCCBPF@?$FLAIMode?$FN?5Thread_SendGameInfo?$CI?$CJ?5@ 0041b318     ServerAppDlg.obj
 0002:00002378       ??_C@_0ED@GKCGBJAB@GAMESERVERMSG_INSERTCHARACTER_A@ 0041b378     ServerAppDlg.obj
 0002:000023c0       ??_C@_0FJ@IGOJOCLB@CServerAppDlg?3?3ThreadUpdate?5Sen@ 0041b3c0     ServerAppDlg.obj
 0002:00002420       ??_C@_0FJ@BOALIPHF@CServerAppDlg?3?3ThreadUpdate?5Sen@ 0041b420     ServerAppDlg.obj
 0002:00002480       ??_C@_0FJ@HNGKKIND@CServerAppDlg?3?3ThreadUpdate?5Sen@ 0041b480     ServerAppDlg.obj
 0002:000024e0       ??_C@_0GN@EKGJFLNH@CServerAppDlg?3?3ThreadUpdate?5Sen@ 0041b4e0     ServerAppDlg.obj
 0002:00002550       ??_C@_0FD@BAOJIFFE@Thread_SendUserInfo?$CI?$CJ?5?5iCharact@ 0041b550     ServerAppDlg.obj
 0002:000025a8       ??_C@_0EA@GOMMNBJL@CServerAppDlg?3?3ThreadUpdate?5?9?5C@ 0041b5a8     ServerAppDlg.obj
 0002:000025e8       ??_C@_0DO@DOJLKLON@CServerAppDlg?3?3ThreadUpdate?5?9?5C@ 0041b5e8     ServerAppDlg.obj
 0002:00002628       ??_C@_0CO@ENFPBBBP@CServerAppDlg?3?3ThreadUpdate?5?9?5S@ 0041b628     ServerAppDlg.obj
 0002:00002658       ??_C@_0CM@EGAFBNIJ@CServerAppDlg?3?3ThreadUpdate?5?9?5S@ 0041b658     ServerAppDlg.obj
 0002:00002684       ??_C@_0DC@GMIOFBC@?$FLUCCLog?$FN?5rez?5file?5download?5succ@ 0041b684     ServerAppDlg.obj
 0002:000026b8       ??_C@_0DJ@PNMLFLAA@?$FLUCCLog?$FN?5rez?5file?5download?5fail@ 0041b6b8     ServerAppDlg.obj
 0002:000026f4       ??_C@_03IEEBNAED@rez@      0041b6f4     ServerAppDlg.obj
 0002:000026f8       ??_C@_08JFAGHOJI@?$CFs?2?$CK?4rez@ 0041b6f8     ServerAppDlg.obj
 0002:00002704       ??_C@_01IDAFKMJL@_@        0041b704     ServerAppDlg.obj
 0002:00002708       ??_C@_0BL@IJJEJKPA@S_P_F?3?5HOST_HEARTBEAT?5?3?5?$CFd@ 0041b708     ServerAppDlg.obj
 0002:00002728       ??_C@_0EP@CPNDGEAA@GAMESERVERMSG_LOAD_MAP?5?9?5tMapIn@ 0041b728     ServerAppDlg.obj
 0002:00002778       ??_C@_0GB@BLONMNPP@Error?5while?5processing?5SendToSe@ 0041b778     ServerAppDlg.obj
 0002:000027e0       ??_C@_0FC@CBEKAGGK@Error?5while?5processing?5SendToSe@ 0041b7e0     ServerAppDlg.obj
 0002:00002834       ??_C@_0CP@ODPBIJII@?$FLRECV?$FN?5tIndex?$FL?$CF02d?$FN?0?5msgID?$FL?$CF02d@ 0041b834     ServerAppDlg.obj
 0002:00002864       ??_C@_0DC@LELNLDON@Not?5Supported?5Message?$CB?$CB?$CB?$CB?$CB?5tInd@ 0041b864     ServerAppDlg.obj
 0002:00002898       ??_C@_0EH@NACBIGCG@?$FLRWPM?$FN?$FLERROR?5?3?5Not?5Supported?$CB?$CB?$FN@ 0041b898     ServerAppDlg.obj
 0002:000028e0       ??_C@_0GC@FCJGOKJC@g_sGameInfos?5?9?5Push?5GameInfo?5Su@ 0041b8e0     ServerAppDlg.obj
 0002:00002948       ??_C@_0FP@EONMPNCI@g_sGameInfos?5?9?5Push?5GameInfo?5Fa@ 0041b948     ServerAppDlg.obj
 0002:000029a8       ??_C@_0GG@NEAGNFAL@g_sUserInfos?5?9?5Push?5UserInfo?5Su@ 0041b9a8     ServerAppDlg.obj
 0002:00002a10       ??_C@_0GD@KPPLLAEO@g_sUserInfos?5?9?5Push?5UserInfo?5Fa@ 0041ba10     ServerAppDlg.obj
 0002:00002a74       ??_C@_0DB@BBOAIBIB@?$FLUCCLog?$FN?5Already?5Has?5the?5rez?5fi@ 0041ba74     ServerAppDlg.obj
 0002:00002aa8       ??_C@_0DA@IPOEBJEM@?$FLUCCLog?$FN?5start?5rez?5file?5downloa@ 0041baa8     ServerAppDlg.obj
 0002:00002ad8       ??_C@_0FK@CANCCIAA@?$FLUCCLog?$FN?5rez?5file?5download?5fail@ 0041bad8     ServerAppDlg.obj
 0002:00002b34       ??_C@_0BI@HNLBPJDH@RunConsoleString?5error?4@ 0041bb34     ServerAppDlg.obj
 0002:00002b4c       ??_C@_0CB@EMGJKHPD@Logger?5Init?5Failed?5?3?5ErrCode?$FL?$CFd@ 0041bb4c     ServerAppDlg.obj
 0002:00002b70       ??_C@_0CC@ILNGBDNH@Log?5Msz?5File?5Load?5Failed?4?5Level@ 0041bb70     ServerAppDlg.obj
 0002:00002b94       ??_C@_0BO@PFCCNDDI@Log?5Msz?5Entering?5Read?5Mode?4?4?4@ 0041bb94     ServerAppDlg.obj
 0002:00002bb4       ??_C@_0CC@OKBOBAOJ@Log?5Msz?5Read?9Mode?5Failed?4?5Level@ 0041bbb4     ServerAppDlg.obj
 0002:00002bd8       ??_C@_0BK@MPHOBHIK@Logger?5USAGE_READ?5Setted?4@ 0041bbd8     ServerAppDlg.obj
 0002:00002bf4       ??_C@_0CC@KAPLEABE@Log?5Msz?5File?5Load?5Failed?4?5Level@ 0041bbf4     ServerAppDlg.obj
 0002:00002c18       ??_C@_0BL@BMLEPNEM@Logger?5USAGE_NOUSE?5Setted?4@ 0041bc18     ServerAppDlg.obj
 0002:00002c34       ??_C@_0P@KCHJOCJL@?9SaveGameInfo?$DN@ 0041bc34     ServerAppDlg.obj
 0002:00002c44       ??_C@_02GMLFBBN@wb@        0041bc44     ServerAppDlg.obj
 0002:00002c48       ??_C@_0P@NBLHLNAC@?9LoadGameInfo?$DN@ 0041bc48     ServerAppDlg.obj
 0002:00002c58       ??_C@_01KDCPPGHE@r@        0041bc58     ServerAppDlg.obj
 0002:00002c5c       ??_C@_06GDNIANOG@?$CFs?5?$CFhd@ 0041bc5c     ServerAppDlg.obj
 0002:00002c64       ??_C@_05DIALNFFA@?$CFs?5?$CFd@ 0041bc64     ServerAppDlg.obj
 0002:00002c6c       ??_C@_05KDNLHNC@?$CFs?5?$CFf@ 0041bc6c     ServerAppDlg.obj
 0002:00002c74       ??_C@_01CLKCMJKC@?5@       0041bc74     ServerAppDlg.obj
 0002:00002c78       ??_C@_0FP@HECBBGFL@?$FLRWPM?$FNSEND?5PostMessage?5Failed?5M@ 0041bc78     ServerAppDlg.obj
 0002:00002cd8       ??_C@_0FI@KBICGMBM@?$FLRWPM?$FNSEND?5PostMessage?5Failed?5H@ 0041bcd8     ServerAppDlg.obj
 0002:00002d30       ??_C@_0EG@EGBOFFPH@?$FLRWPM?$FNSEND?5PostMessage?5Failed?5t@ 0041bd30     ServerAppDlg.obj
 0002:00002d78       ??_C@_0EA@PONNFNHJ@?$FLSEND?$FN?5tIndex?$FL?$CF02d?$FN?0?5msgID?$FL?$CF02d@ 0041bd78     ServerAppDlg.obj
 0002:00002db8       ??_C@_0FB@DAMIMBHN@?$FLRWPM?$FNWriteGSMMemory?5Failed?$CB?$CB?5m@ 0041bdb8     ServerAppDlg.obj
 0002:00002e10       ??_C@_0EI@EHKLMNFO@?$FLRWPM?$FNWriteGSMMemory?5Failed?$CB?$CB?5A@ 0041be10     ServerAppDlg.obj
 0002:00002e58       ??_C@_0EK@LCPIHJD@?$FLRWPM?$FNWriteGSMMemory?5Failed?$CB?$CB?5P@ 0041be58     ServerAppDlg.obj
 0002:00002ea8       ??_C@_0EM@ONMNGCCO@?$FLRWPM?$FNWriteGSMMemory?5Failed?$CB?$CB?5O@ 0041bea8     ServerAppDlg.obj
 0002:00002ef8       ??_C@_0FD@MJOAPBFH@?$FLRWPM?$FNWriteGSMMemory?5Failed?$CB?$CB?5W@ 0041bef8     ServerAppDlg.obj
 0002:00002f50       ??_C@_0FN@CMEINILJ@?$FLRWPM?$FNReadGSMMemory?5Failed?$CB?$CB?5m_@ 0041bf50     ServerAppDlg.obj
 0002:00002fb0       ??_C@_0FE@NEFIKGOD@?$FLRWPM?$FNReadGSMMemory?5Failed?$CB?$CB?5Ad@ 0041bfb0     ServerAppDlg.obj
 0002:00003008       ??_C@_0FG@OFPAPHCO@?$FLRWPM?$FNReadGSMMemory?5Failed?$CB?$CB?5bu@ 0041c008     ServerAppDlg.obj
 0002:00003060       ??_C@_0FJ@FBMAGNKE@?$FLRWPM?$FNReadGSMMemory?5Failed?$CB?$CB?5Pr@ 0041c060     ServerAppDlg.obj
 0002:000030c0       ??_C@_0FI@LNJBBJAM@?$FLRWPM?$FNReadGSMMemory?5Failed?$CB?$CB?5Op@ 0041c0c0     ServerAppDlg.obj
 0002:00003118       ??_C@_0FO@GEJFEOLN@?$FLRWPM?$FNReadGSMMemory?5Failed?$CB?$CB?5Re@ 0041c118     ServerAppDlg.obj
 0002:00003178       ??_C@_0FB@HONOMPA@?$FLRWPM?$FN?$FLERROR?5?3?5New?5Memory?5Error@ 0041c178     ServerAppDlg.obj
 0002:000031cc       ??_C@_06HMJBGFMB@?$FLRECV?$FN@ 0041c1cc     ServerAppDlg.obj
 0002:000031d4       ??_C@_0DE@PGLLLGDD@?$FLRWPM?$FN?$FLERROR?5?3?5New?5Memory?5Error@ 0041c1d4     ServerAppDlg.obj
 0002:00003208       ??_C@_0DI@NEKPHLAC@?$FLRWPM?$FN?$FLERROR?5?3?5New?5Memory?5Error@ 0041c208     ServerAppDlg.obj
 0002:00003240       ??_C@_0DL@INGPPNNG@Recv?5GAMESERVERMSG_INSERTCHARAC@ 0041c240     ServerAppDlg.obj
 0002:00003280       ??_C@_0FC@HOLPKAAP@?$FLRWPM?$FN?$FLERROR?5?3?5New?5Memory?5Error@ 0041c280     ServerAppDlg.obj
 0002:000032d8       ??_C@_0FB@GHOBMMIA@?$FLRWPM?$FN?$FLERROR?5?3?5New?5Memory?5Error@ 0041c2d8     ServerAppDlg.obj
 0002:00003330       ??_C@_0ED@JFDONNGO@?$FLRWPM?$FN?$FLERROR?5?3?5New?5Memory?5Error@ 0041c330     ServerAppDlg.obj
 0002:00003374       ??_C@_0CA@FMNGHFIB@GAMESERVERMSG_USER_DISCONNECTED@ 0041c374     ServerAppDlg.obj
 0002:00003394       ??_C@_0BB@EBJDADCL@?4?2UCCSetting?4ini@ 0041c394     ServerAppDlg.obj
 0002:000033a8       ??_C@_09CNGDDFNE@ServerURL@ 0041c3a8     ServerAppDlg.obj
 0002:000033b4       ??_C@_0O@KMFGOFBD@fileserverurl@ 0041c3b4     ServerAppDlg.obj
 0002:000033c4       ??_C@_04MEDPFIKH@HTTP@     0041c3c4     ServerAppDlg.obj
 0002:000033cc       ??_C@_0M@FHOHKDM@?$CFd?$CF02d?$CF02d_@ 0041c3cc     ServerAppDlg.obj
 0002:000033d8       ??_C@_04FPOLKAEB@?4log@    0041c3d8     ServerAppDlg.obj
 0002:000033e0       ??_C@_03BFHAFKOB@wb?$CL@   0041c3e0     ServerAppDlg.obj
 0002:000033e4       ??_C@_0CL@FMBHHKIH@?$FLucclog?$FN?5UCC?5file?5Write?5Error?5N@ 0041c3e4     ServerAppDlg.obj
 0002:00003410       ??_C@_0EF@JPAKIDCC@?$FLUCCLog?$FN?5rez?5temp?5file?5delete?5f@ 0041c410     ServerAppDlg.obj
 0002:00003458       ??_C@_0DF@KLJPIDKF@?$FLUCCLog?$FN?5rez?5temp?5file?5delete?5s@ 0041c458     ServerAppDlg.obj
 0002:00003490       ??_C@_0M@KHNENFMD@RezFilePath@ 0041c490     ServerAppDlg.obj
 0002:0000349c       ??_C@_0BC@OGNIILDB@rezrepositoryinfo@ 0041c49c     ServerAppDlg.obj
 0002:000034b0       ??_C@_11LOCGONAA@@         0041c4b0     StdAfx.obj
 0002:000074c0       __real@3f466666            004204c0     StdAfx.obj
 0002:000074c4       __real@41800000            004204c4     StdAfx.obj
 0002:000074c8       ??_C@_0BF@IAOALLHJ@C?3?2log?2crossfire?2?$CFs?2@ 004204c8     BugReporter1.obj
 0002:000074e0       ??_C@_04KBDJOJNB@?$FL?$CFd?$FN@ 004204e0     BugReporter1.obj
 0002:000074e8       ??_C@_0L@IFPJGDKC@?$CFd?$CF02d?$CF02d@ 004204e8     BugReporter1.obj
 0002:000074f4       ??_C@_08PNEMGIDK@FullDump@ 004204f4     BugReporter1.obj
 0002:00007500       ??_C@_0BJ@DAFBOCMI@CRS?5Upload?5Succeeded?3?5?$CFs@ 00420500     BugReporter1.obj
 0002:0000751c       ??_C@_0BG@LEKOEBGH@CRS?5Upload?5Failed?3?5?$CFs@ 0042051c     BugReporter1.obj
 0002:00007534       ??_C@_03GIOIKFCO@C?3?2@    00420534     BugReporter1.obj
 0002:00007538       ??_C@_03MGHMBJCF@log@      00420538     BugReporter1.obj
 0002:0000753c       ??_C@_04FNMMLKAG@log?2@    0042053c     BugReporter1.obj
 0002:00007544       ??_C@_09LOKONNNP@crossfire@ 00420544     BugReporter1.obj
 0002:00007550       ??_C@_05BMGBEOOC@?$CFs?2?$CFs@ 00420550     BugReporter1.obj
 0002:00007558       ??_C@_1BA@HDJCCPDO@?$AAC?$AAR?$AAS?$AA?4?$AAi?$AAn?$AAi@ 00420558     crs_uploader1.obj
 0002:00007568       ??_C@_17BHJPJDEN@?$AAU?$AAR?$AAL@ 00420568     crs_uploader1.obj
 0002:00007570       ??_C@_17KFDBOMCI@?$AAC?$AAR?$AAS@ 00420570     crs_uploader1.obj
 0002:00007578       ??_C@_1CG@KLCLFNNP@?$AAD?$AAe?$AAl?$AAe?$AAt?$AAe?$AAM?$AAi?$AAn?$AAi?$AAd?$AAu?$AAm?$AAp?$AAF@ 00420578     crs_uploader1.obj
 0002:000075a0       ??_C@_19FKLFLPMF@?$AAt?$AAr?$AAu?$AAe@ 004205a0     crs_uploader1.obj
 0002:000075ac       ??_C@_1BG@BMKKPDAI@?$AA?$CF?$AAs?$AA?2?$AAC?$AAR?$AAS?$AA?4?$AAi?$AAn?$AAi@ 004205ac     crs_uploader1.obj
 0002:000075c4       ??_C@_1BA@ODBNFJPP@?$AAu?$AAn?$AAk?$AAn?$AAw?$AAo?$AAn@ 004205c4     crs_uploader1.obj
 0002:000075d4       ??_C@_1M@LLCLNBHO@?$AA?$CF?$AAs?$AA_?$AA?$CF?$AAs@ 004205d4     crs_uploader1.obj
 0002:000075e0       ??_C@_0L@CIKECLEP@version?3?$CFd@ 004205e0     crs_uploader1.obj
 0002:000075ec       ??_C@_09BNNAOANA@empty?5url@ 004205ec     crs_uploader1.obj
 0002:000075f8       ??_C@_1O@NBDODAKG@?$AAu?$AAp?$AAl?$AAo?$AAa?$AAd@ 004205f8     crs_uploader1.obj
 0002:00007608       ??_C@_0BL@ININHFIP@output_dir?5is?5empty?5URL?$DN?$CFs@ 00420608     crs_uploader1.obj
 0002:00007624       ??_C@_0BI@LFPNAEAK@invalid?5url?$FL?$CFlu?$FN?5URL?$DN?$CFs@ 00420624     crs_uploader1.obj
 0002:0000763c       ??_C@_0BA@ELPOGNCH@disabled?5URL?$DN?$CFs@ 0042063c     crs_uploader1.obj
 0002:0000764c       ??_C@_0BA@GOHDMMKI@unknown?5path?$DN?$CFs@ 0042064c     crs_uploader1.obj
 0002:0000765c       ??_C@_0BD@BMMMPMLP@exists?5not?5path?$DN?$CFs@ 0042065c     crs_uploader1.obj
 0002:00007670       ??_C@_1BE@KEAGFEAH@?$AA?1?$AAv?$AAe?$AAr?$AAs?$AAi?$AAo?$AAn?$AA?1@ 00420670     crs_uploader1.obj
 0002:00007684       ??_C@_19JLKJCDCM@?$AAP?$AAO?$AAS?$AAT@ 00420684     crs_uploader1.obj
 0002:00007690       ??_C@_0CC@NKABMACB@?$CFs?5WinHttpOpenRequest?$FL?$CFlu?$FN?5URL?$DN@ 00420690     crs_uploader1.obj
 0002:000076b4       ??_C@_0CC@MFDBFDLN@?$CFs?5WinHttpSendRequest?$FL?$CFlu?$FN?5URL?$DN@ 004206b4     crs_uploader1.obj
 0002:000076d8       ??_C@_07CIFAGBMG@unknown@  004206d8     crs_uploader1.obj
 0002:000076e0       ??_C@_0L@KCOBBBIC@?$CFs?$CL0x?$CFI64X@ 004206e0     crs_uploader1.obj
 0002:000076ec       ??_C@_0DE@FBPBPEDJ@?$CD?5Exception?5Infomation?5?3?5EXCEPT@ 004206ec     crs_uploader1.obj
 0002:00007720       ??_C@_0BH@GDOLEHPB@?$CD?5Exception?5Infomation@ 00420720     crs_uploader1.obj
 0002:00007738       ??_C@_08CFKGHCOB@16?319?337@ 00420738     crs_uploader1.obj
 0002:00007744       ??_C@_0M@JEFMNEEL@Feb?519?52021@ 00420744     crs_uploader1.obj
 0002:00007750       ??_C@_0BC@CEMNINJG@?$CD?5DATESTAMP?$DN?$CFs?5?$CFs@ 00420750     crs_uploader1.obj
 0002:00007764       ??_C@_0BB@LJEFLPEH@?$CD?5Address?$DN0x?$CF08X@ 00420764     crs_uploader1.obj
 0002:00007778       ??_C@_0BF@CCECPKIO@?$CD?5ExceptionCode?$DN0x?$CFX@ 00420778     crs_uploader1.obj
 0002:00007790       ??_C@_0BO@HFLEEEGJ@?$CF2d?50x?$CF08X?50x?$CF08X?50x?$CF08X?5?$CI?$CFs?$CJ@ 00420790     crs_uploader1.obj
 0002:000077b0       ??_C@_0BK@ENPPOBB@?$CD?5SymInitialize?5FAIL?$FL?$CFlu?$FN@ 004207b0     crs_uploader1.obj
 0002:000077cc       ??_C@_1BM@PEICEKM@?$AAS?$AAm?$AAi?$AAl?$AAe?$AAG?$AAa?$AAt?$AAe?$AA?5?$AAC?$AAR?$AAS@ 004207cc     crs_uploader1.obj
 0002:000077e8       ??_C@_0BI@JANBAAPF@WinHttpOpen?$FL?$CFlu?$FN?5URL?$DN?$CFs@ 004207e8     crs_uploader1.obj
 0002:00007800       ??_C@_0BL@EFGBFCEJ@WinHttpConnect?$FL?$CFlu?$FN?5URL?$DN?$CFs@ 00420800     crs_uploader1.obj
 0002:0000781c       ??_C@_17NHNHNCOB@?$AAP?$AAU?$AAT@ 0042081c     crs_uploader1.obj
 0002:00007824       ??_C@_0BP@IIOECOIJ@?$CFs?5CreateFile?5READ?$FL?$CFlu?$FN?5URL?$DN?$CFs@ 00420824     crs_uploader1.obj
 0002:00007844       ??_C@_0BL@MLCFLFFE@?$CFs?5GetFileSize?$FL?$CFlu?$FN?5URL?$DN?$CFs@ 00420844     crs_uploader1.obj
 0002:00007860       ??_C@_0BI@GHDKNBPJ@?$CFs?5ReadFile?$FL?$CFlu?$FN?5URL?$DN?$CFs@ 00420860     crs_uploader1.obj
 0002:00007878       ??_C@_0CA@OMIDHMOL@?$CFs?5WinHttpWriteData?$FL?$CFlu?$FN?5URL?$DN?$CFs@ 00420878     crs_uploader1.obj
 0002:00007898       ??_C@_1BA@NCJLFNJB@?$AAc?$AAr?$AAs?$AA?4?$AAl?$AAo?$AAg@ 00420898     crs_uploader1.obj
 0002:000078a8       ??_C@_0CG@LLGLPKJE@?$CFs?5WinHttpReceiveResponse?$FL?$CFlu?$FN?5@ 004208a8     crs_uploader1.obj
 0002:000078d0       ??_C@_0CD@ODMPMKPE@?$CFs?5WinHttpQueryHeaders?$FL?$CFlu?$FN?5URL@ 004208d0     crs_uploader1.obj
 0002:000078f4       ??_C@_0BE@IDLGBAE@?$CFs?5HTTP?$FL?$CFlu?$FN?5URL?$DN?$CFs@ 004208f4     crs_uploader1.obj
 0002:00007908       ??_C@_1FA@CNNLBJGF@?$AA?$CF?$AAs?$AA_?$AA?$CF?$AA0?$AA4?$AAd?$AA?$CF?$AA0?$AA2?$AAd?$AA?$CF?$AA0?$AA2?$AAd@ 00420908     crs_uploader1.obj
 0002:00007958       ??_C@_1M@BHHLEAOO@?$AA?$CF?$AAs?$AA?1?$AA?$CF?$AAs@ 00420958     crs_uploader1.obj
 0002:00007964       ??_C@_19LJDFFCJJ@?$AA?$CF?$AAs?$AA?$CF?$AAs@ 00420964     crs_uploader1.obj
 0002:00007974       ??_7CServerLog@@6B@        00420974     LogMgmt1.obj
 0002:0000797c       ??_7type_info@@6B@         0042097c     msvcrt:std_type_info_static.obj
 0002:00007988       _GUID_ATLVer110            00420988     atls:atlbase.obj
 0002:00007998       ??_C@_1IC@ONKHOIDK@?$AAE?$AAR?$AAR?$AAO?$AAR?$AA?5?$AA?3?$AA?5?$AAU?$AAn?$AAa?$AAb?$AAl?$AAe?$AA?5@ 00420998     atls:atlbase.obj
 0002:00007a1c       ??_C@_01BJJEKLCA@?$CC@     00420a1c     safe_string:safe_string.obj
 0002:00007a20       ??_C@_03JMHOMAJH@?$CJ?5?$CC@ 00420a20     safe_string:safe_string.obj
 0002:00007a24       ??_C@_03MFPIGDOF@?5?$DO?5@ 00420a24     safe_string:safe_string.obj
 0002:00007a28       ??_C@_0BE@EGPJCBFC@?5warning?5sprintf?3?5?$CI@ 00420a28     safe_string:safe_string.obj
 0002:00007a3c       ??_C@_07DNAEFDKF@sprintf@  00420a3c     safe_string:safe_string.obj
 0002:00007a44       ??_C@_0BD@MFEJDGPJ@?5warning?5strcpy?3?5?$CI@ 00420a44     safe_string:safe_string.obj
 0002:00007a58       ??_C@_08IBECHLLM@strcpy_s@ 00420a58     safe_string:safe_string.obj
 0002:00007a64       ??_C@_0BD@JCAAKJFN@warning?5strncpy?3?5?$CI@ 00420a64     safe_string:safe_string.obj
 0002:00007a78       ??_C@_07EDFCNFDJ@strncpy@  00420a78     safe_string:safe_string.obj
 0002:00007a80       ??_C@_0BA@JFNIOLAK@string?5too?5long@ 00420a80     safe_string:safe_string.obj
 0002:00007a90       ??_8?$basic_stringstream@DU?$char_traits@D@std@@V?$allocator@D@2@@std@@7B?$basic_ostream@DU?$char_traits@D@std@@@1@@ 00420a90     safe_string:safe_string.obj
 0002:00007a9c       ??_7?$basic_stringbuf@DU?$char_traits@D@std@@V?$allocator@D@2@@std@@6B@ 00420a9c     safe_string:safe_string.obj
 0002:00007adc       ??_7?$basic_stringstream@DU?$char_traits@D@std@@V?$allocator@D@2@@std@@6B@ 00420adc     safe_string:safe_string.obj
 0002:00007ae0       ??_8?$basic_stringstream@DU?$char_traits@D@std@@V?$allocator@D@2@@std@@7B?$basic_istream@DU?$char_traits@D@std@@@1@@ 00420ae0     safe_string:safe_string.obj
 0002:00007b48       __load_config_used         00420b48     msvcrt:loadcfg.obj
 0002:00007be8       ??_R4CAPIHolderBase@@6B@   00420be8     ltmodule.obj
 0002:00007bfc       ??_R3CAPIHolderBase@@8     00420bfc     ltmodule.obj
 0002:00007c0c       ??_R2CAPIHolderBase@@8     00420c0c     ltmodule.obj
 0002:00007c14       ??_R1A@?0A@EA@CAPIHolderBase@@8 00420c14     ltmodule.obj
 0002:00007c30       ??_R4CInterfaceDatabase@@6B@ 00420c30     ltmodule.obj
 0002:00007c44       ??_R3CInterfaceDatabase@@8 00420c44     ltmodule.obj
 0002:00007c54       ??_R2CInterfaceDatabase@@8 00420c54     ltmodule.obj
 0002:00007c5c       ??_R1A@?0A@EA@CInterfaceDatabase@@8 00420c5c     ltmodule.obj
 0002:00007c78       ??_R4CInterfaceNameMgr@@6B@ 00420c78     ltmodule.obj
 0002:00007c8c       ??_R3CInterfaceNameMgr@@8  00420c8c     ltmodule.obj
 0002:00007c9c       ??_R2CInterfaceNameMgr@@8  00420c9c     ltmodule.obj
 0002:00007ca4       ??_R1A@?0A@EA@CInterfaceNameMgr@@8 00420ca4     ltmodule.obj
 0002:00007cc0       ??_R4CMustSyncObjectLog@@6B@ 00420cc0     HostLogger.obj
 0002:00007cd4       ??_R3CMustSyncObjectLog@@8 00420cd4     HostLogger.obj
 0002:00007ce4       ??_R2CMustSyncObjectLog@@8 00420ce4     HostLogger.obj
 0002:00007cf0       ??_R1A@?0A@EA@CMustSyncObjectLog@@8 00420cf0     HostLogger.obj
 0002:00007d0c       ??_R13?0A@EA@_RTL_CRITICAL_SECTION@@8 00420d0c     HostLogger.obj
 0002:00007d28       ??_R3_RTL_CRITICAL_SECTION@@8 00420d28     HostLogger.obj
 0002:00007d38       ??_R2_RTL_CRITICAL_SECTION@@8 00420d38     HostLogger.obj
 0002:00007d40       ??_R1A@?0A@EA@_RTL_CRITICAL_SECTION@@8 00420d40     HostLogger.obj
 0002:00007d5c       ??_R4FindXlsMsg@@6B@       00420d5c     LoadXlsMsg.obj
 0002:00007d70       ??_R3FindXlsMsg@@8         00420d70     LoadXlsMsg.obj
 0002:00007d80       ??_R2FindXlsMsg@@8         00420d80     LoadXlsMsg.obj
 0002:00007d88       ??_R1A@?0A@EA@FindXlsMsg@@8 00420d88     LoadXlsMsg.obj
 0002:00007da4       ??_R3CObject@@8            00420da4     ServerApp.obj
 0002:00007db4       ??_R2CObject@@8            00420db4     ServerApp.obj
 0002:00007dbc       ??_R1A@?0A@EA@CObject@@8   00420dbc     ServerApp.obj
 0002:00007dd8       ??_R1A@?0A@EA@CCmdTarget@@8 00420dd8     ServerApp.obj
 0002:00007df4       ??_R3CCmdTarget@@8         00420df4     ServerApp.obj
 0002:00007e04       ??_R2CCmdTarget@@8         00420e04     ServerApp.obj
 0002:00007e10       ??_R4CServerAppApp@@6B@    00420e10     ServerApp.obj
 0002:00007e24       ??_R3CServerAppApp@@8      00420e24     ServerApp.obj
 0002:00007e34       ??_R2CServerAppApp@@8      00420e34     ServerApp.obj
 0002:00007e4c       ??_R1A@?0A@EA@CServerAppApp@@8 00420e4c     ServerApp.obj
 0002:00007e68       ??_R1A@?0A@EA@CWinApp@@8   00420e68     ServerApp.obj
 0002:00007e84       ??_R3CWinApp@@8            00420e84     ServerApp.obj
 0002:00007e94       ??_R2CWinApp@@8            00420e94     ServerApp.obj
 0002:00007ea8       ??_R1A@?0A@EA@CWinThread@@8 00420ea8     ServerApp.obj
 0002:00007ec4       ??_R3CWinThread@@8         00420ec4     ServerApp.obj
 0002:00007ed4       ??_R2CWinThread@@8         00420ed4     ServerApp.obj
 0002:00007ee4       ??_R4?$CAPIHolder@VILTCommon@@@@6B@ 00420ee4     ServerAppDlg.obj
 0002:00007ef8       ??_R3?$CAPIHolder@VILTCommon@@@@8 00420ef8     ServerAppDlg.obj
 0002:00007f08       ??_R2?$CAPIHolder@VILTCommon@@@@8 00420f08     ServerAppDlg.obj
 0002:00007f14       ??_R1A@?0A@EA@?$CAPIHolder@VILTCommon@@@@8 00420f14     ServerAppDlg.obj
 0002:00007f30       ??_R1A@?0A@EA@CWnd@@8      00420f30     ServerAppDlg.obj
 0002:00007f4c       ??_R3CWnd@@8               00420f4c     ServerAppDlg.obj
 0002:00007f5c       ??_R2CWnd@@8               00420f5c     ServerAppDlg.obj
 0002:00007f6c       ??_R4CListBox@@6B@         00420f6c     ServerAppDlg.obj
 0002:00007f80       ??_R3CListBox@@8           00420f80     ServerAppDlg.obj
 0002:00007f90       ??_R2CListBox@@8           00420f90     ServerAppDlg.obj
 0002:00007fa4       ??_R1A@?0A@EA@CListBox@@8  00420fa4     ServerAppDlg.obj
 0002:00007fc0       ??_R4CEdit@@6B@            00420fc0     ServerAppDlg.obj
 0002:00007fd4       ??_R3CEdit@@8              00420fd4     ServerAppDlg.obj
 0002:00007fe4       ??_R2CEdit@@8              00420fe4     ServerAppDlg.obj
 0002:00007ff8       ??_R1A@?0A@EA@CEdit@@8     00420ff8     ServerAppDlg.obj
 0002:00008014       ??_R1A@?0A@EA@CDialog@@8   00421014     ServerAppDlg.obj
 0002:00008030       ??_R3CDialog@@8            00421030     ServerAppDlg.obj
 0002:00008040       ??_R2CDialog@@8            00421040     ServerAppDlg.obj
 0002:00008054       ??_R4exception@std@@6B@    00421054     ServerAppDlg.obj
 0002:00008068       ??_R3exception@std@@8      00421068     ServerAppDlg.obj
 0002:00008078       ??_R2exception@std@@8      00421078     ServerAppDlg.obj
 0002:00008080       ??_R1A@?0A@EA@exception@std@@8 00421080     ServerAppDlg.obj
 0002:0000809c       ??_R3GAMEPROTO_COMMON@@8   0042109c     ServerAppDlg.obj
 0002:000080ac       ??_R2GAMEPROTO_COMMON@@8   004210ac     ServerAppDlg.obj
 0002:000080b4       ??_R1A@?0A@EA@GAMEPROTO_COMMON@@8 004210b4     ServerAppDlg.obj
 0002:000080d0       ??_R3GAMEPROTO_SC_COMMON@@8 004210d0     ServerAppDlg.obj
 0002:000080e0       ??_R2GAMEPROTO_SC_COMMON@@8 004210e0     ServerAppDlg.obj
 0002:000080ec       ??_R1A@?0A@EA@GAMEPROTO_SC_COMMON@@8 004210ec     ServerAppDlg.obj
 0002:00008108       ??_R4PROTO_SERVERAPPMSG_INIT@@6B@ 00421108     ServerAppDlg.obj
 0002:0000811c       ??_R3PROTO_SERVERAPPMSG_INIT@@8 0042111c     ServerAppDlg.obj
 0002:0000812c       ??_R2PROTO_SERVERAPPMSG_INIT@@8 0042112c     ServerAppDlg.obj
 0002:0000813c       ??_R1A@?0A@EA@PROTO_SERVERAPPMSG_INIT@@8 0042113c     ServerAppDlg.obj
 0002:00008158       ??_R3ServerAppHandler@@8   00421158     ServerAppDlg.obj
 0002:00008168       ??_R2ServerAppHandler@@8   00421168     ServerAppDlg.obj
 0002:00008170       ??_R1A@?0A@EA@ServerAppHandler@@8 00421170     ServerAppDlg.obj
 0002:0000818c       ??_R4CServerAppDlg@@6B@    0042118c     ServerAppDlg.obj
 0002:000081a0       ??_R3CServerAppDlg@@8      004211a0     ServerAppDlg.obj
 0002:000081b0       ??_R2CServerAppDlg@@8      004211b0     ServerAppDlg.obj
 0002:000081c8       ??_R1A@?0A@EA@CServerAppDlg@@8 004211c8     ServerAppDlg.obj
 0002:000081e4       ??_R4CGameServerAppHandler@@6B@ 004211e4     ServerAppDlg.obj
 0002:000081f8       ??_R3CGameServerAppHandler@@8 004211f8     ServerAppDlg.obj
 0002:00008208       ??_R2CGameServerAppHandler@@8 00421208     ServerAppDlg.obj
 0002:00008214       ??_R1A@?0A@EA@CGameServerAppHandler@@8 00421214     ServerAppDlg.obj
 0002:00008230       ??_R4CServerLog@@6B@       00421230     LogMgmt1.obj
 0002:00008244       ??_R3CServerLog@@8         00421244     LogMgmt1.obj
 0002:00008254       ??_R2CServerLog@@8         00421254     LogMgmt1.obj
 0002:0000825c       ??_R1A@?0A@EA@CServerLog@@8 0042125c     LogMgmt1.obj
 0002:00008278       ??_R4type_info@@6B@        00421278     msvcrt:std_type_info_static.obj
 0002:0000828c       ??_R3type_info@@8          0042128c     msvcrt:std_type_info_static.obj
 0002:0000829c       ??_R2type_info@@8          0042129c     msvcrt:std_type_info_static.obj
 0002:000082a4       ??_R1A@?0A@EA@type_info@@8 004212a4     msvcrt:std_type_info_static.obj
 0002:000082c0       ??_R3?$basic_istream@DU?$char_traits@D@std@@@std@@8 004212c0     safe_string:safe_string.obj
 0002:000082d0       ??_R3?$basic_iostream@DU?$char_traits@D@std@@@std@@8 004212d0     safe_string:safe_string.obj
 0002:000082e0       ??_R1A@?0A@EA@?$basic_istream@DU?$char_traits@D@std@@@std@@8 004212e0     safe_string:safe_string.obj
 0002:000082fc       ??_R2?$basic_stringbuf@DU?$char_traits@D@std@@V?$allocator@D@2@@std@@8 004212fc     safe_string:safe_string.obj
 0002:00008308       ??_R17A@3EA@?$_Iosb@H@std@@8 00421308     safe_string:safe_string.obj
 0002:00008324       ??_R1A@?0A@EA@?$basic_stringstream@DU?$char_traits@D@std@@V?$allocator@D@2@@std@@8 00421324     safe_string:safe_string.obj
 0002:00008340       ??_R1A@?0A@EA@?$basic_streambuf@DU?$char_traits@D@std@@@std@@8 00421340     safe_string:safe_string.obj
 0002:0000835c       ??_R2?$basic_istream@DU?$char_traits@D@std@@@std@@8 0042135c     safe_string:safe_string.obj
 0002:00008370       ??_R3?$basic_stringbuf@DU?$char_traits@D@std@@V?$allocator@D@2@@std@@8 00421370     safe_string:safe_string.obj
 0002:00008380       ??_R2?$basic_ostream@DU?$char_traits@D@std@@@std@@8 00421380     safe_string:safe_string.obj
 0002:00008394       ??_R3?$basic_ios@DU?$char_traits@D@std@@@std@@8 00421394     safe_string:safe_string.obj
 0002:000083a4       ??_R1BA@?0A@EA@?$basic_ostream@DU?$char_traits@D@std@@@std@@8 004213a4     safe_string:safe_string.obj
 0002:000083c0       ??_R1A@?0A@EA@ios_base@std@@8 004213c0     safe_string:safe_string.obj
 0002:000083dc       ??_R1A@?0A@EA@?$basic_ostream@DU?$char_traits@D@std@@@std@@8 004213dc     safe_string:safe_string.obj
 0002:000083f8       ??_R2?$basic_streambuf@DU?$char_traits@D@std@@@std@@8 004213f8     safe_string:safe_string.obj
 0002:00008400       ??_R1A@?0A@EA@?$_Iosb@H@std@@8 00421400     safe_string:safe_string.obj
 0002:0000841c       ??_R1A@?0A@EA@?$basic_stringbuf@DU?$char_traits@D@std@@V?$allocator@D@2@@std@@8 0042141c     safe_string:safe_string.obj
 0002:00008438       ??_R2?$basic_iostream@DU?$char_traits@D@std@@@std@@8 00421438     safe_string:safe_string.obj
 0002:00008460       ??_R2?$basic_stringstream@DU?$char_traits@D@std@@V?$allocator@D@2@@std@@8 00421460     safe_string:safe_string.obj
 0002:0000848c       ??_R4?$basic_stringbuf@DU?$char_traits@D@std@@V?$allocator@D@2@@std@@6B@ 0042148c     safe_string:safe_string.obj
 0002:000084a0       ??_R4?$basic_stringstream@DU?$char_traits@D@std@@V?$allocator@D@2@@std@@6B@ 004214a0     safe_string:safe_string.obj
 0002:000084b4       ??_R1A@A@3FA@?$basic_ios@DU?$char_traits@D@std@@@std@@8 004214b4     safe_string:safe_string.obj
 0002:000084d0       ??_R2ios_base@std@@8       004214d0     safe_string:safe_string.obj
 0002:000084dc       ??_R3?$basic_ostream@DU?$char_traits@D@std@@@std@@8 004214dc     safe_string:safe_string.obj
 0002:000084ec       ??_R1A@?0A@EA@?$basic_iostream@DU?$char_traits@D@std@@@std@@8 004214ec     safe_string:safe_string.obj
 0002:00008508       ??_R3ios_base@std@@8       00421508     safe_string:safe_string.obj
 0002:00008518       ??_R3?$basic_streambuf@DU?$char_traits@D@std@@@std@@8 00421518     safe_string:safe_string.obj
 0002:00008528       ??_R3?$basic_stringstream@DU?$char_traits@D@std@@V?$allocator@D@2@@std@@8 00421528     safe_string:safe_string.obj
 0002:00008538       ??_R2?$_Iosb@H@std@@8      00421538     safe_string:safe_string.obj
 0002:00008540       ??_R1A@A@3EA@ios_base@std@@8 00421540     safe_string:safe_string.obj
 0002:0000855c       ??_R1A@?0A@EA@?$basic_ios@DU?$char_traits@D@std@@@std@@8 0042155c     safe_string:safe_string.obj
 0002:00008578       ??_R3?$_Iosb@H@std@@8      00421578     safe_string:safe_string.obj
 0002:00008588       ??_R17?0A@EA@?$_Iosb@H@std@@8 00421588     safe_string:safe_string.obj
 0002:000085a4       ??_R2?$basic_ios@DU?$char_traits@D@std@@@std@@8 004215a4     safe_string:safe_string.obj
 0002:000085c0       ___safe_se_handler_table   004215c0     <linker-defined>
 0002:00008a00       ___rtc_iaa                 00421a00     msvcrt:initsect.obj
 0002:00008a04       ___rtc_izz                 00421a04     msvcrt:initsect.obj
 0002:00008a08       ___rtc_taa                 00421a08     msvcrt:initsect.obj
 0002:00008a0c       ___rtc_tzz                 00421a0c     msvcrt:initsect.obj
 0002:00009734       __CT??_R0?AVexception@std@@@8??0exception@std@@QAE@ABV01@@Z12 00422734     ServerAppDlg.obj
 0002:00009750       __TI1?AVexception@std@@    00422750     ServerAppDlg.obj
 0002:00009760       __CTA1?AVexception@std@@   00422760     ServerAppDlg.obj
 0002:00009908       __IMPORT_DESCRIPTOR_PSAPI  00422908     Psapi:PSAPI.DLL
 0002:0000991c       __IMPORT_DESCRIPTOR_mfc140 0042291c     mfc140:mfc140.dll
 0002:00009930       __IMPORT_DESCRIPTOR_KERNEL32 00422930     kernel32:KERNEL32.dll
 0002:00009944       __IMPORT_DESCRIPTOR_USER32 00422944     user32:USER32.dll
 0002:00009958       __IMPORT_DESCRIPTOR_SHELL32 00422958     shell32:SHELL32.dll
 0002:0000996c       __IMPORT_DESCRIPTOR_SHLWAPI 0042296c     shlwapi:SHLWAPI.dll
 0002:00009980       __IMPORT_DESCRIPTOR_MSVCP140 00422980     msvcprt:MSVCP140.dll
 0002:00009994       __IMPORT_DESCRIPTOR_WININET 00422994     wininet:WININET.dll
 0002:000099a8       __IMPORT_DESCRIPTOR_WS2_32 004229a8     ws2_32:WS2_32.dll
 0002:000099bc       __IMPORT_DESCRIPTOR_dbghelp 004229bc     DbgHelp:dbghelp.dll
 0002:000099d0       __IMPORT_DESCRIPTOR_WINMM  004229d0     winmm:WINMM.dll
 0002:000099e4       __IMPORT_DESCRIPTOR_WINHTTP 004229e4     winhttp:WINHTTP.dll
 0002:000099f8       __IMPORT_DESCRIPTOR_VCRUNTIME140 004229f8     vcruntime:VCRUNTIME140.dll
 0002:00009a0c       __IMPORT_DESCRIPTOR_api-ms-win-crt-string-l1-1-0 00422a0c     ucrt:api-ms-win-crt-string-l1-1-0.dll
 0002:00009a20       __IMPORT_DESCRIPTOR_api-ms-win-crt-math-l1-1-0 00422a20     ucrt:api-ms-win-crt-math-l1-1-0.dll
 0002:00009a34       __IMPORT_DESCRIPTOR_api-ms-win-crt-runtime-l1-1-0 00422a34     ucrt:api-ms-win-crt-runtime-l1-1-0.dll
 0002:00009a48       __IMPORT_DESCRIPTOR_api-ms-win-crt-stdio-l1-1-0 00422a48     ucrt:api-ms-win-crt-stdio-l1-1-0.dll
 0002:00009a5c       __IMPORT_DESCRIPTOR_api-ms-win-crt-filesystem-l1-1-0 00422a5c     ucrt:api-ms-win-crt-filesystem-l1-1-0.dll
 0002:00009a70       __IMPORT_DESCRIPTOR_api-ms-win-crt-utility-l1-1-0 00422a70     ucrt:api-ms-win-crt-utility-l1-1-0.dll
 0002:00009a84       __IMPORT_DESCRIPTOR_api-ms-win-crt-convert-l1-1-0 00422a84     ucrt:api-ms-win-crt-convert-l1-1-0.dll
 0002:00009a98       __IMPORT_DESCRIPTOR_api-ms-win-crt-time-l1-1-0 00422a98     ucrt:api-ms-win-crt-time-l1-1-0.dll
 0002:00009aac       __IMPORT_DESCRIPTOR_api-ms-win-crt-heap-l1-1-0 00422aac     ucrt:api-ms-win-crt-heap-l1-1-0.dll
 0002:00009ac0       __IMPORT_DESCRIPTOR_api-ms-win-crt-locale-l1-1-0 00422ac0     ucrt:api-ms-win-crt-locale-l1-1-0.dll
 0002:00009ad4       __NULL_IMPORT_DESCRIPTOR   00422ad4     Psapi:PSAPI.DLL
 0003:00000024       ?m_LogLevel@CHLogger@@0IA  00425024     HostLogger.obj
 0003:00000028       ?m_strFileFormat@CHLogger@@0V?$basic_string@DU?$char_traits@D@std@@V?$allocator@D@2@@std@@A 00425028     HostLogger.obj
 0003:00000040       ?m_strBRFileFormat@CHLogger@@0V?$basic_string@DU?$char_traits@D@std@@V?$allocator@D@2@@std@@A 00425040     HostLogger.obj
 0003:00000058       ?m_strKernelFileFormat@CHLogger@@0V?$basic_string@DU?$char_traits@D@std@@V?$allocator@D@2@@std@@A 00425058     HostLogger.obj
 0003:00000070       ?m_strTimeOutFileFormat@CHLogger@@0V?$basic_string@DU?$char_traits@D@std@@V?$allocator@D@2@@std@@A 00425070     HostLogger.obj
 0003:00000088       ?m_strEtcFileFormat@CHLogger@@0V?$basic_string@DU?$char_traits@D@std@@V?$allocator@D@2@@std@@A 00425088     HostLogger.obj
 0003:000000a0       ?m_strPacketFileFormat@CHLogger@@0V?$basic_string@DU?$char_traits@D@std@@V?$allocator@D@2@@std@@A 004250a0     HostLogger.obj
 0003:000000b8       ?m_strModeUserCountFormat@CHLogger@@0V?$basic_string@DU?$char_traits@D@std@@V?$allocator@D@2@@std@@A 004250b8     HostLogger.obj
 0003:000000d0       ?m_strServerAppUseCountFormat@CHLogger@@0V?$basic_string@DU?$char_traits@D@std@@V?$allocator@D@2@@std@@A 004250d0     HostLogger.obj
 0003:000000e8       ?m_strRWProcessMemoryFileFormat@CHLogger@@0V?$basic_string@DU?$char_traits@D@std@@V?$allocator@D@2@@std@@A 004250e8     HostLogger.obj
 0003:00000100       ?m_strIPCMessageFileFormat@CHLogger@@0V?$basic_string@DU?$char_traits@D@std@@V?$allocator@D@2@@std@@A 00425100     HostLogger.obj
 0003:00000118       ?m_strHostName@CHLogger@@0V?$basic_string@DU?$char_traits@D@std@@V?$allocator@D@2@@std@@A 00425118     HostLogger.obj
 0003:00000130       ?m_strServerName@CHLogger@@0V?$basic_string@DU?$char_traits@D@std@@V?$allocator@D@2@@std@@A 00425130     HostLogger.obj
 0003:00000148       ?m_strLogFolder@CHLogger@@0V?$basic_string@DU?$char_traits@D@std@@V?$allocator@D@2@@std@@A 00425148     HostLogger.obj
 0003:00000160       ?m_LogLock@CHLogger@@0VCMustSyncObjectLog@@A 00425160     HostLogger.obj
 0003:0000017c       ?m_LogPacketLock@CHLogger@@0VCMustSyncObjectLog@@A 0042517c     HostLogger.obj
 0003:00000198       ?m_eSharedMemUsage@CLogMsgManager@@0W4ESHARED_MEM_USAGE_TYPE@1@A 00425198     LogMsgManager.obj
 0003:0000019c       ?g_bUseCS@@3_NA            0042519c     ServerAppDlg.obj
 0003:000001a0       ?g_lMinInterval@@3JA       004251a0     ServerAppDlg.obj
 0003:0000022c       ___security_cookie_complement 0042522c     msvcrt:gs_cookie.obj
 0003:00000230       ___security_cookie         00425230     msvcrt:gs_cookie.obj
 0003:00000234       ___scrt_native_dllmain_reason 00425234     msvcrt:utility.obj
 0003:00000238       __fltused                  00425238     msvcrt:fltused.obj
 0003:00000240       ___isa_enabled             00425240     msvcrt:cpu_disp.obj
 0003:00000244       ___scrt_default_matherr    00425244     msvcrt:matherr.obj
 0003:00000248       ___scrt_ucrt_dll_is_in_use 00425248     msvcrt:ucrt_stubs.obj
 0003:00000250       ??_R0?AVCAPIHolderBase@@@8 00425250     ltmodule.obj
 0003:00000270       ??_R0?AVCInterfaceDatabase@@@8 00425270     ltmodule.obj
 0003:00000294       ??_R0?AVCInterfaceNameMgr@@@8 00425294     ltmodule.obj
 0003:000002b4       ??_R0?AVCMustSyncObjectLog@@@8 004252b4     HostLogger.obj
 0003:000002d8       ??_R0?AU_RTL_CRITICAL_SECTION@@@8 004252d8     HostLogger.obj
 0003:000002fc       ??_R0?AVFindXlsMsg@@@8     004252fc     LoadXlsMsg.obj
 0003:00000318       ??_R0?AVCObject@@@8        00425318     ServerApp.obj
 0003:00000330       ??_R0?AVCCmdTarget@@@8     00425330     ServerApp.obj
 0003:0000034c       ??_R0?AVCServerAppApp@@@8  0042534c     ServerApp.obj
 0003:00000368       ??_R0?AVCWinApp@@@8        00425368     ServerApp.obj
 0003:00000380       ??_R0?AVCWinThread@@@8     00425380     ServerApp.obj
 0003:0000039c       ??_R0?AV?$CAPIHolder@VILTCommon@@@@@8 0042539c     ServerAppDlg.obj
 0003:000003c4       ??_R0PAVCException@@@8     004253c4     ServerAppDlg.obj
 0003:000003e0       ??_R0?AVexception@std@@@8  004253e0     ServerAppDlg.obj
 0003:000003fc       ??_R0?AVCWnd@@@8           004253fc     ServerAppDlg.obj
 0003:00000410       ??_R0?AVCListBox@@@8       00425410     ServerAppDlg.obj
 0003:00000428       ??_R0?AVCEdit@@@8          00425428     ServerAppDlg.obj
 0003:0000043c       ??_R0?AVCDialog@@@8        0042543c     ServerAppDlg.obj
 0003:00000454       ??_R0?AUGAMEPROTO_COMMON@@@8 00425454     ServerAppDlg.obj
 0003:00000474       ??_R0?AUGAMEPROTO_SC_COMMON@@@8 00425474     ServerAppDlg.obj
 0003:00000498       ??_R0?AUPROTO_SERVERAPPMSG_INIT@@@8 00425498     ServerAppDlg.obj
 0003:000004c0       ??_R0?AVServerAppHandler@@@8 004254c0     ServerAppDlg.obj
 0003:000004e0       ??_R0?AVCServerAppDlg@@@8  004254e0     ServerAppDlg.obj
 0003:000004fc       ??_R0?AVCGameServerAppHandler@@@8 004254fc     ServerAppDlg.obj
 0003:00000520       ??_R0?AVCServerLog@@@8     00425520     LogMgmt1.obj
 0003:0000053c       ??_R0?AVtype_info@@@8      0042553c     msvcrt:std_type_info_static.obj
 0003:00000558       ??_R0?AV?$basic_stringstream@DU?$char_traits@D@std@@V?$allocator@D@2@@std@@@8 00425558     safe_string:safe_string.obj
 0003:000005a8       ??_R0?AV?$basic_stringbuf@DU?$char_traits@D@std@@V?$allocator@D@2@@std@@@8 004255a8     safe_string:safe_string.obj
 0003:000005f8       ??_R0?AVios_base@std@@@8   004255f8     safe_string:safe_string.obj
 0003:00000614       ??_R0?AV?$basic_iostream@DU?$char_traits@D@std@@@std@@@8 00425614     safe_string:safe_string.obj
 0003:00000650       ??_R0?AV?$_Iosb@H@std@@@8  00425650     safe_string:safe_string.obj
 0003:0000066c       ??_R0?AV?$basic_streambuf@DU?$char_traits@D@std@@@std@@@8 0042566c     safe_string:safe_string.obj
 0003:000006a8       ??_R0?AV?$basic_istream@DU?$char_traits@D@std@@@std@@@8 004256a8     safe_string:safe_string.obj
 0003:000006e4       ??_R0?AV?$basic_ios@DU?$char_traits@D@std@@@std@@@8 004256e4     safe_string:safe_string.obj
 0003:0000071c       ??_R0?AV?$basic_ostream@DU?$char_traits@D@std@@@std@@@8 0042571c     safe_string:safe_string.obj
 0003:00000a00       ?_FILE_SHUTDOWN_var_ltmod_database_@@3V_FILE_SHUTDOWN_class_ltmod_database_@@A 00425a00     ltmodule.obj
 0003:00000a90       ?m_isWriteLog_IPCMsg@CHLogger@@0_NA 00425a90     HostLogger.obj
 0003:00000a91       ?m_isWriteLog_IPCMemory@CHLogger@@0_NA 00425a91     HostLogger.obj
 0003:00000a94       ?m_pXlsLoader@CLogMsgManager@@0PAVFindXlsMsg@@A 00425a94     LogMsgManager.obj
 0003:00000a98       ?m_eLastError@CLogMsgManager@@0W4EERROR_TYPE@1@A 00425a98     LogMsgManager.obj
 0003:00000a9c       ?m_hSizeHandle@CLogMsgManager@@0PAXA 00425a9c     LogMsgManager.obj
 0003:00000aa0       ?m_vectSharedMapHandles@CLogMsgManager@@0V?$vector@PAXV?$allocator@PAX@std@@@std@@A 00425aa0     LogMsgManager.obj
 0003:00000ab0       ?theApp@@3VCServerAppApp@@A 00425ab0     ServerApp.obj
 0003:00000b80       ?g_useDialogConsoleOutput@@3_NA 00425b80     ServerAppDlg.obj
 0003:00000b81       ?g_bCSSet@@3_NA            00425b81     ServerAppDlg.obj
 0003:00000b84       ?g_hServerDll@@3PAUHINSTANCE__@@A 00425b84     ServerAppDlg.obj
 0003:00000b88       ?GAMEGUID@@3TLTGUID@@A     00425b88     ServerAppDlg.obj
 0003:00000b98       ?g_pLTSCommon@@3PAVILTCommon@@A 00425b98     ServerAppDlg.obj
 0003:00000b9c       ?g_cs@@3U_RTL_CRITICAL_SECTION@@A 00425b9c     ServerAppDlg.obj
 0003:00000bb4       ?g_csGameInfoQueue@@3U_RTL_CRITICAL_SECTION@@A 00425bb4     ServerAppDlg.obj
 0003:00000bcc       ?g_csUserInfoQueue@@3U_RTL_CRITICAL_SECTION@@A 00425bcc     ServerAppDlg.obj
 0003:00000be4       ?g_iQueuedGameInfosNum@@3HC 00425be4     ServerAppDlg.obj
 0003:00000be8       ?g_iQueuedUserInfosNum@@3HC 00425be8     ServerAppDlg.obj
 0003:00000bf0       ?g_cServerLog@@3VCServerLog@@A 00425bf0     ServerAppDlg.obj
 0003:00000e00       ?g_sGameInfos@@3PAUPROTO_START_HOST_tag@@A 00425e00     ServerAppDlg.obj
 0003:001f05d0       ?g_sUserInfos@@3PAUPROTO_GAME_USER_INFO_tag@@A 006155d0     ServerAppDlg.obj
 0003:00221828       ?_OptionsStorage@?1??__local_stdio_scanf_options@@9@4_KA 00646828     ServerAppDlg.obj
 0003:00221830       ___@@_PchSym_@00@UwveUfhUeCBADUxorvmgUlyqUcIGUurmzoUhvievizkkUhgwzucOlyq@4B2008FD98C1DD4 00646830     StdAfx.obj
 0003:00221834       ?m_bInitFailed@CAtlBaseModule@ATL@@2_NA 00646834     StdAfx.obj
 0003:00222318       ?m_iLogLevel@CServerLog@@1HA 00647318     LogMgmt1.obj
 0003:00222320       ?m_szHostName@CServerLog@@1PADA 00647320     LogMgmt1.obj
 0003:00222388       ?m_szServerName@CServerLog@@1PADA 00647388     LogMgmt1.obj
 0003:002223f0       ?m_szLogFolder@CServerLog@@1PADA 006473f0     LogMgmt1.obj
 0003:00222588       ?m_szLogErrorFileName@CServerLog@@1PADA 00647588     LogMgmt1.obj
 0003:00222978       ?m_szLogCashFileName@CServerLog@@1PADA 00647978     LogMgmt1.obj
 0003:00222d68       ?m_szLogUnknownDataFileName@CServerLog@@1PADA 00647d68     LogMgmt1.obj
 0003:00223158       ?m_szLogMegaPhoneFileName@CServerLog@@1PADA 00648158     LogMgmt1.obj
 0003:00223548       ?m_szLogGachaFileName@CServerLog@@1PADA 00648548     LogMgmt1.obj
 0003:00223938       ?m_szLogConnectCheckFileName@CServerLog@@1PADA 00648938     LogMgmt1.obj
 0003:00223d28       ?m_szLogMonitoringFileName@CServerLog@@1PADA 00648d28     LogMgmt1.obj
 0003:00224118       ?m_szLogEmergencyStateFileName@CServerLog@@1PADA 00649118     LogMgmt1.obj
 0003:00224508       ?m_szLogHackingFileName@CServerLog@@1PADA 00649508     LogMgmt1.obj
 0003:002248f8       ?m_szLogServerSettingCheckFileName@CServerLog@@1PADA 006498f8     LogMgmt1.obj
 0003:00224ce8       ?m_szLogKickUserFileName@CServerLog@@1PADA 00649ce8     LogMgmt1.obj
 0003:002250d8       ?m_szLogInGameClanFileName@CServerLog@@1PADA 0064a0d8     LogMgmt1.obj
 0003:002254c8       ?m_szLogEtcFileName@CServerLog@@1PADA 0064a4c8     LogMgmt1.obj
 0003:002258b8       ?m_szLogTimeFileName@CServerLog@@1PADA 0064a8b8     LogMgmt1.obj
 0003:00225ca8       ?m_szLogTimeOutFileName@CServerLog@@1PADA 0064aca8     LogMgmt1.obj
 0003:00226098       ?m_szLogHackFileName@CServerLog@@1PADA 0064b098     LogMgmt1.obj
 0003:00226488       ?m_szLogCountFileName@CServerLog@@1PADA 0064b488     LogMgmt1.obj
 0003:00226878       ?m_szLogCriticalErrorPath@CServerLog@@1PADA 0064b878     LogMgmt1.obj
 0003:00226c68       ?m_szLogMgrDataFileName@CServerLog@@1PADA 0064bc68     LogMgmt1.obj
 0003:00227058       ?m_szLogMailerFileName@CServerLog@@1PADA 0064c058     LogMgmt1.obj
 0003:00227448       ?m_szLogTryWeaponItemFileName@CServerLog@@1PADA 0064c448     LogMgmt1.obj
 0003:00227834       __afxForceEXCLUDE          0064c834     mfcs140:nolib.obj
 0003:00227838       __afxForceSTDAFX           0064c838     mfcs140:stdafx.obj
 0003:0022783c       ___scrt_current_native_startup_state 0064c83c     msvcrt:utility.obj
 0003:00227840       ___scrt_native_startup_lock 0064c840     msvcrt:utility.obj
 0003:00227b7c       ___isa_available           0064cb7c     msvcrt:cpu_disp.obj
 0003:00227b80       ___favor                   0064cb80     msvcrt:cpu_disp.obj
 0003:00227b84       ___scrt_debugger_hook_flag 0064cb84     msvcrt:utility_desktop.obj
 0003:00227b88       ?__type_info_root_node@@3U__type_info_node@@A 0064cb88     msvcrt:tncleanup.obj
 0003:00227b90       ?_AtlBaseModule@ATL@@3VCAtlBaseModule@1@A 0064cb90     atls:atlbase.obj
 0003:00227bc8       ___@@_PchSym_@00@UztvmgUPdlipUDUhUrmgvinvwrzgvUexgllohUzgohOmzgrevkilqPBACIAJCBDBUlyqiUcIGUhgwzucOlyq@4B2008FD98C1DD4 0064cbc8     atls:stdafx.obj
 0003:00227bcc       ?_afxInitAppState@@3DA     0064cbcc     mfcs140:appmodul.obj
 0003:00227bd0       ?handler@vars@cf@@2P6AXABV?$basic_string@DU?$char_traits@D@std@@V?$allocator@D@2@@std@@0@ZA 0064cbd0     safe_string:safe_string.obj
 0003:00227bd8       ?_OptionsStorage@?1??__local_stdio_printf_options@@9@4_KA 0064cbd8     safe_string:safe_string.obj
 0003:00227be0       ___dyn_tls_dtor_callback   0064cbe0     <common>
 0003:00227be4       ___dyn_tls_init_callback   0064cbe4     <common>

 entry point at        0001:00015d7e

 Static symbols

 0000:ffdae000       .debug$S                   00400000     mfc140:mfc140.dll
 0000:ffdae000       .debug$S                   00400000     Psapi:PSAPI.DLL
 0000:ffdae000       .debug$S                   00400000     mfc140:mfc140.dll
 0000:ffdae000       .debug$S                   00400000     mfc140:mfc140.dll
 0000:ffdae000       .debug$S                   00400000     mfc140:mfc140.dll
 0000:ffdae000       .debug$S                   00400000     mfc140:mfc140.dll
 0000:ffdae000       .debug$S                   00400000     mfc140:mfc140.dll
 0000:ffdae000       .debug$S                   00400000     mfc140:mfc140.dll
 0000:ffdae000       .debug$S                   00400000     mfc140:mfc140.dll
 0000:ffdae000       .debug$S                   00400000     mfc140:mfc140.dll
 0000:ffdae000       .debug$S                   00400000     mfc140:mfc140.dll
 0000:ffdae000       .debug$S                   00400000     mfc140:mfc140.dll
 0000:ffdae000       .debug$S                   00400000     mfc140:mfc140.dll
 0000:ffdae000       .debug$S                   00400000     mfc140:mfc140.dll
 0000:ffdae000       .debug$S                   00400000     mfc140:mfc140.dll
 0000:ffdae000       .debug$S                   00400000     mfc140:mfc140.dll
 0000:ffdae000       .debug$S                   00400000     mfc140:mfc140.dll
 0000:ffdae000       .debug$S                   00400000     mfc140:mfc140.dll
 0000:ffdae000       .debug$S                   00400000     mfc140:mfc140.dll
 0000:ffdae000       .debug$S                   00400000     mfc140:mfc140.dll
 0000:ffdae000       .debug$S                   00400000     mfc140:mfc140.dll
 0000:ffdae000       .debug$S                   00400000     mfc140:mfc140.dll
 0000:ffdae000       .debug$S                   00400000     mfc140:mfc140.dll
 0000:ffdae000       .debug$S                   00400000     mfc140:mfc140.dll
 0000:ffdae000       .debug$S                   00400000     mfc140:mfc140.dll
 0000:ffdae000       .debug$S                   00400000     mfc140:mfc140.dll
 0000:ffdae000       .debug$S                   00400000     mfc140:mfc140.dll
 0000:ffdae000       .debug$S                   00400000     mfc140:mfc140.dll
 0000:ffdae000       .debug$S                   00400000     mfc140:mfc140.dll
 0000:ffdae000       .debug$S                   00400000     mfc140:mfc140.dll
 0000:ffdae000       .debug$S                   00400000     mfc140:mfc140.dll
 0000:ffdae000       .debug$S                   00400000     mfc140:mfc140.dll
 0000:ffdae000       .debug$S                   00400000     mfc140:mfc140.dll
 0000:ffdae000       .debug$S                   00400000     mfc140:mfc140.dll
 0000:ffdae000       .debug$S                   00400000     mfc140:mfc140.dll
 0000:ffdae000       .debug$S                   00400000     mfc140:mfc140.dll
 0000:ffdae000       .debug$S                   00400000     mfc140:mfc140.dll
 0000:ffdae000       .debug$S                   00400000     mfc140:mfc140.dll
 0000:ffdae000       .debug$S                   00400000     mfc140:mfc140.dll
 0000:ffdae000       .debug$S                   00400000     mfc140:mfc140.dll
 0000:ffdae000       .debug$S                   00400000     mfc140:mfc140.dll
 0000:ffdae000       .debug$S                   00400000     mfc140:mfc140.dll
 0000:ffdae000       .debug$S                   00400000     mfc140:mfc140.dll
 0000:ffdae000       .debug$S                   00400000     mfc140:mfc140.dll
 0000:ffdae000       .debug$S                   00400000     mfc140:mfc140.dll
 0000:ffdae000       .debug$S                   00400000     mfc140:mfc140.dll
 0000:ffdae000       .debug$S                   00400000     mfc140:mfc140.dll
 0000:ffdae000       .debug$S                   00400000     mfc140:mfc140.dll
 0000:ffdae000       .debug$S                   00400000     mfc140:mfc140.dll
 0000:ffdae000       .debug$S                   00400000     mfc140:mfc140.dll
 0000:ffdae000       .debug$S                   00400000     mfc140:mfc140.dll
 0000:ffdae000       .debug$S                   00400000     mfc140:mfc140.dll
 0000:ffdae000       .debug$S                   00400000     ServerApp.exp
 0000:ffdae000       .debug$S                   00400000     mfc140:mfc140.dll
 0000:ffdae000       .debug$S                   00400000     mfc140:mfc140.dll
 0000:ffdae000       .debug$S                   00400000     ucrt:api-ms-win-crt-locale-l1-1-0.dll
 0000:ffdae000       .debug$S                   00400000     msvcprt:MSVCP140.dll
 0000:ffdae000       .debug$S                   00400000     msvcprt:MSVCP140.dll
 0000:ffdae000       .debug$S                   00400000     msvcprt:MSVCP140.dll
 0000:ffdae000       .debug$S                   00400000     msvcprt:MSVCP140.dll
 0000:ffdae000       .debug$S                   00400000     msvcprt:MSVCP140.dll
 0000:ffdae000       .debug$S                   00400000     msvcprt:MSVCP140.dll
 0000:ffdae000       .debug$S                   00400000     msvcprt:MSVCP140.dll
 0000:ffdae000       .debug$S                   00400000     msvcprt:MSVCP140.dll
 0000:ffdae000       .debug$S                   00400000     msvcprt:MSVCP140.dll
 0000:ffdae000       .debug$S                   00400000     msvcprt:MSVCP140.dll
 0000:ffdae000       .debug$S                   00400000     msvcprt:MSVCP140.dll
 0000:ffdae000       .debug$S                   00400000     msvcprt:MSVCP140.dll
 0000:ffdae000       .debug$S                   00400000     msvcprt:MSVCP140.dll
 0000:ffdae000       .debug$S                   00400000     msvcprt:MSVCP140.dll
 0000:ffdae000       .debug$S                   00400000     msvcprt:MSVCP140.dll
 0000:ffdae000       .debug$S                   00400000     msvcprt:MSVCP140.dll
 0000:ffdae000       .debug$S                   00400000     msvcprt:MSVCP140.dll
 0000:ffdae000       .debug$S                   00400000     msvcprt:MSVCP140.dll
 0000:ffdae000       .debug$S                   00400000     msvcprt:MSVCP140.dll
 0000:ffdae000       .debug$S                   00400000     msvcprt:MSVCP140.dll
 0000:ffdae000       .debug$S                   00400000     msvcprt:MSVCP140.dll
 0000:ffdae000       .debug$S                   00400000     msvcprt:MSVCP140.dll
 0000:ffdae000       .debug$S                   00400000     msvcprt:MSVCP140.dll
 0000:ffdae000       .debug$S                   00400000     msvcprt:MSVCP140.dll
 0000:ffdae000       .debug$S                   00400000     msvcprt:MSVCP140.dll
 0000:ffdae000       .debug$S                   00400000     msvcprt:MSVCP140.dll
 0000:ffdae000       .debug$S                   00400000     msvcprt:MSVCP140.dll
 0000:ffdae000       .debug$S                   00400000     msvcprt:MSVCP140.dll
 0000:ffdae000       .debug$S                   00400000     msvcprt:MSVCP140.dll
 0000:ffdae000       .debug$S                   00400000     msvcprt:MSVCP140.dll
 0000:ffdae000       .debug$S                   00400000     msvcprt:MSVCP140.dll
 0000:ffdae000       .debug$S                   00400000     msvcprt:MSVCP140.dll
 0000:ffdae000       .debug$S                   00400000     msvcprt:MSVCP140.dll
 0000:ffdae000       .debug$S                   00400000     msvcprt:MSVCP140.dll
 0000:ffdae000       .debug$S                   00400000     msvcprt:MSVCP140.dll
 0000:ffdae000       .debug$S                   00400000     msvcprt:MSVCP140.dll
 0000:ffdae000       .debug$S                   00400000     msvcprt:MSVCP140.dll
 0000:ffdae000       .debug$S                   00400000     msvcprt:MSVCP140.dll
 0000:ffdae000       .debug$S                   00400000     msvcprt:MSVCP140.dll
 0000:ffdae000       .debug$S                   00400000     msvcprt:MSVCP140.dll
 0000:ffdae000       .debug$S                   00400000     msvcprt:MSVCP140.dll
 0000:ffdae000       .debug$S                   00400000     msvcprt:MSVCP140.dll
 0000:ffdae000       .debug$S                   00400000     msvcprt:MSVCP140.dll
 0000:ffdae000       .debug$S                   00400000     msvcprt:MSVCP140.dll
 0000:ffdae000       .debug$S                   00400000     kernel32:KERNEL32.dll
 0000:ffdae000       .debug$S                   00400000     mfc140:mfc140.dll
 0000:ffdae000       .debug$S                   00400000     mfc140:mfc140.dll
 0000:ffdae000       .debug$S                   00400000     mfc140:mfc140.dll
 0000:ffdae000       .debug$S                   00400000     mfc140:mfc140.dll
 0000:ffdae000       .debug$S                   00400000     mfc140:mfc140.dll
 0000:ffdae000       .debug$S                   00400000     mfc140:mfc140.dll
 0000:ffdae000       .debug$S                   00400000     mfc140:mfc140.dll
 0000:ffdae000       .debug$S                   00400000     mfc140:mfc140.dll
 0000:ffdae000       .debug$S                   00400000     mfc140:mfc140.dll
 0000:ffdae000       .debug$S                   00400000     mfc140:mfc140.dll
 0000:ffdae000       .debug$S                   00400000     mfc140:mfc140.dll
 0000:ffdae000       .debug$S                   00400000     mfc140:mfc140.dll
 0000:ffdae000       .debug$S                   00400000     ucrt:api-ms-win-crt-string-l1-1-0.dll
 0000:ffdae000       .debug$S                   00400000     ucrt:api-ms-win-crt-stdio-l1-1-0.dll
 0000:ffdae000       .debug$S                   00400000     ucrt:api-ms-win-crt-string-l1-1-0.dll
 0000:ffdae000       .debug$S                   00400000     ucrt:api-ms-win-crt-heap-l1-1-0.dll
 0000:ffdae000       .debug$S                   00400000     ucrt:api-ms-win-crt-runtime-l1-1-0.dll
 0000:ffdae000       .debug$S                   00400000     ucrt:api-ms-win-crt-runtime-l1-1-0.dll
 0000:ffdae000       .debug$S                   00400000     ucrt:api-ms-win-crt-runtime-l1-1-0.dll
 0000:ffdae000       .debug$S                   00400000     ucrt:api-ms-win-crt-runtime-l1-1-0.dll
 0000:ffdae000       .debug$S                   00400000     ucrt:api-ms-win-crt-stdio-l1-1-0.dll
 0000:ffdae000       .debug$S                   00400000     ucrt:api-ms-win-crt-heap-l1-1-0.dll
 0000:ffdae000       .debug$S                   00400000     ucrt:api-ms-win-crt-locale-l1-1-0.dll
 0000:ffdae000       .debug$S                   00400000     ucrt:api-ms-win-crt-runtime-l1-1-0.dll
 0000:ffdae000       .debug$S                   00400000     ucrt:api-ms-win-crt-runtime-l1-1-0.dll
 0000:ffdae000       .debug$S                   00400000     ucrt:api-ms-win-crt-stdio-l1-1-0.dll
 0000:ffdae000       .debug$S                   00400000     ucrt:api-ms-win-crt-runtime-l1-1-0.dll
 0000:ffdae000       .debug$S                   00400000     ucrt:api-ms-win-crt-runtime-l1-1-0.dll
 0000:ffdae000       .debug$S                   00400000     ucrt:api-ms-win-crt-runtime-l1-1-0.dll
 0000:ffdae000       .debug$S                   00400000     ucrt:api-ms-win-crt-runtime-l1-1-0.dll
 0000:ffdae000       .debug$S                   00400000     ucrt:api-ms-win-crt-runtime-l1-1-0.dll
 0000:ffdae000       .debug$S                   00400000     ucrt:api-ms-win-crt-math-l1-1-0.dll
 0000:ffdae000       .debug$S                   00400000     ucrt:api-ms-win-crt-runtime-l1-1-0.dll
 0000:ffdae000       .debug$S                   00400000     ucrt:api-ms-win-crt-runtime-l1-1-0.dll
 0000:ffdae000       .debug$S                   00400000     ucrt:api-ms-win-crt-runtime-l1-1-0.dll
 0000:ffdae000       .debug$S                   00400000     ucrt:api-ms-win-crt-runtime-l1-1-0.dll
 0000:ffdae000       .debug$S                   00400000     ucrt:api-ms-win-crt-runtime-l1-1-0.dll
 0000:ffdae000       .debug$S                   00400000     ucrt:api-ms-win-crt-runtime-l1-1-0.dll
 0000:ffdae000       .debug$S                   00400000     ucrt:api-ms-win-crt-runtime-l1-1-0.dll
 0000:ffdae000       .debug$S                   00400000     ucrt:api-ms-win-crt-runtime-l1-1-0.dll
 0000:ffdae000       .debug$S                   00400000     ucrt:api-ms-win-crt-runtime-l1-1-0.dll
 0000:ffdae000       .debug$S                   00400000     ucrt:api-ms-win-crt-runtime-l1-1-0.dll
 0000:ffdae000       .debug$S                   00400000     ucrt:api-ms-win-crt-runtime-l1-1-0.dll
 0000:ffdae000       .debug$S                   00400000     ucrt:api-ms-win-crt-stdio-l1-1-0.dll
 0000:ffdae000       .debug$S                   00400000     ucrt:api-ms-win-crt-stdio-l1-1-0.dll
 0000:ffdae000       .debug$S                   00400000     ucrt:api-ms-win-crt-stdio-l1-1-0.dll
 0000:ffdae000       .debug$S                   00400000     ucrt:api-ms-win-crt-convert-l1-1-0.dll
 0000:ffdae000       .debug$S                   00400000     ucrt:api-ms-win-crt-stdio-l1-1-0.dll
 0000:ffdae000       .debug$S                   00400000     ucrt:api-ms-win-crt-string-l1-1-0.dll
 0000:ffdae000       .debug$S                   00400000     ucrt:api-ms-win-crt-string-l1-1-0.dll
 0000:ffdae000       .debug$S                   00400000     ucrt:api-ms-win-crt-filesystem-l1-1-0.dll
 0000:ffdae000       .debug$S                   00400000     ucrt:api-ms-win-crt-runtime-l1-1-0.dll
 0000:ffdae000       .debug$S                   00400000     ucrt:api-ms-win-crt-stdio-l1-1-0.dll
 0000:ffdae000       .debug$S                   00400000     ucrt:api-ms-win-crt-heap-l1-1-0.dll
 0000:ffdae000       .debug$S                   00400000     ucrt:api-ms-win-crt-runtime-l1-1-0.dll
 0000:ffdae000       .debug$S                   00400000     ucrt:api-ms-win-crt-runtime-l1-1-0.dll
 0000:ffdae000       .debug$S                   00400000     ucrt:api-ms-win-crt-time-l1-1-0.dll
 0000:ffdae000       .debug$S                   00400000     ucrt:api-ms-win-crt-runtime-l1-1-0.dll
 0000:ffdae000       .debug$S                   00400000     ucrt:api-ms-win-crt-runtime-l1-1-0.dll
 0000:ffdae000       .debug$S                   00400000     ucrt:api-ms-win-crt-convert-l1-1-0.dll
 0000:ffdae000       .debug$S                   00400000     ucrt:api-ms-win-crt-convert-l1-1-0.dll
 0000:ffdae000       .debug$S                   00400000     ucrt:api-ms-win-crt-utility-l1-1-0.dll
 0000:ffdae000       .debug$S                   00400000     ucrt:api-ms-win-crt-stdio-l1-1-0.dll
 0000:ffdae000       .debug$S                   00400000     ucrt:api-ms-win-crt-stdio-l1-1-0.dll
 0000:ffdae000       .debug$S                   00400000     ucrt:api-ms-win-crt-filesystem-l1-1-0.dll
 0000:ffdae000       .debug$S                   00400000     ucrt:api-ms-win-crt-filesystem-l1-1-0.dll
 0000:ffdae000       .debug$S                   00400000     ucrt:api-ms-win-crt-stdio-l1-1-0.dll
 0000:ffdae000       .debug$S                   00400000     ucrt:api-ms-win-crt-string-l1-1-0.dll
 0000:ffdae000       .debug$S                   00400000     ucrt:api-ms-win-crt-filesystem-l1-1-0.dll
 0000:ffdae000       .debug$S                   00400000     ucrt:api-ms-win-crt-stdio-l1-1-0.dll
 0000:ffdae000       .debug$S                   00400000     ucrt:api-ms-win-crt-stdio-l1-1-0.dll
 0000:ffdae000       .debug$S                   00400000     ucrt:api-ms-win-crt-stdio-l1-1-0.dll
 0000:ffdae000       .debug$S                   00400000     ucrt:api-ms-win-crt-runtime-l1-1-0.dll
 0000:ffdae000       .debug$S                   00400000     ucrt:api-ms-win-crt-math-l1-1-0.dll
 0000:ffdae000       .debug$S                   00400000     ucrt:api-ms-win-crt-math-l1-1-0.dll
 0000:ffdae000       .debug$S                   00400000     ucrt:api-ms-win-crt-string-l1-1-0.dll
 0000:ffdae000       .debug$S                   00400000     mfc140:mfc140.dll
 0000:ffdae000       .debug$S                   00400000     vcruntime:VCRUNTIME140.dll
 0000:ffdae000       .debug$S                   00400000     vcruntime:VCRUNTIME140.dll
 0000:ffdae000       .debug$S                   00400000     vcruntime:VCRUNTIME140.dll
 0000:ffdae000       .debug$S                   00400000     vcruntime:VCRUNTIME140.dll
 0000:ffdae000       .debug$S                   00400000     vcruntime:VCRUNTIME140.dll
 0000:ffdae000       .debug$S                   00400000     vcruntime:VCRUNTIME140.dll
 0000:ffdae000       .debug$S                   00400000     vcruntime:VCRUNTIME140.dll
 0000:ffdae000       .debug$S                   00400000     vcruntime:VCRUNTIME140.dll
 0000:ffdae000       .debug$S                   00400000     vcruntime:VCRUNTIME140.dll
 0000:ffdae000       .debug$S                   00400000     vcruntime:VCRUNTIME140.dll
 0000:ffdae000       .debug$S                   00400000     vcruntime:VCRUNTIME140.dll
 0000:ffdae000       .debug$S                   00400000     vcruntime:VCRUNTIME140.dll
 0000:ffdae000       .debug$S                   00400000     vcruntime:VCRUNTIME140.dll
 0000:ffdae000       .debug$S                   00400000     vcruntime:VCRUNTIME140.dll
 0000:ffdae000       .debug$S                   00400000     vcruntime:VCRUNTIME140.dll
 0000:ffdae000       .debug$S                   00400000     mfc140:mfc140.dll
 0000:ffdae000       .debug$S                   00400000     winhttp:WINHTTP.dll
 0000:ffdae000       .debug$S                   00400000     winhttp:WINHTTP.dll
 0000:ffdae000       .debug$S                   00400000     winhttp:WINHTTP.dll
 0000:ffdae000       .debug$S                   00400000     winhttp:WINHTTP.dll
 0000:ffdae000       .debug$S                   00400000     winhttp:WINHTTP.dll
 0000:ffdae000       .debug$S                   00400000     winhttp:WINHTTP.dll
 0000:ffdae000       .debug$S                   00400000     winhttp:WINHTTP.dll
 0000:ffdae000       .debug$S                   00400000     winhttp:WINHTTP.dll
 0000:ffdae000       .debug$S                   00400000     winhttp:WINHTTP.dll
 0000:ffdae000       .debug$S                   00400000     mfc140:mfc140.dll
 0000:ffdae000       .debug$S                   00400000     winmm:WINMM.dll
 0000:ffdae000       .debug$S                   00400000     mfc140:mfc140.dll
 0000:ffdae000       .debug$S                   00400000     DbgHelp:dbghelp.dll
 0000:ffdae000       .debug$S                   00400000     DbgHelp:dbghelp.dll
 0000:ffdae000       .debug$S                   00400000     DbgHelp:dbghelp.dll
 0000:ffdae000       .debug$S                   00400000     DbgHelp:dbghelp.dll
 0000:ffdae000       .debug$S                   00400000     DbgHelp:dbghelp.dll
 0000:ffdae000       .debug$S                   00400000     DbgHelp:dbghelp.dll
 0000:ffdae000       .debug$S                   00400000     DbgHelp:dbghelp.dll
 0000:ffdae000       .debug$S                   00400000     DbgHelp:dbghelp.dll
 0000:ffdae000       .debug$S                   00400000     mfc140:mfc140.dll
 0000:ffdae000       .debug$S                   00400000     ws2_32:WS2_32.dll
 0000:ffdae000       .debug$S                   00400000     ws2_32:WS2_32.dll
 0000:ffdae000       .debug$S                   00400000     ws2_32:WS2_32.dll
 0000:ffdae000       .debug$S                   00400000     mfc140:mfc140.dll
 0000:ffdae000       .debug$S                   00400000     wininet:WININET.dll
 0000:ffdae000       .debug$S                   00400000     wininet:WININET.dll
 0000:ffdae000       .debug$S                   00400000     wininet:WININET.dll
 0000:ffdae000       .debug$S                   00400000     wininet:WININET.dll
 0000:ffdae000       .debug$S                   00400000     wininet:WININET.dll
 0000:ffdae000       .debug$S                   00400000     wininet:WININET.dll
 0000:ffdae000       .debug$S                   00400000     wininet:WININET.dll
 0000:ffdae000       .debug$S                   00400000     wininet:WININET.dll
 0000:ffdae000       .debug$S                   00400000     mfc140:mfc140.dll
 0000:ffdae000       .debug$S                   00400000     msvcprt:MSVCP140.dll
 0000:ffdae000       .debug$S                   00400000     msvcprt:MSVCP140.dll
 0002:fffe7000       .idata$6                   00400000     oleaut32:OLEAUT32.dll
 0000:ffdae000       .debug$S                   00400000     oleaut32:OLEAUT32.dll
 0000:ffdae000       .debug$S                   00400000     mfc140:mfc140.dll
 0000:ffdae000       .debug$S                   00400000     mfc140:mfc140.dll
 0000:ffdae000       .debug$S                   00400000     mfc140:mfc140.dll
 0000:ffdae000       .debug$S                   00400000     mfc140:mfc140.dll
 0000:ffdae000       .debug$S                   00400000     shlwapi:SHLWAPI.dll
 0000:ffdae000       .debug$S                   00400000     mfc140:mfc140.dll
 0000:ffdae000       .debug$S                   00400000     shell32:SHELL32.dll
 0000:ffdae000       .debug$S                   00400000     mfc140:mfc140.dll
 0000:ffdae000       .debug$S                   00400000     user32:USER32.dll
 0000:ffdae000       .debug$S                   00400000     user32:USER32.dll
 0000:ffdae000       .debug$S                   00400000     user32:USER32.dll
 0000:ffdae000       .debug$S                   00400000     user32:USER32.dll
 0000:ffdae000       .debug$S                   00400000     user32:USER32.dll
 0000:ffdae000       .debug$S                   00400000     user32:USER32.dll
 0000:ffdae000       .debug$S                   00400000     user32:USER32.dll
 0000:ffdae000       .debug$S                   00400000     user32:USER32.dll
 0000:ffdae000       .debug$S                   00400000     user32:USER32.dll
 0000:ffdae000       .debug$S                   00400000     mfc140:mfc140.dll
 0000:ffdae000       .debug$S                   00400000     kernel32:KERNEL32.dll
 0000:ffdae000       .debug$S                   00400000     kernel32:KERNEL32.dll
 0000:ffdae000       .debug$S                   00400000     kernel32:KERNEL32.dll
 0000:ffdae000       .debug$S                   00400000     kernel32:KERNEL32.dll
 0000:ffdae000       .debug$S                   00400000     kernel32:KERNEL32.dll
 0000:ffdae000       .debug$S                   00400000     kernel32:KERNEL32.dll
 0000:ffdae000       .debug$S                   00400000     kernel32:KERNEL32.dll
 0000:ffdae000       .debug$S                   00400000     kernel32:KERNEL32.dll
 0000:ffdae000       .debug$S                   00400000     kernel32:KERNEL32.dll
 0000:ffdae000       .debug$S                   00400000     kernel32:KERNEL32.dll
 0000:ffdae000       .debug$S                   00400000     kernel32:KERNEL32.dll
 0000:ffdae000       .debug$S                   00400000     kernel32:KERNEL32.dll
 0000:ffdae000       .debug$S                   00400000     kernel32:KERNEL32.dll
 0000:ffdae000       .debug$S                   00400000     kernel32:KERNEL32.dll
 0000:ffdae000       .debug$S                   00400000     kernel32:KERNEL32.dll
 0000:ffdae000       .debug$S                   00400000     kernel32:KERNEL32.dll
 0000:ffdae000       .debug$S                   00400000     kernel32:KERNEL32.dll
 0000:ffdae000       .debug$S                   00400000     kernel32:KERNEL32.dll
 0000:ffdae000       .debug$S                   00400000     kernel32:KERNEL32.dll
 0000:ffdae000       .debug$S                   00400000     kernel32:KERNEL32.dll
 0000:ffdae000       .debug$S                   00400000     kernel32:KERNEL32.dll
 0000:ffdae000       .debug$S                   00400000     kernel32:KERNEL32.dll
 0000:ffdae000       .debug$S                   00400000     kernel32:KERNEL32.dll
 0000:ffdae000       .debug$S                   00400000     kernel32:KERNEL32.dll
 0000:ffdae000       .debug$S                   00400000     kernel32:KERNEL32.dll
 0000:ffdae000       .debug$S                   00400000     kernel32:KERNEL32.dll
 0000:ffdae000       .debug$S                   00400000     kernel32:KERNEL32.dll
 0000:ffdae000       .debug$S                   00400000     kernel32:KERNEL32.dll
 0000:ffdae000       .debug$S                   00400000     kernel32:KERNEL32.dll
 0000:ffdae000       .debug$S                   00400000     kernel32:KERNEL32.dll
 0000:ffdae000       .debug$S                   00400000     kernel32:KERNEL32.dll
 0000:ffdae000       .debug$S                   00400000     kernel32:KERNEL32.dll
 0000:ffdae000       .debug$S                   00400000     kernel32:KERNEL32.dll
 0000:ffdae000       .debug$S                   00400000     kernel32:KERNEL32.dll
 0000:ffdae000       .debug$S                   00400000     kernel32:KERNEL32.dll
 0000:ffdae000       .debug$S                   00400000     kernel32:KERNEL32.dll
 0000:ffdae000       .debug$S                   00400000     kernel32:KERNEL32.dll
 0000:ffdae000       .debug$S                   00400000     kernel32:KERNEL32.dll
 0000:ffdae000       .debug$S                   00400000     kernel32:KERNEL32.dll
 0000:ffdae000       .debug$S                   00400000     kernel32:KERNEL32.dll
 0000:ffdae000       .debug$S                   00400000     kernel32:KERNEL32.dll
 0000:ffdae000       .debug$S                   00400000     kernel32:KERNEL32.dll
 0000:ffdae000       .debug$S                   00400000     kernel32:KERNEL32.dll
 0000:ffdae000       .debug$S                   00400000     kernel32:KERNEL32.dll
 0000:ffdae000       .debug$S                   00400000     kernel32:KERNEL32.dll
 0000:ffdae000       .debug$S                   00400000     kernel32:KERNEL32.dll
 0000:ffdae000       .debug$S                   00400000     kernel32:KERNEL32.dll
 0000:ffdae000       .debug$S                   00400000     kernel32:KERNEL32.dll
 0000:ffdae000       .debug$S                   00400000     kernel32:KERNEL32.dll
 0000:ffdae000       .debug$S                   00400000     kernel32:KERNEL32.dll
 0000:ffdae000       .debug$S                   00400000     kernel32:KERNEL32.dll
 0000:ffdae000       .debug$S                   00400000     kernel32:KERNEL32.dll
 0000:ffdae000       .debug$S                   00400000     kernel32:KERNEL32.dll
 0000:ffdae000       .debug$S                   00400000     kernel32:KERNEL32.dll
 0000:ffdae000       .debug$S                   00400000     kernel32:KERNEL32.dll
 0000:ffdae000       .debug$S                   00400000     kernel32:KERNEL32.dll
 0000:ffdae000       .debug$S                   00400000     kernel32:KERNEL32.dll
 0000:ffdae000       .debug$S                   00400000     kernel32:KERNEL32.dll
 0000:ffdae000       .debug$S                   00400000     kernel32:KERNEL32.dll
 0000:ffdae000       .debug$S                   00400000     kernel32:KERNEL32.dll
 0000:ffdae000       .debug$S                   00400000     kernel32:KERNEL32.dll
 0000:ffdae000       .debug$S                   00400000     kernel32:KERNEL32.dll
 0000:ffdae000       .debug$S                   00400000     kernel32:KERNEL32.dll
 0000:ffdae000       .debug$S                   00400000     kernel32:KERNEL32.dll
 0000:ffdae000       .debug$S                   00400000     kernel32:KERNEL32.dll
 0000:ffdae000       .debug$S                   00400000     kernel32:KERNEL32.dll
 0000:ffdae000       .debug$S                   00400000     kernel32:KERNEL32.dll
 0000:ffdae000       .debug$S                   00400000     kernel32:KERNEL32.dll
 0000:ffdae000       .debug$S                   00400000     kernel32:KERNEL32.dll
 0000:ffdae000       .debug$S                   00400000     kernel32:KERNEL32.dll
 0000:ffdae000       .debug$S                   00400000     kernel32:KERNEL32.dll
 0000:ffdae000       .debug$S                   00400000     kernel32:KERNEL32.dll
 0000:ffdae000       .debug$S                   00400000     mfc140:mfc140.dll
 0000:ffdae000       .debug$S                   00400000     mfc140:mfc140.dll
 0000:ffdae000       .debug$S                   00400000     mfc140:mfc140.dll
 0000:ffdae000       .debug$S                   00400000     mfc140:mfc140.dll
 0000:ffdae000       .debug$S                   00400000     mfc140:mfc140.dll
 0000:ffdae000       .debug$S                   00400000     mfc140:mfc140.dll
 0000:ffdae000       .debug$S                   00400000     mfc140:mfc140.dll
 0000:ffdae000       .debug$S                   00400000     mfc140:mfc140.dll
 0000:ffdae000       .debug$S                   00400000     mfc140:mfc140.dll
 0000:ffdae000       .debug$S                   00400000     mfc140:mfc140.dll
 0000:ffdae000       .debug$S                   00400000     mfc140:mfc140.dll
 0000:ffdae000       .debug$S                   00400000     mfc140:mfc140.dll
 0000:ffdae000       .debug$S                   00400000     mfc140:mfc140.dll
 0000:ffdae000       .debug$S                   00400000     mfc140:mfc140.dll
 0000:ffdae000       .debug$S                   00400000     mfc140:mfc140.dll
 0000:ffdae000       .debug$S                   00400000     mfc140:mfc140.dll
 0000:ffdae000       .debug$S                   00400000     mfc140:mfc140.dll
 0000:ffdae000       .debug$S                   00400000     mfc140:mfc140.dll
 0000:ffdae000       .debug$S                   00400000     mfc140:mfc140.dll
 0000:ffdae000       .debug$S                   00400000     mfc140:mfc140.dll
 0000:ffdae000       .debug$S                   00400000     mfc140:mfc140.dll
 0000:ffdae000       .debug$S                   00400000     mfc140:mfc140.dll
 0000:ffdae000       .debug$S                   00400000     mfc140:mfc140.dll
 0000:ffdae000       .debug$S                   00400000     mfc140:mfc140.dll
 0000:ffdae000       .debug$S                   00400000     mfc140:mfc140.dll
 0000:ffdae000       .debug$S                   00400000     mfc140:mfc140.dll
 0000:ffdae000       .debug$S                   00400000     mfc140:mfc140.dll
 0000:ffdae000       .debug$S                   00400000     mfc140:mfc140.dll
 0000:ffdae000       .debug$S                   00400000     mfc140:mfc140.dll
 0000:ffdae000       .debug$S                   00400000     mfc140:mfc140.dll
 0000:ffdae000       .debug$S                   00400000     mfc140:mfc140.dll
 0000:ffdae000       .debug$S                   00400000     mfc140:mfc140.dll
 0000:ffdae000       .debug$S                   00400000     mfc140:mfc140.dll
 0000:ffdae000       .debug$S                   00400000     mfc140:mfc140.dll
 0000:ffdae000       .debug$S                   00400000     mfc140:mfc140.dll
 0000:ffdae000       .debug$S                   00400000     mfc140:mfc140.dll
 0000:ffdae000       .debug$S                   00400000     mfc140:mfc140.dll
 0000:ffdae000       .debug$S                   00400000     mfc140:mfc140.dll
 0000:ffdae000       .debug$S                   00400000     mfc140:mfc140.dll
 0000:ffdae000       .debug$S                   00400000     mfc140:mfc140.dll
 0000:ffdae000       .debug$S                   00400000     mfc140:mfc140.dll
 0000:ffdae000       .debug$S                   00400000     mfc140:mfc140.dll
 0000:ffdae000       .debug$S                   00400000     mfc140:mfc140.dll
 0000:ffdae000       .debug$S                   00400000     mfc140:mfc140.dll
 0000:ffdae000       .debug$S                   00400000     mfc140:mfc140.dll
 0000:ffdae000       .debug$S                   00400000     mfc140:mfc140.dll
 0000:ffdae000       .debug$S                   00400000     mfc140:mfc140.dll
 0000:ffdae000       .debug$S                   00400000     mfc140:mfc140.dll
 0000:ffdae000       .debug$S                   00400000     mfc140:mfc140.dll
 0000:ffdae000       .debug$S                   00400000     mfc140:mfc140.dll
 0000:ffdae000       .debug$S                   00400000     mfc140:mfc140.dll
 0000:ffdae000       .debug$S                   00400000     mfc140:mfc140.dll
 0000:ffdae000       .debug$S                   00400000     mfc140:mfc140.dll
 0000:ffdae000       .debug$S                   00400000     mfc140:mfc140.dll
 0000:ffdae000       .debug$S                   00400000     mfc140:mfc140.dll
 0000:ffdae000       .debug$S                   00400000     mfc140:mfc140.dll
 0000:ffdae000       .debug$S                   00400000     mfc140:mfc140.dll
 0000:ffdae000       .debug$S                   00400000     mfc140:mfc140.dll
 0000:ffdae000       .debug$S                   00400000     mfc140:mfc140.dll
 0000:ffdae000       .debug$S                   00400000     mfc140:mfc140.dll
 0000:ffdae000       .debug$S                   00400000     mfc140:mfc140.dll
 0000:ffdae000       .debug$S                   00400000     mfc140:mfc140.dll
 0000:ffdae000       .debug$S                   00400000     mfc140:mfc140.dll
 0000:ffdae000       .debug$S                   00400000     mfc140:mfc140.dll
 0000:ffdae000       .debug$S                   00400000     mfc140:mfc140.dll
 0000:ffdae000       .debug$S                   00400000     mfc140:mfc140.dll
 0000:ffdae000       .debug$S                   00400000     mfc140:mfc140.dll
 0000:ffdae000       .debug$S                   00400000     mfc140:mfc140.dll
 0000:ffdae000       .debug$S                   00400000     mfc140:mfc140.dll
 0000:ffdae000       .debug$S                   00400000     mfc140:mfc140.dll
 0000:ffdae000       .debug$S                   00400000     mfc140:mfc140.dll
 0000:ffdae000       .debug$S                   00400000     mfc140:mfc140.dll
 0000:ffdae000       .debug$S                   00400000     mfc140:mfc140.dll
 0000:ffdae000       .debug$S                   00400000     mfc140:mfc140.dll
 0000:ffdae000       .debug$S                   00400000     mfc140:mfc140.dll
 0000:ffdae000       .debug$S                   00400000     mfc140:mfc140.dll
 0000:ffdae000       .debug$S                   00400000     mfc140:mfc140.dll
 0000:ffdae000       .debug$S                   00400000     mfc140:mfc140.dll
 0000:ffdae000       .debug$S                   00400000     mfc140:mfc140.dll
 0000:ffdae000       .debug$S                   00400000     mfc140:mfc140.dll
 0000:ffdae000       .debug$S                   00400000     mfc140:mfc140.dll
 0000:ffdae000       .debug$S                   00400000     mfc140:mfc140.dll
 0000:ffdae000       .debug$S                   00400000     mfc140:mfc140.dll
 0000:ffdae000       .debug$S                   00400000     mfc140:mfc140.dll
 0000:ffdae000       .debug$S                   00400000     mfc140:mfc140.dll
 0000:ffdae000       .debug$S                   00400000     mfc140:mfc140.dll
 0000:ffdae000       .debug$S                   00400000     mfc140:mfc140.dll
 0000:ffdae000       .debug$S                   00400000     mfc140:mfc140.dll
 0000:ffdae000       .debug$S                   00400000     mfc140:mfc140.dll
 0000:ffdae000       .debug$S                   00400000     mfc140:mfc140.dll
 0000:ffdae000       .debug$S                   00400000     mfc140:mfc140.dll
 0000:ffdae000       .debug$S                   00400000     mfc140:mfc140.dll
 0000:ffdae000       .debug$S                   00400000     mfc140:mfc140.dll
 0000:ffdae000       .debug$S                   00400000     mfc140:mfc140.dll
 0000:ffdae000       .debug$S                   00400000     mfc140:mfc140.dll
 0000:ffdae000       .debug$S                   00400000     mfc140:mfc140.dll
 0000:ffdae000       .debug$S                   00400000     mfc140:mfc140.dll
 0000:ffdae000       .debug$S                   00400000     mfc140:mfc140.dll
 0000:ffdae000       .debug$S                   00400000     mfc140:mfc140.dll
 0000:ffdae000       .debug$S                   00400000     mfc140:mfc140.dll
 0000:ffdae000       .debug$S                   00400000     mfc140:mfc140.dll
 0000:ffdae000       .debug$S                   00400000     mfc140:mfc140.dll
 0000:ffdae000       .debug$S                   00400000     mfc140:mfc140.dll
 0000:ffdae000       .debug$S                   00400000     mfc140:mfc140.dll
 0000:ffdae000       .debug$S                   00400000     mfc140:mfc140.dll
 0000:ffdae000       .debug$S                   00400000     mfc140:mfc140.dll
 0000:ffdae000       .debug$S                   00400000     mfc140:mfc140.dll
 0000:ffdae000       .debug$S                   00400000     mfc140:mfc140.dll
 0000:ffdae000       .debug$S                   00400000     mfc140:mfc140.dll
 0000:ffdae000       .debug$S                   00400000     mfc140:mfc140.dll
 0000:ffdae000       .debug$S                   00400000     mfc140:mfc140.dll
 0000:ffdae000       .debug$S                   00400000     mfc140:mfc140.dll
 0000:ffdae000       .debug$S                   00400000     mfc140:mfc140.dll
 0000:ffdae000       .debug$S                   00400000     mfc140:mfc140.dll
 0000:ffdae000       .debug$S                   00400000     mfc140:mfc140.dll
 0000:ffdae000       .debug$S                   00400000     mfc140:mfc140.dll
 0000:ffdae000       .debug$S                   00400000     mfc140:mfc140.dll
 0000:ffdae000       .debug$S                   00400000     mfc140:mfc140.dll
 0000:ffdae000       .debug$S                   00400000     mfc140:mfc140.dll
 0000:ffdae000       .debug$S                   00400000     mfc140:mfc140.dll
 0000:ffdae000       .debug$S                   00400000     mfc140:mfc140.dll
 0001:00000000       ??__EA@VectorSinConstantsSSE@@YAXXZ 00401000 f   ltmodule.obj
 0001:00000020       ??__EAllMask@GlobalVectorConstants@@YAXXZ 00401020 f   ltmodule.obj
 0001:00000030       ??__EB@VectorSinConstantsSSE@@YAXXZ 00401030 f   ltmodule.obj
 0001:00000050       ??__EBigNumber@GlobalVectorConstants@@YAXXZ 00401050 f   ltmodule.obj
 0001:00000060       ??__EDEGREES_PER_RADIAN@@YAXXZ 00401060 f   ltmodule.obj
 0001:00000080       ??__EDEG_TO_RAD@GlobalVectorConstants@@YAXXZ 00401080 f   ltmodule.obj
 0001:00000090       ??__EDEG_TO_RAD_HALF@GlobalVectorConstants@@YAXXZ 00401090 f   ltmodule.obj
 0001:000000a0       ??__EFloat0001@GlobalVectorConstants@@YAXXZ 004010a0 f   ltmodule.obj
 0001:000000b0       ??__EFloat111_Minus1@GlobalVectorConstants@@YAXXZ 004010b0 f   ltmodule.obj
 0001:000000c0       ??__EFloat127@GlobalVectorConstants@@YAXXZ 004010c0 f   ltmodule.obj
 0001:000000d0       ??__EFloat180@GlobalVectorConstants@@YAXXZ 004010d0 f   ltmodule.obj
 0001:000000e0       ??__EFloat255@GlobalVectorConstants@@YAXXZ 004010e0 f   ltmodule.obj
 0001:000000f0       ??__EFloat360@GlobalVectorConstants@@YAXXZ 004010f0 f   ltmodule.obj
 0001:00000100       ??__EFloatAlmostTwo@GlobalVectorConstants@@YAXXZ 00401100 f   ltmodule.obj
 0001:00000110       ??__EFloatInfinity@GlobalVectorConstants@@YAXXZ 00401110 f   ltmodule.obj
 0001:00000120       ??__EFloatMinus1_111@GlobalVectorConstants@@YAXXZ 00401120 f   ltmodule.obj
 0001:00000130       ??__EFloatMinusOne@GlobalVectorConstants@@YAXXZ 00401130 f   ltmodule.obj
 0001:00000140       ??__EFloatMinusOneHalf@GlobalVectorConstants@@YAXXZ 00401140 f   ltmodule.obj
 0001:00000150       ??__EFloatNeg127@GlobalVectorConstants@@YAXXZ 00401150 f   ltmodule.obj
 0001:00000160       ??__EFloatOne@GlobalVectorConstants@@YAXXZ 00401160 f   ltmodule.obj
 0001:00000170       ??__EFloatOneHalf@GlobalVectorConstants@@YAXXZ 00401170 f   ltmodule.obj
 0001:00000180       ??__EFloatOneHundredth@GlobalVectorConstants@@YAXXZ 00401180 f   ltmodule.obj
 0001:00000190       ??__EFloatTwo@GlobalVectorConstants@@YAXXZ 00401190 f   ltmodule.obj
 0001:000001a0       ??__EFloatZero@GlobalVectorConstants@@YAXXZ 004011a0 f   ltmodule.obj
 0001:000001b0       ??__EIntAllMask@GlobalVectorConstants@@YAXXZ 004011b0 f   ltmodule.obj
 0001:000001c0       ??__EIntMinusOne@GlobalVectorConstants@@YAXXZ 004011c0 f   ltmodule.obj
 0001:000001d0       ??__EIntOne@GlobalVectorConstants@@YAXXZ 004011d0 f   ltmodule.obj
 0001:000001e0       ??__EIntSignBit@GlobalVectorConstants@@YAXXZ 004011e0 f   ltmodule.obj
 0001:000001f0       ??__EIntSignMask@GlobalVectorConstants@@YAXXZ 004011f0 f   ltmodule.obj
 0001:00000200       ??__EIntZero@GlobalVectorConstants@@YAXXZ 00401200 f   ltmodule.obj
 0001:00000210       ??__EKindaSmallNumber@GlobalVectorConstants@@YAXXZ 00401210 f   ltmodule.obj
 0001:00000220       ??__EOneOverPi@GlobalVectorConstants@@YAXXZ 00401220 f   ltmodule.obj
 0001:00000230       ??__EOneOverTwoPi@GlobalVectorConstants@@YAXXZ 00401230 f   ltmodule.obj
 0001:00000240       ??__EPI@@YAXXZ             00401240 f   ltmodule.obj
 0001:00000270       ??__EPI_2@@YAXXZ           00401270 f   ltmodule.obj
 0001:00000290       ??__EPI_3@@YAXXZ           00401290 f   ltmodule.obj
 0001:000002b0       ??__EPI_4@@YAXXZ           004012b0 f   ltmodule.obj
 0001:000002d0       ??__EPi@GlobalVectorConstants@@YAXXZ 004012d0 f   ltmodule.obj
 0001:000002e0       ??__EPiByFour@GlobalVectorConstants@@YAXXZ 004012e0 f   ltmodule.obj
 0001:000002f0       ??__EPiByTwo@GlobalVectorConstants@@YAXXZ 004012f0 f   ltmodule.obj
 0001:00000300       ??__EQINV_SIGN_MASK@GlobalVectorConstants@@YAXXZ 00401300 f   ltmodule.obj
 0001:00000310       ??__EQMULTI_SIGN_MASK0@GlobalVectorConstants@@YAXXZ 00401310 f   ltmodule.obj
 0001:00000320       ??__EQMULTI_SIGN_MASK1@GlobalVectorConstants@@YAXXZ 00401320 f   ltmodule.obj
 0001:00000330       ??__EQMULTI_SIGN_MASK2@GlobalVectorConstants@@YAXXZ 00401330 f   ltmodule.obj
 0001:00000340       ??__ERADIANS_PER_DEGREE@@YAXXZ 00401340 f   ltmodule.obj
 0001:00000360       ??__ERAD_TO_DEG@GlobalVectorConstants@@YAXXZ 00401360 f   ltmodule.obj
 0001:00000370       ??__ESignBit@GlobalVectorConstants@@YAXXZ 00401370 f   ltmodule.obj
 0001:00000380       ??__ESignMask@GlobalVectorConstants@@YAXXZ 00401380 f   ltmodule.obj
 0001:00000390       ??__ESmallLengthThreshold@GlobalVectorConstants@@YAXXZ 00401390 f   ltmodule.obj
 0001:000003a0       ??__ESmallNumber@GlobalVectorConstants@@YAXXZ 004013a0 f   ltmodule.obj
 0001:000003b0       ??__EThreshQuatNormalized@GlobalVectorConstants@@YAXXZ 004013b0 f   ltmodule.obj
 0001:000003c0       ??__ETwoPi@GlobalVectorConstants@@YAXXZ 004013c0 f   ltmodule.obj
 0001:000003d0       ??__EXYZMask@GlobalVectorConstants@@YAXXZ 004013d0 f   ltmodule.obj
 0001:000003e0       ??__E_FILE_SHUTDOWN_var_ltmod_database_@@YAXXZ 004013e0 f   ltmodule.obj
 0001:000003f0       ??__Ea@VectorSinConstantsSSE@@YAXXZ 004013f0 f   ltmodule.obj
 0001:00000420       ??__Eb@VectorSinConstantsSSE@@YAXXZ 00401420 f   ltmodule.obj
 0001:00000450       ??__E?m_LogLock@CHLogger@@0VCMustSyncObjectLog@@A@@YAXXZ 00401450 f   HostLogger.obj
 0001:00000470       ??__E?m_LogPacketLock@CHLogger@@0VCMustSyncObjectLog@@A@@YAXXZ 00401470 f   HostLogger.obj
 0001:00000490       ??__E?m_strBRFileFormat@CHLogger@@0V?$basic_string@DU?$char_traits@D@std@@V?$allocator@D@2@@std@@A@@YAXXZ 00401490 f   HostLogger.obj
 0001:000004a0       ??__E?m_strEtcFileFormat@CHLogger@@0V?$basic_string@DU?$char_traits@D@std@@V?$allocator@D@2@@std@@A@@YAXXZ 004014a0 f   HostLogger.obj
 0001:000004b0       ??__E?m_strFileFormat@CHLogger@@0V?$basic_string@DU?$char_traits@D@std@@V?$allocator@D@2@@std@@A@@YAXXZ 004014b0 f   HostLogger.obj
 0001:000004c0       ??__E?m_strHostName@CHLogger@@0V?$basic_string@DU?$char_traits@D@std@@V?$allocator@D@2@@std@@A@@YAXXZ 004014c0 f   HostLogger.obj
 0001:000004d0       ??__E?m_strIPCMessageFileFormat@CHLogger@@0V?$basic_string@DU?$char_traits@D@std@@V?$allocator@D@2@@std@@A@@YAXXZ 004014d0 f   HostLogger.obj
 0001:000004e0       ??__E?m_strKernelFileFormat@CHLogger@@0V?$basic_string@DU?$char_traits@D@std@@V?$allocator@D@2@@std@@A@@YAXXZ 004014e0 f   HostLogger.obj
 0001:000004f0       ??__E?m_strLogFolder@CHLogger@@0V?$basic_string@DU?$char_traits@D@std@@V?$allocator@D@2@@std@@A@@YAXXZ 004014f0 f   HostLogger.obj
 0001:00000500       ??__E?m_strModeUserCountFormat@CHLogger@@0V?$basic_string@DU?$char_traits@D@std@@V?$allocator@D@2@@std@@A@@YAXXZ 00401500 f   HostLogger.obj
 0001:00000510       ??__E?m_strPacketFileFormat@CHLogger@@0V?$basic_string@DU?$char_traits@D@std@@V?$allocator@D@2@@std@@A@@YAXXZ 00401510 f   HostLogger.obj
 0001:00000520       ??__E?m_strRWProcessMemoryFileFormat@CHLogger@@0V?$basic_string@DU?$char_traits@D@std@@V?$allocator@D@2@@std@@A@@YAXXZ 00401520 f   HostLogger.obj
 0001:00000530       ??__E?m_strServerAppUseCountFormat@CHLogger@@0V?$basic_string@DU?$char_traits@D@std@@V?$allocator@D@2@@std@@A@@YAXXZ 00401530 f   HostLogger.obj
 0001:00000540       ??__E?m_strServerName@CHLogger@@0V?$basic_string@DU?$char_traits@D@std@@V?$allocator@D@2@@std@@A@@YAXXZ 00401540 f   HostLogger.obj
 0001:00000550       ??__E?m_strTimeOutFileFormat@CHLogger@@0V?$basic_string@DU?$char_traits@D@std@@V?$allocator@D@2@@std@@A@@YAXXZ 00401550 f   HostLogger.obj
 0001:00000560       ??__E?m_vectSharedMapHandles@CLogMsgManager@@0V?$vector@PAXV?$allocator@PAX@std@@@std@@A@@YAXXZ 00401560 f   LogMsgManager.obj
 0001:00000570       ??__EtheApp@@YAXXZ         00401570 f   ServerApp.obj
 0001:00000590       ??__E__api_holder_ILTCommon_Server_g_pLTSCommon__@@YAXXZ 00401590 f   ServerAppDlg.obj
 0001:000005c0       ??__Eg_cServerLog@@YAXXZ   004015c0 f   ServerAppDlg.obj
 0001:000005e0       ??__Eg_sGameInfos@@YAXXZ   004015e0 f   ServerAppDlg.obj
 0001:00000650       ??__Eg_sUserInfos@@YAXXZ   00401650 f   ServerAppDlg.obj
 0001:00000680       ??__EA@VectorSinConstantsSSE@@YAXXZ 00401680 f   StdAfx.obj
 0001:000006a0       ??__EAllMask@GlobalVectorConstants@@YAXXZ 004016a0 f   StdAfx.obj
 0001:000006b0       ??__EB@VectorSinConstantsSSE@@YAXXZ 004016b0 f   StdAfx.obj
 0001:000006d0       ??__EBigNumber@GlobalVectorConstants@@YAXXZ 004016d0 f   StdAfx.obj
 0001:000006e0       ??__EDEGREES_PER_RADIAN@@YAXXZ 004016e0 f   StdAfx.obj
 0001:00000700       ??__EDEG_TO_RAD@GlobalVectorConstants@@YAXXZ 00401700 f   StdAfx.obj
 0001:00000710       ??__EDEG_TO_RAD_HALF@GlobalVectorConstants@@YAXXZ 00401710 f   StdAfx.obj
 0001:00000720       ??__EFloat0001@GlobalVectorConstants@@YAXXZ 00401720 f   StdAfx.obj
 0001:00000730       ??__EFloat111_Minus1@GlobalVectorConstants@@YAXXZ 00401730 f   StdAfx.obj
 0001:00000740       ??__EFloat127@GlobalVectorConstants@@YAXXZ 00401740 f   StdAfx.obj
 0001:00000750       ??__EFloat180@GlobalVectorConstants@@YAXXZ 00401750 f   StdAfx.obj
 0001:00000760       ??__EFloat255@GlobalVectorConstants@@YAXXZ 00401760 f   StdAfx.obj
 0001:00000770       ??__EFloat360@GlobalVectorConstants@@YAXXZ 00401770 f   StdAfx.obj
 0001:00000780       ??__EFloatAlmostTwo@GlobalVectorConstants@@YAXXZ 00401780 f   StdAfx.obj
 0001:00000790       ??__EFloatInfinity@GlobalVectorConstants@@YAXXZ 00401790 f   StdAfx.obj
 0001:000007a0       ??__EFloatMinus1_111@GlobalVectorConstants@@YAXXZ 004017a0 f   StdAfx.obj
 0001:000007b0       ??__EFloatMinusOne@GlobalVectorConstants@@YAXXZ 004017b0 f   StdAfx.obj
 0001:000007c0       ??__EFloatMinusOneHalf@GlobalVectorConstants@@YAXXZ 004017c0 f   StdAfx.obj
 0001:000007d0       ??__EFloatNeg127@GlobalVectorConstants@@YAXXZ 004017d0 f   StdAfx.obj
 0001:000007e0       ??__EFloatOne@GlobalVectorConstants@@YAXXZ 004017e0 f   StdAfx.obj
 0001:000007f0       ??__EFloatOneHalf@GlobalVectorConstants@@YAXXZ 004017f0 f   StdAfx.obj
 0001:00000800       ??__EFloatOneHundredth@GlobalVectorConstants@@YAXXZ 00401800 f   StdAfx.obj
 0001:00000810       ??__EFloatTwo@GlobalVectorConstants@@YAXXZ 00401810 f   StdAfx.obj
 0001:00000820       ??__EFloatZero@GlobalVectorConstants@@YAXXZ 00401820 f   StdAfx.obj
 0001:00000830       ??__EIntAllMask@GlobalVectorConstants@@YAXXZ 00401830 f   StdAfx.obj
 0001:00000840       ??__EIntMinusOne@GlobalVectorConstants@@YAXXZ 00401840 f   StdAfx.obj
 0001:00000850       ??__EIntOne@GlobalVectorConstants@@YAXXZ 00401850 f   StdAfx.obj
 0001:00000860       ??__EIntSignBit@GlobalVectorConstants@@YAXXZ 00401860 f   StdAfx.obj
 0001:00000870       ??__EIntSignMask@GlobalVectorConstants@@YAXXZ 00401870 f   StdAfx.obj
 0001:00000880       ??__EIntZero@GlobalVectorConstants@@YAXXZ 00401880 f   StdAfx.obj
 0001:00000890       ??__EKindaSmallNumber@GlobalVectorConstants@@YAXXZ 00401890 f   StdAfx.obj
 0001:000008a0       ??__EOneOverPi@GlobalVectorConstants@@YAXXZ 004018a0 f   StdAfx.obj
 0001:000008b0       ??__EOneOverTwoPi@GlobalVectorConstants@@YAXXZ 004018b0 f   StdAfx.obj
 0001:000008c0       ??__EPI@@YAXXZ             004018c0 f   StdAfx.obj
 0001:000008f0       ??__EPI_2@@YAXXZ           004018f0 f   StdAfx.obj
 0001:00000910       ??__EPI_3@@YAXXZ           00401910 f   StdAfx.obj
 0001:00000930       ??__EPI_4@@YAXXZ           00401930 f   StdAfx.obj
 0001:00000950       ??__EPi@GlobalVectorConstants@@YAXXZ 00401950 f   StdAfx.obj
 0001:00000960       ??__EPiByFour@GlobalVectorConstants@@YAXXZ 00401960 f   StdAfx.obj
 0001:00000970       ??__EPiByTwo@GlobalVectorConstants@@YAXXZ 00401970 f   StdAfx.obj
 0001:00000980       ??__EQINV_SIGN_MASK@GlobalVectorConstants@@YAXXZ 00401980 f   StdAfx.obj
 0001:00000990       ??__EQMULTI_SIGN_MASK0@GlobalVectorConstants@@YAXXZ 00401990 f   StdAfx.obj
 0001:000009a0       ??__EQMULTI_SIGN_MASK1@GlobalVectorConstants@@YAXXZ 004019a0 f   StdAfx.obj
 0001:000009b0       ??__EQMULTI_SIGN_MASK2@GlobalVectorConstants@@YAXXZ 004019b0 f   StdAfx.obj
 0001:000009c0       ??__ERADIANS_PER_DEGREE@@YAXXZ 004019c0 f   StdAfx.obj
 0001:000009e0       ??__ERAD_TO_DEG@GlobalVectorConstants@@YAXXZ 004019e0 f   StdAfx.obj
 0001:000009f0       ??__ESignBit@GlobalVectorConstants@@YAXXZ 004019f0 f   StdAfx.obj
 0001:00000a00       ??__ESignMask@GlobalVectorConstants@@YAXXZ 00401a00 f   StdAfx.obj
 0001:00000a10       ??__ESmallLengthThreshold@GlobalVectorConstants@@YAXXZ 00401a10 f   StdAfx.obj
 0001:00000a20       ??__ESmallNumber@GlobalVectorConstants@@YAXXZ 00401a20 f   StdAfx.obj
 0001:00000a30       ??__EThreshQuatNormalized@GlobalVectorConstants@@YAXXZ 00401a30 f   StdAfx.obj
 0001:00000a40       ??__ETwoPi@GlobalVectorConstants@@YAXXZ 00401a40 f   StdAfx.obj
 0001:00000a50       ??__EXYZMask@GlobalVectorConstants@@YAXXZ 00401a50 f   StdAfx.obj
 0001:00000a60       ??__Ea@VectorSinConstantsSSE@@YAXXZ 00401a60 f   StdAfx.obj
 0001:00000a90       ??__Eb@VectorSinConstantsSSE@@YAXXZ 00401a90 f   StdAfx.obj
 0001:00000abf       ??__E_AtlBaseModule@ATL@@YAXXZ 00401abf f   atls:atlbase.obj
 0001:00000ad5       ??__E_afxInitAppState@@YAXXZ 00401ad5 f   mfcs140:appmodul.obj
 0001:00001ea5       __catch$??$?6U?$char_traits@D@std@@@std@@YAAAV?$basic_ostream@DU?$char_traits@D@std@@@0@AAV10@PBD@Z$0 00402ea5 f i safe_string:safe_string.obj
 0001:00005fd4       $LN35                      00406fd4     HostLogger.obj
 0001:00007267       __catch$??$_Insert_hint@AAU?$pair@$$CB_JV?$basic_string@DU?$char_traits@D@std@@V?$allocator@D@2@@std@@@std@@PAU?$_Tree_node@U?$pair@$$CB_JV?$basic_string@DU?$char_traits@D@std@@V?$allocator@D@2@@std@@@std@@PAX@2@@?$_Tree@V?$_Tmap_traits@_JV?$basic_string@DU?$char_traits@D@std@@V?$allocator@D@2@@std@@U?$less@_J@2@V?$allocator@U?$pair@$$CB_JV?$basic_string@DU?$char_traits@D@std@@V?$allocator@D@2@@std@@@std@@@2@$0A@@std@@@std@@IAE?AV?$_Tree_iterator@V?$_Tree_val@U?$_Tree_simple_types@U?$pair@$$CB_JV?$basic_string@DU?$char_traits@D@std@@V?$allocator@D@2@@std@@@std@@@std@@@std@@@1@V?$_Tree_const_iterator@V?$_Tree_val@U?$_Tree_simple_types@U?$pair@$$CB_JV?$basic_string@DU?$char_traits@D@std@@V?$allocator@D@2@@std@@@std@@@std@@@std@@@1@AAU?$pair@$$CB_JV?$basic_string@DU?$char_traits@D@std@@V?$allocator@D@2@@std@@@1@PAU?$_Tree_node@U?$pair@$$CB_JV?$basic_string@DU?$char_traits@D@std@@V?$allocator@D@2@@std@@@std@@PAX@1@@Z$0 00408267 f i LoadXlsMsg.obj
 0001:000073a8       __catch$??$_Insert_nohint@AAU?$pair@$$CB_JV?$basic_string@DU?$char_traits@D@std@@V?$allocator@D@2@@std@@@std@@PAU?$_Tree_node@U?$pair@$$CB_JV?$basic_string@DU?$char_traits@D@std@@V?$allocator@D@2@@std@@@std@@PAX@2@@?$_Tree@V?$_Tmap_traits@_JV?$basic_string@DU?$char_traits@D@std@@V?$allocator@D@2@@std@@U?$less@_J@2@V?$allocator@U?$pair@$$CB_JV?$basic_string@DU?$char_traits@D@std@@V?$allocator@D@2@@std@@@std@@@2@$0A@@std@@@std@@IAE?AU?$pair@V?$_Tree_iterator@V?$_Tree_val@U?$_Tree_simple_types@U?$pair@$$CB_JV?$basic_string@DU?$char_traits@D@std@@V?$allocator@D@2@@std@@@std@@@std@@@std@@@std@@_N@1@_NAAU?$pair@$$CB_JV?$basic_string@DU?$char_traits@D@std@@V?$allocator@D@2@@std@@@1@PAU?$_Tree_node@U?$pair@$$CB_JV?$basic_string@DU?$char_traits@D@std@@V?$allocator@D@2@@std@@@std@@PAX@1@@Z$0 004083a8 f i LoadXlsMsg.obj
 0001:00008c11       __catch$??1CWaitCursor@@QAE@XZ$0 00409c11 f i ServerAppDlg.obj
 0001:000094a4       $LN87                      0040a4a4     ServerAppDlg.obj
 0001:0000bc00       $LN84                      0040cc00     ServerAppDlg.obj
 0001:0000bc34       $LN80                      0040cc34     ServerAppDlg.obj
 0001:0000e868       $LN948                     0040f868     ServerAppDlg.obj
 0001:0000e8f0       $LN924                     0040f8f0     ServerAppDlg.obj
 0001:0000f650       ?RTIDUSNtoString@EXPAND_USN@@YA?AV?$basic_string@DU?$char_traits@D@std@@V?$allocator@D@2@@std@@HFF_J@Z 00410650 f   ServerAppDlg.obj
 0001:00012220       ?USNtoStr@EXPAND_USN@@YA?AV?$basic_string@DU?$char_traits@D@std@@V?$allocator@D@2@@std@@_J@Z 00413220 f   ServerAppDlg.obj
 0001:000127b0       ?CRSUploader@@YAAAVUploader@crs@@XZ 004137b0 f   BugReporter1.obj
 0001:00012880       ?GetVersionName@@YAHXZ     00413880 f   BugReporter1.obj
 0001:00012880       ?GetVersionName@@YAHXZ     00413880 f   crs_uploader1.obj
 0001:00013280       ?EnumModuleDetail@ModuleInfo@?1??makeExceptionLog@Uploader@crs@@QAEXPAU_EXCEPTION_POINTERS@@AAVLogBuffer@4@@Z@SGHPBD_KKPAX@Z 00414280 f   crs_uploader1.obj
 0001:0001586b       ?find_pe_section@@YAPAU_IMAGE_SECTION_HEADER@@QAEI@Z 0041686b f   msvcrt:utility.obj
 0001:00015b10       $$000000                   00416b10     msvcrt:chkstk.obj
 0001:00015b3d       ?pre_c_initialization@@YAHXZ 00416b3d f   msvcrt:exe_winmain.obj
 0001:00015be8       ?post_pgo_initialization@@YAHXZ 00416be8 f   msvcrt:exe_winmain.obj
 0001:00015bf0       ?pre_cpp_initialization@@YAXXZ 00416bf0 f   msvcrt:exe_winmain.obj
 0001:00015c02       ?__scrt_common_main_seh@@YAHXZ 00416c02 f   msvcrt:exe_winmain.obj
 0001:00015d90       $$000000                   00416d90     msvcrt:sehprolg4.obj
 0001:00015df0       $$000000                   00416df0     msvcrt:sehprolg4gs.obj
 0001:0001631d       ___get_entropy             0041731d f   msvcrt:gs_support.obj
 0001:00016690       __unwindfunclet$?sprintf_s@internal@cf@@YAHPADIPBDAAPAD@Z$0 00417690 f   safe_string:safe_string.obj
 0001:0001669b       __unwindfunclet$?sprintf_s@internal@cf@@YAHPADIPBDAAPAD@Z$1 0041769b f   safe_string:safe_string.obj
 0001:000166a3       __unwindfunclet$?sprintf_s@internal@cf@@YAHPADIPBDAAPAD@Z$2 004176a3 f   safe_string:safe_string.obj
 0001:000166ab       __ehhandler$?sprintf_s@internal@cf@@YAHPADIPBDAAPAD@Z 004176ab f   safe_string:safe_string.obj
 0001:000166e0       __unwindfunclet$?strcpy_s@cf@@YAHPADIPBD@Z$0 004176e0 f   safe_string:safe_string.obj
 0001:000166eb       __unwindfunclet$?strcpy_s@cf@@YAHPADIPBD@Z$1 004176eb f   safe_string:safe_string.obj
 0001:000166f3       __unwindfunclet$?strcpy_s@cf@@YAHPADIPBD@Z$2 004176f3 f   safe_string:safe_string.obj
 0001:000166fb       __ehhandler$?strcpy_s@cf@@YAHPADIPBD@Z 004176fb f   safe_string:safe_string.obj
 0001:00016730       __unwindfunclet$?strncpy_s@cf@@YAHPADIPBDI@Z$0 00417730 f   safe_string:safe_string.obj
 0001:0001673b       __unwindfunclet$?strncpy_s@cf@@YAHPADIPBDI@Z$1 0041773b f   safe_string:safe_string.obj
 0001:00016743       __unwindfunclet$?strncpy_s@cf@@YAHPADIPBDI@Z$2 00417743 f   safe_string:safe_string.obj
 0001:0001674b       __ehhandler$?strncpy_s@cf@@YAHPADIPBDI@Z 0041774b f   safe_string:safe_string.obj
 0001:00016780       __unwindfunclet$?str@?$basic_stringstream@DU?$char_traits@D@std@@V?$allocator@D@2@@std@@QBE?AV?$basic_string@DU?$char_traits@D@std@@V?$allocator@D@2@@2@XZ$1 00417780 f   safe_string:safe_string.obj
 0001:00016799       __ehhandler$?str@?$basic_stringstream@DU?$char_traits@D@std@@V?$allocator@D@2@@std@@QBE?AV?$basic_string@DU?$char_traits@D@std@@V?$allocator@D@2@@2@XZ 00417799 f   safe_string:safe_string.obj
 0001:000167c0       __unwindfunclet$??0?$basic_stringstream@DU?$char_traits@D@std@@V?$allocator@D@2@@std@@QAE@H@Z$0 004177c0 f   safe_string:safe_string.obj
 0001:000167dd       __unwindfunclet$??0?$basic_stringstream@DU?$char_traits@D@std@@V?$allocator@D@2@@std@@QAE@H@Z$1 004177dd f   safe_string:safe_string.obj
 0001:000167e9       __ehhandler$??0?$basic_stringstream@DU?$char_traits@D@std@@V?$allocator@D@2@@std@@QAE@H@Z 004177e9 f   safe_string:safe_string.obj
 0001:00016810       __ehhandler$??1sentry@?$basic_ostream@DU?$char_traits@D@std@@@std@@QAE@XZ 00417810 f   safe_string:safe_string.obj
 0001:00016830       __ehhandler$??1_Sentry_base@?$basic_ostream@DU?$char_traits@D@std@@@std@@QAE@XZ 00417830 f   safe_string:safe_string.obj
 0001:00016850       __unwindfunclet$??$?6U?$char_traits@D@std@@@std@@YAAAV?$basic_ostream@DU?$char_traits@D@std@@@0@AAV10@PBD@Z$3 00417850 f   safe_string:safe_string.obj
 0001:00016858       __unwindfunclet$??$?6U?$char_traits@D@std@@@std@@YAAAV?$basic_ostream@DU?$char_traits@D@std@@@0@AAV10@PBD@Z$2 00417858 f   safe_string:safe_string.obj
 0001:00016860       __ehhandler$??$?6U?$char_traits@D@std@@@std@@YAAAV?$basic_ostream@DU?$char_traits@D@std@@@0@AAV10@PBD@Z 00417860 f   safe_string:safe_string.obj
 0001:00016880       __unwindfunclet$??0CInterfaceDatabase@@QAE@XZ$0 00417880 f   ltmodule.obj
 0001:0001688b       __unwindfunclet$??0CInterfaceDatabase@@QAE@XZ$1 0041788b f   ltmodule.obj
 0001:0001689a       __ehhandler$??0CInterfaceDatabase@@QAE@XZ 0041789a f   ltmodule.obj
 0001:000168c0       __unwindfunclet$??0CInterfaceNameMgr@@QAE@PBDH@Z$0 004178c0 f   ltmodule.obj
 0001:000168cf       __unwindfunclet$??0CInterfaceNameMgr@@QAE@PBDH@Z$1 004178cf f   ltmodule.obj
 0001:000168de       __unwindfunclet$??0CInterfaceNameMgr@@QAE@PBDH@Z$2 004178de f   ltmodule.obj
 0001:000168ed       __ehhandler$??0CInterfaceNameMgr@@QAE@PBDH@Z 004178ed f   ltmodule.obj
 0001:00016910       __unwindfunclet$?Add@CInterfaceDatabase@@EAEXPAVCInterfaceChooser@@@Z$0 00417910 f   ltmodule.obj
 0001:00016910       __unwindfunclet$?Add@CInterfaceDatabase@@EAEXPAVCAPIHolderBase@@@Z$0 00417910 f   ltmodule.obj
 0001:0001691f       __ehhandler$?Add@CInterfaceDatabase@@EAEXPAVCAPIHolderBase@@@Z 0041791f f   ltmodule.obj
 0001:0001691f       __ehhandler$?Add@CInterfaceDatabase@@EAEXPAVCInterfaceChooser@@@Z 0041791f f   ltmodule.obj
 0001:00016940       __unwindfunclet$?Add@CInterfaceDatabase@@EAEXPAVIBase@@PBDH@Z$0 00417940 f   ltmodule.obj
 0001:0001694f       __ehhandler$?Add@CInterfaceDatabase@@EAEXPAVIBase@@PBDH@Z 0041794f f   ltmodule.obj
 0001:00016970       __unwindfunclet$?GetMasterDatabase@@YAPAVCInterfaceDatabase@@XZ$0 00417970 f   ltmodule.obj
 0001:00016970       __unwindfunclet$?AddHolder@CInterfaceDatabase@@SAXPAVCAPIHolderBase@@@Z$0 00417970 f   ltmodule.obj
 0001:00016970       __unwindfunclet$?AddAPI@CInterfaceDatabase@@SAXPAVIBase@@PBDH@Z$0 00417970 f   ltmodule.obj
 0001:00016970       __unwindfunclet$?AddChooser@CInterfaceDatabase@@SAXPAVCInterfaceChooser@@@Z$0 00417970 f   ltmodule.obj
 0001:0001697f       __ehhandler$?GetMasterDatabase@@YAPAVCInterfaceDatabase@@XZ 0041797f f   ltmodule.obj
 0001:0001697f       __ehhandler$?AddChooser@CInterfaceDatabase@@SAXPAVCInterfaceChooser@@@Z 0041797f f   ltmodule.obj
 0001:0001697f       __ehhandler$?AddHolder@CInterfaceDatabase@@SAXPAVCAPIHolderBase@@@Z 0041797f f   ltmodule.obj
 0001:0001697f       __ehhandler$?AddAPI@CInterfaceDatabase@@SAXPAVIBase@@PBDH@Z 0041797f f   ltmodule.obj
 0001:000169a0       __unwindfunclet$?TransferFrom@CInterfaceDatabase@@UAEXPAV1@@Z$0 004179a0 f   ltmodule.obj
 0001:000169af       __ehhandler$?TransferFrom@CInterfaceDatabase@@UAEXPAV1@@Z 004179af f   ltmodule.obj
 0001:000169d0       __unwindfunclet$?LogPacket@CHLogger@@SAXPBDZZ$0 004179d0 f   HostLogger.obj
 0001:000169db       __ehhandler$?LogPacket@CHLogger@@SAXPBDZZ 004179db f   HostLogger.obj
 0001:00016a10       __unwindfunclet$?_BuildDirectory@CHLogger@@CAXABU_SYSTEMTIME@@@Z$0 00417a10 f   HostLogger.obj
 0001:00016a1b       __unwindfunclet$?_BuildDirectory@CHLogger@@CAXABU_SYSTEMTIME@@@Z$1 00417a1b f   HostLogger.obj
 0001:00016a26       __unwindfunclet$?_BuildDirectory@CHLogger@@CAXABU_SYSTEMTIME@@@Z$2 00417a26 f   HostLogger.obj
 0001:00016a31       __ehhandler$?_BuildDirectory@CHLogger@@CAXABU_SYSTEMTIME@@@Z 00417a31 f   HostLogger.obj
 0001:00016a60       __unwindfunclet$?_DoLogWithLevel@CHLogger@@CAXPBDW4ELOG_LEVEL@1@0PAD@Z$0 00417a60 f   HostLogger.obj
 0001:00016a6b       __ehhandler$?_DoLogWithLevel@CHLogger@@CAXPBDW4ELOG_LEVEL@1@0PAD@Z 00417a6b f   HostLogger.obj
 0001:00016aa0       __unwindfunclet$?Init@CLogMsgManager@@SA_NW4ESHARED_MEM_USAGE_TYPE@1@@Z$1 00417aa0 f   LogMsgManager.obj
 0001:00016aaf       __unwindfunclet$?Init@CLogMsgManager@@SA_NW4ESHARED_MEM_USAGE_TYPE@1@@Z$0 00417aaf f   LogMsgManager.obj
 0001:00016abe       __ehhandler$?Init@CLogMsgManager@@SA_NW4ESHARED_MEM_USAGE_TYPE@1@@Z 00417abe f   LogMsgManager.obj
 0001:00016ae0       __unwindfunclet$?_WriteXlsDataToSharedMemory@CLogMsgManager@@CA_NXZ$0 00417ae0 f   LogMsgManager.obj
 0001:00016ae8       __ehhandler$?_WriteXlsDataToSharedMemory@CLogMsgManager@@CA_NXZ 00417ae8 f   LogMsgManager.obj
 0001:00016b10       __ehhandler$??$_Insert_hint@AAU?$pair@$$CB_JV?$basic_string@DU?$char_traits@D@std@@V?$allocator@D@2@@std@@@std@@PAU?$_Tree_node@U?$pair@$$CB_JV?$basic_string@DU?$char_traits@D@std@@V?$allocator@D@2@@std@@@std@@PAX@2@@?$_Tree@V?$_Tmap_traits@_JV?$basic_string@DU?$char_traits@D@std@@V?$allocator@D@2@@std@@U?$less@_J@2@V?$allocator@U?$pair@$$CB_JV?$basic_string@DU?$char_traits@D@std@@V?$allocator@D@2@@std@@@std@@@2@$0A@@std@@@std@@IAE?AV?$_Tree_iterator@V?$_Tree_val@U?$_Tree_simple_types@U?$pair@$$CB_JV?$basic_string@DU?$char_traits@D@std@@V?$allocator@D@2@@std@@@std@@@std@@@std@@@1@V?$_Tree_const_iterator@V?$_Tree_val@U?$_Tree_simple_types@U?$pair@$$CB_JV?$basic_string@DU?$char_traits@D@std@@V?$allocator@D@2@@std@@@std@@@std@@@std@@@1@AAU?$pair@$$CB_JV?$basic_string@DU?$char_traits@D@std@@V?$allocator@D@2@@std@@@1@PAU?$_Tree_node@U?$pair@$$CB_JV?$basic_string@DU?$char_traits@D@std@@V?$allocator@D@2@@std@@@std@@PAX@1@@Z 00417b10 f   LoadXlsMsg.obj
 0001:00016b30       __ehhandler$??$_Insert_nohint@AAU?$pair@$$CB_JV?$basic_string@DU?$char_traits@D@std@@V?$allocator@D@2@@std@@@std@@PAU?$_Tree_node@U?$pair@$$CB_JV?$basic_string@DU?$char_traits@D@std@@V?$allocator@D@2@@std@@@std@@PAX@2@@?$_Tree@V?$_Tmap_traits@_JV?$basic_string@DU?$char_traits@D@std@@V?$allocator@D@2@@std@@U?$less@_J@2@V?$allocator@U?$pair@$$CB_JV?$basic_string@DU?$char_traits@D@std@@V?$allocator@D@2@@std@@@std@@@2@$0A@@std@@@std@@IAE?AU?$pair@V?$_Tree_iterator@V?$_Tree_val@U?$_Tree_simple_types@U?$pair@$$CB_JV?$basic_string@DU?$char_traits@D@std@@V?$allocator@D@2@@std@@@std@@@std@@@std@@@std@@_N@1@_NAAU?$pair@$$CB_JV?$basic_string@DU?$char_traits@D@std@@V?$allocator@D@2@@std@@@1@PAU?$_Tree_node@U?$pair@$$CB_JV?$basic_string@DU?$char_traits@D@std@@V?$allocator@D@2@@std@@@std@@PAX@1@@Z 00417b30 f   LoadXlsMsg.obj
 0001:00016b50       __ehhandler$??1FindXlsMsg@@UAE@XZ 00417b50 f   LoadXlsMsg.obj
 0001:00016b70       __unwindfunclet$?LoadWMszFile@FindXlsMsg@@QAE_NPAD@Z$0 00417b70 f   LoadXlsMsg.obj
 0001:00016b7b       __ehhandler$?LoadWMszFile@FindXlsMsg@@QAE_NPAD@Z 00417b7b f   LoadXlsMsg.obj
 0001:00016bb0       __unwindfunclet$?Run@CServerAppApp@@UAEHXZ$0 00417bb0 f   ServerApp.obj
 0001:00016bbb       __ehhandler$?Run@CServerAppApp@@UAEHXZ 00417bbb f   ServerApp.obj
 0001:00016bf0       __unwindfunclet$??$?HDU?$char_traits@D@std@@V?$allocator@D@1@@std@@YA?AV?$basic_string@DU?$char_traits@D@std@@V?$allocator@D@2@@0@ABV10@0@Z$0 00417bf0 f   ServerAppDlg.obj
 0001:00016c09       __ehhandler$??$?HDU?$char_traits@D@std@@V?$allocator@D@1@@std@@YA?AV?$basic_string@DU?$char_traits@D@std@@V?$allocator@D@2@@0@ABV10@0@Z 00417c09 f   ServerAppDlg.obj
 0001:00016c30       __unwindfunclet$??0?$CAPIHolder@VILTCommon@@@@QAE@PBDAAPAVILTCommon@@H@Z$0 00417c30 f   ServerAppDlg.obj
 0001:00016c38       __ehhandler$??0?$CAPIHolder@VILTCommon@@@@QAE@PBDAAPAVILTCommon@@H@Z 00417c38 f   ServerAppDlg.obj
 0001:00016c60       __unwindfunclet$??0CServerAppDlg@@QAE@PAVCWnd@@@Z$0 00417c60 f   ServerAppDlg.obj
 0001:00016c68       __unwindfunclet$??0CServerAppDlg@@QAE@PAVCWnd@@@Z$1 00417c68 f   ServerAppDlg.obj
 0001:00016c77       __unwindfunclet$??0CServerAppDlg@@QAE@PAVCWnd@@@Z$2 00417c77 f   ServerAppDlg.obj
 0001:00016c85       __unwindfunclet$??0CServerAppDlg@@QAE@PAVCWnd@@@Z$3 00417c85 f   ServerAppDlg.obj
 0001:00016c93       __unwindfunclet$??0CServerAppDlg@@QAE@PAVCWnd@@@Z$4 00417c93 f   ServerAppDlg.obj
 0001:00016ca1       __unwindfunclet$??0CServerAppDlg@@QAE@PAVCWnd@@@Z$5 00417ca1 f   ServerAppDlg.obj
 0001:00016caf       __ehhandler$??0CServerAppDlg@@QAE@PAVCWnd@@@Z 00417caf f   ServerAppDlg.obj
 0001:00016cd0       __ehhandler$??1?$CAPIHolder@VILTCommon@@@@UAE@XZ 00417cd0 f   ServerAppDlg.obj
 0001:00016cd0       __ehhandler$??1CServerAppDlg@@UAE@XZ 00417cd0 f   ServerAppDlg.obj
 0001:00016cf0       __unwindfunclet$??1CWaitCursor@@QAE@XZ$2 00417cf0 f   ServerAppDlg.obj
 0001:00016cfc       __ehhandler$??1CWaitCursor@@QAE@XZ 00417cfc f   ServerAppDlg.obj
 0001:00016d30       __unwindfunclet$?AddResources@CServerAppDlg@@QAE_NXZ$0 00417d30 f   ServerAppDlg.obj
 0001:00016d3b       __unwindfunclet$?AddResources@CServerAppDlg@@QAE_NXZ$1 00417d3b f   ServerAppDlg.obj
 0001:00016d46       __unwindfunclet$?AddResources@CServerAppDlg@@QAE_NXZ$2 00417d46 f   ServerAppDlg.obj
 0001:00016d52       __unwindfunclet$?AddResources@CServerAppDlg@@QAE_NXZ$3 00417d52 f   ServerAppDlg.obj
 0001:00016d5e       __unwindfunclet$?AddResources@CServerAppDlg@@QAE_NXZ$4 00417d5e f   ServerAppDlg.obj
 0001:00016d69       __unwindfunclet$?AddResources@CServerAppDlg@@QAE_NXZ$5 00417d69 f   ServerAppDlg.obj
 0001:00016d75       __unwindfunclet$?AddResources@CServerAppDlg@@QAE_NXZ$6 00417d75 f   ServerAppDlg.obj
 0001:00016d81       __unwindfunclet$?AddResources@CServerAppDlg@@QAE_NXZ$7 00417d81 f   ServerAppDlg.obj
 0001:00016d8d       __ehhandler$?AddResources@CServerAppDlg@@QAE_NXZ 00417d8d f   ServerAppDlg.obj
 0001:00016dc0       __unwindfunclet$?AddServerMsg@CServerAppDlg@@QAEXPBDH@Z$0 00417dc0 f   ServerAppDlg.obj
 0001:00016dc8       __ehhandler$?AddServerMsg@CServerAppDlg@@QAEXPBDH@Z 00417dc8 f   ServerAppDlg.obj
 0001:00016df0       __unwindfunclet$?ConsoleOutputFn@CGameServerAppHandler@@UAEIHHPBD@Z$0 00417df0 f   ServerAppDlg.obj
 0001:00016dfb       __ehhandler$?ConsoleOutputFn@CGameServerAppHandler@@UAEIHHPBD@Z 00417dfb f   ServerAppDlg.obj
 0001:00016e30       __unwindfunclet$?DoHost@CServerAppDlg@@QAE_NXZ$0 00417e30 f   ServerAppDlg.obj
 0001:00016e3b       __ehhandler$?DoHost@CServerAppDlg@@QAE_NXZ 00417e3b f   ServerAppDlg.obj
 0001:00016e70       __unwindfunclet$?DownloadUCCMapFile_HTTP@CServerAppDlg@@AAE?AW4UCCMAPDOWNLOADREAULT@@V?$basic_string@DU?$char_traits@D@std@@V?$allocator@D@2@@std@@@Z$0 00417e70 f   ServerAppDlg.obj
 0001:00016e78       __unwindfunclet$?DownloadUCCMapFile_HTTP@CServerAppDlg@@AAE?AW4UCCMAPDOWNLOADREAULT@@V?$basic_string@DU?$char_traits@D@std@@V?$allocator@D@2@@std@@@Z$1 00417e78 f   ServerAppDlg.obj
 0001:00016e83       __unwindfunclet$?DownloadUCCMapFile_HTTP@CServerAppDlg@@AAE?AW4UCCMAPDOWNLOADREAULT@@V?$basic_string@DU?$char_traits@D@std@@V?$allocator@D@2@@std@@@Z$2 00417e83 f   ServerAppDlg.obj
 0001:00016e8e       __unwindfunclet$?DownloadUCCMapFile_HTTP@CServerAppDlg@@AAE?AW4UCCMAPDOWNLOADREAULT@@V?$basic_string@DU?$char_traits@D@std@@V?$allocator@D@2@@std@@@Z$4 00417e8e f   ServerAppDlg.obj
 0001:00016e99       __unwindfunclet$?DownloadUCCMapFile_HTTP@CServerAppDlg@@AAE?AW4UCCMAPDOWNLOADREAULT@@V?$basic_string@DU?$char_traits@D@std@@V?$allocator@D@2@@std@@@Z$14 00417e99 f   ServerAppDlg.obj
 0001:00016ebb       __unwindfunclet$?DownloadUCCMapFile_HTTP@CServerAppDlg@@AAE?AW4UCCMAPDOWNLOADREAULT@@V?$basic_string@DU?$char_traits@D@std@@V?$allocator@D@2@@std@@@Z$6 00417ebb f   ServerAppDlg.obj
 0001:00016ec6       __unwindfunclet$?DownloadUCCMapFile_HTTP@CServerAppDlg@@AAE?AW4UCCMAPDOWNLOADREAULT@@V?$basic_string@DU?$char_traits@D@std@@V?$allocator@D@2@@std@@@Z$7 00417ec6 f   ServerAppDlg.obj
 0001:00016ed1       __unwindfunclet$?DownloadUCCMapFile_HTTP@CServerAppDlg@@AAE?AW4UCCMAPDOWNLOADREAULT@@V?$basic_string@DU?$char_traits@D@std@@V?$allocator@D@2@@std@@@Z$8 00417ed1 f   ServerAppDlg.obj
 0001:00016edc       __ehhandler$?DownloadUCCMapFile_HTTP@CServerAppDlg@@AAE?AW4UCCMAPDOWNLOADREAULT@@V?$basic_string@DU?$char_traits@D@std@@V?$allocator@D@2@@std@@@Z 00417edc f   ServerAppDlg.obj
 0001:00016f10       __unwindfunclet$?GetDownloadPath@CServerAppDlg@@AAE?AV?$basic_string@DU?$char_traits@D@std@@V?$allocator@D@2@@std@@XZ$0 00417f10 f   ServerAppDlg.obj
 0001:00016f32       __ehhandler$?GetDownloadPath@CServerAppDlg@@AAE?AV?$basic_string@DU?$char_traits@D@std@@V?$allocator@D@2@@std@@XZ 00417f32 f   ServerAppDlg.obj
 0001:00016f60       __unwindfunclet$?GetOptionValueString@CServerAppDlg@@IAE?AV?$basic_string@DU?$char_traits@D@std@@V?$allocator@D@2@@std@@V23@00@Z$0 00417f60 f   ServerAppDlg.obj
 0001:00016f68       __unwindfunclet$?GetOptionValueString@CServerAppDlg@@IAE?AV?$basic_string@DU?$char_traits@D@std@@V?$allocator@D@2@@std@@V23@00@Z$1 00417f68 f   ServerAppDlg.obj
 0001:00016f70       __unwindfunclet$?GetOptionValueString@CServerAppDlg@@IAE?AV?$basic_string@DU?$char_traits@D@std@@V?$allocator@D@2@@std@@V23@00@Z$2 00417f70 f   ServerAppDlg.obj
 0001:00016f78       __unwindfunclet$?GetOptionValueString@CServerAppDlg@@IAE?AV?$basic_string@DU?$char_traits@D@std@@V?$allocator@D@2@@std@@V23@00@Z$3 00417f78 f   ServerAppDlg.obj
 0001:00016f80       __ehhandler$?GetOptionValueString@CServerAppDlg@@IAE?AV?$basic_string@DU?$char_traits@D@std@@V?$allocator@D@2@@std@@V23@00@Z 00417f80 f   ServerAppDlg.obj
 0001:00016fb0       __unwindfunclet$?LoadHostGameInfo@CServerAppDlg@@IAEXXZ$0 00417fb0 f   ServerAppDlg.obj
 0001:00016fb8       __unwindfunclet$?LoadHostGameInfo@CServerAppDlg@@IAEXXZ$1 00417fb8 f   ServerAppDlg.obj
 0001:00016fc3       __unwindfunclet$?LoadHostGameInfo@CServerAppDlg@@IAEXXZ$2 00417fc3 f   ServerAppDlg.obj
 0001:00016fce       __ehhandler$?LoadHostGameInfo@CServerAppDlg@@IAEXXZ 00417fce f   ServerAppDlg.obj
 0001:00017000       __unwindfunclet$?LoadServer@CServerAppDlg@@QAE_NXZ$0 00418000 f   ServerAppDlg.obj
 0001:00017008       __unwindfunclet$?LoadServer@CServerAppDlg@@QAE_NXZ$1 00418008 f   ServerAppDlg.obj
 0001:00017011       __unwindfunclet$?LoadServer@CServerAppDlg@@QAE_NXZ$2 00418011 f   ServerAppDlg.obj
 0001:0001701a       __unwindfunclet$?LoadServer@CServerAppDlg@@QAE_NXZ$3 0041801a f   ServerAppDlg.obj
 0001:00017023       __unwindfunclet$?LoadServer@CServerAppDlg@@QAE_NXZ$4 00418023 f   ServerAppDlg.obj
 0001:0001702b       __unwindfunclet$?LoadServer@CServerAppDlg@@QAE_NXZ$5 0041802b f   ServerAppDlg.obj
 0001:00017033       __ehhandler$?LoadServer@CServerAppDlg@@QAE_NXZ 00418033 f   ServerAppDlg.obj
 0001:00017060       __unwindfunclet$?OnButtonStartServer@CServerAppDlg@@QAEHXZ$0 00418060 f   ServerAppDlg.obj
 0001:00017068       __unwindfunclet$?OnButtonStartServer@CServerAppDlg@@QAEHXZ$1 00418068 f   ServerAppDlg.obj
 0001:00017070       __ehhandler$?OnButtonStartServer@CServerAppDlg@@QAEHXZ 00418070 f   ServerAppDlg.obj
 0001:000170a0       __unwindfunclet$?OnCopyData@CServerAppDlg@@IAEHPAVCWnd@@PAUtagCOPYDATASTRUCT@@@Z$0 004180a0 f   ServerAppDlg.obj
 0001:000170ab       __unwindfunclet$?OnCopyData@CServerAppDlg@@IAEHPAVCWnd@@PAUtagCOPYDATASTRUCT@@@Z$1 004180ab f   ServerAppDlg.obj
 0001:000170b6       __unwindfunclet$?OnCopyData@CServerAppDlg@@IAEHPAVCWnd@@PAUtagCOPYDATASTRUCT@@@Z$2 004180b6 f   ServerAppDlg.obj
 0001:000170be       __unwindfunclet$?OnCopyData@CServerAppDlg@@IAEHPAVCWnd@@PAUtagCOPYDATASTRUCT@@@Z$3 004180be f   ServerAppDlg.obj
 0001:000170c6       __unwindfunclet$?OnCopyData@CServerAppDlg@@IAEHPAVCWnd@@PAUtagCOPYDATASTRUCT@@@Z$4 004180c6 f   ServerAppDlg.obj
 0001:000170d2       __unwindfunclet$?OnCopyData@CServerAppDlg@@IAEHPAVCWnd@@PAUtagCOPYDATASTRUCT@@@Z$5 004180d2 f   ServerAppDlg.obj
 0001:000170da       __unwindfunclet$?OnCopyData@CServerAppDlg@@IAEHPAVCWnd@@PAUtagCOPYDATASTRUCT@@@Z$6 004180da f   ServerAppDlg.obj
 0001:000170e5       __unwindfunclet$?OnCopyData@CServerAppDlg@@IAEHPAVCWnd@@PAUtagCOPYDATASTRUCT@@@Z$7 004180e5 f   ServerAppDlg.obj
 0001:000170ed       __ehhandler$?OnCopyData@CServerAppDlg@@IAEHPAVCWnd@@PAUtagCOPYDATASTRUCT@@@Z 004180ed f   ServerAppDlg.obj
 0001:00017120       __unwindfunclet$?OnGameServerMsg@CServerAppDlg@@IAEJIJ@Z$0 00418120 f   ServerAppDlg.obj
 0001:00017128       __unwindfunclet$?OnGameServerMsg@CServerAppDlg@@IAEJIJ@Z$1 00418128 f   ServerAppDlg.obj
 0001:00017130       __unwindfunclet$?OnGameServerMsg@CServerAppDlg@@IAEJIJ@Z$2 00418130 f   ServerAppDlg.obj
 0001:00017138       __ehhandler$?OnGameServerMsg@CServerAppDlg@@IAEJIJ@Z 00418138 f   ServerAppDlg.obj
 0001:00017160       __unwindfunclet$?OnInitDialog@CServerAppDlg@@MAEHXZ$0 00418160 f   ServerAppDlg.obj
 0001:0001716b       __unwindfunclet$?OnInitDialog@CServerAppDlg@@MAEHXZ$1 0041816b f   ServerAppDlg.obj
 0001:00017177       __unwindfunclet$?OnInitDialog@CServerAppDlg@@MAEHXZ$2 00418177 f   ServerAppDlg.obj
 0001:00017182       __unwindfunclet$?OnInitDialog@CServerAppDlg@@MAEHXZ$3 00418182 f   ServerAppDlg.obj
 0001:0001718e       __unwindfunclet$?OnInitDialog@CServerAppDlg@@MAEHXZ$4 0041818e f   ServerAppDlg.obj
 0001:00017199       __unwindfunclet$?OnInitDialog@CServerAppDlg@@MAEHXZ$5 00418199 f   ServerAppDlg.obj
 0001:000171a4       __ehhandler$?OnInitDialog@CServerAppDlg@@MAEHXZ 004181a4 f   ServerAppDlg.obj
 0001:000171d0       __unwindfunclet$?OnShellMessage@CServerAppDlg@@QAEXAAVILTMessage_Read@@@Z$0 004181d0 f   ServerAppDlg.obj
 0001:000171d8       __unwindfunclet$?OnShellMessage@CServerAppDlg@@QAEXAAVILTMessage_Read@@@Z$1 004181d8 f   ServerAppDlg.obj
 0001:000171e0       __unwindfunclet$?OnShellMessage@CServerAppDlg@@QAEXAAVILTMessage_Read@@@Z$3 004181e0 f   ServerAppDlg.obj
 0001:000171e8       __unwindfunclet$?OnShellMessage@CServerAppDlg@@QAEXAAVILTMessage_Read@@@Z$4 004181e8 f   ServerAppDlg.obj
 0001:000171f0       __unwindfunclet$?OnShellMessage@CServerAppDlg@@QAEXAAVILTMessage_Read@@@Z$5 004181f0 f   ServerAppDlg.obj
 0001:000171f8       __unwindfunclet$?OnShellMessage@CServerAppDlg@@QAEXAAVILTMessage_Read@@@Z$6 004181f8 f   ServerAppDlg.obj
 0001:00017200       __unwindfunclet$?OnShellMessage@CServerAppDlg@@QAEXAAVILTMessage_Read@@@Z$7 00418200 f   ServerAppDlg.obj
 0001:0001720b       __ehhandler$?OnShellMessage@CServerAppDlg@@QAEXAAVILTMessage_Read@@@Z 0041820b f   ServerAppDlg.obj
 0001:00017240       __unwindfunclet$?OnTimer@CServerAppDlg@@QAEXI@Z$0 00418240 f   ServerAppDlg.obj
 0001:0001724b       __ehhandler$?OnTimer@CServerAppDlg@@QAEXI@Z 0041824b f   ServerAppDlg.obj
 0001:00017280       __unwindfunclet$?OutOfMemory@CGameServerAppHandler@@UAEIXZ$0 00418280 f   ServerAppDlg.obj
 0001:00017288       __ehhandler$?OutOfMemory@CGameServerAppHandler@@UAEIXZ 00418288 f   ServerAppDlg.obj
 0001:000172b0       __unwindfunclet$?RECV_MSG_AIITEM_DEC@CServerAppDlg@@AAEXJ@Z$1 004182b0 f   ServerAppDlg.obj
 0001:000172b8       __ehhandler$?RECV_MSG_AIITEM_DEC@CServerAppDlg@@AAEXJ@Z 004182b8 f   ServerAppDlg.obj
 0001:000172e0       __unwindfunclet$?SendServerAppInit@CServerAppDlg@@AAEXXZ$0 004182e0 f   ServerAppDlg.obj
 0001:000172e0       __unwindfunclet$?RECV_MSG_AIITEM_GROUP_RATE_RESULT@CServerAppDlg@@AAEXJ@Z$1 004182e0 f   ServerAppDlg.obj
 0001:000172e8       __ehhandler$?SendServerAppInit@CServerAppDlg@@AAEXXZ 004182e8 f   ServerAppDlg.obj
 0001:000172e8       __ehhandler$?RECV_MSG_AIITEM_GROUP_RATE_RESULT@CServerAppDlg@@AAEXJ@Z 004182e8 f   ServerAppDlg.obj
 0001:00017310       __unwindfunclet$?RECV_MSG_INSERTCHARACTER@CServerAppDlg@@AAEXJ@Z$1 00418310 f   ServerAppDlg.obj
 0001:00017318       __unwindfunclet$?RECV_MSG_INSERTCHARACTER@CServerAppDlg@@AAEXJ@Z$2 00418318 f   ServerAppDlg.obj
 0001:00017320       __ehhandler$?RECV_MSG_INSERTCHARACTER@CServerAppDlg@@AAEXJ@Z 00418320 f   ServerAppDlg.obj
 0001:00017350       __unwindfunclet$?RECV_MSG_USER_DISCONNECTED@CServerAppDlg@@AAEXJ@Z$0 00418350 f   ServerAppDlg.obj
 0001:00017358       __ehhandler$?RECV_MSG_USER_DISCONNECTED@CServerAppDlg@@AAEXJ@Z 00418358 f   ServerAppDlg.obj
 0001:00017380       __unwindfunclet$?RTIDUSNtoString@EXPAND_USN@@YA?AV?$basic_string@DU?$char_traits@D@std@@V?$allocator@D@2@@std@@HFF_J@Z$0 00418380 f   ServerAppDlg.obj
 0001:00017388       __ehhandler$?RTIDUSNtoString@EXPAND_USN@@YA?AV?$basic_string@DU?$char_traits@D@std@@V?$allocator@D@2@@std@@HFF_J@Z 00418388 f   ServerAppDlg.obj
 0001:000173b0       __unwindfunclet$?RunServer@CServerAppDlg@@QAE_NXZ$0 004183b0 f   ServerAppDlg.obj
 0001:000173b8       __unwindfunclet$?RunServer@CServerAppDlg@@QAE_NXZ$1 004183b8 f   ServerAppDlg.obj
 0001:000173c0       __unwindfunclet$?RunServer@CServerAppDlg@@QAE_NXZ$2 004183c0 f   ServerAppDlg.obj
 0001:000173c8       __unwindfunclet$?RunServer@CServerAppDlg@@QAE_NXZ$3 004183c8 f   ServerAppDlg.obj
 0001:000173d0       __ehhandler$?RunServer@CServerAppDlg@@QAE_NXZ 004183d0 f   ServerAppDlg.obj
 0001:00017400       __unwindfunclet$?SaveHostGameInfo@CServerAppDlg@@IAEXXZ$0 00418400 f   ServerAppDlg.obj
 0001:00017408       __unwindfunclet$?SaveHostGameInfo@CServerAppDlg@@IAEXXZ$1 00418408 f   ServerAppDlg.obj
 0001:00017410       __unwindfunclet$?SaveHostGameInfo@CServerAppDlg@@IAEXXZ$2 00418410 f   ServerAppDlg.obj
 0001:00017418       __ehhandler$?SaveHostGameInfo@CServerAppDlg@@IAEXXZ 00418418 f   ServerAppDlg.obj
 0001:00017440       __unwindfunclet$?SendServerAppInitFail@CServerAppDlg@@AAEXHH@Z$0 00418440 f   ServerAppDlg.obj
 0001:00017449       __unwindfunclet$?SendServerAppInitFail@CServerAppDlg@@AAEXHH@Z$1 00418449 f   ServerAppDlg.obj
 0001:00017451       __ehhandler$?SendServerAppInitFail@CServerAppDlg@@AAEXHH@Z 00418451 f   ServerAppDlg.obj
 0001:00017480       __unwindfunclet$?ServerUpdate@CServerAppDlg@@QAEXXZ$0 00418480 f   ServerAppDlg.obj
 0001:0001748b       __ehhandler$?ServerUpdate@CServerAppDlg@@QAEXXZ 0041848b f   ServerAppDlg.obj
 0001:000174c0       __unwindfunclet$?StopServer@CServerAppDlg@@QAE_NXZ$0 004184c0 f   ServerAppDlg.obj
 0001:000174c8       __ehhandler$?StopServer@CServerAppDlg@@QAE_NXZ 004184c8 f   ServerAppDlg.obj
 0001:000174f0       __unwindfunclet$?ThreadUpdate@CServerAppDlg@@SAXPAX@Z$0 004184f0 f   ServerAppDlg.obj
 0001:000174f8       __unwindfunclet$?ThreadUpdate@CServerAppDlg@@SAXPAX@Z$1 004184f8 f   ServerAppDlg.obj
 0001:00017500       __ehhandler$?ThreadUpdate@CServerAppDlg@@SAXPAX@Z 00418500 f   ServerAppDlg.obj
 0001:00017530       __unwindfunclet$?Thread_SendGameInfo@@YAXPAVCServerAppDlg@@AAUPROTO_START_HOST_tag@@@Z$0 00418530 f   ServerAppDlg.obj
 0001:00017538       __unwindfunclet$?Thread_SendGameInfo@@YAXPAVCServerAppDlg@@AAUPROTO_START_HOST_tag@@@Z$1 00418538 f   ServerAppDlg.obj
 0001:00017540       __unwindfunclet$?Thread_SendGameInfo@@YAXPAVCServerAppDlg@@AAUPROTO_START_HOST_tag@@@Z$2 00418540 f   ServerAppDlg.obj
 0001:00017548       __unwindfunclet$?Thread_SendGameInfo@@YAXPAVCServerAppDlg@@AAUPROTO_START_HOST_tag@@@Z$3 00418548 f   ServerAppDlg.obj
 0001:00017550       __unwindfunclet$?Thread_SendGameInfo@@YAXPAVCServerAppDlg@@AAUPROTO_START_HOST_tag@@@Z$4 00418550 f   ServerAppDlg.obj
 0001:00017558       __unwindfunclet$?Thread_SendGameInfo@@YAXPAVCServerAppDlg@@AAUPROTO_START_HOST_tag@@@Z$5 00418558 f   ServerAppDlg.obj
 0001:00017560       __unwindfunclet$?Thread_SendGameInfo@@YAXPAVCServerAppDlg@@AAUPROTO_START_HOST_tag@@@Z$6 00418560 f   ServerAppDlg.obj
 0001:00017568       __ehhandler$?Thread_SendGameInfo@@YAXPAVCServerAppDlg@@AAUPROTO_START_HOST_tag@@@Z 00418568 f   ServerAppDlg.obj
 0001:00017590       __unwindfunclet$?Thread_SendUserInfo@@YAXPAVCServerAppDlg@@AAUPROTO_GAME_USER_INFO_tag@@@Z$0 00418590 f   ServerAppDlg.obj
 0001:00017598       __unwindfunclet$?Thread_SendUserInfo@@YAXPAVCServerAppDlg@@AAUPROTO_GAME_USER_INFO_tag@@@Z$1 00418598 f   ServerAppDlg.obj
 0001:000175a0       __ehhandler$?Thread_SendUserInfo@@YAXPAVCServerAppDlg@@AAUPROTO_GAME_USER_INFO_tag@@@Z 004185a0 f   ServerAppDlg.obj
 0001:000175d0       __unwindfunclet$?CRSUploader@@YAAAVUploader@crs@@XZ$0 004185d0 f   BugReporter1.obj
 0001:000175de       __ehhandler$?CRSUploader@@YAAAVUploader@crs@@XZ 004185de f   BugReporter1.obj
 0001:00017600       __unwindfunclet$?threadCreateDumpFile@@YGKPAX@Z$0 00418600 f   BugReporter1.obj
 0001:0001760b       __ehhandler$?threadCreateDumpFile@@YGKPAX@Z 0041860b f   BugReporter1.obj
 0001:00017640       __unwindfunclet$??0Uploader@crs@@QAE@XZ$0 00418640 f   crs_uploader1.obj
 0001:0001764f       __unwindfunclet$??0Uploader@crs@@QAE@XZ$7 0041864f f   crs_uploader1.obj
 0001:00017657       __ehhandler$??0Uploader@crs@@QAE@XZ 00418657 f   crs_uploader1.obj
 0001:00017680       __unwindfunclet$?init@Uploader@crs@@QAE_N_NPAD1@Z$0 00418680 f   crs_uploader1.obj
 0001:0001768b       __ehhandler$?init@Uploader@crs@@QAE_N_NPAD1@Z 0041868b f   crs_uploader1.obj
 0001:000176c0       __unwindfunclet$?readURL@Uploader@crs@@AAEXAAV?$basic_string@_WU?$char_traits@_W@std@@V?$allocator@_W@2@@std@@@Z$0 004186c0 f   crs_uploader1.obj
 0001:000176cb       __unwindfunclet$?readURL@Uploader@crs@@AAEXAAV?$basic_string@_WU?$char_traits@_W@std@@V?$allocator@_W@2@@std@@@Z$1 004186cb f   crs_uploader1.obj
 0001:000176d6       __ehhandler$?readURL@Uploader@crs@@AAEXAAV?$basic_string@_WU?$char_traits@_W@std@@V?$allocator@_W@2@@std@@@Z 004186d6 f   crs_uploader1.obj
 0001:00017700       ??__F_FILE_SHUTDOWN_var_ltmod_database_@@YAXXZ 00418700 f   ltmodule.obj
 0001:00017710       ??__F?m_LogLock@CHLogger@@0VCMustSyncObjectLog@@A@@YAXXZ 00418710 f   HostLogger.obj
 0001:00017730       ??__F?m_LogPacketLock@CHLogger@@0VCMustSyncObjectLog@@A@@YAXXZ 00418730 f   HostLogger.obj
 0001:00017750       ??__F?m_strBRFileFormat@CHLogger@@0V?$basic_string@DU?$char_traits@D@std@@V?$allocator@D@2@@std@@A@@YAXXZ 00418750 f   HostLogger.obj
 0001:000177b0       ??__F?m_strEtcFileFormat@CHLogger@@0V?$basic_string@DU?$char_traits@D@std@@V?$allocator@D@2@@std@@A@@YAXXZ 004187b0 f   HostLogger.obj
 0001:00017810       ??__F?m_strFileFormat@CHLogger@@0V?$basic_string@DU?$char_traits@D@std@@V?$allocator@D@2@@std@@A@@YAXXZ 00418810 f   HostLogger.obj
 0001:00017870       ??__F?m_strHostName@CHLogger@@0V?$basic_string@DU?$char_traits@D@std@@V?$allocator@D@2@@std@@A@@YAXXZ 00418870 f   HostLogger.obj
 0001:000178d0       ??__F?m_strIPCMessageFileFormat@CHLogger@@0V?$basic_string@DU?$char_traits@D@std@@V?$allocator@D@2@@std@@A@@YAXXZ 004188d0 f   HostLogger.obj
 0001:00017930       ??__F?m_strKernelFileFormat@CHLogger@@0V?$basic_string@DU?$char_traits@D@std@@V?$allocator@D@2@@std@@A@@YAXXZ 00418930 f   HostLogger.obj
 0001:00017990       ??__F?m_strLogFolder@CHLogger@@0V?$basic_string@DU?$char_traits@D@std@@V?$allocator@D@2@@std@@A@@YAXXZ 00418990 f   HostLogger.obj
 0001:000179f0       ??__F?m_strModeUserCountFormat@CHLogger@@0V?$basic_string@DU?$char_traits@D@std@@V?$allocator@D@2@@std@@A@@YAXXZ 004189f0 f   HostLogger.obj
 0001:00017a50       ??__F?m_strPacketFileFormat@CHLogger@@0V?$basic_string@DU?$char_traits@D@std@@V?$allocator@D@2@@std@@A@@YAXXZ 00418a50 f   HostLogger.obj
 0001:00017ab0       ??__F?m_strRWProcessMemoryFileFormat@CHLogger@@0V?$basic_string@DU?$char_traits@D@std@@V?$allocator@D@2@@std@@A@@YAXXZ 00418ab0 f   HostLogger.obj
 0001:00017b10       ??__F?m_strServerAppUseCountFormat@CHLogger@@0V?$basic_string@DU?$char_traits@D@std@@V?$allocator@D@2@@std@@A@@YAXXZ 00418b10 f   HostLogger.obj
 0001:00017b70       ??__F?m_strServerName@CHLogger@@0V?$basic_string@DU?$char_traits@D@std@@V?$allocator@D@2@@std@@A@@YAXXZ 00418b70 f   HostLogger.obj
 0001:00017bd0       ??__F?m_strTimeOutFileFormat@CHLogger@@0V?$basic_string@DU?$char_traits@D@std@@V?$allocator@D@2@@std@@A@@YAXXZ 00418bd0 f   HostLogger.obj
 0001:00017c30       ??__F?m_vectSharedMapHandles@CLogMsgManager@@0V?$vector@PAXV?$allocator@PAX@std@@@std@@A@@YAXXZ 00418c30 f   LogMsgManager.obj
 0001:00017c90       ??__FtheApp@@YAXXZ         00418c90 f   ServerApp.obj
 0001:00017ca0       ??__F__api_holder_ILTCommon_Server_g_pLTSCommon__@@YAXXZ 00418ca0 f   ServerAppDlg.obj
 0001:00017cb0       ??__Fg_cServerLog@@YAXXZ   00418cb0 f   ServerAppDlg.obj
 0001:00017cc0       ??__Fcrs_uploader@?1??CRSUploader@@YAAAVUploader@crs@@XZ@YAXXZ 00418cc0 f   BugReporter1.obj
 0001:00017cca       ??__F_AtlBaseModule@ATL@@YAXXZ 00418cca f   atls:atlbase.obj
 0002:00000684       ?pre_cpp_initializer@@3P6AXXZA 00419684     msvcrt:exe_winmain.obj
 0002:00000688       ?_AtlBaseModule$initializer$@ATL@@3P6AXXZA 00419688     atls:atlbase.obj
 0002:0000068c       ?_afxInitAppState$initializer$@@3P6AXXZA 0041968c     mfcs140:appmodul.obj
 0002:00000690       ?FloatOne$initializer$@GlobalVectorConstants@@3P6AXXZA 00419690     ltmodule.obj
 0002:00000694       ?FloatZero$initializer$@GlobalVectorConstants@@3P6AXXZA 00419694     ltmodule.obj
 0002:00000698       ?FloatMinusOne$initializer$@GlobalVectorConstants@@3P6AXXZA 00419698     ltmodule.obj
 0002:0000069c       ?Float0001$initializer$@GlobalVectorConstants@@3P6AXXZA 0041969c     ltmodule.obj
 0002:000006a0       ?SmallLengthThreshold$initializer$@GlobalVectorConstants@@3P6AXXZA 004196a0     ltmodule.obj
 0002:000006a4       ?FloatOneHundredth$initializer$@GlobalVectorConstants@@3P6AXXZA 004196a4     ltmodule.obj
 0002:000006a8       ?Float111_Minus1$initializer$@GlobalVectorConstants@@3P6AXXZA 004196a8     ltmodule.obj
 0002:000006ac       ?FloatMinus1_111$initializer$@GlobalVectorConstants@@3P6AXXZA 004196ac     ltmodule.obj
 0002:000006b0       ?FloatOneHalf$initializer$@GlobalVectorConstants@@3P6AXXZA 004196b0     ltmodule.obj
 0002:000006b4       ?FloatMinusOneHalf$initializer$@GlobalVectorConstants@@3P6AXXZA 004196b4     ltmodule.obj
 0002:000006b8       ?KindaSmallNumber$initializer$@GlobalVectorConstants@@3P6AXXZA 004196b8     ltmodule.obj
 0002:000006bc       ?SmallNumber$initializer$@GlobalVectorConstants@@3P6AXXZA 004196bc     ltmodule.obj
 0002:000006c0       ?ThreshQuatNormalized$initializer$@GlobalVectorConstants@@3P6AXXZA 004196c0     ltmodule.obj
 0002:000006c4       ?BigNumber$initializer$@GlobalVectorConstants@@3P6AXXZA 004196c4     ltmodule.obj
 0002:000006c8       ?IntOne$initializer$@GlobalVectorConstants@@3P6AXXZA 004196c8     ltmodule.obj
 0002:000006cc       ?IntZero$initializer$@GlobalVectorConstants@@3P6AXXZA 004196cc     ltmodule.obj
 0002:000006d0       ?IntMinusOne$initializer$@GlobalVectorConstants@@3P6AXXZA 004196d0     ltmodule.obj
 0002:000006d4       ?QINV_SIGN_MASK$initializer$@GlobalVectorConstants@@3P6AXXZA 004196d4     ltmodule.obj
 0002:000006d8       ?QMULTI_SIGN_MASK0$initializer$@GlobalVectorConstants@@3P6AXXZA 004196d8     ltmodule.obj
 0002:000006dc       ?QMULTI_SIGN_MASK1$initializer$@GlobalVectorConstants@@3P6AXXZA 004196dc     ltmodule.obj
 0002:000006e0       ?QMULTI_SIGN_MASK2$initializer$@GlobalVectorConstants@@3P6AXXZA 004196e0     ltmodule.obj
 0002:000006e4       ?DEG_TO_RAD$initializer$@GlobalVectorConstants@@3P6AXXZA 004196e4     ltmodule.obj
 0002:000006e8       ?DEG_TO_RAD_HALF$initializer$@GlobalVectorConstants@@3P6AXXZA 004196e8     ltmodule.obj
 0002:000006ec       ?RAD_TO_DEG$initializer$@GlobalVectorConstants@@3P6AXXZA 004196ec     ltmodule.obj
 0002:000006f0       ?XYZMask$initializer$@GlobalVectorConstants@@3P6AXXZA 004196f0     ltmodule.obj
 0002:000006f4       ?SignBit$initializer$@GlobalVectorConstants@@3P6AXXZA 004196f4     ltmodule.obj
 0002:000006f8       ?SignMask$initializer$@GlobalVectorConstants@@3P6AXXZA 004196f8     ltmodule.obj
 0002:000006fc       ?IntSignBit$initializer$@GlobalVectorConstants@@3P6AXXZA 004196fc     ltmodule.obj
 0002:00000700       ?IntSignMask$initializer$@GlobalVectorConstants@@3P6AXXZA 00419700     ltmodule.obj
 0002:00000704       ?AllMask$initializer$@GlobalVectorConstants@@3P6AXXZA 00419704     ltmodule.obj
 0002:00000708       ?IntAllMask$initializer$@GlobalVectorConstants@@3P6AXXZA 00419708     ltmodule.obj
 0002:0000070c       ?FloatInfinity$initializer$@GlobalVectorConstants@@3P6AXXZA 0041970c     ltmodule.obj
 0002:00000710       ?Pi$initializer$@GlobalVectorConstants@@3P6AXXZA 00419710     ltmodule.obj
 0002:00000714       ?TwoPi$initializer$@GlobalVectorConstants@@3P6AXXZA 00419714     ltmodule.obj
 0002:00000718       ?PiByTwo$initializer$@GlobalVectorConstants@@3P6AXXZA 00419718     ltmodule.obj
 0002:0000071c       ?PiByFour$initializer$@GlobalVectorConstants@@3P6AXXZA 0041971c     ltmodule.obj
 0002:00000720       ?OneOverPi$initializer$@GlobalVectorConstants@@3P6AXXZA 00419720     ltmodule.obj
 0002:00000724       ?OneOverTwoPi$initializer$@GlobalVectorConstants@@3P6AXXZA 00419724     ltmodule.obj
 0002:00000728       ?Float255$initializer$@GlobalVectorConstants@@3P6AXXZA 00419728     ltmodule.obj
 0002:0000072c       ?Float127$initializer$@GlobalVectorConstants@@3P6AXXZA 0041972c     ltmodule.obj
 0002:00000730       ?FloatNeg127$initializer$@GlobalVectorConstants@@3P6AXXZA 00419730     ltmodule.obj
 0002:00000734       ?Float360$initializer$@GlobalVectorConstants@@3P6AXXZA 00419734     ltmodule.obj
 0002:00000738       ?Float180$initializer$@GlobalVectorConstants@@3P6AXXZA 00419738     ltmodule.obj
 0002:0000073c       ?FloatTwo$initializer$@GlobalVectorConstants@@3P6AXXZA 0041973c     ltmodule.obj
 0002:00000740       ?FloatAlmostTwo$initializer$@GlobalVectorConstants@@3P6AXXZA 00419740     ltmodule.obj
 0002:00000744       ?a$initializer$@VectorSinConstantsSSE@@3P6AXXZA 00419744     ltmodule.obj
 0002:00000748       ?b$initializer$@VectorSinConstantsSSE@@3P6AXXZA 00419748     ltmodule.obj
 0002:0000074c       ?A$initializer$@VectorSinConstantsSSE@@3P6AXXZA 0041974c     ltmodule.obj
 0002:00000750       ?B$initializer$@VectorSinConstantsSSE@@3P6AXXZA 00419750     ltmodule.obj
 0002:00000754       ?PI$initializer$@@3P6AXXZA 00419754     ltmodule.obj
 0002:00000758       ?PI_2$initializer$@@3P6AXXZA 00419758     ltmodule.obj
 0002:0000075c       ?PI_3$initializer$@@3P6AXXZA 0041975c     ltmodule.obj
 0002:00000760       ?PI_4$initializer$@@3P6AXXZA 00419760     ltmodule.obj
 0002:00000764       ?RADIANS_PER_DEGREE$initializer$@@3P6AXXZA 00419764     ltmodule.obj
 0002:00000768       ?DEGREES_PER_RADIAN$initializer$@@3P6AXXZA 00419768     ltmodule.obj
 0002:0000076c       ?_FILE_SHUTDOWN_var_ltmod_database_$initializer$@@3P6AXXZA 0041976c     ltmodule.obj
 0002:00000770       ??m_strFileFormat$initializer$@CHLogger@@0P6AXXZA@@3P6AXXZA 00419770     HostLogger.obj
 0002:00000774       ??m_strBRFileFormat$initializer$@CHLogger@@0P6AXXZA@@3P6AXXZA 00419774     HostLogger.obj
 0002:00000778       ??m_strKernelFileFormat$initializer$@CHLogger@@0P6AXXZA@@3P6AXXZA 00419778     HostLogger.obj
 0002:0000077c       ??m_strEtcFileFormat$initializer$@CHLogger@@0P6AXXZA@@3P6AXXZA 0041977c     HostLogger.obj
 0002:00000780       ??m_strRWProcessMemoryFileFormat$initializer$@CHLogger@@0P6AXXZA@@3P6AXXZA 00419780     HostLogger.obj
 0002:00000784       ??m_strIPCMessageFileFormat$initializer$@CHLogger@@0P6AXXZA@@3P6AXXZA 00419784     HostLogger.obj
 0002:00000788       ??m_strTimeOutFileFormat$initializer$@CHLogger@@0P6AXXZA@@3P6AXXZA 00419788     HostLogger.obj
 0002:0000078c       ??m_strPacketFileFormat$initializer$@CHLogger@@0P6AXXZA@@3P6AXXZA 0041978c     HostLogger.obj
 0002:00000790       ??m_strHostName$initializer$@CHLogger@@0P6AXXZA@@3P6AXXZA 00419790     HostLogger.obj
 0002:00000794       ??m_strServerName$initializer$@CHLogger@@0P6AXXZA@@3P6AXXZA 00419794     HostLogger.obj
 0002:00000798       ??m_strLogFolder$initializer$@CHLogger@@0P6AXXZA@@3P6AXXZA 00419798     HostLogger.obj
 0002:0000079c       ??m_strModeUserCountFormat$initializer$@CHLogger@@0P6AXXZA@@3P6AXXZA 0041979c     HostLogger.obj
 0002:000007a0       ??m_strServerAppUseCountFormat$initializer$@CHLogger@@0P6AXXZA@@3P6AXXZA 004197a0     HostLogger.obj
 0002:000007a4       ??m_LogLock$initializer$@CHLogger@@0P6AXXZA@@3P6AXXZA 004197a4     HostLogger.obj
 0002:000007a8       ??m_LogPacketLock$initializer$@CHLogger@@0P6AXXZA@@3P6AXXZA 004197a8     HostLogger.obj
 0002:000007ac       ??m_vectSharedMapHandles$initializer$@CLogMsgManager@@0P6AXXZA@@3P6AXXZA 004197ac     LogMsgManager.obj
 0002:000007b0       ?theApp$initializer$@@3P6AXXZA 004197b0     ServerApp.obj
 0002:000007b4       ?g_cServerLog$initializer$@@3P6AXXZA 004197b4     ServerAppDlg.obj
 0002:000007b8       ?__api_holder_ILTCommon_Server_g_pLTSCommon__$initializer$@@3P6AXXZA 004197b8     ServerAppDlg.obj
 0002:000007bc       ?g_sGameInfos$initializer$@@3P6AXXZA 004197bc     ServerAppDlg.obj
 0002:000007c0       ?g_sUserInfos$initializer$@@3P6AXXZA 004197c0     ServerAppDlg.obj
 0002:000007c4       ?FloatOne$initializer$@GlobalVectorConstants@@3P6AXXZA 004197c4     StdAfx.obj
 0002:000007c8       ?FloatZero$initializer$@GlobalVectorConstants@@3P6AXXZA 004197c8     StdAfx.obj
 0002:000007cc       ?FloatMinusOne$initializer$@GlobalVectorConstants@@3P6AXXZA 004197cc     StdAfx.obj
 0002:000007d0       ?Float0001$initializer$@GlobalVectorConstants@@3P6AXXZA 004197d0     StdAfx.obj
 0002:000007d4       ?SmallLengthThreshold$initializer$@GlobalVectorConstants@@3P6AXXZA 004197d4     StdAfx.obj
 0002:000007d8       ?FloatOneHundredth$initializer$@GlobalVectorConstants@@3P6AXXZA 004197d8     StdAfx.obj
 0002:000007dc       ?Float111_Minus1$initializer$@GlobalVectorConstants@@3P6AXXZA 004197dc     StdAfx.obj
 0002:000007e0       ?FloatMinus1_111$initializer$@GlobalVectorConstants@@3P6AXXZA 004197e0     StdAfx.obj
 0002:000007e4       ?FloatOneHalf$initializer$@GlobalVectorConstants@@3P6AXXZA 004197e4     StdAfx.obj
 0002:000007e8       ?FloatMinusOneHalf$initializer$@GlobalVectorConstants@@3P6AXXZA 004197e8     StdAfx.obj
 0002:000007ec       ?KindaSmallNumber$initializer$@GlobalVectorConstants@@3P6AXXZA 004197ec     StdAfx.obj
 0002:000007f0       ?SmallNumber$initializer$@GlobalVectorConstants@@3P6AXXZA 004197f0     StdAfx.obj
 0002:000007f4       ?ThreshQuatNormalized$initializer$@GlobalVectorConstants@@3P6AXXZA 004197f4     StdAfx.obj
 0002:000007f8       ?BigNumber$initializer$@GlobalVectorConstants@@3P6AXXZA 004197f8     StdAfx.obj
 0002:000007fc       ?IntOne$initializer$@GlobalVectorConstants@@3P6AXXZA 004197fc     StdAfx.obj
 0002:00000800       ?IntZero$initializer$@GlobalVectorConstants@@3P6AXXZA 00419800     StdAfx.obj
 0002:00000804       ?IntMinusOne$initializer$@GlobalVectorConstants@@3P6AXXZA 00419804     StdAfx.obj
 0002:00000808       ?QINV_SIGN_MASK$initializer$@GlobalVectorConstants@@3P6AXXZA 00419808     StdAfx.obj
 0002:0000080c       ?QMULTI_SIGN_MASK0$initializer$@GlobalVectorConstants@@3P6AXXZA 0041980c     StdAfx.obj
 0002:00000810       ?QMULTI_SIGN_MASK1$initializer$@GlobalVectorConstants@@3P6AXXZA 00419810     StdAfx.obj
 0002:00000814       ?QMULTI_SIGN_MASK2$initializer$@GlobalVectorConstants@@3P6AXXZA 00419814     StdAfx.obj
 0002:00000818       ?DEG_TO_RAD$initializer$@GlobalVectorConstants@@3P6AXXZA 00419818     StdAfx.obj
 0002:0000081c       ?DEG_TO_RAD_HALF$initializer$@GlobalVectorConstants@@3P6AXXZA 0041981c     StdAfx.obj
 0002:00000820       ?RAD_TO_DEG$initializer$@GlobalVectorConstants@@3P6AXXZA 00419820     StdAfx.obj
 0002:00000824       ?XYZMask$initializer$@GlobalVectorConstants@@3P6AXXZA 00419824     StdAfx.obj
 0002:00000828       ?SignBit$initializer$@GlobalVectorConstants@@3P6AXXZA 00419828     StdAfx.obj
 0002:0000082c       ?SignMask$initializer$@GlobalVectorConstants@@3P6AXXZA 0041982c     StdAfx.obj
 0002:00000830       ?IntSignBit$initializer$@GlobalVectorConstants@@3P6AXXZA 00419830     StdAfx.obj
 0002:00000834       ?IntSignMask$initializer$@GlobalVectorConstants@@3P6AXXZA 00419834     StdAfx.obj
 0002:00000838       ?AllMask$initializer$@GlobalVectorConstants@@3P6AXXZA 00419838     StdAfx.obj
 0002:0000083c       ?IntAllMask$initializer$@GlobalVectorConstants@@3P6AXXZA 0041983c     StdAfx.obj
 0002:00000840       ?FloatInfinity$initializer$@GlobalVectorConstants@@3P6AXXZA 00419840     StdAfx.obj
 0002:00000844       ?Pi$initializer$@GlobalVectorConstants@@3P6AXXZA 00419844     StdAfx.obj
 0002:00000848       ?TwoPi$initializer$@GlobalVectorConstants@@3P6AXXZA 00419848     StdAfx.obj
 0002:0000084c       ?PiByTwo$initializer$@GlobalVectorConstants@@3P6AXXZA 0041984c     StdAfx.obj
 0002:00000850       ?PiByFour$initializer$@GlobalVectorConstants@@3P6AXXZA 00419850     StdAfx.obj
 0002:00000854       ?OneOverPi$initializer$@GlobalVectorConstants@@3P6AXXZA 00419854     StdAfx.obj
 0002:00000858       ?OneOverTwoPi$initializer$@GlobalVectorConstants@@3P6AXXZA 00419858     StdAfx.obj
 0002:0000085c       ?Float255$initializer$@GlobalVectorConstants@@3P6AXXZA 0041985c     StdAfx.obj
 0002:00000860       ?Float127$initializer$@GlobalVectorConstants@@3P6AXXZA 00419860     StdAfx.obj
 0002:00000864       ?FloatNeg127$initializer$@GlobalVectorConstants@@3P6AXXZA 00419864     StdAfx.obj
 0002:00000868       ?Float360$initializer$@GlobalVectorConstants@@3P6AXXZA 00419868     StdAfx.obj
 0002:0000086c       ?Float180$initializer$@GlobalVectorConstants@@3P6AXXZA 0041986c     StdAfx.obj
 0002:00000870       ?FloatTwo$initializer$@GlobalVectorConstants@@3P6AXXZA 00419870     StdAfx.obj
 0002:00000874       ?FloatAlmostTwo$initializer$@GlobalVectorConstants@@3P6AXXZA 00419874     StdAfx.obj
 0002:00000878       ?a$initializer$@VectorSinConstantsSSE@@3P6AXXZA 00419878     StdAfx.obj
 0002:0000087c       ?b$initializer$@VectorSinConstantsSSE@@3P6AXXZA 0041987c     StdAfx.obj
 0002:00000880       ?A$initializer$@VectorSinConstantsSSE@@3P6AXXZA 00419880     StdAfx.obj
 0002:00000884       ?B$initializer$@VectorSinConstantsSSE@@3P6AXXZA 00419884     StdAfx.obj
 0002:00000888       ?PI$initializer$@@3P6AXXZA 00419888     StdAfx.obj
 0002:0000088c       ?PI_2$initializer$@@3P6AXXZA 0041988c     StdAfx.obj
 0002:00000890       ?PI_3$initializer$@@3P6AXXZA 00419890     StdAfx.obj
 0002:00000894       ?PI_4$initializer$@@3P6AXXZA 00419894     StdAfx.obj
 0002:00000898       ?RADIANS_PER_DEGREE$initializer$@@3P6AXXZA 00419898     StdAfx.obj
 0002:0000089c       ?DEGREES_PER_RADIAN$initializer$@@3P6AXXZA 0041989c     StdAfx.obj
 0002:000008a8       ?pre_c_initializer@@3P6AHXZA 004198a8     msvcrt:exe_winmain.obj
 0002:000008ac       ?post_pgo_initializer@@3P6AHXZA 004198ac     msvcrt:exe_winmain.obj
 0002:00000ee0       ?AlmostTwoBits@GlobalVectorConstants@@3IB 00419ee0     ltmodule.obj
 0002:00001423       ?piecewise_construct@std@@3Upiecewise_construct_t@1@B 0041a423     LoadXlsMsg.obj
 0002:0000155c       ?_messageEntries@?1??GetThisMessageMap@CServerAppApp@@KGPBUAFX_MSGMAP@@XZ@4QBUAFX_MSGMAP_ENTRY@@B 0041a55c     ServerApp.obj
 0002:0000158c       ?messageMap@?1??GetThisMessageMap@CServerAppApp@@KGPBUAFX_MSGMAP@@XZ@4U3@B 0041a58c     ServerApp.obj
 0002:00001cc0       ?_messageEntries@?1??GetThisMessageMap@CServerAppDlg@@KGPBUAFX_MSGMAP@@XZ@4QBUAFX_MSGMAP_ENTRY@@B 0041acc0     ServerAppDlg.obj
 0002:00001d68       ?messageMap@?1??GetThisMessageMap@CServerAppDlg@@KGPBUAFX_MSGMAP@@XZ@4U3@B 0041ad68     ServerAppDlg.obj
 0002:000034b8       ?AlmostTwoBits@GlobalVectorConstants@@3IB 0041c4b8     StdAfx.obj
 0002:000034c0       ?g_szCommonAnimNames@@3QAY0IA@$$CBDA 0041c4c0     StdAfx.obj
 0002:00007980       _GS_ExceptionPointers      00420980     msvcrt:gs_report.obj
 0002:00008a10       __ehfuncinfo$?sprintf_s@internal@cf@@YAHPADIPBDAAPAD@Z 00421a10     safe_string:safe_string.obj
 0002:00008a34       __unwindtable$?sprintf_s@internal@cf@@YAHPADIPBDAAPAD@Z 00421a34     safe_string:safe_string.obj
 0002:00008a4c       __ehfuncinfo$?strcpy_s@cf@@YAHPADIPBD@Z 00421a4c     safe_string:safe_string.obj
 0002:00008a70       __unwindtable$?strcpy_s@cf@@YAHPADIPBD@Z 00421a70     safe_string:safe_string.obj
 0002:00008a88       __ehfuncinfo$?strncpy_s@cf@@YAHPADIPBDI@Z 00421a88     safe_string:safe_string.obj
 0002:00008aac       __unwindtable$?strncpy_s@cf@@YAHPADIPBDI@Z 00421aac     safe_string:safe_string.obj
 0002:00008ac4       __ehfuncinfo$?str@?$basic_stringstream@DU?$char_traits@D@std@@V?$allocator@D@2@@std@@QBE?AV?$basic_string@DU?$char_traits@D@std@@V?$allocator@D@2@@2@XZ 00421ac4     safe_string:safe_string.obj
 0002:00008ae8       __unwindtable$?str@?$basic_stringstream@DU?$char_traits@D@std@@V?$allocator@D@2@@std@@QBE?AV?$basic_string@DU?$char_traits@D@std@@V?$allocator@D@2@@2@XZ 00421ae8     safe_string:safe_string.obj
 0002:00008af0       __ehfuncinfo$??0?$basic_stringstream@DU?$char_traits@D@std@@V?$allocator@D@2@@std@@QAE@H@Z 00421af0     safe_string:safe_string.obj
 0002:00008b14       __unwindtable$??0?$basic_stringstream@DU?$char_traits@D@std@@V?$allocator@D@2@@std@@QAE@H@Z 00421b14     safe_string:safe_string.obj
 0002:00008b24       __ehfuncinfo$??1sentry@?$basic_ostream@DU?$char_traits@D@std@@@std@@QAE@XZ 00421b24     safe_string:safe_string.obj
 0002:00008b48       __unwindtable$??1sentry@?$basic_ostream@DU?$char_traits@D@std@@@std@@QAE@XZ 00421b48     safe_string:safe_string.obj
 0002:00008b50       __ehfuncinfo$??1_Sentry_base@?$basic_ostream@DU?$char_traits@D@std@@@std@@QAE@XZ 00421b50     safe_string:safe_string.obj
 0002:00008b50       __ehfuncinfo$??1CServerAppDlg@@UAE@XZ 00421b50     ServerAppDlg.obj
 0002:00008b50       __ehfuncinfo$??1?$CAPIHolder@VILTCommon@@@@UAE@XZ 00421b50     ServerAppDlg.obj
 0002:00008b74       __ehfuncinfo$??$?6U?$char_traits@D@std@@@std@@YAAAV?$basic_ostream@DU?$char_traits@D@std@@@0@AAV10@PBD@Z 00421b74     safe_string:safe_string.obj
 0002:00008b98       __unwindtable$??$?6U?$char_traits@D@std@@@std@@YAAAV?$basic_ostream@DU?$char_traits@D@std@@@0@AAV10@PBD@Z 00421b98     safe_string:safe_string.obj
 0002:00008bc8       __tryblocktable$??$?6U?$char_traits@D@std@@@std@@YAAAV?$basic_ostream@DU?$char_traits@D@std@@@0@AAV10@PBD@Z 00421bc8     safe_string:safe_string.obj
 0002:00008bdc       __catchsym$??$?6U?$char_traits@D@std@@@std@@YAAAV?$basic_ostream@DU?$char_traits@D@std@@@0@AAV10@PBD@Z$6 00421bdc     safe_string:safe_string.obj
 0002:00008bec       __unwindtable$?GetMasterDatabase@@YAPAVCInterfaceDatabase@@XZ 00421bec     ltmodule.obj
 0002:00008bec       __unwindtable$?AddAPI@CInterfaceDatabase@@SAXPAVIBase@@PBDH@Z 00421bec     ltmodule.obj
 0002:00008bec       __unwindtable$?AddHolder@CInterfaceDatabase@@SAXPAVCAPIHolderBase@@@Z 00421bec     ltmodule.obj
 0002:00008bec       __unwindtable$?AddChooser@CInterfaceDatabase@@SAXPAVCInterfaceChooser@@@Z 00421bec     ltmodule.obj
 0002:00008bf4       __ehfuncinfo$?AddChooser@CInterfaceDatabase@@SAXPAVCInterfaceChooser@@@Z 00421bf4     ltmodule.obj
 0002:00008bf4       __ehfuncinfo$?AddAPI@CInterfaceDatabase@@SAXPAVIBase@@PBDH@Z 00421bf4     ltmodule.obj
 0002:00008bf4       __ehfuncinfo$?GetMasterDatabase@@YAPAVCInterfaceDatabase@@XZ 00421bf4     ltmodule.obj
 0002:00008bf4       __ehfuncinfo$?AddHolder@CInterfaceDatabase@@SAXPAVCAPIHolderBase@@@Z 00421bf4     ltmodule.obj
 0002:00008c18       __unwindtable$??0CInterfaceDatabase@@QAE@XZ 00421c18     ltmodule.obj
 0002:00008c28       __ehfuncinfo$??0CInterfaceDatabase@@QAE@XZ 00421c28     ltmodule.obj
 0002:00008c4c       __unwindtable$?TransferFrom@CInterfaceDatabase@@UAEXPAV1@@Z 00421c4c     ltmodule.obj
 0002:00008c54       __ehfuncinfo$?TransferFrom@CInterfaceDatabase@@UAEXPAV1@@Z 00421c54     ltmodule.obj
 0002:00008c78       __unwindtable$?Add@CInterfaceDatabase@@EAEXPAVIBase@@PBDH@Z 00421c78     ltmodule.obj
 0002:00008c80       __ehfuncinfo$?Add@CInterfaceDatabase@@EAEXPAVIBase@@PBDH@Z 00421c80     ltmodule.obj
 0002:00008ca4       __unwindtable$?Add@CInterfaceDatabase@@EAEXPAVCAPIHolderBase@@@Z 00421ca4     ltmodule.obj
 0002:00008ca4       __unwindtable$?Add@CInterfaceDatabase@@EAEXPAVCInterfaceChooser@@@Z 00421ca4     ltmodule.obj
 0002:00008cac       __ehfuncinfo$?Add@CInterfaceDatabase@@EAEXPAVCAPIHolderBase@@@Z 00421cac     ltmodule.obj
 0002:00008cac       __ehfuncinfo$?Add@CInterfaceDatabase@@EAEXPAVCInterfaceChooser@@@Z 00421cac     ltmodule.obj
 0002:00008cd0       __unwindtable$??0CInterfaceNameMgr@@QAE@PBDH@Z 00421cd0     ltmodule.obj
 0002:00008ce8       __ehfuncinfo$??0CInterfaceNameMgr@@QAE@PBDH@Z 00421ce8     ltmodule.obj
 0002:00008d0c       __unwindtable$?LogPacket@CHLogger@@SAXPBDZZ 00421d0c     HostLogger.obj
 0002:00008d14       __ehfuncinfo$?LogPacket@CHLogger@@SAXPBDZZ 00421d14     HostLogger.obj
 0002:00008d38       __unwindtable$?_BuildDirectory@CHLogger@@CAXABU_SYSTEMTIME@@@Z 00421d38     HostLogger.obj
 0002:00008d50       __ehfuncinfo$?_BuildDirectory@CHLogger@@CAXABU_SYSTEMTIME@@@Z 00421d50     HostLogger.obj
 0002:00008d74       __unwindtable$?_DoLogWithLevel@CHLogger@@CAXPBDW4ELOG_LEVEL@1@0PAD@Z 00421d74     HostLogger.obj
 0002:00008d7c       __ehfuncinfo$?_DoLogWithLevel@CHLogger@@CAXPBDW4ELOG_LEVEL@1@0PAD@Z 00421d7c     HostLogger.obj
 0002:00008da0       __unwindtable$?Init@CLogMsgManager@@SA_NW4ESHARED_MEM_USAGE_TYPE@1@@Z 00421da0     LogMsgManager.obj
 0002:00008db0       __ehfuncinfo$?Init@CLogMsgManager@@SA_NW4ESHARED_MEM_USAGE_TYPE@1@@Z 00421db0     LogMsgManager.obj
 0002:00008dd4       __unwindtable$?_WriteXlsDataToSharedMemory@CLogMsgManager@@CA_NXZ 00421dd4     LogMsgManager.obj
 0002:00008ddc       __ehfuncinfo$?_WriteXlsDataToSharedMemory@CLogMsgManager@@CA_NXZ 00421ddc     LogMsgManager.obj
 0002:00008e00       __unwindtable$??1FindXlsMsg@@UAE@XZ 00421e00     LoadXlsMsg.obj
 0002:00008e10       __ehfuncinfo$??1FindXlsMsg@@UAE@XZ 00421e10     LoadXlsMsg.obj
 0002:00008e34       __unwindtable$?LoadWMszFile@FindXlsMsg@@QAE_NPAD@Z 00421e34     LoadXlsMsg.obj
 0002:00008e3c       __ehfuncinfo$?LoadWMszFile@FindXlsMsg@@QAE_NPAD@Z 00421e3c     LoadXlsMsg.obj
 0002:00008e60       __catchsym$??$_Insert_hint@AAU?$pair@$$CB_JV?$basic_string@DU?$char_traits@D@std@@V?$allocator@D@2@@std@@@std@@PAU?$_Tree_node@U?$pair@$$CB_JV?$basic_string@DU?$char_traits@D@std@@V?$allocator@D@2@@std@@@std@@PAX@2@@?$_Tree@V?$_Tmap_traits@_JV?$basic_string@DU?$char_traits@D@std@@V?$allocator@D@2@@std@@U?$less@_J@2@V?$allocator@U?$pair@$$CB_JV?$basic_string@DU?$char_traits@D@std@@V?$allocator@D@2@@std@@@std@@@2@$0A@@std@@@std@@IAE?AV?$_Tree_iterator@V?$_Tree_val@U?$_Tree_simple_types@U?$pair@$$CB_JV?$basic_string@DU?$char_traits@D@std@@V?$allocator@D@2@@std@@@std@@@std@@@std@@@1@V?$_Tree_const_iterator@V?$_Tree_val@U?$_Tree_simple_types@U?$pair@$$CB_JV?$basic_string@DU?$char_traits@D@std@@V?$allocator@D@2@@std@@@std@@@std@@@std@@@1@AAU?$pair@$$CB_JV?$basic_string@DU?$char_traits@D@std@@V?$allocator@D@2@@std@@@1@PAU?$_Tree_node@U?$pair@$$CB_JV?$basic_string@DU?$char_traits@D@std@@V?$allocator@D@2@@std@@@std@@PAX@1@@Z$2 00421e60     LoadXlsMsg.obj
 0002:00008e70       __unwindtable$??$_Insert_hint@AAU?$pair@$$CB_JV?$basic_string@DU?$char_traits@D@std@@V?$allocator@D@2@@std@@@std@@PAU?$_Tree_node@U?$pair@$$CB_JV?$basic_string@DU?$char_traits@D@std@@V?$allocator@D@2@@std@@@std@@PAX@2@@?$_Tree@V?$_Tmap_traits@_JV?$basic_string@DU?$char_traits@D@std@@V?$allocator@D@2@@std@@U?$less@_J@2@V?$allocator@U?$pair@$$CB_JV?$basic_string@DU?$char_traits@D@std@@V?$allocator@D@2@@std@@@std@@@2@$0A@@std@@@std@@IAE?AV?$_Tree_iterator@V?$_Tree_val@U?$_Tree_simple_types@U?$pair@$$CB_JV?$basic_string@DU?$char_traits@D@std@@V?$allocator@D@2@@std@@@std@@@std@@@std@@@1@V?$_Tree_const_iterator@V?$_Tree_val@U?$_Tree_simple_types@U?$pair@$$CB_JV?$basic_string@DU?$char_traits@D@std@@V?$allocator@D@2@@std@@@std@@@std@@@std@@@1@AAU?$pair@$$CB_JV?$basic_string@DU?$char_traits@D@std@@V?$allocator@D@2@@std@@@1@PAU?$_Tree_node@U?$pair@$$CB_JV?$basic_string@DU?$char_traits@D@std@@V?$allocator@D@2@@std@@@std@@PAX@1@@Z 00421e70     LoadXlsMsg.obj
 0002:00008e80       __tryblocktable$??$_Insert_hint@AAU?$pair@$$CB_JV?$basic_string@DU?$char_traits@D@std@@V?$allocator@D@2@@std@@@std@@PAU?$_Tree_node@U?$pair@$$CB_JV?$basic_string@DU?$char_traits@D@std@@V?$allocator@D@2@@std@@@std@@PAX@2@@?$_Tree@V?$_Tmap_traits@_JV?$basic_string@DU?$char_traits@D@std@@V?$allocator@D@2@@std@@U?$less@_J@2@V?$allocator@U?$pair@$$CB_JV?$basic_string@DU?$char_traits@D@std@@V?$allocator@D@2@@std@@@std@@@2@$0A@@std@@@std@@IAE?AV?$_Tree_iterator@V?$_Tree_val@U?$_Tree_simple_types@U?$pair@$$CB_JV?$basic_string@DU?$char_traits@D@std@@V?$allocator@D@2@@std@@@std@@@std@@@std@@@1@V?$_Tree_const_iterator@V?$_Tree_val@U?$_Tree_simple_types@U?$pair@$$CB_JV?$basic_string@DU?$char_traits@D@std@@V?$allocator@D@2@@std@@@std@@@std@@@std@@@1@AAU?$pair@$$CB_JV?$basic_string@DU?$char_traits@D@std@@V?$allocator@D@2@@std@@@1@PAU?$_Tree_node@U?$pair@$$CB_JV?$basic_string@DU?$char_traits@D@std@@V?$allocator@D@2@@std@@@std@@PAX@1@@Z 00421e80     LoadXlsMsg.obj
 0002:00008e94       __ehfuncinfo$??$_Insert_hint@AAU?$pair@$$CB_JV?$basic_string@DU?$char_traits@D@std@@V?$allocator@D@2@@std@@@std@@PAU?$_Tree_node@U?$pair@$$CB_JV?$basic_string@DU?$char_traits@D@std@@V?$allocator@D@2@@std@@@std@@PAX@2@@?$_Tree@V?$_Tmap_traits@_JV?$basic_string@DU?$char_traits@D@std@@V?$allocator@D@2@@std@@U?$less@_J@2@V?$allocator@U?$pair@$$CB_JV?$basic_string@DU?$char_traits@D@std@@V?$allocator@D@2@@std@@@std@@@2@$0A@@std@@@std@@IAE?AV?$_Tree_iterator@V?$_Tree_val@U?$_Tree_simple_types@U?$pair@$$CB_JV?$basic_string@DU?$char_traits@D@std@@V?$allocator@D@2@@std@@@std@@@std@@@std@@@1@V?$_Tree_const_iterator@V?$_Tree_val@U?$_Tree_simple_types@U?$pair@$$CB_JV?$basic_string@DU?$char_traits@D@std@@V?$allocator@D@2@@std@@@std@@@std@@@std@@@1@AAU?$pair@$$CB_JV?$basic_string@DU?$char_traits@D@std@@V?$allocator@D@2@@std@@@1@PAU?$_Tree_node@U?$pair@$$CB_JV?$basic_string@DU?$char_traits@D@std@@V?$allocator@D@2@@std@@@std@@PAX@1@@Z 00421e94     LoadXlsMsg.obj
 0002:00008eb8       __catchsym$??$_Insert_nohint@AAU?$pair@$$CB_JV?$basic_string@DU?$char_traits@D@std@@V?$allocator@D@2@@std@@@std@@PAU?$_Tree_node@U?$pair@$$CB_JV?$basic_string@DU?$char_traits@D@std@@V?$allocator@D@2@@std@@@std@@PAX@2@@?$_Tree@V?$_Tmap_traits@_JV?$basic_string@DU?$char_traits@D@std@@V?$allocator@D@2@@std@@U?$less@_J@2@V?$allocator@U?$pair@$$CB_JV?$basic_string@DU?$char_traits@D@std@@V?$allocator@D@2@@std@@@std@@@2@$0A@@std@@@std@@IAE?AU?$pair@V?$_Tree_iterator@V?$_Tree_val@U?$_Tree_simple_types@U?$pair@$$CB_JV?$basic_string@DU?$char_traits@D@std@@V?$allocator@D@2@@std@@@std@@@std@@@std@@@std@@_N@1@_NAAU?$pair@$$CB_JV?$basic_string@DU?$char_traits@D@std@@V?$allocator@D@2@@std@@@1@PAU?$_Tree_node@U?$pair@$$CB_JV?$basic_string@DU?$char_traits@D@std@@V?$allocator@D@2@@std@@@std@@PAX@1@@Z$2 00421eb8     LoadXlsMsg.obj
 0002:00008ec8       __unwindtable$??$_Insert_nohint@AAU?$pair@$$CB_JV?$basic_string@DU?$char_traits@D@std@@V?$allocator@D@2@@std@@@std@@PAU?$_Tree_node@U?$pair@$$CB_JV?$basic_string@DU?$char_traits@D@std@@V?$allocator@D@2@@std@@@std@@PAX@2@@?$_Tree@V?$_Tmap_traits@_JV?$basic_string@DU?$char_traits@D@std@@V?$allocator@D@2@@std@@U?$less@_J@2@V?$allocator@U?$pair@$$CB_JV?$basic_string@DU?$char_traits@D@std@@V?$allocator@D@2@@std@@@std@@@2@$0A@@std@@@std@@IAE?AU?$pair@V?$_Tree_iterator@V?$_Tree_val@U?$_Tree_simple_types@U?$pair@$$CB_JV?$basic_string@DU?$char_traits@D@std@@V?$allocator@D@2@@std@@@std@@@std@@@std@@@std@@_N@1@_NAAU?$pair@$$CB_JV?$basic_string@DU?$char_traits@D@std@@V?$allocator@D@2@@std@@@1@PAU?$_Tree_node@U?$pair@$$CB_JV?$basic_string@DU?$char_traits@D@std@@V?$allocator@D@2@@std@@@std@@PAX@1@@Z 00421ec8     LoadXlsMsg.obj
 0002:00008ed8       __tryblocktable$??$_Insert_nohint@AAU?$pair@$$CB_JV?$basic_string@DU?$char_traits@D@std@@V?$allocator@D@2@@std@@@std@@PAU?$_Tree_node@U?$pair@$$CB_JV?$basic_string@DU?$char_traits@D@std@@V?$allocator@D@2@@std@@@std@@PAX@2@@?$_Tree@V?$_Tmap_traits@_JV?$basic_string@DU?$char_traits@D@std@@V?$allocator@D@2@@std@@U?$less@_J@2@V?$allocator@U?$pair@$$CB_JV?$basic_string@DU?$char_traits@D@std@@V?$allocator@D@2@@std@@@std@@@2@$0A@@std@@@std@@IAE?AU?$pair@V?$_Tree_iterator@V?$_Tree_val@U?$_Tree_simple_types@U?$pair@$$CB_JV?$basic_string@DU?$char_traits@D@std@@V?$allocator@D@2@@std@@@std@@@std@@@std@@@std@@_N@1@_NAAU?$pair@$$CB_JV?$basic_string@DU?$char_traits@D@std@@V?$allocator@D@2@@std@@@1@PAU?$_Tree_node@U?$pair@$$CB_JV?$basic_string@DU?$char_traits@D@std@@V?$allocator@D@2@@std@@@std@@PAX@1@@Z 00421ed8     LoadXlsMsg.obj
 0002:00008eec       __ehfuncinfo$??$_Insert_nohint@AAU?$pair@$$CB_JV?$basic_string@DU?$char_traits@D@std@@V?$allocator@D@2@@std@@@std@@PAU?$_Tree_node@U?$pair@$$CB_JV?$basic_string@DU?$char_traits@D@std@@V?$allocator@D@2@@std@@@std@@PAX@2@@?$_Tree@V?$_Tmap_traits@_JV?$basic_string@DU?$char_traits@D@std@@V?$allocator@D@2@@std@@U?$less@_J@2@V?$allocator@U?$pair@$$CB_JV?$basic_string@DU?$char_traits@D@std@@V?$allocator@D@2@@std@@@std@@@2@$0A@@std@@@std@@IAE?AU?$pair@V?$_Tree_iterator@V?$_Tree_val@U?$_Tree_simple_types@U?$pair@$$CB_JV?$basic_string@DU?$char_traits@D@std@@V?$allocator@D@2@@std@@@std@@@std@@@std@@@std@@_N@1@_NAAU?$pair@$$CB_JV?$basic_string@DU?$char_traits@D@std@@V?$allocator@D@2@@std@@@1@PAU?$_Tree_node@U?$pair@$$CB_JV?$basic_string@DU?$char_traits@D@std@@V?$allocator@D@2@@std@@@std@@PAX@1@@Z 00421eec     LoadXlsMsg.obj
 0002:00008f10       __unwindtable$?Run@CServerAppApp@@UAEHXZ 00421f10     ServerApp.obj
 0002:00008f18       __ehfuncinfo$?Run@CServerAppApp@@UAEHXZ 00421f18     ServerApp.obj
 0002:00008f3c       __catchsym$??1CWaitCursor@@QAE@XZ$3 00421f3c     ServerAppDlg.obj
 0002:00008f4c       __tryblocktable$??1CWaitCursor@@QAE@XZ 00421f4c     ServerAppDlg.obj
 0002:00008f60       __unwindtable$??1CWaitCursor@@QAE@XZ 00421f60     ServerAppDlg.obj
 0002:00008f78       __ehfuncinfo$??1CWaitCursor@@QAE@XZ 00421f78     ServerAppDlg.obj
 0002:00008f9c       __unwindtable$?RTIDUSNtoString@EXPAND_USN@@YA?AV?$basic_string@DU?$char_traits@D@std@@V?$allocator@D@2@@std@@HFF_J@Z 00421f9c     ServerAppDlg.obj
 0002:00008fa4       __ehfuncinfo$?RTIDUSNtoString@EXPAND_USN@@YA?AV?$basic_string@DU?$char_traits@D@std@@V?$allocator@D@2@@std@@HFF_J@Z 00421fa4     ServerAppDlg.obj
 0002:00008fc8       __unwindtable$?OutOfMemory@CGameServerAppHandler@@UAEIXZ 00421fc8     ServerAppDlg.obj
 0002:00008fd0       __ehfuncinfo$?OutOfMemory@CGameServerAppHandler@@UAEIXZ 00421fd0     ServerAppDlg.obj
 0002:00008ff4       __unwindtable$?ConsoleOutputFn@CGameServerAppHandler@@UAEIHHPBD@Z 00421ff4     ServerAppDlg.obj
 0002:00008ffc       __ehfuncinfo$?ConsoleOutputFn@CGameServerAppHandler@@UAEIHHPBD@Z 00421ffc     ServerAppDlg.obj
 0002:00009020       __ehfuncinfo$??0CServerAppDlg@@QAE@PAVCWnd@@@Z 00422020     ServerAppDlg.obj
 0002:00009044       __unwindtable$??0CServerAppDlg@@QAE@PAVCWnd@@@Z 00422044     ServerAppDlg.obj
 0002:00009074       __ehfuncinfo$?OnShellMessage@CServerAppDlg@@QAEXAAVILTMessage_Read@@@Z 00422074     ServerAppDlg.obj
 0002:00009098       __unwindtable$?OnShellMessage@CServerAppDlg@@QAEXAAVILTMessage_Read@@@Z 00422098     ServerAppDlg.obj
 0002:000090d0       __unwindtable$?AddServerMsg@CServerAppDlg@@QAEXPBDH@Z 004220d0     ServerAppDlg.obj
 0002:000090d8       __ehfuncinfo$?AddServerMsg@CServerAppDlg@@QAEXPBDH@Z 004220d8     ServerAppDlg.obj
 0002:000090fc       __unwindtable$?ThreadUpdate@CServerAppDlg@@SAXPAX@Z 004220fc     ServerAppDlg.obj
 0002:0000910c       __ehfuncinfo$?ThreadUpdate@CServerAppDlg@@SAXPAX@Z 0042210c     ServerAppDlg.obj
 0002:00009130       __unwindtable$?ServerUpdate@CServerAppDlg@@QAEXXZ 00422130     ServerAppDlg.obj
 0002:00009138       __ehfuncinfo$?ServerUpdate@CServerAppDlg@@QAEXXZ 00422138     ServerAppDlg.obj
 0002:0000915c       __ehfuncinfo$?LoadServer@CServerAppDlg@@QAE_NXZ 0042215c     ServerAppDlg.obj
 0002:00009180       __unwindtable$?LoadServer@CServerAppDlg@@QAE_NXZ 00422180     ServerAppDlg.obj
 0002:000091b0       __unwindtable$?RunServer@CServerAppDlg@@QAE_NXZ 004221b0     ServerAppDlg.obj
 0002:000091d0       __ehfuncinfo$?RunServer@CServerAppDlg@@QAE_NXZ 004221d0     ServerAppDlg.obj
 0002:000091f4       __unwindtable$?StopServer@CServerAppDlg@@QAE_NXZ 004221f4     ServerAppDlg.obj
 0002:000091fc       __ehfuncinfo$?StopServer@CServerAppDlg@@QAE_NXZ 004221fc     ServerAppDlg.obj
 0002:00009220       __unwindtable$?DoHost@CServerAppDlg@@QAE_NXZ 00422220     ServerAppDlg.obj
 0002:00009228       __ehfuncinfo$?DoHost@CServerAppDlg@@QAE_NXZ 00422228     ServerAppDlg.obj
 0002:0000924c       __ehfuncinfo$?AddResources@CServerAppDlg@@QAE_NXZ 0042224c     ServerAppDlg.obj
 0002:00009270       __unwindtable$?AddResources@CServerAppDlg@@QAE_NXZ 00422270     ServerAppDlg.obj
 0002:000092b0       __unwindtable$?SaveHostGameInfo@CServerAppDlg@@IAEXXZ 004222b0     ServerAppDlg.obj
 0002:000092c8       __ehfuncinfo$?SaveHostGameInfo@CServerAppDlg@@IAEXXZ 004222c8     ServerAppDlg.obj
 0002:000092ec       __unwindtable$?LoadHostGameInfo@CServerAppDlg@@IAEXXZ 004222ec     ServerAppDlg.obj
 0002:00009304       __ehfuncinfo$?LoadHostGameInfo@CServerAppDlg@@IAEXXZ 00422304     ServerAppDlg.obj
 0002:00009328       __unwindtable$?GetOptionValueString@CServerAppDlg@@IAE?AV?$basic_string@DU?$char_traits@D@std@@V?$allocator@D@2@@std@@V23@00@Z 00422328     ServerAppDlg.obj
 0002:00009348       __ehfuncinfo$?GetOptionValueString@CServerAppDlg@@IAE?AV?$basic_string@DU?$char_traits@D@std@@V?$allocator@D@2@@std@@V23@00@Z 00422348     ServerAppDlg.obj
 0002:0000936c       __unwindtable$?SendServerAppInit@CServerAppDlg@@AAEXXZ 0042236c     ServerAppDlg.obj
 0002:0000936c       __unwindtable$?RECV_MSG_AIITEM_GROUP_RATE_RESULT@CServerAppDlg@@AAEXJ@Z 0042236c     ServerAppDlg.obj
 0002:00009374       __ehfuncinfo$?SendServerAppInit@CServerAppDlg@@AAEXXZ 00422374     ServerAppDlg.obj
 0002:00009374       __ehfuncinfo$?RECV_MSG_AIITEM_GROUP_RATE_RESULT@CServerAppDlg@@AAEXJ@Z 00422374     ServerAppDlg.obj
 0002:00009398       __unwindtable$?SendServerAppInitFail@CServerAppDlg@@AAEXHH@Z 00422398     ServerAppDlg.obj
 0002:000093a8       __ehfuncinfo$?SendServerAppInitFail@CServerAppDlg@@AAEXHH@Z 004223a8     ServerAppDlg.obj
 0002:000093cc       __ehfuncinfo$?OnInitDialog@CServerAppDlg@@MAEHXZ 004223cc     ServerAppDlg.obj
 0002:000093f0       __unwindtable$?OnInitDialog@CServerAppDlg@@MAEHXZ 004223f0     ServerAppDlg.obj
 0002:00009420       __unwindtable$?OnGameServerMsg@CServerAppDlg@@IAEJIJ@Z 00422420     ServerAppDlg.obj
 0002:00009438       __ehfuncinfo$?OnGameServerMsg@CServerAppDlg@@IAEJIJ@Z 00422438     ServerAppDlg.obj
 0002:0000945c       __ehfuncinfo$?OnCopyData@CServerAppDlg@@IAEHPAVCWnd@@PAUtagCOPYDATASTRUCT@@@Z 0042245c     ServerAppDlg.obj
 0002:00009480       __unwindtable$?OnCopyData@CServerAppDlg@@IAEHPAVCWnd@@PAUtagCOPYDATASTRUCT@@@Z 00422480     ServerAppDlg.obj
 0002:000094c0       __unwindtable$?OnTimer@CServerAppDlg@@QAEXI@Z 004224c0     ServerAppDlg.obj
 0002:000094c8       __ehfuncinfo$?OnTimer@CServerAppDlg@@QAEXI@Z 004224c8     ServerAppDlg.obj
 0002:000094ec       __unwindtable$?OnButtonStartServer@CServerAppDlg@@QAEHXZ 004224ec     ServerAppDlg.obj
 0002:000094fc       __ehfuncinfo$?OnButtonStartServer@CServerAppDlg@@QAEHXZ 004224fc     ServerAppDlg.obj
 0002:00009520       __unwindtable$?RECV_MSG_INSERTCHARACTER@CServerAppDlg@@AAEXJ@Z 00422520     ServerAppDlg.obj
 0002:00009530       __ehfuncinfo$?RECV_MSG_INSERTCHARACTER@CServerAppDlg@@AAEXJ@Z 00422530     ServerAppDlg.obj
 0002:00009554       __unwindtable$?RECV_MSG_AIITEM_DEC@CServerAppDlg@@AAEXJ@Z 00422554     ServerAppDlg.obj
 0002:0000955c       __ehfuncinfo$?RECV_MSG_AIITEM_DEC@CServerAppDlg@@AAEXJ@Z 0042255c     ServerAppDlg.obj
 0002:00009580       __unwindtable$?RECV_MSG_USER_DISCONNECTED@CServerAppDlg@@AAEXJ@Z 00422580     ServerAppDlg.obj
 0002:00009588       __ehfuncinfo$?RECV_MSG_USER_DISCONNECTED@CServerAppDlg@@AAEXJ@Z 00422588     ServerAppDlg.obj
 0002:000095ac       __ehfuncinfo$?DownloadUCCMapFile_HTTP@CServerAppDlg@@AAE?AW4UCCMAPDOWNLOADREAULT@@V?$basic_string@DU?$char_traits@D@std@@V?$allocator@D@2@@std@@@Z 004225ac     ServerAppDlg.obj
 0002:000095d0       __unwindtable$?DownloadUCCMapFile_HTTP@CServerAppDlg@@AAE?AW4UCCMAPDOWNLOADREAULT@@V?$basic_string@DU?$char_traits@D@std@@V?$allocator@D@2@@std@@@Z 004225d0     ServerAppDlg.obj
 0002:00009620       __unwindtable$?GetDownloadPath@CServerAppDlg@@AAE?AV?$basic_string@DU?$char_traits@D@std@@V?$allocator@D@2@@std@@XZ 00422620     ServerAppDlg.obj
 0002:00009628       __ehfuncinfo$?GetDownloadPath@CServerAppDlg@@AAE?AV?$basic_string@DU?$char_traits@D@std@@V?$allocator@D@2@@std@@XZ 00422628     ServerAppDlg.obj
 0002:0000964c       __unwindtable$??0?$CAPIHolder@VILTCommon@@@@QAE@PBDAAPAVILTCommon@@H@Z 0042264c     ServerAppDlg.obj
 0002:00009654       __ehfuncinfo$??0?$CAPIHolder@VILTCommon@@@@QAE@PBDAAPAVILTCommon@@H@Z 00422654     ServerAppDlg.obj
 0002:00009678       __ehfuncinfo$?Thread_SendGameInfo@@YAXPAVCServerAppDlg@@AAUPROTO_START_HOST_tag@@@Z 00422678     ServerAppDlg.obj
 0002:0000969c       __unwindtable$?Thread_SendGameInfo@@YAXPAVCServerAppDlg@@AAUPROTO_START_HOST_tag@@@Z 0042269c     ServerAppDlg.obj
 0002:000096d4       __unwindtable$?Thread_SendUserInfo@@YAXPAVCServerAppDlg@@AAUPROTO_GAME_USER_INFO_tag@@@Z 004226d4     ServerAppDlg.obj
 0002:000096e4       __ehfuncinfo$?Thread_SendUserInfo@@YAXPAVCServerAppDlg@@AAUPROTO_GAME_USER_INFO_tag@@@Z 004226e4     ServerAppDlg.obj
 0002:00009708       __unwindtable$??$?HDU?$char_traits@D@std@@V?$allocator@D@1@@std@@YA?AV?$basic_string@DU?$char_traits@D@std@@V?$allocator@D@2@@0@ABV10@0@Z 00422708     ServerAppDlg.obj
 0002:00009710       __ehfuncinfo$??$?HDU?$char_traits@D@std@@V?$allocator@D@1@@std@@YA?AV?$basic_string@DU?$char_traits@D@std@@V?$allocator@D@2@@0@ABV10@0@Z 00422710     ServerAppDlg.obj
 0002:00009768       __unwindtable$?CRSUploader@@YAAAVUploader@crs@@XZ 00422768     BugReporter1.obj
 0002:00009770       __ehfuncinfo$?CRSUploader@@YAAAVUploader@crs@@XZ 00422770     BugReporter1.obj
 0002:00009794       __unwindtable$?threadCreateDumpFile@@YGKPAX@Z 00422794     BugReporter1.obj
 0002:0000979c       __ehfuncinfo$?threadCreateDumpFile@@YGKPAX@Z 0042279c     BugReporter1.obj
 0002:000097c0       __unwindtable$??0Uploader@crs@@QAE@XZ 004227c0     crs_uploader1.obj
 0002:000097d0       __ehfuncinfo$??0Uploader@crs@@QAE@XZ 004227d0     crs_uploader1.obj
 0002:000097f4       __unwindtable$?init@Uploader@crs@@QAE_N_NPAD1@Z 004227f4     crs_uploader1.obj
 0002:000097fc       __ehfuncinfo$?init@Uploader@crs@@QAE_N_NPAD1@Z 004227fc     crs_uploader1.obj
 0002:00009820       __unwindtable$?readURL@Uploader@crs@@AAEXAAV?$basic_string@_WU?$char_traits@_W@std@@V?$allocator@_W@2@@std@@@Z 00422820     crs_uploader1.obj
 0002:00009838       __ehfuncinfo$?readURL@Uploader@crs@@AAEXAAV?$basic_string@_WU?$char_traits@_W@std@@V?$allocator@_W@2@@std@@@Z 00422838     crs_uploader1.obj
 0002:00009860       __sehtable$___scrt_is_nonwritable_in_current_image 00422860     msvcrt:utility.obj
 0002:00009880       __sehtable$?__scrt_common_main_seh@@YAHXZ 00422880     msvcrt:exe_winmain.obj
 0002:000098a0       .edata                     004228a0     ServerApp.exp
 0002:000098c8       rgpv                       004228c8     ServerApp.exp
 0002:000098d0       rgszName                   004228d0     ServerApp.exp
 0002:000098d8       rgwOrd                     004228d8     ServerApp.exp
 0002:000098dc       szName                     004228dc     ServerApp.exp
 0002:000098ea       $N00001                    004228ea     ServerApp.exp
 0002:000098f6       $N00002                    004228f6     ServerApp.exp
 0002:0000a17c       .idata$6                   0042317c     Psapi:PSAPI.DLL
 0002:0000a186       .idata$6                   00423186     mfc140:mfc140.dll
 0002:0000a616       .idata$6                   00423616     kernel32:KERNEL32.dll
 0002:0000a6a0       .idata$6                   004236a0     user32:USER32.dll
 0002:0000a6c4       .idata$6                   004236c4     shell32:SHELL32.dll
 0002:0000a6e2       .idata$6                   004236e2     shlwapi:SHLWAPI.dll
 0002:0000a72e       .idata$6                   0042372e     msvcprt:MSVCP140.dll
 0002:0000a78a       .idata$6                   0042378a     wininet:WININET.dll
 0002:0000a796       .idata$6                   00423796     ws2_32:WS2_32.dll
 0002:0000a840       .idata$6                   00423840     DbgHelp:dbghelp.dll
 0002:0000a85a       .idata$6                   0042385a     winmm:WINMM.dll
 0002:0000a91c       .idata$6                   0042391c     winhttp:WINHTTP.dll
 0002:0000aa0c       .idata$6                   00423a0c     vcruntime:VCRUNTIME140.dll
 0002:0000adfa       .idata$6                   00423dfa     ucrt:api-ms-win-crt-string-l1-1-0.dll
 0002:0000ae1c       .idata$6                   00423e1c     ucrt:api-ms-win-crt-math-l1-1-0.dll
 0002:0000ae3c       .idata$6                   00423e3c     ucrt:api-ms-win-crt-runtime-l1-1-0.dll
 0002:0000ae5e       .idata$6                   00423e5e     ucrt:api-ms-win-crt-stdio-l1-1-0.dll
 0002:0000ae7e       .idata$6                   00423e7e     ucrt:api-ms-win-crt-filesystem-l1-1-0.dll
 0002:0000aea4       .idata$6                   00423ea4     ucrt:api-ms-win-crt-utility-l1-1-0.dll
 0002:0000aec6       .idata$6                   00423ec6     ucrt:api-ms-win-crt-convert-l1-1-0.dll
 0002:0000aee8       .idata$6                   00423ee8     ucrt:api-ms-win-crt-time-l1-1-0.dll
 0002:0000af08       .idata$6                   00423f08     ucrt:api-ms-win-crt-heap-l1-1-0.dll
 0002:0000af28       .idata$6                   00423f28     ucrt:api-ms-win-crt-locale-l1-1-0.dll
 0003:00000000       ?WORLD_RIGHT@@3V?$LTVector3@M@@B 00425000     ltmodule.obj
 0003:0000000c       ?WORLD_FORWARD@@3V?$LTVector3@M@@B 0042500c     ltmodule.obj
 0003:00000018       ?WORLD_UP@@3V?$LTVector3@M@@B 00425018     ltmodule.obj
 0003:000001a4       ?WORLD_RIGHT@@3V?$LTVector3@M@@B 004251a4     StdAfx.obj
 0003:000001b0       ?WORLD_FORWARD@@3V?$LTVector3@M@@B 004251b0     StdAfx.obj
 0003:000001bc       ?WORLD_UP@@3V?$LTVector3@M@@B 004251bc     StdAfx.obj
 0003:000001c8       ?szDmp_Folder@@3PADA       004251c8     BugReporter1.obj
 0003:000001cc       ?szDmp_ErrorFile@@3PADA    004251cc     BugReporter1.obj
 0003:000001d0       ?g_szDmp_FileName_Format@@3PADA 004251d0     BugReporter1.obj
 0003:000001d4       ?prefix@?1??uploadVersion@Uploader@crs@@QAE_NXZ@4PADA 004251d4     crs_uploader1.obj
 0003:000001dc       ?prefix@?1??uploadLOG@Uploader@crs@@AAE_NAAVHttpHandle@3@AAU_SYSTEMTIME@@AAVLogBuffer@3@@Z@4PADA 004251dc     crs_uploader1.obj
 0003:000001e0       ?szLog_Folder@@3PADA       004251e0     LogMgmt1.obj
 0003:000001e4       ?szLog_ErrorFile@@3PADA    004251e4     LogMgmt1.obj
 0003:000001e8       ?szLog_EtcFile@@3PADA      004251e8     LogMgmt1.obj
 0003:000001ec       ?szLog_TimeFile@@3PADA     004251ec     LogMgmt1.obj
 0003:000001f0       ?szLog_TimeOutFile@@3PADA  004251f0     LogMgmt1.obj
 0003:000001f4       ?szLog_HackFile@@3PADA     004251f4     LogMgmt1.obj
 0003:000001f8       ?szLog_CountFile@@3PADA    004251f8     LogMgmt1.obj
 0003:000001fc       ?szLog_CashFile@@3PADA     004251fc     LogMgmt1.obj
 0003:00000200       ?szLog_UnknownDataFile@@3PADA 00425200     LogMgmt1.obj
 0003:00000204       ?szLog_MagaPhone@@3PADA    00425204     LogMgmt1.obj
 0003:00000208       ?szLog_ConnectCheck@@3PADA 00425208     LogMgmt1.obj
 0003:0000020c       ?szLog_EmergencyState@@3PADA 0042520c     LogMgmt1.obj
 0003:00000210       ?szLog_Hacking@@3PADA      00425210     LogMgmt1.obj
 0003:00000214       ?szLog_KickUser@@3PADA     00425214     LogMgmt1.obj
 0003:00000218       ?szLog_ServerSettingCheck@@3PADA 00425218     LogMgmt1.obj
 0003:0000021c       ?szLog_MgrDataFile@@3PADA  0042521c     LogMgmt1.obj
 0003:00000220       ?szLog_GachaFile@@3PADA    00425220     LogMgmt1.obj
 0003:00000224       ?szLog_MailerFile@@3PADA   00425224     LogMgmt1.obj
 0003:00000228       ?szLog_TryWeaponItemFile@@3PADA 00425228     LogMgmt1.obj
 0003:00000760       ?a@VectorSinConstantsSSE@@3MB 00425760     ltmodule.obj
 0003:00000764       ?RADIANS_PER_DEGREE@@3MB   00425764     ltmodule.obj
 0003:00000768       ?b@VectorSinConstantsSSE@@3MB 00425768     ltmodule.obj
 0003:0000076c       ?PI_3@@3MB                 0042576c     ltmodule.obj
 0003:00000770       ?PiByTwo@GlobalVectorConstants@@3T__m128@@B 00425770     ltmodule.obj
 0003:00000780       ?FloatMinusOneHalf@GlobalVectorConstants@@3T__m128@@B 00425780     ltmodule.obj
 0003:00000790       ?IntAllMask@GlobalVectorConstants@@3T__m128i@@B 00425790     ltmodule.obj
 0003:000007a0       ?TwoPi@GlobalVectorConstants@@3T__m128@@B 004257a0     ltmodule.obj
 0003:000007b0       ?SmallLengthThreshold@GlobalVectorConstants@@3T__m128@@B 004257b0     ltmodule.obj
 0003:000007c0       ?OneOverPi@GlobalVectorConstants@@3T__m128@@B 004257c0     ltmodule.obj
 0003:000007d0       ?AllMask@GlobalVectorConstants@@3T__m128@@B 004257d0     ltmodule.obj
 0003:000007e0       ?ThreshQuatNormalized@GlobalVectorConstants@@3T__m128@@B 004257e0     ltmodule.obj
 0003:000007f0       ?SignBit@GlobalVectorConstants@@3T__m128@@B 004257f0     ltmodule.obj
 0003:00000800       ?Float360@GlobalVectorConstants@@3T__m128@@B 00425800     ltmodule.obj
 0003:00000810       ?QMULTI_SIGN_MASK0@GlobalVectorConstants@@3T__m128@@B 00425810     ltmodule.obj
 0003:00000820       ?OneOverTwoPi@GlobalVectorConstants@@3T__m128@@B 00425820     ltmodule.obj
 0003:00000830       ?DEG_TO_RAD@GlobalVectorConstants@@3T__m128@@B 00425830     ltmodule.obj
 0003:00000840       ?BigNumber@GlobalVectorConstants@@3T__m128@@B 00425840     ltmodule.obj
 0003:00000850       ?FloatOneHundredth@GlobalVectorConstants@@3T__m128@@B 00425850     ltmodule.obj
 0003:00000860       ?FloatTwo@GlobalVectorConstants@@3T__m128@@B 00425860     ltmodule.obj
 0003:00000870       ?Float0001@GlobalVectorConstants@@3T__m128@@B 00425870     ltmodule.obj
 0003:00000880       ?FloatAlmostTwo@GlobalVectorConstants@@3T__m128@@B 00425880     ltmodule.obj
 0003:00000890       ?QMULTI_SIGN_MASK2@GlobalVectorConstants@@3T__m128@@B 00425890     ltmodule.obj
 0003:000008a0       ?SignMask@GlobalVectorConstants@@3T__m128@@B 004258a0     ltmodule.obj
 0003:000008b0       ?FloatMinus1_111@GlobalVectorConstants@@3T__m128@@B 004258b0     ltmodule.obj
 0003:000008c0       ?QMULTI_SIGN_MASK1@GlobalVectorConstants@@3T__m128@@B 004258c0     ltmodule.obj
 0003:000008d0       ?IntMinusOne@GlobalVectorConstants@@3T__m128i@@B 004258d0     ltmodule.obj
 0003:000008e0       ?FloatOneHalf@GlobalVectorConstants@@3T__m128@@B 004258e0     ltmodule.obj
 0003:000008f0       ?FloatZero@GlobalVectorConstants@@3T__m128@@B 004258f0     ltmodule.obj
 0003:00000900       ?B@VectorSinConstantsSSE@@3T__m128@@B 00425900     ltmodule.obj
 0003:00000910       ?Float255@GlobalVectorConstants@@3T__m128@@B 00425910     ltmodule.obj
 0003:00000920       ?Float127@GlobalVectorConstants@@3T__m128@@B 00425920     ltmodule.obj
 0003:00000930       ?QINV_SIGN_MASK@GlobalVectorConstants@@3T__m128@@B 00425930     ltmodule.obj
 0003:00000940       ?DEG_TO_RAD_HALF@GlobalVectorConstants@@3T__m128@@B 00425940     ltmodule.obj
 0003:00000950       ?FloatOne@GlobalVectorConstants@@3T__m128@@B 00425950     ltmodule.obj
 0003:00000960       ?A@VectorSinConstantsSSE@@3T__m128@@B 00425960     ltmodule.obj
 0003:00000970       ?IntSignBit@GlobalVectorConstants@@3T__m128i@@B 00425970     ltmodule.obj
 0003:00000980       ?FloatMinusOne@GlobalVectorConstants@@3T__m128@@B 00425980     ltmodule.obj
 0003:00000990       ?FloatNeg127@GlobalVectorConstants@@3T__m128@@B 00425990     ltmodule.obj
 0003:000009a0       ?Float111_Minus1@GlobalVectorConstants@@3T__m128@@B 004259a0     ltmodule.obj
 0003:000009b0       ?XYZMask@GlobalVectorConstants@@3T__m128@@B 004259b0     ltmodule.obj
 0003:000009c0       ?KindaSmallNumber@GlobalVectorConstants@@3T__m128@@B 004259c0     ltmodule.obj
 0003:000009d0       ?IntOne@GlobalVectorConstants@@3T__m128i@@B 004259d0     ltmodule.obj
 0003:000009e0       ?SmallNumber@GlobalVectorConstants@@3T__m128@@B 004259e0     ltmodule.obj
 0003:000009f0       ?PiByFour@GlobalVectorConstants@@3T__m128@@B 004259f0     ltmodule.obj
 0003:00000a10       ?Pi@GlobalVectorConstants@@3T__m128@@B 00425a10     ltmodule.obj
 0003:00000a20       ?DEGREES_PER_RADIAN@@3MB   00425a20     ltmodule.obj
 0003:00000a24       ?PI@@3MB                   00425a24     ltmodule.obj
 0003:00000a28       ?PI_4@@3MB                 00425a28     ltmodule.obj
 0003:00000a30       ?FloatInfinity@GlobalVectorConstants@@3T__m128@@B 00425a30     ltmodule.obj
 0003:00000a40       ?IntZero@GlobalVectorConstants@@3T__m128i@@B 00425a40     ltmodule.obj
 0003:00000a50       ?IntSignMask@GlobalVectorConstants@@3T__m128i@@B 00425a50     ltmodule.obj
 0003:00000a60       ?RAD_TO_DEG@GlobalVectorConstants@@3T__m128@@B 00425a60     ltmodule.obj
 0003:00000a70       ?PI_2@@3MB                 00425a70     ltmodule.obj
 0003:00000a74       ?ptrs@@3PAVCDatabasePtrs@@A 00425a74     ltmodule.obj
 0003:00000a78       ?database_item_count@@3HA  00425a78     ltmodule.obj
 0003:00000a80       ?Float180@GlobalVectorConstants@@3T__m128@@B 00425a80     ltmodule.obj
 0003:00000dec       ?__api_holder_ILTCommon_Server_g_pLTSCommon__@@3V?$CAPIHolder@VILTCommon@@@@A 00425dec     ServerAppDlg.obj
 0003:00221840       ?a@VectorSinConstantsSSE@@3MB 00646840     StdAfx.obj
 0003:00221844       ?RADIANS_PER_DEGREE@@3MB   00646844     StdAfx.obj
 0003:00221848       ?b@VectorSinConstantsSSE@@3MB 00646848     StdAfx.obj
 0003:0022184c       ?PI_3@@3MB                 0064684c     StdAfx.obj
 0003:00221850       ?PiByTwo@GlobalVectorConstants@@3T__m128@@B 00646850     StdAfx.obj
 0003:00221860       ?FloatMinusOneHalf@GlobalVectorConstants@@3T__m128@@B 00646860     StdAfx.obj
 0003:00221870       ?IntAllMask@GlobalVectorConstants@@3T__m128i@@B 00646870     StdAfx.obj
 0003:00221880       ?TwoPi@GlobalVectorConstants@@3T__m128@@B 00646880     StdAfx.obj
 0003:00221890       ?SmallLengthThreshold@GlobalVectorConstants@@3T__m128@@B 00646890     StdAfx.obj
 0003:002218a0       ?OneOverPi@GlobalVectorConstants@@3T__m128@@B 006468a0     StdAfx.obj
 0003:002218b0       ?AllMask@GlobalVectorConstants@@3T__m128@@B 006468b0     StdAfx.obj
 0003:002218c0       ?ThreshQuatNormalized@GlobalVectorConstants@@3T__m128@@B 006468c0     StdAfx.obj
 0003:002218d0       ?SignBit@GlobalVectorConstants@@3T__m128@@B 006468d0     StdAfx.obj
 0003:002218e0       ?Float360@GlobalVectorConstants@@3T__m128@@B 006468e0     StdAfx.obj
 0003:002218f0       ?QMULTI_SIGN_MASK0@GlobalVectorConstants@@3T__m128@@B 006468f0     StdAfx.obj
 0003:00221900       ?OneOverTwoPi@GlobalVectorConstants@@3T__m128@@B 00646900     StdAfx.obj
 0003:00221910       ?DEG_TO_RAD@GlobalVectorConstants@@3T__m128@@B 00646910     StdAfx.obj
 0003:00221920       ?BigNumber@GlobalVectorConstants@@3T__m128@@B 00646920     StdAfx.obj
 0003:00221930       ?FloatOneHundredth@GlobalVectorConstants@@3T__m128@@B 00646930     StdAfx.obj
 0003:00221940       ?FloatTwo@GlobalVectorConstants@@3T__m128@@B 00646940     StdAfx.obj
 0003:00221950       ?Float0001@GlobalVectorConstants@@3T__m128@@B 00646950     StdAfx.obj
 0003:00221960       ?FloatAlmostTwo@GlobalVectorConstants@@3T__m128@@B 00646960     StdAfx.obj
 0003:00221970       ?QMULTI_SIGN_MASK2@GlobalVectorConstants@@3T__m128@@B 00646970     StdAfx.obj
 0003:00221980       ?SignMask@GlobalVectorConstants@@3T__m128@@B 00646980     StdAfx.obj
 0003:00221990       ?FloatMinus1_111@GlobalVectorConstants@@3T__m128@@B 00646990     StdAfx.obj
 0003:002219a0       ?QMULTI_SIGN_MASK1@GlobalVectorConstants@@3T__m128@@B 006469a0     StdAfx.obj
 0003:002219b0       ?IntMinusOne@GlobalVectorConstants@@3T__m128i@@B 006469b0     StdAfx.obj
 0003:002219c0       ?FloatOneHalf@GlobalVectorConstants@@3T__m128@@B 006469c0     StdAfx.obj
 0003:002219d0       ?FloatZero@GlobalVectorConstants@@3T__m128@@B 006469d0     StdAfx.obj
 0003:002219e0       ?B@VectorSinConstantsSSE@@3T__m128@@B 006469e0     StdAfx.obj
 0003:002219f0       ?Float255@GlobalVectorConstants@@3T__m128@@B 006469f0     StdAfx.obj
 0003:00221a00       ?Float127@GlobalVectorConstants@@3T__m128@@B 00646a00     StdAfx.obj
 0003:00221a10       ?QINV_SIGN_MASK@GlobalVectorConstants@@3T__m128@@B 00646a10     StdAfx.obj
 0003:00221a20       ?DEG_TO_RAD_HALF@GlobalVectorConstants@@3T__m128@@B 00646a20     StdAfx.obj
 0003:00221a30       ?FloatOne@GlobalVectorConstants@@3T__m128@@B 00646a30     StdAfx.obj
 0003:00221a40       ?A@VectorSinConstantsSSE@@3T__m128@@B 00646a40     StdAfx.obj
 0003:00221a50       ?IntSignBit@GlobalVectorConstants@@3T__m128i@@B 00646a50     StdAfx.obj
 0003:00221a60       ?FloatMinusOne@GlobalVectorConstants@@3T__m128@@B 00646a60     StdAfx.obj
 0003:00221a70       ?FloatNeg127@GlobalVectorConstants@@3T__m128@@B 00646a70     StdAfx.obj
 0003:00221a80       ?Float111_Minus1@GlobalVectorConstants@@3T__m128@@B 00646a80     StdAfx.obj
 0003:00221a90       ?XYZMask@GlobalVectorConstants@@3T__m128@@B 00646a90     StdAfx.obj
 0003:00221aa0       ?KindaSmallNumber@GlobalVectorConstants@@3T__m128@@B 00646aa0     StdAfx.obj
 0003:00221ab0       ?IntOne@GlobalVectorConstants@@3T__m128i@@B 00646ab0     StdAfx.obj
 0003:00221ac0       ?SmallNumber@GlobalVectorConstants@@3T__m128@@B 00646ac0     StdAfx.obj
 0003:00221ad0       ?PiByFour@GlobalVectorConstants@@3T__m128@@B 00646ad0     StdAfx.obj
 0003:00221ae0       ?Pi@GlobalVectorConstants@@3T__m128@@B 00646ae0     StdAfx.obj
 0003:00221af0       ?DEGREES_PER_RADIAN@@3MB   00646af0     StdAfx.obj
 0003:00221af4       ?PI@@3MB                   00646af4     StdAfx.obj
 0003:00221af8       ?PI_4@@3MB                 00646af8     StdAfx.obj
 0003:00221afc       ?PI_2@@3MB                 00646afc     StdAfx.obj
 0003:00221b00       ?FloatInfinity@GlobalVectorConstants@@3T__m128@@B 00646b00     StdAfx.obj
 0003:00221b10       ?IntZero@GlobalVectorConstants@@3T__m128i@@B 00646b10     StdAfx.obj
 0003:00221b20       ?IntSignMask@GlobalVectorConstants@@3T__m128i@@B 00646b20     StdAfx.obj
 0003:00221b30       ?RAD_TO_DEG@GlobalVectorConstants@@3T__m128@@B 00646b30     StdAfx.obj
 0003:00221b40       ?Float180@GlobalVectorConstants@@3T__m128@@B 00646b40     StdAfx.obj
 0003:00221b50       ?g_szHostName@@3PADA       00646b50     BugReporter1.obj
 0003:00221bb8       ?g_szServerName@@3PADA     00646bb8     BugReporter1.obj
 0003:00221c20       ?g_szDmpFolder@@3PADA      00646c20     BugReporter1.obj
 0003:00221db8       ?g_szDmpFileName@@3PADA    00646db8     BugReporter1.obj
 0003:002221a8       ?g_szSubDir@@3PADA         006471a8     BugReporter1.obj
 0003:00222210       ?crs_uploader@?1??CRSUploader@@YAAAVUploader@crs@@XZ@4V23@A 00647210     BugReporter1.obj
 0003:00222314       ?$S15@?1??CRSUploader@@YAAAVUploader@crs@@XZ@4IA 00647314     BugReporter1.obj
 0003:00227844       ?is_initialized_as_dll@@3_NA 0064c844     msvcrt:utility.obj
 0003:00227845       ?module_local_atexit_table_initialized@@3_NA 0064c845     msvcrt:utility.obj
 0003:00227848       ?module_local_atexit_table@@3U_onexit_table_t@@A 0064c848     msvcrt:utility.obj
 0003:00227854       ?module_local_at_quick_exit_table@@3U_onexit_table_t@@A 0064c854     msvcrt:utility.obj
 0003:00227860       _GS_ExceptionRecord        0064c860     msvcrt:gs_report.obj
 0003:002278b0       _GS_ContextRecord          0064c8b0     msvcrt:gs_report.obj
 0004:000001b0       $R000000                   0064d1b0     ServerApp.res
 0004:00000498       $R0002E8                   0064d498     ServerApp.res
 0004:000005c0       $R000410                   0064d5c0     ServerApp.res
 0004:000005e8       $R000438                   0064d5e8     ServerApp.res
 0004:00000710       $R000560                   0064d710     ServerApp.res
 0004:000009c0       $R000810                   0064d9c0     ServerApp.res

 Exports

  ordinal    name

        1    _IsDebugMode
               exported name: IsDebugMode
        2    _SetMasterDatabase
               exported name: SetMasterDatabase
